 fontmanager

 Timestamp is ffffffff (Sun Feb  7 06:28:15 2106)

 Preferred load address is 10000000

 Start         Length     Name                   Class
 0001:00000000 000705bcH .text$mn                CODE
 0002:00000000 00000200H .idata$5                DATA
 0002:00000200 00000004H .00cfg                  DATA
 0002:00000204 00000004H .CRT$XCA                DATA
 0002:00000208 00000004H .CRT$XCZ                DATA
 0002:0000020c 00000004H .CRT$XIA                DATA
 0002:00000210 00000004H .CRT$XIZ                DATA
 0002:00000214 00000004H .CRT$XPA                DATA
 0002:00000218 00000004H .CRT$XPZ                DATA
 0002:0000021c 00000004H .CRT$XTA                DATA
 0002:00000220 00000010H .CRT$XTZ                DATA
 0002:00000224 00000000H .gfids$y                DATA
 0002:00000230 00035058H .rdata                  DATA
 0002:00035288 00000004H .rdata$sxdata           DATA
 0002:0003528c 00000288H .rdata$zzzdbg           DATA
 0002:00035514 00000004H .rtc$IAA                DATA
 0002:00035518 00000004H .rtc$IZZ                DATA
 0002:0003551c 00000004H .rtc$TAA                DATA
 0002:00035520 00000008H .rtc$TZZ                DATA
 0002:00035528 00000088H .xdata$x                DATA
 0002:000355b0 00000958H .edata                  DATA
 0002:00035f08 0000012cH .idata$2                DATA
 0002:00036034 00000014H .idata$3                DATA
 0002:00036048 00000200H .idata$4                DATA
 0002:00036248 000009fcH .idata$6                DATA
 0003:00000000 000007c0H .data                   DATA
 0003:000007c0 00000ce0H .bss                    DATA
 0004:00000000 00000060H .rsrc$01                DATA
 0004:00000060 00000330H .rsrc$02                DATA

  Address         Publics by Value              Rva+Base       Lib:Object

 0000:00000000       ___hybrid_auxiliary_iat    00000000     <absolute>
 0000:00000000       ___arm64x_extra_rfe_table  00000000     <absolute>
 0000:00000000       ___arm64x_redirection_metadata 00000000     <absolute>
 0000:00000000       ___guard_eh_cont_count     00000000     <absolute>
 0000:00000000       ___volatile_metadata       00000000     <absolute>
 0000:00000000       ___x64_code_ranges_to_entry_points 00000000     <absolute>
 0000:00000000       ___guard_longjmp_table     00000000     <absolute>
 0000:00000000       ___AbsoluteZero            00000000     <absolute>
 0000:00000000       ___guard_eh_cont_table     00000000     <absolute>
 0000:00000000       ___hybrid_code_map         00000000     <absolute>
 0000:00000000       ___x64_code_ranges_to_entry_points_count 00000000     <absolute>
 0000:00000000       ___guard_longjmp_count     00000000     <absolute>
 0000:00000000       ___arm64x_redirection_metadata_count 00000000     <absolute>
 0000:00000000       ___dynamic_value_reloc_table 00000000     <absolute>
 0000:00000000       ___guard_iat_count         00000000     <absolute>
 0000:00000000       ___arm64x_extra_rfe_table_size 00000000     <absolute>
 0000:00000000       ___guard_fids_count        00000000     <absolute>
 0000:00000000       ___hybrid_code_map_count   00000000     <absolute>
 0000:00000000       ___arm64x_native_entrypoint 00000000     <absolute>
 0000:00000000       ___guard_fids_table        00000000     <absolute>
 0000:00000000       ___guard_iat_table         00000000     <absolute>
 0000:00000000       ___enclave_config          00000000     <absolute>
 0000:00000001       ___safe_se_handler_count   00000001     <absolute>
 0000:00000100       ___guard_flags             00000100     <absolute>
 0000:00000000       ___ImageBase               10000000     <linker-defined>
 0001:000000b0       _Java_sun_font_ColorGlyphSurfaceData_initOps@8 100010b0 f   ColorGlyphSurfaceData.obj
 0001:000000e0       _Java_sun_font_ColorGlyphSurfaceData_setCurrentGlyph@16 100010e0 f   ColorGlyphSurfaceData.obj
 0001:00000100       _Java_sun_java2d_loops_DrawGlyphListAA_DrawGlyphListAA@28 10001100 f   DrawGlyphList.obj
 0001:00000100       _Java_sun_java2d_loops_DrawGlyphList_DrawGlyphList@28 10001100 f   DrawGlyphList.obj
 0001:00000180       _Java_sun_java2d_loops_DrawGlyphListLCD_DrawGlyphListLCD@28 10001180 f   DrawGlyphList.obj
 0001:00000230       _RefineBounds              10001230 f   DrawGlyphList.obj
 0001:000006f0       _initLCDGammaTables        100016f0 f   DrawGlyphList.obj
 0001:00000730       _initLUT                   10001730 f   DrawGlyphList.obj
 0001:00000860       _setupBlitVector           10001860 f   DrawGlyphList.obj
 0001:00000cf0       _setupLCDBlitVector        10001cf0 f   DrawGlyphList.obj
 0001:000013b0       _Java_sun_font_SunLayoutEngine_shape@68 100023b0 f   HBShaper.obj
 0001:00001780       _storeGVData               10002780 f   HBShaper.obj
 0001:00002120       _Java_sun_awt_Win32FontManager_getFontPath@12 10003120 f   fontpath.obj
 0001:000022b0       _Java_sun_awt_Win32FontManager_populateFontFileNameMap0@24 100032b0 f   fontpath.obj
 0001:00002c40       _Java_sun_font_FreetypeFontScaler_createScalerContextNative@36 10003c40 f   freetypeScaler.obj
 0001:00002e40       _Java_sun_font_FreetypeFontScaler_disposeNativeScaler@20 10003e40 f   freetypeScaler.obj
 0001:00002eb0       _Java_sun_font_FreetypeFontScaler_getFontMetricsNative@28 10003eb0 f   freetypeScaler.obj
 0001:000031c0       _Java_sun_font_FreetypeFontScaler_getGlyphAdvanceNative@32 100041c0 f   freetypeScaler.obj
 0001:00003220       _Java_sun_font_FreetypeFontScaler_getGlyphCodeNative@24 10004220 f   freetypeScaler.obj
 0001:000032d0       _Java_sun_font_FreetypeFontScaler_getGlyphImageNative@32 100042d0 f   freetypeScaler.obj
 0001:00003300       _Java_sun_font_FreetypeFontScaler_getGlyphMetricsNative@36 10004300 f   freetypeScaler.obj
 0001:000033c0       _Java_sun_font_FreetypeFontScaler_getGlyphOutlineBoundsNative@32 100043c0 f   freetypeScaler.obj
 0001:00003540       _Java_sun_font_FreetypeFontScaler_getGlyphOutlineNative@40 10004540 f   freetypeScaler.obj
 0001:000036b0       _Java_sun_font_FreetypeFontScaler_getGlyphPointNative@36 100046b0 f   freetypeScaler.obj
 0001:00003780       _Java_sun_font_FreetypeFontScaler_getGlyphVectorOutlineNative@44 10004780 f   freetypeScaler.obj
 0001:00003980       _Java_sun_font_FreetypeFontScaler_getMissingGlyphCodeNative@16 10004980 f   freetypeScaler.obj
 0001:00003990       _Java_sun_font_FreetypeFontScaler_getNumGlyphsNative@16 10004990 f   freetypeScaler.obj
 0001:00003a20       _Java_sun_font_FreetypeFontScaler_getUnitsPerEMNative@16 10004a20 f   freetypeScaler.obj
 0001:00003a40       _Java_sun_font_FreetypeFontScaler_initIDs@12 10004a40 f   freetypeScaler.obj
 0001:00003a70       _Java_sun_font_FreetypeFontScaler_initNativeScaler@28 10004a70 f   freetypeScaler.obj
 0001:00004840       ??$?0PBU?$KernSubTable@UKernAATSubTableHeader@OT@@@OT@@@hb_sanitize_with_object_t@@QAE@PAUhb_sanitize_context_t@@ABQBU?$KernSubTable@UKernAATSubTableHeader@OT@@@OT@@@Z 10005840 f i hb-ot-layout.obj
 0001:00004840       ??$?0PBUKerxSubTable@AAT@@@hb_sanitize_with_object_t@@QAE@PAUhb_sanitize_context_t@@ABQBUKerxSubTable@AAT@@@Z 10005840 f i hb-aat-layout.obj
 0001:00004840       ??$?0PBU?$ChainSubtable@UExtendedTypes@AAT@@@AAT@@@hb_sanitize_with_object_t@@QAE@PAUhb_sanitize_context_t@@ABQBU?$ChainSubtable@UExtendedTypes@AAT@@@AAT@@@Z 10005840 f i hb-aat-layout.obj
 0001:000048c0       ??$?0PBU?$ChainSubtable@UObsoleteTypes@AAT@@@AAT@@@hb_sanitize_with_object_t@@QAE@PAUhb_sanitize_context_t@@ABQBU?$ChainSubtable@UObsoleteTypes@AAT@@@AAT@@@Z 100058c0 f i hb-aat-layout.obj
 0001:000049e0       __hb_ot_shaper_font_data_destroy 100059e0 f   hb-ot-shape.obj
 0001:000049e0       @_guard_check_icall_nop@4  100059e0 f   MSVCRT:guard_support.obj
 0001:000049e0       __hb_ot_shaper_face_data_destroy 100059e0 f   hb-ot-shape.obj
 0001:000049e0       __hb_fallback_shaper_face_data_destroy 100059e0 f   hb-fallback-shape.obj
 0001:000049e0       __hb_fallback_shaper_font_data_destroy 100059e0 f   hb-fallback-shape.obj
 0001:000049e0       ?hb_ot_layout_position_finish_advances@@YAXPAUhb_font_t@@PAUhb_buffer_t@@@Z 100059e0 f   hb-ot-layout.obj
 0001:000049f0       ??$check_array@U?$IntType@G$01@OT@@@hb_sanitize_context_t@@QBE_NPBU?$IntType@G$01@OT@@I@Z 100059f0 f i hb-aat-layout.obj
 0001:00004a20       ??$check_range@U?$IntType@E$00@OT@@@hb_sanitize_context_t@@QBE_NPBU?$IntType@E$00@OT@@II@Z 10005a20 f i hb-aat-layout.obj
 0001:00004a60       ??$check_struct@U?$IntType@E$00@OT@@@hb_sanitize_context_t@@QBE_NPBU?$IntType@E$00@OT@@@Z 10005a60 f i hb-aat-layout.obj
 0001:00004ad0       ??$dispatch@UCoverage@OT@@$$V@hb_sanitize_context_t@@QAE_NABUCoverage@OT@@@Z 10005ad0 f i hb-aat-layout.obj
 0001:00004b60       ??$dispatch@UVariationStore@OT@@$$V@hb_sanitize_context_t@@QAE_NABUVariationStore@OT@@@Z 10005b60 f i hb-aat-layout.obj
 0001:00004c20       ??$dispatch@Uhb_aat_apply_context_t@AAT@@$$V@?$ChainSubtable@UExtendedTypes@AAT@@@AAT@@QBE_NPAUhb_aat_apply_context_t@1@@Z 10005c20 f i hb-aat-layout.obj
 0001:00004fe0       ??$dispatch@Uhb_aat_apply_context_t@AAT@@$$V@?$ChainSubtable@UObsoleteTypes@AAT@@@AAT@@QBE_NPAUhb_aat_apply_context_t@1@@Z 10005fe0 f i hb-aat-layout.obj
 0001:00005340       ??$dispatch@Uhb_aat_apply_context_t@AAT@@$$V@KerxSubTable@AAT@@QBE_NPAUhb_aat_apply_context_t@1@@Z 10006340 f i hb-aat-layout.obj
 0001:00005640       ??$dispatch@Uhb_sanitize_context_t@@$$V@?$ChainSubtable@UExtendedTypes@AAT@@@AAT@@QBE_NPAUhb_sanitize_context_t@@@Z 10006640 f i hb-aat-layout.obj
 0001:00005930       ??$dispatch@Uhb_sanitize_context_t@@$$V@?$ChainSubtable@UObsoleteTypes@AAT@@@AAT@@QBE_NPAUhb_sanitize_context_t@@@Z 10006930 f i hb-aat-layout.obj
 0001:00005b40       ??$dispatch@Uhb_sanitize_context_t@@$$V@KerxSubTable@AAT@@QBE_NPAUhb_sanitize_context_t@@@Z 10006b40 f i hb-aat-layout.obj
 0001:00005df0       ??$drive@Udriver_context_t@?$ContextualSubtable@UExtendedTypes@AAT@@@AAT@@@?$StateTableDriver@UExtendedTypes@AAT@@UEntryData@?$ContextualSubtable@UExtendedTypes@AAT@@@2@@AAT@@QAEXPAUdriver_context_t@?$ContextualSubtable@UExtendedTypes@AAT@@@1@@Z 10006df0 f i hb-aat-layout.obj
 0001:00006170       ??$drive@Udriver_context_t@?$ContextualSubtable@UObsoleteTypes@AAT@@@AAT@@@?$StateTableDriver@UObsoleteTypes@AAT@@UEntryData@?$ContextualSubtable@UObsoleteTypes@AAT@@@2@@AAT@@QAEXPAUdriver_context_t@?$ContextualSubtable@UObsoleteTypes@AAT@@@1@@Z 10007170 f i hb-aat-layout.obj
 0001:00006520       ??$drive@Udriver_context_t@?$InsertionSubtable@UExtendedTypes@AAT@@@AAT@@@?$StateTableDriver@UExtendedTypes@AAT@@UEntryData@?$InsertionSubtable@UExtendedTypes@AAT@@@2@@AAT@@QAEXPAUdriver_context_t@?$InsertionSubtable@UExtendedTypes@AAT@@@1@@Z 10007520 f i hb-aat-layout.obj
 0001:000068f0       ??$drive@Udriver_context_t@?$InsertionSubtable@UObsoleteTypes@AAT@@@AAT@@@?$StateTableDriver@UObsoleteTypes@AAT@@UEntryData@?$InsertionSubtable@UObsoleteTypes@AAT@@@2@@AAT@@QAEXPAUdriver_context_t@?$InsertionSubtable@UObsoleteTypes@AAT@@@1@@Z 100078f0 f i hb-aat-layout.obj
 0001:00006cc0       ??$drive@Udriver_context_t@?$KerxSubTableFormat1@UKerxSubTableHeader@AAT@@@AAT@@@?$StateTableDriver@UExtendedTypes@AAT@@UEntryData@?$Format1Entry@$00@2@@AAT@@QAEXPAUdriver_context_t@?$KerxSubTableFormat1@UKerxSubTableHeader@AAT@@@1@@Z 10007cc0 f i hb-aat-layout.obj
 0001:00007070       ??$drive@Udriver_context_t@?$KerxSubTableFormat4@UKerxSubTableHeader@AAT@@@AAT@@@?$StateTableDriver@UExtendedTypes@AAT@@UEntryData@?$KerxSubTableFormat4@UKerxSubTableHeader@AAT@@@2@@AAT@@QAEXPAUdriver_context_t@?$KerxSubTableFormat4@UKerxSubTableHeader@AAT@@@1@@Z 10008070 f i hb-aat-layout.obj
 0001:00007410       ??$drive@Udriver_context_t@?$LigatureSubtable@UExtendedTypes@AAT@@@AAT@@@?$StateTableDriver@UExtendedTypes@AAT@@UEntryData@?$LigatureEntry@$00@2@@AAT@@QAEXPAUdriver_context_t@?$LigatureSubtable@UExtendedTypes@AAT@@@1@@Z 10008410 f i hb-aat-layout.obj
 0001:000077b0       ??$drive@Udriver_context_t@?$LigatureSubtable@UObsoleteTypes@AAT@@@AAT@@@?$StateTableDriver@UObsoleteTypes@AAT@@X@AAT@@QAEXPAUdriver_context_t@?$LigatureSubtable@UObsoleteTypes@AAT@@@1@@Z 100087b0 f i hb-aat-layout.obj
 0001:00007a90       ??$drive@Udriver_context_t@?$RearrangementSubtable@UExtendedTypes@AAT@@@AAT@@@?$StateTableDriver@UExtendedTypes@AAT@@X@AAT@@QAEXPAUdriver_context_t@?$RearrangementSubtable@UExtendedTypes@AAT@@@1@@Z 10008a90 f i hb-aat-layout.obj
 0001:00007de0       ??$drive@Udriver_context_t@?$RearrangementSubtable@UObsoleteTypes@AAT@@@AAT@@@?$StateTableDriver@UObsoleteTypes@AAT@@X@AAT@@QAEXPAUdriver_context_t@?$RearrangementSubtable@UObsoleteTypes@AAT@@@1@@Z 10008de0 f i hb-aat-layout.obj
 0001:00008150       ??$replace_glyphs@I@hb_buffer_t@@QAE_NIIPBI@Z 10009150 f i hb-aat-layout.obj
 0001:00008200       ??$replace_glyphs@UHBGlyphID16@OT@@@hb_buffer_t@@QAE_NIIPBUHBGlyphID16@OT@@@Z 10009200 f i hb-aat-layout.obj
 0001:000082d0       ??$sanitize@$$V@?$ArrayOf@UHBGlyphID16@OT@@U?$IntType@G$01@2@@OT@@QBE_NPAUhb_sanitize_context_t@@@Z 100092d0 f i hb-aat-layout.obj
 0001:00008310       ??$sanitize@$$V@?$OffsetTo@U?$ArrayOf@UAnchor@AAT@@U?$IntType@I$03@OT@@@OT@@U?$IntType@G$01@2@$0A@@OT@@QBE_NPAUhb_sanitize_context_t@@PBX@Z 10009310 f i hb-aat-layout.obj
 0001:000083f0       ??$sanitize@$$V@?$OffsetTo@U?$ClassTable@U?$IntType@E$00@OT@@@AAT@@U?$IntType@G$01@OT@@$0A@@OT@@QBE_NPAUhb_sanitize_context_t@@PBX@Z 100093f0 f i hb-aat-layout.obj
 0001:00008520       ??$sanitize@$$V@?$OffsetTo@U?$Lookup@U?$IntType@G$01@OT@@@AAT@@U?$IntType@I$03@OT@@$0A@@OT@@QBE_NPAUhb_sanitize_context_t@@PBX@Z 10009520 f i hb-aat-layout.obj
 0001:000085e0       ??$sanitize@$$V@?$OffsetTo@U?$Lookup@U?$IntType@I$03@OT@@@AAT@@U?$IntType@I$03@OT@@$0A@@OT@@QBE_NPAUhb_sanitize_context_t@@PBX@Z 100095e0 f i hb-aat-layout.obj
 0001:000086a0       ??$sanitize@$$V@?$OffsetTo@UClassDef@OT@@U?$IntType@G$01@2@$00@OT@@QBE_NPAUhb_sanitize_context_t@@PBX@Z 100096a0 f i hb-aat-layout.obj
 0001:00008770       ??$sanitize@$$V@?$OffsetTo@UCoverage@OT@@U?$IntType@G$01@2@$00@OT@@QBE_NPAUhb_sanitize_context_t@@PBX@Z 10009770 f i hb-aat-layout.obj
 0001:00008840       ??$sanitize@$$V@?$OffsetTo@UDevice@OT@@U?$IntType@G$01@2@$00@OT@@QBE_NPAUhb_sanitize_context_t@@PBX@Z 10009840 f i hb-aat-layout.obj
 0001:00008910       ??$sanitize@$$V@?$OffsetTo@UVarRegionList@OT@@U?$IntType@I$03@2@$00@OT@@QBE_NPAUhb_sanitize_context_t@@PBX@Z 10009910 f i hb-aat-layout.obj
 0001:00008a90       ??$sanitize@$$V@?$OffsetTo@UVariationStore@OT@@U?$IntType@I$03@2@$00@OT@@QBE_NPAUhb_sanitize_context_t@@PBX@Z 10009a90 f i hb-aat-layout.obj
 0001:00008c10       ??$sanitize@$$V@?$UnsizedListOfOffset16To@U?$Lookup@UHBGlyphID16@OT@@@AAT@@U?$IntType@G$01@OT@@$0A@@OT@@QBE_NPAUhb_sanitize_context_t@@I@Z 10009c10 f i hb-aat-layout.obj
 0001:00008d10       ??$sanitize@$$V@?$UnsizedListOfOffset16To@U?$Lookup@UHBGlyphID16@OT@@@AAT@@U?$IntType@I$03@OT@@$0A@@OT@@QBE_NPAUhb_sanitize_context_t@@I@Z 10009d10 f i hb-aat-layout.obj
 0001:00008e30       ??$sanitize@AAPBX@?$UnsizedArrayOf@U?$OffsetTo@U?$ArrayOf@UAnchor@AAT@@U?$IntType@I$03@OT@@@OT@@U?$IntType@G$01@2@$0A@@OT@@@OT@@QBE_NPAUhb_sanitize_context_t@@IAAPBX@Z 10009e30 f i hb-aat-layout.obj
 0001:00008e90       ??$sanitize@AAPBX@?$VarSizedBinSearchArrayOf@U?$LookupSegmentSingle@U?$OffsetTo@U?$ArrayOf@UAnchor@AAT@@U?$IntType@I$03@OT@@@OT@@U?$IntType@G$01@2@$0A@@OT@@@AAT@@@OT@@QBE_NPAUhb_sanitize_context_t@@AAPBX@Z 10009e90 f i hb-aat-layout.obj
 0001:00009000       ??$sanitize@AAPBX@?$VarSizedBinSearchArrayOf@U?$LookupSingle@U?$OffsetTo@U?$ArrayOf@UAnchor@AAT@@U?$IntType@I$03@OT@@@OT@@U?$IntType@G$01@2@$0A@@OT@@@AAT@@@OT@@QBE_NPAUhb_sanitize_context_t@@AAPBX@Z 1000a000 f i hb-aat-layout.obj
 0001:00009170       ??$sanitize@PBU?$LookupFormat4@U?$IntType@G$01@OT@@@AAT@@@?$VarSizedBinSearchArrayOf@U?$LookupSegmentArray@U?$IntType@G$01@OT@@@AAT@@@OT@@QBE_NPAUhb_sanitize_context_t@@$$QAPBU?$LookupFormat4@U?$IntType@G$01@OT@@@AAT@@@Z 1000a170 f i hb-aat-layout.obj
 0001:00009170       ??$sanitize@PBU?$LookupFormat4@UHBGlyphID16@OT@@@AAT@@@?$VarSizedBinSearchArrayOf@U?$LookupSegmentArray@UHBGlyphID16@OT@@@AAT@@@OT@@QBE_NPAUhb_sanitize_context_t@@$$QAPBU?$LookupFormat4@UHBGlyphID16@OT@@@AAT@@@Z 1000a170 f i hb-aat-layout.obj
 0001:000093a0       ??$sanitize@PBU?$LookupFormat4@U?$IntType@I$03@OT@@@AAT@@@?$VarSizedBinSearchArrayOf@U?$LookupSegmentArray@U?$IntType@I$03@OT@@@AAT@@@OT@@QBE_NPAUhb_sanitize_context_t@@$$QAPBU?$LookupFormat4@U?$IntType@I$03@OT@@@AAT@@@Z 1000a3a0 f i hb-aat-layout.obj
 0001:000095d0       ??$sanitize@PBU?$LookupFormat4@U?$OffsetTo@U?$ArrayOf@UAnchor@AAT@@U?$IntType@I$03@OT@@@OT@@U?$IntType@G$01@2@$0A@@OT@@@AAT@@AAPBX@?$VarSizedBinSearchArrayOf@U?$LookupSegmentArray@U?$OffsetTo@U?$ArrayOf@UAnchor@AAT@@U?$IntType@I$03@OT@@@OT@@U?$IntType@G$01@2@$0A@@OT@@@AAT@@@OT@@QBE_NPAUhb_sanitize_context_t@@$$QAPBU?$LookupFormat4@U?$OffsetTo@U?$ArrayOf@UAnchor@AAT@@U?$IntType@I$03@OT@@@OT@@U?$IntType@G$01@2@$0A@@OT@@@AAT@@AAPBX@Z 1000a5d0 f i hb-aat-layout.obj
 0001:00009800       ??$sanitize@PBUAttachList@OT@@@?$ArrayOf@U?$OffsetTo@UAttachPoint@OT@@U?$IntType@G$01@2@$00@OT@@U?$IntType@G$01@2@@OT@@QBE_NPAUhb_sanitize_context_t@@$$QAPBUAttachList@1@@Z 1000a800 f i hb-aat-layout.obj
 0001:00009960       ??$sanitize@PBULigCaretList@OT@@@?$ArrayOf@U?$OffsetTo@ULigGlyph@OT@@U?$IntType@G$01@2@$00@OT@@U?$IntType@G$01@2@@OT@@QBE_NPAUhb_sanitize_context_t@@$$QAPBULigCaretList@1@@Z 1000a960 f i hb-aat-layout.obj
 0001:00009ab0       ??$sanitize@PBULigGlyph@OT@@@?$ArrayOf@U?$OffsetTo@UCaretValue@OT@@U?$IntType@G$01@2@$00@OT@@U?$IntType@G$01@2@@OT@@QBE_NPAUhb_sanitize_context_t@@$$QAPBULigGlyph@1@@Z 1000aab0 f i hb-aat-layout.obj
 0001:00009bf0       ??$sanitize@PBUMarkGlyphSetsFormat1@OT@@@?$ArrayOf@U?$OffsetTo@UCoverage@OT@@U?$IntType@I$03@2@$00@OT@@U?$IntType@G$01@2@@OT@@QBE_NPAUhb_sanitize_context_t@@$$QAPBUMarkGlyphSetsFormat1@1@@Z 1000abf0 f i hb-aat-layout.obj
 0001:00009d30       ??$sanitize@PBUVariationStore@OT@@@?$ArrayOf@U?$OffsetTo@UVarData@OT@@U?$IntType@I$03@2@$00@OT@@U?$IntType@G$01@2@@OT@@QBE_NPAUhb_sanitize_context_t@@$$QAPBUVariationStore@1@@Z 1000ad30 f i hb-aat-layout.obj
 0001:00009e70       ??$sanitize@PBUtrak@AAT@@@?$OffsetTo@UTrackData@AAT@@U?$IntType@G$01@OT@@$00@OT@@QBE_NPAUhb_sanitize_context_t@@PBX$$QAPBUtrak@AAT@@@Z 1000ae70 f i hb-aat-layout.obj
 0001:00009f50       ??$sanitize_blob@UGDEF@OT@@@hb_sanitize_context_t@@QAEPAUhb_blob_t@@PAU1@@Z 1000af50 f i hb-aat-layout.obj
 0001:0000a0d0       ??$sanitize_blob@Uankr@AAT@@@hb_sanitize_context_t@@QAEPAUhb_blob_t@@PAU1@@Z 1000b0d0 f i hb-aat-layout.obj
 0001:0000a480       ??$sanitize_blob@Ufeat@AAT@@@hb_sanitize_context_t@@QAEPAUhb_blob_t@@PAU1@@Z 1000b480 f i hb-aat-layout.obj
 0001:0000a600       ??$sanitize_blob@Ukerx@AAT@@@hb_sanitize_context_t@@QAEPAUhb_blob_t@@PAU1@@Z 1000b600 f i hb-aat-layout.obj
 0001:0000a780       ??$sanitize_blob@Umort@AAT@@@hb_sanitize_context_t@@QAEPAUhb_blob_t@@PAU1@@Z 1000b780 f i hb-aat-layout.obj
 0001:0000a900       ??$sanitize_blob@Umorx@AAT@@@hb_sanitize_context_t@@QAEPAUhb_blob_t@@PAU1@@Z 1000b900 f i hb-aat-layout.obj
 0001:0000abf0       ??$sanitize_blob@Utrak@AAT@@@hb_sanitize_context_t@@QAEPAUhb_blob_t@@PAU1@@Z 1000bbf0 f i hb-aat-layout.obj
 0001:0000ae20       ??0hb_aat_apply_context_t@AAT@@QAE@PBUhb_ot_shape_plan_t@@PAUhb_font_t@@PAUhb_buffer_t@@PAUhb_blob_t@@@Z 1000be20 f   hb-aat-layout.obj
 0001:0000af10       ??0hb_ot_apply_context_t@OT@@QAE@IPAUhb_font_t@@PAUhb_buffer_t@@@Z 1000bf10 f i hb-aat-layout.obj
 0001:0000b0f0       ??0hb_sanitize_context_t@@QAE@XZ 1000c0f0 f i hb-aat-layout.obj
 0001:0000b140       ??1hb_aat_apply_context_t@AAT@@QAE@XZ 1000c140 f   hb-aat-layout.obj
 0001:0000b190       ??A?$hb_vector_t@I$0A@@@QBEABIH@Z 1000c190 f i hb-aat-layout.obj
 0001:0000b1b0       ?to_int@?$FixedVersion@U?$IntType@G$01@OT@@@OT@@QBEIXZ 1000c1b0 f i hb-aat-layout.obj
 0001:0000b1b0       ??B?$IntType@I$03@OT@@QBEIXZ 1000c1b0 f i hb-aat-layout.obj
 0001:0000b1d0       ??C?$hb_lazy_loader_t@UGDEF_accelerator_t@OT@@U?$hb_face_lazy_loader_t@UGDEF_accelerator_t@OT@@$0BH@@@Uhb_face_t@@$0BH@U12@@@QBEPBUGDEF_accelerator_t@OT@@XZ 1000c1d0 f i hb-aat-layout.obj
 0001:0000b300       ??C?$hb_lazy_loader_t@Ufeat@AAT@@U?$hb_table_lazy_loader_t@Ufeat@AAT@@$0CB@$0A@@@Uhb_face_t@@$0CB@Uhb_blob_t@@@@QBEPBUfeat@AAT@@XZ 1000c300 f i hb-aat-layout.obj
 0001:0000b3e0       ?_infos_find_min_cluster@hb_buffer_t@@SAIPBUhb_glyph_info_t@@III@Z 1000c3e0 f i hb-aat-layout.obj
 0001:0000b420       ?_infos_set_glyph_flags@hb_buffer_t@@QAEXPAUhb_glyph_info_t@@IIII@Z 1000c420 f i hb-aat-layout.obj
 0001:0000b460       ?alloc@?$hb_vector_t@PAUobject_t@hb_serialize_context_t@@$0A@@@QAE_NI@Z 1000c460 f i hb-face.obj
 0001:0000b460       ?alloc@?$hb_vector_t@I$0A@@@QAE_NI@Z 1000c460 f i hb-aat-layout.obj
 0001:0000b460       ?alloc@?$hb_vector_t@PAUchunk_t@?$hb_pool_t@Uobject_t@hb_serialize_context_t@@$0BA@@@$0A@@@QAE_NI@Z 1000c460 f i hb-face.obj
 0001:0000b4d0       ?apply@?$Chain@UExtendedTypes@AAT@@@AAT@@QBEXPAUhb_aat_apply_context_t@2@I@Z 1000c4d0 f i hb-aat-layout.obj
 0001:0000b680       ?apply@?$Chain@UObsoleteTypes@AAT@@@AAT@@QBEXPAUhb_aat_apply_context_t@2@I@Z 1000c680 f i hb-aat-layout.obj
 0001:0000b810       ?apply@?$KerxTable@Ukerx@AAT@@@AAT@@QBE_NPAUhb_aat_apply_context_t@2@@Z 1000c810 f i hb-aat-layout.obj
 0001:0000ba50       ?apply@trak@AAT@@QBE_NPAUhb_aat_apply_context_t@2@@Z 1000ca50 f i hb-aat-layout.obj
 0001:0000bd30       ?backtrack_len@hb_buffer_t@@QBEIXZ 1000cd30 f i hb-aat-layout.obj
 0001:0000bd40       ?check_glyph_property@hb_ot_apply_context_t@OT@@QBE_NPBUhb_glyph_info_t@@I@Z 1000cd40 f i hb-aat-layout.obj
 0001:0000be90       ?check_range@hb_sanitize_context_t@@QBE_NPBXI@Z 1000ce90 f i hb-aat-layout.obj
 0001:0000bf10       ?compile_flags@?$Chain@UExtendedTypes@AAT@@@AAT@@QBEIPBUhb_aat_map_builder_t@@@Z 1000cf10 f i hb-aat-layout.obj
 0001:0000c0b0       ?compile_flags@?$Chain@UObsoleteTypes@AAT@@@AAT@@QBEIPBUhb_aat_map_builder_t@@@Z 1000d0b0 f i hb-aat-layout.obj
 0001:0000c240       ?copy_glyph@hb_buffer_t@@QAE_NXZ 1000d240 f i hb-aat-layout.obj
 0001:0000c2a0       ?create_cache@VariationStore@OT@@QBEPAMXZ 1000d2a0 f i hb-aat-layout.obj
 0001:0000c310       ?em_scale_x@hb_font_t@@QAEHF@Z 1000d310 f i hb-aat-layout.obj
 0001:0000c340       ?em_scale_y@hb_font_t@@QAEHF@Z 1000d340 f i hb-aat-layout.obj
 0001:0000c370       ?em_scalef_x@hb_font_t@@QAEHM@Z 1000d370 f i hb-aat-layout.obj
 0001:0000c3c0       ?em_scalef_y@hb_font_t@@QAEHM@Z 1000d3c0 f i hb-aat-layout.obj
 0001:0000c410       ?end_processing@hb_sanitize_context_t@@QAEXXZ 1000d410 f i hb-aat-layout.obj
 0001:0000c460       ?get@?$hb_lazy_loader_t@Utrak@AAT@@U?$hb_table_lazy_loader_t@Utrak@AAT@@$0BP@$0A@@@Uhb_face_t@@$0BP@Uhb_blob_t@@@@QBEPBUtrak@AAT@@XZ 1000d460 f i hb-aat-layout.obj
 0001:0000c530       ?get_anchor@ankr@AAT@@QBEABUAnchor@2@III@Z 1000d530 f i hb-aat-layout.obj
 0001:0000c5e0       ?get_class@ClassDef@OT@@QBEII@Z 1000d5e0 f i hb-aat-layout.obj
 0001:0000c6c0       ?get_coverage@Coverage@OT@@QBEII@Z 1000d6c0 f i hb-aat-layout.obj
 0001:0000c7e0       ?get_entry@?$StateTable@UExtendedTypes@AAT@@UEntryData@?$InsertionSubtable@UExtendedTypes@AAT@@@2@@AAT@@QBEABU?$Entry@UEntryData@?$InsertionSubtable@UExtendedTypes@AAT@@@AAT@@@2@HI@Z 1000d7e0 f i hb-aat-layout.obj
 0001:0000c7e0       ?get_entry@?$StateTable@UExtendedTypes@AAT@@UEntryData@?$ContextualSubtable@UExtendedTypes@AAT@@@2@@AAT@@QBEABU?$Entry@UEntryData@?$ContextualSubtable@UExtendedTypes@AAT@@@AAT@@@2@HI@Z 1000d7e0 f i hb-aat-layout.obj
 0001:0000c880       ?get_entry@?$StateTable@UExtendedTypes@AAT@@UEntryData@?$Format1Entry@$00@2@@AAT@@QBEABU?$Entry@UEntryData@?$Format1Entry@$00@AAT@@@2@HI@Z 1000d880 f i hb-aat-layout.obj
 0001:0000c880       ?get_entry@?$StateTable@UExtendedTypes@AAT@@UEntryData@?$LigatureEntry@$00@2@@AAT@@QBEABU?$Entry@UEntryData@?$LigatureEntry@$00@AAT@@@2@HI@Z 1000d880 f i hb-aat-layout.obj
 0001:0000c880       ?get_entry@?$StateTable@UExtendedTypes@AAT@@UEntryData@?$KerxSubTableFormat4@UKerxSubTableHeader@AAT@@@2@@AAT@@QBEABU?$Entry@UEntryData@?$KerxSubTableFormat4@UKerxSubTableHeader@AAT@@@AAT@@@2@HI@Z 1000d880 f i hb-aat-layout.obj
 0001:0000c920       ?get_entry@?$StateTable@UExtendedTypes@AAT@@X@AAT@@QBEABU?$Entry@X@2@HI@Z 1000d920 f i hb-aat-layout.obj
 0001:0000c9c0       ?get_feature@feat@AAT@@QBEABUFeatureName@2@W4hb_aat_layout_feature_type_t@@@Z 1000d9c0 f i hb-aat-layout.obj
 0001:0000ca30       ?get_glyph_contour_point_for_origin@hb_font_t@@QAEHIIW4hb_direction_t@@PAH1@Z 1000da30 f i hb-aat-layout.obj
 0001:0000cbe0       ?get_glyph_h_origin_with_fallback@hb_font_t@@QAEXIPAH0@Z 1000dbe0 f i hb-aat-layout.obj
 0001:0000cc70       ?get_glyph_props@GDEF@OT@@QBEII@Z 1000dc70 f i hb-aat-layout.obj
 0001:0000cd20       ?get_glyph_v_origin_with_fallback@hb_font_t@@QAEXIPAH0@Z 1000dd20 f i hb-aat-layout.obj
 0001:0000cdb0       ?get_h_extents_with_fallback@hb_font_t@@QAEXPAUhb_font_extents_t@@@Z 1000ddb0 f i hb-aat-layout.obj
 0001:0000ce10       ?get_kerning@?$KerxSubTableFormat0@UKerxSubTableHeader@AAT@@@AAT@@QBEHIIPAUhb_aat_apply_context_t@2@@Z 1000de10 f i hb-aat-layout.obj
 0001:0000cf40       ?get_kerning@?$KerxSubTableFormat2@UKerxSubTableHeader@AAT@@@AAT@@QBEHIIPAUhb_aat_apply_context_t@2@@Z 1000df40 f i hb-aat-layout.obj
 0001:0000d090       ?get_kerning@?$KerxSubTableFormat6@UKerxSubTableHeader@AAT@@@AAT@@QBEHIIPAUhb_aat_apply_context_t@2@@Z 1000e090 f i hb-aat-layout.obj
 0001:0000d2d0       ?get_length@?$VarSizedBinSearchArrayOf@U?$LookupSegmentSingle@U?$IntType@G$01@OT@@@AAT@@@OT@@QBEIXZ 1000e2d0 f i hb-aat-layout.obj
 0001:0000d2d0       ?get_length@?$VarSizedBinSearchArrayOf@U?$LookupSegmentSingle@U?$OffsetTo@U?$ArrayOf@UAnchor@AAT@@U?$IntType@I$03@OT@@@OT@@U?$IntType@G$01@2@$0A@@OT@@@AAT@@@OT@@QBEIXZ 1000e2d0 f i hb-aat-layout.obj
 0001:0000d2d0       ?get_length@?$VarSizedBinSearchArrayOf@U?$LookupSegmentArray@UHBGlyphID16@OT@@@AAT@@@OT@@QBEIXZ 1000e2d0 f i hb-aat-layout.obj
 0001:0000d2d0       ?get_length@?$VarSizedBinSearchArrayOf@U?$LookupSegmentSingle@UHBGlyphID16@OT@@@AAT@@@OT@@QBEIXZ 1000e2d0 f i hb-aat-layout.obj
 0001:0000d2d0       ?get_length@?$VarSizedBinSearchArrayOf@U?$LookupSegmentSingle@U?$IntType@I$03@OT@@@AAT@@@OT@@QBEIXZ 1000e2d0 f i hb-aat-layout.obj
 0001:0000d2d0       ?get_length@?$VarSizedBinSearchArrayOf@U?$LookupSegmentArray@U?$IntType@I$03@OT@@@AAT@@@OT@@QBEIXZ 1000e2d0 f i hb-aat-layout.obj
 0001:0000d2d0       ?get_length@?$VarSizedBinSearchArrayOf@U?$LookupSegmentArray@U?$IntType@G$01@OT@@@AAT@@@OT@@QBEIXZ 1000e2d0 f i hb-aat-layout.obj
 0001:0000d2d0       ?get_length@?$VarSizedBinSearchArrayOf@U?$LookupSegmentArray@U?$OffsetTo@U?$ArrayOf@UAnchor@AAT@@U?$IntType@I$03@OT@@@OT@@U?$IntType@G$01@2@$0A@@OT@@@AAT@@@OT@@QBEIXZ 1000e2d0 f i hb-aat-layout.obj
 0001:0000d350       ?get_length@?$VarSizedBinSearchArrayOf@U?$LookupSingle@U?$IntType@I$03@OT@@@AAT@@@OT@@QBEIXZ 1000e350 f i hb-aat-layout.obj
 0001:0000d350       ?get_length@?$VarSizedBinSearchArrayOf@U?$LookupSingle@U?$IntType@G$01@OT@@@AAT@@@OT@@QBEIXZ 1000e350 f i hb-aat-layout.obj
 0001:0000d350       ?get_length@?$VarSizedBinSearchArrayOf@U?$LookupSingle@U?$OffsetTo@U?$ArrayOf@UAnchor@AAT@@U?$IntType@I$03@OT@@@OT@@U?$IntType@G$01@2@$0A@@OT@@@AAT@@@OT@@QBEIXZ 1000e350 f i hb-aat-layout.obj
 0001:0000d350       ?get_length@?$VarSizedBinSearchArrayOf@U?$LookupSingle@UHBGlyphID16@OT@@@AAT@@@OT@@QBEIXZ 1000e350 f i hb-aat-layout.obj
 0001:0000d3b0       ?get_row_size@VarData@OT@@QBEIXZ 1000e3b0 f i hb-aat-layout.obj
 0001:0000d400       ?get_size@HintingDevice@OT@@QBEIXZ 1000e400 f i hb-aat-layout.obj
 0001:0000d470       ?get_stored@?$hb_lazy_loader_t@Ukerx@AAT@@U?$hb_table_lazy_loader_t@Ukerx@AAT@@$0BN@$0A@@@Uhb_face_t@@$0BN@Uhb_blob_t@@@@QBEPAUhb_blob_t@@XZ 1000e470 f i hb-aat-layout.obj
 0001:0000d540       ?get_stored@?$hb_lazy_loader_t@Umort@AAT@@U?$hb_table_lazy_loader_t@Umort@AAT@@$0BM@$0A@@@Uhb_face_t@@$0BM@Uhb_blob_t@@@@QBEPAUhb_blob_t@@XZ 1000e540 f i hb-aat-layout.obj
 0001:0000d610       ?get_stored@?$hb_lazy_loader_t@Umorx@AAT@@U?$hb_table_lazy_loader_t@Umorx@AAT@@$0BL@$0A@@@Uhb_face_t@@$0BL@Uhb_blob_t@@@@QBEPAUhb_blob_t@@XZ 1000e610 f i hb-aat-layout.obj
 0001:0000d6e0       ?get_tracking@TrackData@AAT@@QBEHPBXM@Z 1000e6e0 f i hb-aat-layout.obj
 0001:0000d8a0       ?get_value@?$Lookup@U?$IntType@G$01@OT@@@AAT@@QBEPBU?$IntType@G$01@OT@@II@Z 1000e8a0 f i hb-aat-layout.obj
 0001:0000d8a0       ?get_value@?$Lookup@U?$OffsetTo@U?$ArrayOf@UAnchor@AAT@@U?$IntType@I$03@OT@@@OT@@U?$IntType@G$01@2@$0A@@OT@@@AAT@@QBEPBU?$OffsetTo@U?$ArrayOf@UAnchor@AAT@@U?$IntType@I$03@OT@@@OT@@U?$IntType@G$01@2@$0A@@OT@@II@Z 1000e8a0 f i hb-aat-layout.obj
 0001:0000d8a0       ?get_value@?$Lookup@UHBGlyphID16@OT@@@AAT@@QBEPBUHBGlyphID16@OT@@II@Z 1000e8a0 f i hb-aat-layout.obj
 0001:0000daf0       ?get_value@?$Lookup@U?$IntType@I$03@OT@@@AAT@@QBEPBU?$IntType@I$03@OT@@II@Z 1000eaf0 f i hb-aat-layout.obj
 0001:0000dd40       ?get_value_or_null@?$Lookup@U?$IntType@G$01@OT@@@AAT@@QBE?BGII@Z 1000ed40 f i hb-aat-layout.obj
 0001:0000de10       ?get_value_or_null@?$Lookup@U?$IntType@I$03@OT@@@AAT@@QBE?BIII@Z 1000ee10 f i hb-aat-layout.obj
 0001:0000df00       ?guess_v_origin_minus_h_origin@hb_font_t@@QAEXIPAH0@Z 1000ef00 f i hb-aat-layout.obj
 0001:0000dfb0       ?hb_aat_layout_compile_map@@YAXPBUhb_aat_map_builder_t@@PAUhb_aat_map_t@@@Z 1000efb0 f   hb-aat-layout.obj
 0001:0000e140       ?hb_aat_layout_find_feature_mapping@@YAPBUhb_aat_feature_mapping_t@@I@Z 1000f140 f   hb-aat-layout.obj
 0001:0000e190       ?hb_aat_layout_position@@YAXPBUhb_ot_shape_plan_t@@PAUhb_font_t@@PAUhb_buffer_t@@@Z 1000f190 f   hb-aat-layout.obj
 0001:0000e320       ?hb_aat_layout_remove_deleted_glyphs@@YAXPAUhb_buffer_t@@@Z 1000f320 f   hb-aat-layout.obj
 0001:0000e340       ?hb_aat_layout_substitute@@YAXPBUhb_ot_shape_plan_t@@PAUhb_font_t@@PAUhb_buffer_t@@@Z 1000f340 f   hb-aat-layout.obj
 0001:0000e5b0       ?hb_aat_layout_track@@YAXPBUhb_ot_shape_plan_t@@PAUhb_font_t@@PAUhb_buffer_t@@@Z 1000f5b0 f   hb-aat-layout.obj
 0001:0000e630       ?hb_aat_layout_zero_width_deleted_glyphs@@YAXPAUhb_buffer_t@@@Z 1000f630 f   hb-aat-layout.obj
 0001:0000e680       ?init_iters@hb_ot_apply_context_t@OT@@QAEXXZ 1000f680 f i hb-aat-layout.obj
 0001:0000e720       ?interpolate_at@TrackData@AAT@@QBEMIMABUTrackTableEntry@2@PBX@Z 1000f720 f i hb-aat-layout.obj
 0001:0000e890       ?is_actionable@driver_context_t@?$ContextualSubtable@UObsoleteTypes@AAT@@@AAT@@QAE_NPAU?$StateTableDriver@UObsoleteTypes@AAT@@UEntryData@?$ContextualSubtable@UObsoleteTypes@AAT@@@2@@3@ABU?$Entry@UEntryData@?$ContextualSubtable@UObsoleteTypes@AAT@@@AAT@@@3@@Z 1000f890 f i hb-aat-layout.obj
 0001:0000e890       ?is_actionable@driver_context_t@?$ContextualSubtable@UExtendedTypes@AAT@@@AAT@@QAE_NPAU?$StateTableDriver@UExtendedTypes@AAT@@UEntryData@?$ContextualSubtable@UExtendedTypes@AAT@@@2@@3@ABU?$Entry@UEntryData@?$ContextualSubtable@UExtendedTypes@AAT@@@AAT@@@3@@Z 1000f890 f i hb-aat-layout.obj
 0001:0000e900       ?kern@?$hb_kern_machine_t@Uaccelerator_t@?$KerxSubTableFormat0@UKerxSubTableHeader@AAT@@@AAT@@@OT@@QBEXPAUhb_font_t@@PAUhb_buffer_t@@I_N@Z 1000f900 f i hb-aat-layout.obj
 0001:0000ecf0       ?kern@?$hb_kern_machine_t@Uaccelerator_t@?$KerxSubTableFormat2@UKerxSubTableHeader@AAT@@@AAT@@@OT@@QBEXPAUhb_font_t@@PAUhb_buffer_t@@I_N@Z 1000fcf0 f i hb-aat-layout.obj
 0001:0000f0e0       ?kern@?$hb_kern_machine_t@Uaccelerator_t@?$KerxSubTableFormat6@UKerxSubTableHeader@AAT@@@AAT@@@OT@@QBEXPAUhb_font_t@@PAUhb_buffer_t@@I_N@Z 100100e0 f i hb-aat-layout.obj
 0001:0000f530       ?may_edit@hb_sanitize_context_t@@QAE_NPBXI@Z 10010530 f i hb-aat-layout.obj
 0001:0000f590       ?may_skip@matcher_t@hb_ot_apply_context_t@OT@@QBE?AW4may_skip_t@123@PBU23@ABUhb_glyph_info_t@@@Z 10010590 f i hb-aat-layout.obj
 0001:0000f610       ?merge_clusters@hb_buffer_t@@QAEXII@Z 10010610 f i hb-aat-layout.obj
 0001:0000f630       ?message@hb_buffer_t@@QAA_NPAUhb_font_t@@PBDZZ 10010630 f i hb-aat-layout.obj
 0001:0000f670       ?next@skipping_iterator_t@hb_ot_apply_context_t@OT@@QAE_NPAI@Z 10010670 f i hb-aat-layout.obj
 0001:0000f790       ?next_glyph@hb_buffer_t@@QAE_NXZ 10010790 f i hb-aat-layout.obj
 0001:0000f7f0       ?replace_glyph@hb_buffer_t@@QAE_NI@Z 100107f0 f i hb-aat-layout.obj
 0001:0000f860       ?reverse_range@hb_buffer_t@@QAEXII@Z 10010860 f i hb-aat-layout.obj
 0001:0000f930       ?sanitize@?$Chain@UExtendedTypes@AAT@@@AAT@@QBE_NPAUhb_sanitize_context_t@@I@Z 10010930 f i hb-aat-layout.obj
 0001:0000fae0       ?sanitize@?$ChainSubtable@UObsoleteTypes@AAT@@@AAT@@QBE_NPAUhb_sanitize_context_t@@@Z 10010ae0 f i hb-aat-layout.obj
 0001:0000fb60       ?sanitize@?$FixedVersion@U?$IntType@G$01@OT@@@OT@@QBE_NPAUhb_sanitize_context_t@@@Z 10010b60 f i hb-aat-layout.obj
 0001:0000fb60       ?sanitize@?$IntType@H$03@OT@@QBE_NPAUhb_sanitize_context_t@@@Z 10010b60 f i hb-aat-layout.obj
 0001:0000fb60       ?sanitize@?$IntType@I$03@OT@@QBE_NPAUhb_sanitize_context_t@@@Z 10010b60 f i hb-aat-layout.obj
 0001:0000fbe0       ?sanitize@?$IntType@E$00@OT@@QBE_NPAUhb_sanitize_context_t@@@Z 10010be0 f i hb-aat-layout.obj
 0001:0000fc50       ?sanitize@?$IntType@G$01@OT@@QBE_NPAUhb_sanitize_context_t@@@Z 10010c50 f i hb-aat-layout.obj
 0001:0000fc50       ?sanitize@?$IntType@F$01@OT@@QBE_NPAUhb_sanitize_context_t@@@Z 10010c50 f i hb-aat-layout.obj
 0001:0000fcd0       ?sanitize@?$KerxSubTableFormat6@UKerxSubTableHeader@AAT@@@AAT@@QBE_NPAUhb_sanitize_context_t@@@Z 10010cd0 f i hb-aat-layout.obj
 0001:0000fe10       ?sanitize@?$KerxTable@Ukerx@AAT@@@AAT@@QBE_NPAUhb_sanitize_context_t@@@Z 10010e10 f i hb-aat-layout.obj
 0001:0000ff70       ?sanitize@?$Lookup@U?$IntType@G$01@OT@@@AAT@@QBE_NPAUhb_sanitize_context_t@@@Z 10010f70 f i hb-aat-layout.obj
 0001:0000ff70       ?sanitize@?$Lookup@UHBGlyphID16@OT@@@AAT@@QBE_NPAUhb_sanitize_context_t@@@Z 10010f70 f i hb-aat-layout.obj
 0001:000101e0       ?sanitize@?$Lookup@U?$IntType@I$03@OT@@@AAT@@QBE_NPAUhb_sanitize_context_t@@@Z 100111e0 f i hb-aat-layout.obj
 0001:00010460       ?sanitize@?$Lookup@U?$OffsetTo@U?$ArrayOf@UAnchor@AAT@@U?$IntType@I$03@OT@@@OT@@U?$IntType@G$01@2@$0A@@OT@@@AAT@@QBE_NPAUhb_sanitize_context_t@@PBX@Z 10011460 f i hb-aat-layout.obj
 0001:000105f0       ?sanitize@?$StateTable@UExtendedTypes@AAT@@UEntryData@?$ContextualSubtable@UExtendedTypes@AAT@@@2@@AAT@@QBE_NPAUhb_sanitize_context_t@@PAI@Z 100115f0 f i hb-aat-layout.obj
 0001:000105f0       ?sanitize@?$StateTable@UExtendedTypes@AAT@@UEntryData@?$InsertionSubtable@UExtendedTypes@AAT@@@2@@AAT@@QBE_NPAUhb_sanitize_context_t@@PAI@Z 100115f0 f i hb-aat-layout.obj
 0001:00010970       ?sanitize@?$StateTable@UExtendedTypes@AAT@@UEntryData@?$KerxSubTableFormat4@UKerxSubTableHeader@AAT@@@2@@AAT@@QBE_NPAUhb_sanitize_context_t@@PAI@Z 10011970 f i hb-aat-layout.obj
 0001:00010970       ?sanitize@?$StateTable@UExtendedTypes@AAT@@UEntryData@?$LigatureEntry@$00@2@@AAT@@QBE_NPAUhb_sanitize_context_t@@PAI@Z 10011970 f i hb-aat-layout.obj
 0001:00010970       ?sanitize@?$StateTable@UExtendedTypes@AAT@@UEntryData@?$Format1Entry@$00@2@@AAT@@QBE_NPAUhb_sanitize_context_t@@PAI@Z 10011970 f i hb-aat-layout.obj
 0001:00010cf0       ?sanitize@?$StateTable@UExtendedTypes@AAT@@X@AAT@@QBE_NPAUhb_sanitize_context_t@@PAI@Z 10011cf0 f i hb-aat-layout.obj
 0001:00011070       ?sanitize@?$StateTable@UObsoleteTypes@AAT@@UEntryData@?$ContextualSubtable@UObsoleteTypes@AAT@@@2@@AAT@@QBE_NPAUhb_sanitize_context_t@@PAI@Z 10012070 f i hb-aat-layout.obj
 0001:00011070       ?sanitize@?$StateTable@UObsoleteTypes@AAT@@UEntryData@?$InsertionSubtable@UObsoleteTypes@AAT@@@2@@AAT@@QBE_NPAUhb_sanitize_context_t@@PAI@Z 10012070 f i hb-aat-layout.obj
 0001:000113a0       ?sanitize@?$StateTable@UObsoleteTypes@AAT@@X@AAT@@QBE_NPAUhb_sanitize_context_t@@PAI@Z 100123a0 f i hb-aat-layout.obj
 0001:000116d0       ?sanitize@?$mortmorx@UExtendedTypes@AAT@@$0GNGPHCHI@@AAT@@QBE_NPAUhb_sanitize_context_t@@@Z 100126d0 f i hb-aat-layout.obj
 0001:000117a0       ?sanitize@?$mortmorx@UObsoleteTypes@AAT@@$0GNGPHCHE@@AAT@@QBE_NPAUhb_sanitize_context_t@@@Z 100127a0 f i hb-aat-layout.obj
 0001:00011940       ?sanitize@CaretValue@OT@@QBE_NPAUhb_sanitize_context_t@@@Z 10012940 f i hb-aat-layout.obj
 0001:00011a70       ?sanitize@ClassDef@OT@@QBE_NPAUhb_sanitize_context_t@@@Z 10012a70 f i hb-aat-layout.obj
 0001:00011b70       ?sanitize@Device@OT@@QBE_NPAUhb_sanitize_context_t@@@Z 10012b70 f i hb-aat-layout.obj
 0001:00011cb0       ?sanitize@GDEF@OT@@QBE_NPAUhb_sanitize_context_t@@@Z 10012cb0 f i hb-aat-layout.obj
 0001:00011ff0       ?sanitize@SBitLineMetrics@OT@@QBE_NPAUhb_sanitize_context_t@@@Z 10012ff0 f i hb-ot-color.obj
 0001:00011ff0       ?sanitize@KerxSubTableHeader@AAT@@QBE_NPAUhb_sanitize_context_t@@@Z 10012ff0 f i hb-aat-layout.obj
 0001:00012070       ?sanitize@TrackData@AAT@@QBE_NPAUhb_sanitize_context_t@@PBX@Z 10013070 f i hb-aat-layout.obj
 0001:00012210       ?sanitize@TrackTableEntry@AAT@@QBE_NPAUhb_sanitize_context_t@@PBXI@Z 10013210 f i hb-aat-layout.obj
 0001:00012330       ?sanitize@VarData@OT@@QBE_NPAUhb_sanitize_context_t@@@Z 10013330 f i hb-aat-layout.obj
 0001:00012460       ?sanitize@VarSizedBinSearchHeader@OT@@QBE_NPAUhb_sanitize_context_t@@@Z 10013460 f i hb-aat-layout.obj
 0001:000124e0       ?sanitize@VariationStore@OT@@QBE_NPAUhb_sanitize_context_t@@@Z 100134e0 f i hb-aat-layout.obj
 0001:000125a0       ?sanitize@ankr@AAT@@QBE_NPAUhb_sanitize_context_t@@@Z 100135a0 f i hb-aat-layout.obj
 0001:00012750       ?sanitize@feat@AAT@@QBE_NPAUhb_sanitize_context_t@@@Z 10013750 f i hb-aat-layout.obj
 0001:00012910       ?sanitize@trak@AAT@@QBE_NPAUhb_sanitize_context_t@@@Z 10013910 f i hb-aat-layout.obj
 0001:000129e0       ?sanitize_shallow@?$OffsetTo@U?$UnsizedListOfOffset16To@U?$Lookup@UHBGlyphID16@OT@@@AAT@@U?$IntType@G$01@OT@@$0A@@OT@@U?$IntType@G$01@2@$0A@@OT@@QBE_NPAUhb_sanitize_context_t@@PBX@Z 100139e0 f i hb-aat-layout.obj
 0001:00012a70       ?sanitize_shallow@?$OffsetTo@U?$UnsizedListOfOffset16To@U?$Lookup@UHBGlyphID16@OT@@@AAT@@U?$IntType@I$03@OT@@$0A@@OT@@U?$IntType@I$03@2@$0A@@OT@@QBE_NPAUhb_sanitize_context_t@@PBX@Z 10013a70 f i hb-aat-layout.obj
 0001:00012b10       ?start_processing@hb_sanitize_context_t@@QAEXXZ 10013b10 f i hb-aat-layout.obj
 0001:00012b90       ?transition@driver_context_t@?$ContextualSubtable@UExtendedTypes@AAT@@@AAT@@QAEXPAU?$StateTableDriver@UExtendedTypes@AAT@@UEntryData@?$ContextualSubtable@UExtendedTypes@AAT@@@2@@3@ABU?$Entry@UEntryData@?$ContextualSubtable@UExtendedTypes@AAT@@@AAT@@@3@@Z 10013b90 f i hb-aat-layout.obj
 0001:00012dd0       ?transition@driver_context_t@?$ContextualSubtable@UObsoleteTypes@AAT@@@AAT@@QAEXPAU?$StateTableDriver@UObsoleteTypes@AAT@@UEntryData@?$ContextualSubtable@UObsoleteTypes@AAT@@@2@@3@ABU?$Entry@UEntryData@?$ContextualSubtable@UObsoleteTypes@AAT@@@AAT@@@3@@Z 10013dd0 f i hb-aat-layout.obj
 0001:00012ff0       ?transition@driver_context_t@?$InsertionSubtable@UObsoleteTypes@AAT@@@AAT@@QAEXPAU?$StateTableDriver@UObsoleteTypes@AAT@@UEntryData@?$InsertionSubtable@UObsoleteTypes@AAT@@@2@@3@ABU?$Entry@UEntryData@?$InsertionSubtable@UObsoleteTypes@AAT@@@AAT@@@3@@Z 10013ff0 f i hb-aat-layout.obj
 0001:00012ff0       ?transition@driver_context_t@?$InsertionSubtable@UExtendedTypes@AAT@@@AAT@@QAEXPAU?$StateTableDriver@UExtendedTypes@AAT@@UEntryData@?$InsertionSubtable@UExtendedTypes@AAT@@@2@@3@ABU?$Entry@UEntryData@?$InsertionSubtable@UExtendedTypes@AAT@@@AAT@@@3@@Z 10013ff0 f i hb-aat-layout.obj
 0001:00013230       ?transition@driver_context_t@?$KerxSubTableFormat1@UKerxSubTableHeader@AAT@@@AAT@@QAEXPAU?$StateTableDriver@UExtendedTypes@AAT@@UEntryData@?$Format1Entry@$00@2@@3@ABU?$Entry@UEntryData@?$Format1Entry@$00@AAT@@@3@@Z 10014230 f i hb-aat-layout.obj
 0001:000135d0       ?transition@driver_context_t@?$KerxSubTableFormat4@UKerxSubTableHeader@AAT@@@AAT@@QAEXPAU?$StateTableDriver@UExtendedTypes@AAT@@UEntryData@?$KerxSubTableFormat4@UKerxSubTableHeader@AAT@@@2@@3@ABU?$Entry@UEntryData@?$KerxSubTableFormat4@UKerxSubTableHeader@AAT@@@AAT@@@3@@Z 100145d0 f i hb-aat-layout.obj
 0001:00013ad0       ?transition@driver_context_t@?$LigatureSubtable@UExtendedTypes@AAT@@@AAT@@QAEXPAU?$StateTableDriver@UExtendedTypes@AAT@@UEntryData@?$LigatureEntry@$00@2@@3@ABU?$Entry@UEntryData@?$LigatureEntry@$00@AAT@@@3@@Z 10014ad0 f i hb-aat-layout.obj
 0001:00013e70       ?transition@driver_context_t@?$LigatureSubtable@UObsoleteTypes@AAT@@@AAT@@QAEXPAU?$StateTableDriver@UObsoleteTypes@AAT@@X@3@ABU?$Entry@X@3@@Z 10014e70 f i hb-aat-layout.obj
 0001:00014220       ?transition@driver_context_t@?$RearrangementSubtable@UObsoleteTypes@AAT@@@AAT@@QAEXPAU?$StateTableDriver@UObsoleteTypes@AAT@@X@3@ABU?$Entry@X@3@@Z 10015220 f i hb-aat-layout.obj
 0001:00014220       ?transition@driver_context_t@?$RearrangementSubtable@UExtendedTypes@AAT@@@AAT@@QAEXPAU?$StateTableDriver@UExtendedTypes@AAT@@X@3@ABU?$Entry@X@3@@Z 10015220 f i hb-aat-layout.obj
 0001:000144a0       ?unsafe_to_break@hb_buffer_t@@QAEXII@Z 100154a0 f i hb-aat-layout.obj
 0001:000144f0       ?unsafe_to_break_from_outbuffer@hb_buffer_t@@QAEXII@Z 100154f0 f i hb-aat-layout.obj
 0001:00014590       ?unsafe_to_concat@hb_buffer_t@@QAEXII@Z 10015590 f i hb-aat-layout.obj
 0001:000145e0       _hb_aat_layout_has_positioning 100155e0 f   hb-aat-layout.obj
 0001:00014620       _hb_aat_layout_has_substitution 10015620 f   hb-aat-layout.obj
 0001:00014690       _hb_aat_layout_has_tracking 10015690 f   hb-aat-layout.obj
 0001:000149f0       ?add_feature@hb_aat_map_builder_t@@QAEXII@Z 100159f0 f   hb-aat-map.obj
 0001:00014b40       ?cmp@feature_info_t@hb_aat_map_builder_t@@SAHPBX0@Z 10015b40 f i hb-aat-map.obj
 0001:00014bb0       ?compile@hb_aat_map_builder_t@@QAEXAAUhb_aat_map_t@@@Z 10015bb0 f   hb-aat-map.obj
 0001:00014d30       ?push@?$hb_vector_t@Ufeature_info_t@hb_aat_map_builder_t@@$00@@QAEPAUfeature_info_t@hb_aat_map_builder_t@@XZ 10015d30 f i hb-aat-map.obj
 0001:00014de0       _hb_blob_destroy           10015de0 f   hb-blob.obj
 0001:00014e50       ?fini@hb_user_data_array_t@@QAEXXZ 10015e50 f i hb-blob.obj
 0001:00014f50       ?try_make_writable@hb_blob_t@@QAE_NXZ 10015f50 f   hb-blob.obj
 0001:00015010       _hb_blob_create            10016010 f   hb-blob.obj
 0001:00015060       _hb_blob_create_or_fail    10016060 f   hb-blob.obj
 0001:00015100       _hb_blob_create_sub_blob   10016100 f   hb-blob.obj
 0001:00015220       _hb_blob_get_data_writable 10016220 f   hb-blob.obj
 0001:00015260       _hb_blob_get_empty         10016260 f   hb-blob.obj
 0001:00015270       _hb_blob_make_immutable    10016270 f   hb-blob.obj
 0001:00015270       _hb_font_funcs_make_immutable 10016270 f   hb-font.obj
 0001:00015270       _hb_face_make_immutable    10016270 f   hb-face.obj
 0001:00015270       _hb_unicode_funcs_make_immutable 10016270 f   hb-unicode.obj
 0001:00015290       _hb_face_reference         10016290 f   hb-face.obj
 0001:00015290       _hb_unicode_funcs_reference 10016290 f   hb-unicode.obj
 0001:00015290       _hb_blob_reference         10016290 f   hb-blob.obj
 0001:000152b0       ___local_stdio_printf_options 100162b0 f i hb-buffer-serialize.obj
 0001:000152c0       _hb_buffer_serialize_unicode 100162c0 f   hb-buffer-serialize.obj
 0001:000155a0       _snprintf                  100165a0 f i hb-buffer-serialize.obj
 0001:00015c50       ?verify@hb_buffer_t@@QAE_NPAU1@PAUhb_font_t@@PBUhb_feature_t@@IPBQBD@Z 10016c50 f   hb-buffer-verify.obj
 0001:00015dc0       _fprintf                   10016dc0 f i hb-buffer-verify.obj
 0001:00016000       ??$reverse_groups@$$A6A_NABUhb_glyph_info_t@@0@Z@hb_buffer_t@@QAEXA6A_NABUhb_glyph_info_t@@0@Z_N@Z 10017000 f i hb-buffer.obj
 0001:000161a0       ?clear@hb_buffer_t@@QAEXXZ 100171a0 f   hb-buffer.obj
 0001:00016220       ?clear_output@hb_buffer_t@@QAEXXZ 10017220 f   hb-buffer.obj
 0001:00016240       ?clear_positions@hb_buffer_t@@QAEXXZ 10017240 f   hb-buffer.obj
 0001:00016270       ?delete_glyph@hb_buffer_t@@QAEXXZ 10017270 f   hb-buffer.obj
 0001:00016300       ?enlarge@hb_buffer_t@@QAE_NI@Z 10017300 f   hb-buffer.obj
 0001:000163d0       ?ensure@hb_buffer_t@@QAE_NI@Z 100173d0 f i hb-buffer.obj
 0001:000164c0       ?enter@hb_buffer_t@@QAEXXZ 100174c0 f   hb-buffer.obj
 0001:00016520       ?leave@hb_buffer_t@@QAEXXZ 10017520 f   hb-buffer.obj
 0001:00016540       ?make_room_for@hb_buffer_t@@QAE_NII@Z 10017540 f   hb-buffer.obj
 0001:000165a0       ?merge_clusters_impl@hb_buffer_t@@QAEXII@Z 100175a0 f   hb-buffer.obj
 0001:00016730       ?merge_out_clusters@hb_buffer_t@@QAEXII@Z 10017730 f   hb-buffer.obj
 0001:00016880       ?message_impl@hb_buffer_t@@QAE_NPAUhb_font_t@@PBDPAD@Z 10017880 f   hb-buffer.obj
 0001:000168f0       ?move_to@hb_buffer_t@@QAE_NI@Z 100178f0 f   hb-buffer.obj
 0001:00016a40       ?next@?$hb_utf16_xe_t@G@@SAPBGPBG0PAII@Z 10017a40 f i hb-buffer.obj
 0001:00016ab0       ?set_masks@hb_buffer_t@@QAEXIIII@Z 10017ab0 f   hb-buffer.obj
 0001:00016b00       ?sort@hb_buffer_t@@QAEXIIP6AHPBUhb_glyph_info_t@@0@Z@Z 10017b00 f   hb-buffer.obj
 0001:00016bf0       ?sync@hb_buffer_t@@QAEXXZ  10017bf0 f   hb-buffer.obj
 0001:00016c90       _hb_buffer_add_utf16       10017c90 f   hb-buffer.obj
 0001:00016ca0       _hb_buffer_append          10017ca0 f   hb-buffer.obj
 0001:00017020       _hb_buffer_clear_contents  10018020 f   hb-buffer.obj
 0001:00017030       _hb_buffer_create          10018030 f   hb-buffer.obj
 0001:000170c0       _hb_buffer_create_similar  100180c0 f   hb-buffer.obj
 0001:00017190       _hb_buffer_destroy         10018190 f   hb-buffer.obj
 0001:00017210       _hb_buffer_diff            10018210 f   hb-buffer.obj
 0001:00017390       _hb_buffer_get_direction   10018390 f   hb-buffer.obj
 0001:000173a0       _hb_buffer_get_flags       100183a0 f   hb-buffer.obj
 0001:000173b0       _hb_buffer_get_glyph_infos 100183b0 f   hb-buffer.obj
 0001:000173d0       _hb_buffer_get_glyph_positions 100183d0 f   hb-buffer.obj
 0001:00017430       _hb_buffer_get_length      10018430 f   hb-buffer.obj
 0001:00017440       _hb_buffer_get_segment_properties 10018440 f   hb-buffer.obj
 0001:00017460       _hb_buffer_reverse         10018460 f   hb-buffer.obj
 0001:00017470       _hb_buffer_set_cluster_level 10018470 f   hb-buffer.obj
 0001:00017490       _hb_buffer_set_direction   10018490 f   hb-buffer.obj
 0001:000174b0       _hb_buffer_set_flags       100184b0 f   hb-buffer.obj
 0001:000174d0       _hb_buffer_set_language    100184d0 f   hb-buffer.obj
 0001:000174f0       _hb_buffer_set_length      100184f0 f   hb-buffer.obj
 0001:00017590       _hb_buffer_set_script      10018590 f   hb-buffer.obj
 0001:000175b0       _hb_buffer_set_segment_properties 100185b0 f   hb-buffer.obj
 0001:000175d0       _hb_segment_properties_equal 100185d0 f   hb-buffer.obj
 0001:00017610       ??$sanitize_blob@Uhead@OT@@@hb_sanitize_context_t@@QAEPAUhb_blob_t@@PAU1@@Z 10018610 f i hb-common.obj
 0001:00017820       ??$sanitize_blob@Umaxp@OT@@@hb_sanitize_context_t@@QAEPAUhb_blob_t@@PAU1@@Z 10018820 f i hb-common.obj
 0001:00017aa0       ??C?$hb_lazy_loader_t@Umaxp@OT@@U?$hb_table_lazy_loader_t@Umaxp@OT@@$01$00@@Uhb_face_t@@$01Uhb_blob_t@@@@QBEPBUmaxp@OT@@XZ 10018aa0 f i hb-common.obj
 0001:00017b40       ?_hb_options_init@@YAXXZ   10018b40 f   hb-common.obj
 0001:00017be0       ?get@?$hb_lazy_loader_t@Uhead@OT@@U?$hb_table_lazy_loader_t@Uhead@OT@@$00$00@@Uhb_face_t@@$00Uhb_blob_t@@@@QBEPBUhead@OT@@XZ 10018be0 f i hb-common.obj
 0001:00017c80       ?get_blob@?$hb_table_lazy_loader_t@Uloca@OT@@$0O@$00@@QBEPAUhb_blob_t@@XZ 10018c80 f i hb-common.obj
 0001:00017e90       ?load_num_glyphs@hb_face_t@@ABEIXZ 10018e90 f   hb-common.obj
 0001:00017f00       ?load_upem@hb_face_t@@ABEIXZ 10018f00 f   hb-common.obj
 0001:000182f0       ?sanitize@head@OT@@QBE_NPAUhb_sanitize_context_t@@@Z 100192f0 f i hb-common.obj
 0001:000183b0       ?sanitize@maxp@OT@@QBE_NPAUhb_sanitize_context_t@@@Z 100193b0 f i hb-common.obj
 0001:000184d0       _hb_feature_from_string    100194d0 f   hb-common.obj
 0001:00018530       _hb_language_from_string   10019530 f   hb-common.obj
 0001:000185c0       _hb_language_to_string     100195c0 f   hb-common.obj
 0001:000185d0       _hb_script_get_horizontal_direction 100195d0 f   hb-common.obj
 0001:00018750       _hb_tag_from_string        10019750 f   hb-common.obj
 0001:000187e0       _hb_tag_to_string          100197e0 f   hb-common.obj
 0001:000188b0       ?close_path@hb_draw_funcs_t@@QAEXPAXAAUhb_draw_state_t@@@Z 100198b0 f i hb-draw.obj
 0001:00018950       ?cubic_to@hb_draw_funcs_t@@QAEXPAXAAUhb_draw_state_t@@MMMMMM@Z 10019950 f i hb-draw.obj
 0001:00018a20       ?line_to@hb_draw_funcs_t@@QAEXPAXAAUhb_draw_state_t@@MM@Z 10019a20 f i hb-draw.obj
 0001:00018ac0       ?quadratic_to@hb_draw_funcs_t@@QAEXPAXAAUhb_draw_state_t@@MMMM@Z 10019ac0 f i hb-draw.obj
 0001:00018b80       ??$?RPBUobject_t@hb_serialize_context_t@@@<unnamed-type-hb_hash>@@QBEIABQBUobject_t@hb_serialize_context_t@@@Z 10019b80 f i hb-face.obj
 0001:00018c10       ??$bsearch@I@?$SortedArrayOf@UCmapSubtableLongGroup@OT@@U?$IntType@I$03@2@@OT@@QBEABUCmapSubtableLongGroup@1@ABIABU21@@Z 10019c10 f i hb-face.obj
 0001:00018cc0       ??$bsearch@I@?$SortedArrayOf@UVariationSelectorRecord@OT@@U?$IntType@I$03@2@@OT@@QBEABUVariationSelectorRecord@1@ABIABU21@@Z 10019cc0 f i hb-face.obj
 0001:00018d40       ??$get_glyph_from@UCmapSubtable@OT@@@accelerator_t@cmap@OT@@KA_NPBXIPAI@Z 10019d40 f i hb-face.obj
 0001:00018d60       ??$get_glyph_from@UCmapSubtableFormat12@OT@@@accelerator_t@cmap@OT@@KA_NPBXIPAI@Z 10019d60 f i hb-face.obj
 0001:00018e70       ??$propagate_error@AAU?$hb_hashmap_t@PBUobject_t@hb_serialize_context_t@@I$0A@@@@hb_serialize_context_t@@QAE_NAAU?$hb_hashmap_t@PBUobject_t@hb_serialize_context_t@@I$0A@@@@Z 10019e70 f i hb-face.obj
 0001:00018ea0       ??$sanitize@$$V@?$ArrayOf@UCmapSubtableLongGroup@OT@@U?$IntType@I$03@2@@OT@@QBE_NPAUhb_sanitize_context_t@@@Z 10019ea0 f i hb-face.obj
 0001:00018f00       ??$sanitize_blob@UOS2@OT@@@hb_sanitize_context_t@@QAEPAUhb_blob_t@@PAU1@@Z 10019f00 f i hb-face.obj
 0001:00019260       ??$sanitize_blob@Ucmap@OT@@@hb_sanitize_context_t@@QAEPAUhb_blob_t@@PAU1@@Z 1001a260 f i hb-face.obj
 0001:00019580       ??0accelerator_t@cmap@OT@@QAE@PAUhb_face_t@@@Z 1001a580 f i hb-face.obj
 0001:000198e0       ??0hb_serialize_context_t@@QAE@PAXI@Z 1001a8e0 f i hb-face.obj
 0001:00019a60       ??1hb_serialize_context_t@@QAE@XZ 1001aa60 f i hb-face.obj
 0001:00019b10       ??8item_t@?$hb_hashmap_t@PBUobject_t@hb_serialize_context_t@@I$0A@@@QAE_NABQBUobject_t@hb_serialize_context_t@@@Z 1001ab10 f i hb-face.obj
 0001:00019b90       ??A?$ArrayOf@UHBGlyphID16@OT@@U?$IntType@G$01@2@@OT@@QBEABUHBGlyphID16@1@H@Z 1001ab90 f i hb-face.obj
 0001:00019bc0       ??C?$hb_lazy_loader_t@UOS2@OT@@U?$hb_table_lazy_loader_t@UOS2@OT@@$05$0A@@@Uhb_face_t@@$05Uhb_blob_t@@@@QBEPBUOS2@OT@@XZ 1001abc0 f i hb-face.obj
 0001:00019cb0       ??C?$hb_lazy_loader_t@Ucmap_accelerator_t@OT@@U?$hb_face_lazy_loader_t@Ucmap_accelerator_t@OT@@$02@@Uhb_face_t@@$02U12@@@QBEPBUcmap_accelerator_t@OT@@XZ 1001acb0 f i hb-face.obj
 0001:00019e30       ?alloc@?$hb_pool_t@Uobject_t@hb_serialize_context_t@@$0BA@@@QAEPAUobject_t@hb_serialize_context_t@@XZ 1001ae30 f i hb-face.obj
 0001:00019ed0       ?alloc@?$hb_vector_t@Ucontour_point_t@OT@@$0A@@@QAE_NI@Z 1001aed0 f i hb-ot-font.obj
 0001:00019ed0       ?alloc@?$hb_vector_t@Ulink_t@object_t@hb_serialize_context_t@@$0A@@@QAE_NI@Z 1001aed0 f i hb-face.obj
 0001:00019f40       ?bucket_for_hash@?$hb_hashmap_t@PBUobject_t@hb_serialize_context_t@@I$0A@@@IBEIABQBUobject_t@hb_serialize_context_t@@I@Z 1001af40 f i hb-face.obj
 0001:0001a070       ?end_serialize@hb_serialize_context_t@@QAEXXZ 1001b070 f i hb-face.obj
 0001:0001a110       ?find_subtable@cmap@OT@@IBEPBUCmapSubtable@2@II@Z 1001b110 f i hb-face.obj
 0001:0001a2a0       ?fini@?$hb_pool_t@Uobject_t@hb_serialize_context_t@@$0BA@@@QAEXXZ 1001b2a0 f i hb-face.obj
 0001:0001a360       ?fini@hb_serialize_context_t@@QAEXXZ 1001b360 f i hb-face.obj
 0001:0001a520       ?fini@object_t@hb_serialize_context_t@@QAEXXZ 1001b520 f i hb-face.obj
 0001:0001a580       ?get_glyph@?$CmapSubtableLongSegmented@UCmapSubtableFormat12@OT@@@OT@@QBE_NIPAI@Z 1001b580 f i hb-face.obj
 0001:0001a5c0       ?get_glyph@CmapSubtable@OT@@QBE_NIPAI@Z 1001b5c0 f i hb-face.obj
 0001:0001a7c0       ?get_glyph@accelerator_t@CmapSubtableFormat4@OT@@QBE_NIPAI@Z 1001b7c0 f i hb-face.obj
 0001:0001a8e0       ?get_glyph_func@accelerator_t@CmapSubtableFormat4@OT@@SA_NPBXIPAI@Z 1001b8e0 f i hb-face.obj
 0001:0001a900       ?group_get_glyph@CmapSubtableFormat12@OT@@SAIABUCmapSubtableLongGroup@2@I@Z 1001b900 f i hb-face.obj
 0001:0001aa10       ?init@accelerator_t@CmapSubtableFormat4@OT@@QAEXPBU23@@Z 1001ba10 f i hb-face.obj
 0001:0001aa70       ?pop_pack@hb_serialize_context_t@@QAEI_N@Z 1001ba70 f i hb-face.obj
 0001:0001ad70       ?resize@?$hb_hashmap_t@PBUobject_t@hb_serialize_context_t@@I$0A@@@QAE_NI@Z 1001bd70 f i hb-face.obj
 0001:0001b0f0       ?resolve_links@hb_serialize_context_t@@QAEXXZ 1001c0f0 f i hb-face.obj
 0001:0001b420       ?sanitize@CmapSubtable@OT@@QBE_NPAUhb_sanitize_context_t@@@Z 1001c420 f i hb-face.obj
 0001:0001b8d0       ?sanitize@EncodingRecord@OT@@QBE_NPAUhb_sanitize_context_t@@PBX@Z 1001c8d0 f i hb-face.obj
 0001:0001ba10       ?sanitize@OS2@OT@@QBE_NPAUhb_sanitize_context_t@@@Z 1001ca10 f i hb-face.obj
 0001:0001bc10       ?sanitize@VariationSelectorRecord@OT@@QBE_NPAUhb_sanitize_context_t@@PBX@Z 1001cc10 f i hb-face.obj
 0001:0001bea0       ?sanitize@cmap@OT@@QBE_NPAUhb_sanitize_context_t@@@Z 1001cea0 f i hb-face.obj
 0001:0001bfa0       _hb_face_create_for_tables 1001cfa0 f   hb-face.obj
 0001:0001c020       _hb_face_destroy           1001d020 f   hb-face.obj
 0001:0001c0e0       _hb_face_get_empty         1001d0e0 f   hb-face.obj
 0001:0001c0f0       _hb_face_get_glyph_count   1001d0f0 f   hb-face.obj
 0001:0001c110       _hb_face_get_upem          1001d110 f   hb-face.obj
 0001:0001c120       _hb_face_reference_table   1001d120 f   hb-face.obj
 0001:0001c150       __hb_fallback_shape        1001d150 f   hb-fallback-shape.obj
 0001:0001c530       __hb_ot_shaper_face_data_create 1001d530 f   hb-ot-shape.obj
 0001:0001c530       __hb_fallback_shaper_font_data_create 1001d530 f   hb-fallback-shape.obj
 0001:0001c530       __hb_fallback_shaper_face_data_create 1001d530 f   hb-fallback-shape.obj
 0001:0001c530       __hb_ot_shaper_font_data_create 1001d530 f   hb-ot-shape.obj
 0001:0001ccb0       ___scrt_stub_for_is_c_termination_complete 1001dcb0 f   MSVCRT:ucrt_stubs.obj
 0001:0001ccb0       __is_c_termination_complete 1001dcb0 f   MSVCRT:ucrt_stubs.obj
 0001:0001d230       ??$sanitize_blob@Uavar@OT@@@hb_sanitize_context_t@@QAEPAUhb_blob_t@@PAU1@@Z 1001e230 f i hb-font.obj
 0001:0001d5d0       ??$sanitize_blob@Ufvar@OT@@@hb_sanitize_context_t@@QAEPAUhb_blob_t@@PAU1@@Z 1001e5d0 f i hb-font.obj
 0001:0001d9b0       ??C?$hb_lazy_loader_t@Uavar@OT@@U?$hb_table_lazy_loader_t@Uavar@OT@@$0BD@$0A@@@Uhb_face_t@@$0BD@Uhb_blob_t@@@@QBEPBUavar@OT@@XZ 1001e9b0 f i hb-font.obj
 0001:0001db30       ?get@?$hb_lazy_loader_t@Ufvar@OT@@U?$hb_table_lazy_loader_t@Ufvar@OT@@$0BC@$0A@@@Uhb_face_t@@$0BC@Uhb_blob_t@@@@QBEPBUfvar@OT@@XZ 1001eb30 f i hb-font.obj
 0001:0001dc00       ?get_axes@fvar@OT@@QBE?AU?$hb_array_t@$$CBUAxisRecord@OT@@@@XZ 1001ec00 f i hb-font.obj
 0001:0001dc50       ?get_coordinates@AxisRecord@OT@@IBEXAAM00@Z 1001ec50 f i hb-font.obj
 0001:0001dd10       ?get_instance@fvar@OT@@QBEPBUInstanceRecord@2@I@Z 1001ed10 f i hb-font.obj
 0001:0001dd80       ?has_func@hb_font_t@@QAE_NI@Z 1001ed80 f   hb-font.obj
 0001:0001ddc0       ?map@SegmentMaps@OT@@QBEHHII@Z 1001edc0 f i hb-font.obj
 0001:0001e030       ?map_coords@avar@OT@@QBEXPAHI@Z 1001f030 f i hb-font.obj
 0001:0001e090       ?mults_changed@hb_font_t@@QAEXXZ 1001f090 f i hb-font.obj
 0001:0001e1f0       ?parent_scale_position@hb_font_t@@QAEXPAH0@Z 1001f1f0 f i hb-font.obj
 0001:0001e260       ?sanitize@avar@OT@@QBE_NPAUhb_sanitize_context_t@@@Z 1001f260 f i hb-font.obj
 0001:0001e3d0       ?sanitize@fvar@OT@@QBE_NPAUhb_sanitize_context_t@@@Z 1001f3d0 f i hb-font.obj
 0001:0001e540       _hb_font_create            1001f540 f   hb-font.obj
 0001:0001e6b0       _hb_font_destroy           1001f6b0 f   hb-font.obj
 0001:0001e770       _hb_font_funcs_create      1001f770 f   hb-font.obj
 0001:0001e7e0       _hb_font_funcs_destroy     1001f7e0 f   hb-font.obj
 0001:0001ea20       _hb_font_funcs_get_empty   1001fa20 f   hb-font.obj
 0001:0001ea30       _hb_font_funcs_set_font_h_extents_func 1001fa30 f   hb-font.obj
 0001:0001eb20       _hb_font_funcs_set_font_v_extents_func 1001fb20 f   hb-font.obj
 0001:0001ec20       _hb_font_funcs_set_glyph_contour_point_func 1001fc20 f   hb-font.obj
 0001:0001ed20       _hb_font_funcs_set_glyph_extents_func 1001fd20 f   hb-font.obj
 0001:0001ee20       _hb_font_funcs_set_glyph_from_name_func 1001fe20 f   hb-font.obj
 0001:0001ef20       _hb_font_funcs_set_glyph_h_advance_func 1001ff20 f   hb-font.obj
 0001:0001f020       _hb_font_funcs_set_glyph_h_advances_func 10020020 f   hb-font.obj
 0001:0001f120       _hb_font_funcs_set_glyph_h_kerning_func 10020120 f   hb-font.obj
 0001:0001f220       _hb_font_funcs_set_glyph_h_origin_func 10020220 f   hb-font.obj
 0001:0001f320       _hb_font_funcs_set_glyph_name_func 10020320 f   hb-font.obj
 0001:0001f420       _hb_font_funcs_set_glyph_shape_func 10020420 f   hb-font.obj
 0001:0001f520       _hb_font_funcs_set_glyph_v_advance_func 10020520 f   hb-font.obj
 0001:0001f620       _hb_font_funcs_set_glyph_v_advances_func 10020620 f   hb-font.obj
 0001:0001f720       _hb_font_funcs_set_glyph_v_kerning_func 10020720 f   hb-font.obj
 0001:0001f820       _hb_font_funcs_set_glyph_v_origin_func 10020820 f   hb-font.obj
 0001:0001f920       _hb_font_funcs_set_nominal_glyph_func 10020920 f   hb-font.obj
 0001:0001fa20       _hb_font_funcs_set_nominal_glyphs_func 10020a20 f   hb-font.obj
 0001:0001fb20       _hb_font_funcs_set_variation_glyph_func 10020b20 f   hb-font.obj
 0001:0001fc20       _hb_font_get_glyph         10020c20 f   hb-font.obj
 0001:0001fc90       _hb_font_get_glyph_h_advance 10020c90 f   hb-font.obj
 0001:0001fcd0       _hb_font_set_funcs         10020cd0 f   hb-font.obj
 0001:0001fd50       _hb_font_set_scale         10020d50 f   hb-font.obj
 0001:0001fd80       ?CallIntMethod@JNIEnv_@@QAAJPAV_jobject@@PAU_jmethodID@@ZZ 10020d80 f i hb-jdk-font.obj
 0001:0001fda0       ?CallObjectMethod@JNIEnv_@@QAAPAV_jobject@@PAV2@PAU_jmethodID@@ZZ 10020da0 f i hb-jdk-font.obj
 0001:00020110       _Java_sun_font_SunLayoutEngine_createFace@20 10021110 f   hb-jdk-font.obj
 0001:00020190       _Java_sun_font_SunLayoutEngine_disposeFace@16 10021190 f   hb-jdk-font.obj
 0001:000201a0       _hb_jdk_font_create        100211a0 f   hb-jdk-font.obj
 0001:00020310       ?hb_parse_double@@YA_NPAPBDPBDPAN_N@Z 10021310 f   hb-number.obj
 0001:00020360       ?hb_parse_int@@YA_NPAPBDPBDPAH_N@Z 10021360 f   hb-number.obj
 0001:00020730       ??$?0$$CBUaccelerator_t@cff1@OT@@@cff1_cs_interp_env_t@CFF@@QAE@ABU?$hb_array_t@$$CBE@@ABUaccelerator_t@cff1@OT@@I@Z 10021730 f i hb-ot-cff1-table.obj
 0001:00020930       ??$bsearch@I@?$hb_sorted_array_t@$$CBUsid_to_gid_t@@@@QAEPBUsid_to_gid_t@@ABIPBU1@@Z 10021930 f i hb-ot-cff1-table.obj
 0001:000209a0       ??0?$interp_env_t@Unumber_t@CFF@@@CFF@@QAE@ABU?$hb_array_t@$$CBE@@@Z 100219a0 f i hb-ot-cff1-table.obj
 0001:00020a20       ??A?$CFFIndex@U?$IntType@G$01@OT@@@CFF@@QBE?AU?$hb_array_t@$$CBE@@I@Z 10021a20 f i hb-ot-cff1-table.obj
 0001:00020da0       ?avail@byte_str_ref_t@CFF@@QBE_NI@Z 10021da0 f i hb-ot-cff1-table.obj
 0001:00020dc0       ?call_subr@?$cs_interp_env_t@Unumber_t@CFF@@U?$Subrs@U?$IntType@G$01@OT@@@2@@CFF@@QAEXABU?$biased_subrs_t@U?$Subrs@U?$IntType@G$01@OT@@@CFF@@@2@W4cs_type_t@2@@Z 10021dc0 f i hb-ot-cff1-table.obj
 0001:00020f30       ?check_width@?$cff1_cs_opset_t@Ucff1_cs_opset_extents_t@@Ucff1_extents_param_t@@Ucff1_path_procs_extents_t@@@CFF@@SAXIAAUcff1_cs_interp_env_t@2@AAUcff1_extents_param_t@@@Z 10021f30 f i hb-ot-cff1-table.obj
 0001:00020f30       ?check_width@?$cff1_cs_opset_t@Ucff1_cs_opset_path_t@@Ucff1_path_param_t@@Ucff1_path_procs_path_t@@@CFF@@SAXIAAUcff1_cs_interp_env_t@2@AAUcff1_path_param_t@@@Z 10021f30 f i hb-ot-cff1-table.obj
 0001:00020fc0       ?clear_args@?$interp_env_t@Unumber_t@CFF@@@CFF@@QAEXXZ 10021fc0 f i hb-ot-cff1-table.obj
 0001:00020fe0       ?curve@cff1_path_procs_extents_t@@SAXAAUcff1_cs_interp_env_t@CFF@@AAUcff1_extents_param_t@@ABUpoint_t@3@22@Z 10021fe0 f i hb-ot-cff1-table.obj
 0001:000211f0       ?curve@cff1_path_procs_path_t@@SAXAAUcff1_cs_interp_env_t@CFF@@AAUcff1_path_param_t@@ABUpoint_t@3@22@Z 100221f0 f i hb-ot-cff1-table.obj
 0001:00021350       ?fetch_op@?$interp_env_t@Unumber_t@CFF@@@CFF@@QAEIXZ 10022350 f i hb-ot-cff1-table.obj
 0001:000213e0       ?flex1@?$path_procs_t@Ucff1_path_procs_extents_t@@Ucff1_cs_interp_env_t@CFF@@Ucff1_extents_param_t@@@CFF@@SAXAAUcff1_cs_interp_env_t@2@AAUcff1_extents_param_t@@@Z 100223e0 f i hb-ot-cff1-table.obj
 0001:00021790       ?flex1@?$path_procs_t@Ucff1_path_procs_path_t@@Ucff1_cs_interp_env_t@CFF@@Ucff1_path_param_t@@@CFF@@SAXAAUcff1_cs_interp_env_t@2@AAUcff1_path_param_t@@@Z 10022790 f i hb-ot-cff1-table.obj
 0001:00021b40       ?flex@?$path_procs_t@Ucff1_path_procs_extents_t@@Ucff1_cs_interp_env_t@CFF@@Ucff1_extents_param_t@@@CFF@@SAXAAUcff1_cs_interp_env_t@2@AAUcff1_extents_param_t@@@Z 10022b40 f i hb-ot-cff1-table.obj
 0001:00021e10       ?flex@?$path_procs_t@Ucff1_path_procs_path_t@@Ucff1_cs_interp_env_t@CFF@@Ucff1_path_param_t@@@CFF@@SAXAAUcff1_cs_interp_env_t@2@AAUcff1_path_param_t@@@Z 10022e10 f i hb-ot-cff1-table.obj
 0001:000220e0       ?process_post_flex@?$cs_opset_t@Unumber_t@CFF@@Ucff1_cs_opset_extents_t@@Ucff1_cs_interp_env_t@2@Ucff1_extents_param_t@@Ucff1_path_procs_extents_t@@@CFF@@SAXIAAUcff1_cs_interp_env_t@2@AAUcff1_extents_param_t@@@Z 100230e0 f i hb-ot-cff1-table.obj
 0001:000220e0       ?process_post_path@?$cs_opset_t@Unumber_t@CFF@@Ucff1_cs_opset_path_t@@Ucff1_cs_interp_env_t@2@Ucff1_path_param_t@@Ucff1_path_procs_path_t@@@CFF@@SAXIAAUcff1_cs_interp_env_t@2@AAUcff1_path_param_t@@@Z 100230e0 f i hb-ot-cff1-table.obj
 0001:000220e0       ?flush_args_and_op@?$cs_opset_t@Unumber_t@CFF@@Ucff1_cs_opset_path_t@@Ucff1_cs_interp_env_t@2@Ucff1_path_param_t@@Ucff1_path_procs_path_t@@@CFF@@SAXIAAUcff1_cs_interp_env_t@2@AAUcff1_path_param_t@@@Z 100230e0 f i hb-ot-cff1-table.obj
 0001:000220e0       ?flush_args_and_op@?$cs_opset_t@Unumber_t@CFF@@Ucff1_cs_opset_extents_t@@Ucff1_cs_interp_env_t@2@Ucff1_extents_param_t@@Ucff1_path_procs_extents_t@@@CFF@@SAXIAAUcff1_cs_interp_env_t@2@AAUcff1_extents_param_t@@@Z 100230e0 f i hb-ot-cff1-table.obj
 0001:000220e0       ?process_post_flex@?$cs_opset_t@Unumber_t@CFF@@Ucff1_cs_opset_path_t@@Ucff1_cs_interp_env_t@2@Ucff1_path_param_t@@Ucff1_path_procs_path_t@@@CFF@@SAXIAAUcff1_cs_interp_env_t@2@AAUcff1_path_param_t@@@Z 100230e0 f i hb-ot-cff1-table.obj
 0001:000220e0       ?process_post_path@?$cs_opset_t@Unumber_t@CFF@@Ucff1_cs_opset_extents_t@@Ucff1_cs_interp_env_t@2@Ucff1_extents_param_t@@Ucff1_path_procs_extents_t@@@CFF@@SAXIAAUcff1_cs_interp_env_t@2@AAUcff1_extents_param_t@@@Z 100230e0 f i hb-ot-cff1-table.obj
 0001:00022120       ?get_extents@accelerator_t@cff1@OT@@QBE_NPAUhb_font_t@@IPAUhb_glyph_extents_t@@@Z 10023120 f   hb-ot-cff1-table.obj
 0001:000222c0       ?get_fd@FDSelect@CFF@@QBEII@Z 100232c0 f i hb-ot-cff1-table.obj
 0001:00022390       ?get_glyph@Charset@CFF@@QBEIII@Z 10023390 f i hb-ot-cff1-table.obj
 0001:000224d0       ?get_path@accelerator_t@cff1@OT@@QBE_NPAUhb_font_t@@IAAUhb_draw_session_t@@@Z 100234d0 f   hb-ot-cff1-table.obj
 0001:000224f0       ?hflex1@?$path_procs_t@Ucff1_path_procs_extents_t@@Ucff1_cs_interp_env_t@CFF@@Ucff1_extents_param_t@@@CFF@@SAXAAUcff1_cs_interp_env_t@2@AAUcff1_extents_param_t@@@Z 100234f0 f i hb-ot-cff1-table.obj
 0001:00022760       ?hflex1@?$path_procs_t@Ucff1_path_procs_path_t@@Ucff1_cs_interp_env_t@CFF@@Ucff1_path_param_t@@@CFF@@SAXAAUcff1_cs_interp_env_t@2@AAUcff1_path_param_t@@@Z 10023760 f i hb-ot-cff1-table.obj
 0001:000229d0       ?hflex@?$path_procs_t@Ucff1_path_procs_extents_t@@Ucff1_cs_interp_env_t@CFF@@Ucff1_extents_param_t@@@CFF@@SAXAAUcff1_cs_interp_env_t@2@AAUcff1_extents_param_t@@@Z 100239d0 f i hb-ot-cff1-table.obj
 0001:00022bf0       ?hflex@?$path_procs_t@Ucff1_path_procs_path_t@@Ucff1_cs_interp_env_t@CFF@@Ucff1_path_param_t@@@CFF@@SAXAAUcff1_cs_interp_env_t@2@AAUcff1_path_param_t@@@Z 10023bf0 f i hb-ot-cff1-table.obj
 0001:00022e10       ?hhcurveto@?$path_procs_t@Ucff1_path_procs_extents_t@@Ucff1_cs_interp_env_t@CFF@@Ucff1_extents_param_t@@@CFF@@SAXAAUcff1_cs_interp_env_t@2@AAUcff1_extents_param_t@@@Z 10023e10 f i hb-ot-cff1-table.obj
 0001:00023170       ?hhcurveto@?$path_procs_t@Ucff1_path_procs_path_t@@Ucff1_cs_interp_env_t@CFF@@Ucff1_path_param_t@@@CFF@@SAXAAUcff1_cs_interp_env_t@2@AAUcff1_path_param_t@@@Z 10024170 f i hb-ot-cff1-table.obj
 0001:000233c0       ?hlineto@?$path_procs_t@Ucff1_path_procs_extents_t@@Ucff1_cs_interp_env_t@CFF@@Ucff1_extents_param_t@@@CFF@@SAXAAUcff1_cs_interp_env_t@2@AAUcff1_extents_param_t@@@Z 100243c0 f i hb-ot-cff1-table.obj
 0001:00023840       ?hlineto@?$path_procs_t@Ucff1_path_procs_path_t@@Ucff1_cs_interp_env_t@CFF@@Ucff1_path_param_t@@@CFF@@SAXAAUcff1_cs_interp_env_t@2@AAUcff1_path_param_t@@@Z 10024840 f i hb-ot-cff1-table.obj
 0001:00023b00       ?hvcurveto@?$path_procs_t@Ucff1_path_procs_extents_t@@Ucff1_cs_interp_env_t@CFF@@Ucff1_extents_param_t@@@CFF@@SAXAAUcff1_cs_interp_env_t@2@AAUcff1_extents_param_t@@@Z 10024b00 f i hb-ot-cff1-table.obj
 0001:00024840       ?hvcurveto@?$path_procs_t@Ucff1_path_procs_path_t@@Ucff1_cs_interp_env_t@CFF@@Ucff1_path_param_t@@@CFF@@SAXAAUcff1_cs_interp_env_t@2@AAUcff1_path_param_t@@@Z 10025840 f i hb-ot-cff1-table.obj
 0001:00025250       ?in_error@?$interp_env_t@Unumber_t@CFF@@@CFF@@QBE_NXZ 10026250 f i hb-ot-cff1-table.obj
 0001:00025270       ?interpret@?$cs_interpreter_t@Ucff1_cs_interp_env_t@CFF@@Ucff1_cs_opset_extents_t@@Ucff1_extents_param_t@@@CFF@@QAE_NAAUcff1_extents_param_t@@@Z 10026270 f i hb-ot-cff1-table.obj
 0001:00025450       ?interpret@?$cs_interpreter_t@Ucff1_cs_interp_env_t@CFF@@Ucff1_cs_opset_path_t@@Ucff1_path_param_t@@@CFF@@QAE_NAAUcff1_path_param_t@@@Z 10026450 f i hb-ot-cff1-table.obj
 0001:00025630       ?lookup_expert_charset_for_glyph@cff1@OT@@KAII@Z 10026630 f   hb-ot-cff1-table.obj
 0001:00025670       ?lookup_expert_charset_for_sid@cff1@OT@@KAII@Z 10026670 f   hb-ot-cff1-table.obj
 0001:00025690       ?lookup_expert_subset_charset_for_glyph@cff1@OT@@KAII@Z 10026690 f   hb-ot-cff1-table.obj
 0001:000256d0       ?lookup_expert_subset_charset_for_sid@cff1@OT@@KAII@Z 100266d0 f   hb-ot-cff1-table.obj
 0001:000256f0       ?merge@bounds_t@@QAEXABU1@@Z 100266f0 f i hb-ot-cff1-table.obj
 0001:000257a0       ?move_to@hb_draw_session_t@@QAEXMM@Z 100267a0 f i hb-ot-cff1-table.obj
 0001:00025800       ?moveto@cff1_path_procs_path_t@@SAXAAUcff1_cs_interp_env_t@CFF@@AAUcff1_path_param_t@@ABUpoint_t@3@@Z 10026800 f i hb-ot-cff1-table.obj
 0001:000258c0       ?offset_at@?$CFFIndex@U?$IntType@G$01@OT@@@CFF@@ABEII@Z 100268c0 f i hb-ot-cff1-table.obj
 0001:000258f0       ?process_op@?$cs_opset_t@Unumber_t@CFF@@Ucff1_cs_opset_extents_t@@Ucff1_cs_interp_env_t@2@Ucff1_extents_param_t@@Ucff1_path_procs_extents_t@@@CFF@@SAXIAAUcff1_cs_interp_env_t@2@AAUcff1_extents_param_t@@@Z 100268f0 f i hb-ot-cff1-table.obj
 0001:00025f90       ?process_op@?$cs_opset_t@Unumber_t@CFF@@Ucff1_cs_opset_path_t@@Ucff1_cs_interp_env_t@2@Ucff1_path_param_t@@Ucff1_path_procs_path_t@@@CFF@@SAXIAAUcff1_cs_interp_env_t@2@AAUcff1_path_param_t@@@Z 10026f90 f i hb-ot-cff1-table.obj
 0001:000267d0       ?process_op@?$opset_t@Unumber_t@CFF@@@CFF@@SAXIAAU?$interp_env_t@Unumber_t@CFF@@@2@@Z 100277d0 f i hb-ot-cff1-table.obj
 0001:00026ac0       ?process_post_move@?$cs_opset_t@Unumber_t@CFF@@Ucff1_cs_opset_path_t@@Ucff1_cs_interp_env_t@2@Ucff1_path_param_t@@Ucff1_path_procs_path_t@@@CFF@@SAXIAAUcff1_cs_interp_env_t@2@AAUcff1_path_param_t@@@Z 10027ac0 f i hb-ot-cff1-table.obj
 0001:00026ac0       ?process_post_move@?$cs_opset_t@Unumber_t@CFF@@Ucff1_cs_opset_extents_t@@Ucff1_cs_interp_env_t@2@Ucff1_extents_param_t@@Ucff1_path_procs_extents_t@@@CFF@@SAXIAAUcff1_cs_interp_env_t@2@AAUcff1_extents_param_t@@@Z 10027ac0 f i hb-ot-cff1-table.obj
 0001:00026b40       ?process_seac@cff1_cs_opset_extents_t@@SAXAAUcff1_cs_interp_env_t@CFF@@AAUcff1_extents_param_t@@@Z 10027b40 f i hb-ot-cff1-table.obj
 0001:00026dc0       ?process_seac@cff1_cs_opset_path_t@@SAXAAUcff1_cs_interp_env_t@CFF@@AAUcff1_path_param_t@@@Z 10027dc0 f i hb-ot-cff1-table.obj
 0001:00026fb0       ?push_fixed_from_substr@?$arg_stack_t@Unumber_t@CFF@@@CFF@@QAE_NAAUbyte_str_ref_t@2@@Z 10027fb0 f i hb-ot-cff1-table.obj
 0001:00027070       ?rcurveline@?$path_procs_t@Ucff1_path_procs_extents_t@@Ucff1_cs_interp_env_t@CFF@@Ucff1_extents_param_t@@@CFF@@SAXAAUcff1_cs_interp_env_t@2@AAUcff1_extents_param_t@@@Z 10028070 f i hb-ot-cff1-table.obj
 0001:000275a0       ?rcurveline@?$path_procs_t@Ucff1_path_procs_path_t@@Ucff1_cs_interp_env_t@CFF@@Ucff1_path_param_t@@@CFF@@SAXAAUcff1_cs_interp_env_t@2@AAUcff1_path_param_t@@@Z 100285a0 f i hb-ot-cff1-table.obj
 0001:00027970       ?return_from_subr@?$cs_interp_env_t@Unumber_t@CFF@@U?$Subrs@U?$IntType@G$01@OT@@@2@@CFF@@QAEXXZ 10028970 f i hb-ot-cff1-table.obj
 0001:00027970       ?return_from_subr@?$cs_interp_env_t@Unumber_t@CFF@@U?$Subrs@U?$IntType@I$03@OT@@@2@@CFF@@QAEXXZ 10028970 f i hb-ot-cff2-table.obj
 0001:000279f0       ?rlinecurve@?$path_procs_t@Ucff1_path_procs_extents_t@@Ucff1_cs_interp_env_t@CFF@@Ucff1_extents_param_t@@@CFF@@SAXAAUcff1_cs_interp_env_t@2@AAUcff1_extents_param_t@@@Z 100289f0 f i hb-ot-cff1-table.obj
 0001:00027d80       ?rlinecurve@?$path_procs_t@Ucff1_path_procs_path_t@@Ucff1_cs_interp_env_t@CFF@@Ucff1_path_param_t@@@CFF@@SAXAAUcff1_cs_interp_env_t@2@AAUcff1_path_param_t@@@Z 10028d80 f i hb-ot-cff1-table.obj
 0001:00028070       ?rlineto@?$path_procs_t@Ucff1_path_procs_extents_t@@Ucff1_cs_interp_env_t@CFF@@Ucff1_extents_param_t@@@CFF@@SAXAAUcff1_cs_interp_env_t@2@AAUcff1_extents_param_t@@@Z 10029070 f i hb-ot-cff1-table.obj
 0001:00028270       ?rrcurveto@?$path_procs_t@Ucff1_path_procs_extents_t@@Ucff1_cs_interp_env_t@CFF@@Ucff1_extents_param_t@@@CFF@@SAXAAUcff1_cs_interp_env_t@2@AAUcff1_extents_param_t@@@Z 10029270 f i hb-ot-cff1-table.obj
 0001:000285e0       ?rrcurveto@?$path_procs_t@Ucff1_path_procs_path_t@@Ucff1_cs_interp_env_t@CFF@@Ucff1_path_param_t@@@CFF@@SAXAAUcff1_cs_interp_env_t@2@AAUcff1_path_param_t@@@Z 100295e0 f i hb-ot-cff1-table.obj
 0001:00028890       ?set_width@cff1_cs_interp_env_t@CFF@@QAEX_N@Z 10029890 f i hb-ot-cff1-table.obj
 0001:00028900       ?vhcurveto@?$path_procs_t@Ucff1_path_procs_extents_t@@Ucff1_cs_interp_env_t@CFF@@Ucff1_extents_param_t@@@CFF@@SAXAAUcff1_cs_interp_env_t@2@AAUcff1_extents_param_t@@@Z 10029900 f i hb-ot-cff1-table.obj
 0001:00029640       ?vhcurveto@?$path_procs_t@Ucff1_path_procs_path_t@@Ucff1_cs_interp_env_t@CFF@@Ucff1_path_param_t@@@CFF@@SAXAAUcff1_cs_interp_env_t@2@AAUcff1_path_param_t@@@Z 1002a640 f i hb-ot-cff1-table.obj
 0001:0002a040       ?vlineto@?$path_procs_t@Ucff1_path_procs_extents_t@@Ucff1_cs_interp_env_t@CFF@@Ucff1_extents_param_t@@@CFF@@SAXAAUcff1_cs_interp_env_t@2@AAUcff1_extents_param_t@@@Z 1002b040 f i hb-ot-cff1-table.obj
 0001:0002a4c0       ?vlineto@?$path_procs_t@Ucff1_path_procs_path_t@@Ucff1_cs_interp_env_t@CFF@@Ucff1_path_param_t@@@CFF@@SAXAAUcff1_cs_interp_env_t@2@AAUcff1_path_param_t@@@Z 1002b4c0 f i hb-ot-cff1-table.obj
 0001:0002a780       ?vvcurveto@?$path_procs_t@Ucff1_path_procs_extents_t@@Ucff1_cs_interp_env_t@CFF@@Ucff1_extents_param_t@@@CFF@@SAXAAUcff1_cs_interp_env_t@2@AAUcff1_extents_param_t@@@Z 1002b780 f i hb-ot-cff1-table.obj
 0001:0002aae0       ?vvcurveto@?$path_procs_t@Ucff1_path_procs_path_t@@Ucff1_cs_interp_env_t@CFF@@Ucff1_path_param_t@@@CFF@@SAXAAUcff1_cs_interp_env_t@2@AAUcff1_path_param_t@@@Z 1002bae0 f i hb-ot-cff1-table.obj
 0001:0002ad30       ??$?0$$CBUaccelerator_t@cff2@OT@@@?$cff2_cs_interp_env_t@Unumber_t@CFF@@@CFF@@QAE@ABU?$hb_array_t@$$CBE@@ABUaccelerator_t@cff2@OT@@IPBHI@Z 1002bd30 f i hb-ot-cff2-table.obj
 0001:0002aff0       ??A?$ArrayOf@U?$FDSelect3_4_Range@U?$IntType@I$03@OT@@U?$IntType@G$01@2@@CFF@@U?$IntType@I$03@OT@@@OT@@QBEABU?$FDSelect3_4_Range@U?$IntType@I$03@OT@@U?$IntType@G$01@2@@CFF@@H@Z 1002bff0 f i hb-ot-cff2-table.obj
 0001:0002b030       ??A?$CFFIndex@U?$IntType@I$03@OT@@@CFF@@QBE?AU?$hb_array_t@$$CBE@@I@Z 1002c030 f i hb-ot-cff2-table.obj
 0001:0002b190       ?blend_deltas@?$cff2_cs_interp_env_t@Unumber_t@CFF@@@CFF@@QBENU?$hb_array_t@$$CBUnumber_t@CFF@@@@@Z 1002c190 f i hb-ot-cff2-table.obj
 0001:0002b210       ?call_subr@?$cs_interp_env_t@Unumber_t@CFF@@U?$Subrs@U?$IntType@I$03@OT@@@2@@CFF@@QAEXABU?$biased_subrs_t@U?$Subrs@U?$IntType@I$03@OT@@@CFF@@@2@W4cs_type_t@2@@Z 1002c210 f i hb-ot-cff2-table.obj
 0001:0002b3b0       ?curve2@?$path_procs_t@Ucff2_path_procs_path_t@@U?$cff2_cs_interp_env_t@Unumber_t@CFF@@@CFF@@Ucff2_path_param_t@@@CFF@@KAXAAU?$cff2_cs_interp_env_t@Unumber_t@CFF@@@2@AAUcff2_path_param_t@@ABUpoint_t@2@22222@Z 1002c3b0 f i hb-ot-cff2-table.obj
 0001:0002b570       ?curve@cff2_path_procs_extents_t@@SAXAAU?$cff2_cs_interp_env_t@Unumber_t@CFF@@@CFF@@AAUcff2_extents_param_t@@ABUpoint_t@3@22@Z 1002c570 f i hb-ot-cff2-table.obj
 0001:0002b790       ?data_base@?$CFFIndex@U?$IntType@I$03@OT@@@CFF@@ABEPBEXZ 1002c790 f i hb-ot-cff2-table.obj
 0001:0002b7c0       ?flex1@?$path_procs_t@Ucff2_path_procs_extents_t@@U?$cff2_cs_interp_env_t@Unumber_t@CFF@@@CFF@@Ucff2_extents_param_t@@@CFF@@SAXAAU?$cff2_cs_interp_env_t@Unumber_t@CFF@@@2@AAUcff2_extents_param_t@@@Z 1002c7c0 f i hb-ot-cff2-table.obj
 0001:0002bb60       ?flex1@?$path_procs_t@Ucff2_path_procs_path_t@@U?$cff2_cs_interp_env_t@Unumber_t@CFF@@@CFF@@Ucff2_path_param_t@@@CFF@@SAXAAU?$cff2_cs_interp_env_t@Unumber_t@CFF@@@2@AAUcff2_path_param_t@@@Z 1002cb60 f i hb-ot-cff2-table.obj
 0001:0002bf00       ?flex@?$path_procs_t@Ucff2_path_procs_extents_t@@U?$cff2_cs_interp_env_t@Unumber_t@CFF@@@CFF@@Ucff2_extents_param_t@@@CFF@@SAXAAU?$cff2_cs_interp_env_t@Unumber_t@CFF@@@2@AAUcff2_extents_param_t@@@Z 1002cf00 f i hb-ot-cff2-table.obj
 0001:0002c1d0       ?flex@?$path_procs_t@Ucff2_path_procs_path_t@@U?$cff2_cs_interp_env_t@Unumber_t@CFF@@@CFF@@Ucff2_path_param_t@@@CFF@@SAXAAU?$cff2_cs_interp_env_t@Unumber_t@CFF@@@2@AAUcff2_path_param_t@@@Z 1002d1d0 f i hb-ot-cff2-table.obj
 0001:0002c4a0       ?flush_args_and_op@?$cs_opset_t@Unumber_t@CFF@@Ucff2_cs_opset_extents_t@@U?$cff2_cs_interp_env_t@Unumber_t@CFF@@@2@Ucff2_extents_param_t@@Ucff2_path_procs_extents_t@@@CFF@@SAXIAAU?$cff2_cs_interp_env_t@Unumber_t@CFF@@@2@AAUcff2_extents_param_t@@@Z 1002d4a0 f i hb-ot-cff2-table.obj
 0001:0002c4a0       ?process_post_path@?$cs_opset_t@Unumber_t@CFF@@Ucff2_cs_opset_extents_t@@U?$cff2_cs_interp_env_t@Unumber_t@CFF@@@2@Ucff2_extents_param_t@@Ucff2_path_procs_extents_t@@@CFF@@SAXIAAU?$cff2_cs_interp_env_t@Unumber_t@CFF@@@2@AAUcff2_extents_param_t@@@Z 1002d4a0 f i hb-ot-cff2-table.obj
 0001:0002c4a0       ?process_post_path@?$cs_opset_t@Unumber_t@CFF@@Ucff2_cs_opset_path_t@@U?$cff2_cs_interp_env_t@Unumber_t@CFF@@@2@Ucff2_path_param_t@@Ucff2_path_procs_path_t@@@CFF@@SAXIAAU?$cff2_cs_interp_env_t@Unumber_t@CFF@@@2@AAUcff2_path_param_t@@@Z 1002d4a0 f i hb-ot-cff2-table.obj
 0001:0002c4a0       ?flush_args_and_op@?$cs_opset_t@Unumber_t@CFF@@Ucff2_cs_opset_path_t@@U?$cff2_cs_interp_env_t@Unumber_t@CFF@@@2@Ucff2_path_param_t@@Ucff2_path_procs_path_t@@@CFF@@SAXIAAU?$cff2_cs_interp_env_t@Unumber_t@CFF@@@2@AAUcff2_path_param_t@@@Z 1002d4a0 f i hb-ot-cff2-table.obj
 0001:0002c4c0       ?get_extents@accelerator_t@cff2@OT@@QBE_NPAUhb_font_t@@IPAUhb_glyph_extents_t@@@Z 1002d4c0 f   hb-ot-cff2-table.obj
 0001:0002c760       ?get_fd@CFF2FDSelect@CFF@@QBEII@Z 1002d760 f i hb-ot-cff2-table.obj
 0001:0002c960       ?get_path@accelerator_t@cff2@OT@@QBE_NPAUhb_font_t@@IAAUhb_draw_session_t@@@Z 1002d960 f   hb-ot-cff2-table.obj
 0001:0002ca90       ?get_region_scalars@VarData@OT@@QBEXPBHIABUVarRegionList@2@PAMI@Z 1002da90 f i hb-ot-cff2-table.obj
 0001:0002cc60       ?hflex1@?$path_procs_t@Ucff2_path_procs_extents_t@@U?$cff2_cs_interp_env_t@Unumber_t@CFF@@@CFF@@Ucff2_extents_param_t@@@CFF@@SAXAAU?$cff2_cs_interp_env_t@Unumber_t@CFF@@@2@AAUcff2_extents_param_t@@@Z 1002dc60 f i hb-ot-cff2-table.obj
 0001:0002ced0       ?hflex1@?$path_procs_t@Ucff2_path_procs_path_t@@U?$cff2_cs_interp_env_t@Unumber_t@CFF@@@CFF@@Ucff2_path_param_t@@@CFF@@SAXAAU?$cff2_cs_interp_env_t@Unumber_t@CFF@@@2@AAUcff2_path_param_t@@@Z 1002ded0 f i hb-ot-cff2-table.obj
 0001:0002d130       ?hflex@?$path_procs_t@Ucff2_path_procs_extents_t@@U?$cff2_cs_interp_env_t@Unumber_t@CFF@@@CFF@@Ucff2_extents_param_t@@@CFF@@SAXAAU?$cff2_cs_interp_env_t@Unumber_t@CFF@@@2@AAUcff2_extents_param_t@@@Z 1002e130 f i hb-ot-cff2-table.obj
 0001:0002d350       ?hflex@?$path_procs_t@Ucff2_path_procs_path_t@@U?$cff2_cs_interp_env_t@Unumber_t@CFF@@@CFF@@Ucff2_path_param_t@@@CFF@@SAXAAU?$cff2_cs_interp_env_t@Unumber_t@CFF@@@2@AAUcff2_path_param_t@@@Z 1002e350 f i hb-ot-cff2-table.obj
 0001:0002d560       ?hhcurveto@?$path_procs_t@Ucff2_path_procs_extents_t@@U?$cff2_cs_interp_env_t@Unumber_t@CFF@@@CFF@@Ucff2_extents_param_t@@@CFF@@SAXAAU?$cff2_cs_interp_env_t@Unumber_t@CFF@@@2@AAUcff2_extents_param_t@@@Z 1002e560 f i hb-ot-cff2-table.obj
 0001:0002d8d0       ?hhcurveto@?$path_procs_t@Ucff2_path_procs_path_t@@U?$cff2_cs_interp_env_t@Unumber_t@CFF@@@CFF@@Ucff2_path_param_t@@@CFF@@SAXAAU?$cff2_cs_interp_env_t@Unumber_t@CFF@@@2@AAUcff2_path_param_t@@@Z 1002e8d0 f i hb-ot-cff2-table.obj
 0001:0002daf0       ?hlineto@?$path_procs_t@Ucff2_path_procs_extents_t@@U?$cff2_cs_interp_env_t@Unumber_t@CFF@@@CFF@@Ucff2_extents_param_t@@@CFF@@SAXAAU?$cff2_cs_interp_env_t@Unumber_t@CFF@@@2@AAUcff2_extents_param_t@@@Z 1002eaf0 f i hb-ot-cff2-table.obj
 0001:0002df70       ?hlineto@?$path_procs_t@Ucff2_path_procs_path_t@@U?$cff2_cs_interp_env_t@Unumber_t@CFF@@@CFF@@Ucff2_path_param_t@@@CFF@@SAXAAU?$cff2_cs_interp_env_t@Unumber_t@CFF@@@2@AAUcff2_path_param_t@@@Z 1002ef70 f i hb-ot-cff2-table.obj
 0001:0002e1e0       ?hvcurveto@?$path_procs_t@Ucff2_path_procs_extents_t@@U?$cff2_cs_interp_env_t@Unumber_t@CFF@@@CFF@@Ucff2_extents_param_t@@@CFF@@SAXAAU?$cff2_cs_interp_env_t@Unumber_t@CFF@@@2@AAUcff2_extents_param_t@@@Z 1002f1e0 f i hb-ot-cff2-table.obj
 0001:0002ef90       ?hvcurveto@?$path_procs_t@Ucff2_path_procs_path_t@@U?$cff2_cs_interp_env_t@Unumber_t@CFF@@@CFF@@Ucff2_path_param_t@@@CFF@@SAXAAU?$cff2_cs_interp_env_t@Unumber_t@CFF@@@2@AAUcff2_path_param_t@@@Z 1002ff90 f i hb-ot-cff2-table.obj
 0001:0002f8f0       ?in_error@?$cs_interp_env_t@Unumber_t@CFF@@U?$Subrs@U?$IntType@I$03@OT@@@2@@CFF@@QBE_NXZ 100308f0 f i hb-ot-cff2-table.obj
 0001:0002f920       ?offset_at@?$CFFIndex@U?$IntType@I$03@OT@@@CFF@@ABEII@Z 10030920 f i hb-ot-cff2-table.obj
 0001:0002f950       ?pop_uint@?$arg_stack_t@Unumber_t@CFF@@@CFF@@QAEIXZ 10030950 f i hb-ot-cff2-table.obj
 0001:0002f990       ?process_blend@?$cff2_cs_interp_env_t@Unumber_t@CFF@@@CFF@@QAEXXZ 10030990 f i hb-ot-cff2-table.obj
 0001:0002fbf0       ?process_op@?$cff2_cs_opset_t@Ucff2_cs_opset_extents_t@@Ucff2_extents_param_t@@Unumber_t@CFF@@Ucff2_path_procs_extents_t@@@CFF@@SAXIAAU?$cff2_cs_interp_env_t@Unumber_t@CFF@@@2@AAUcff2_extents_param_t@@@Z 10030bf0 f i hb-ot-cff2-table.obj
 0001:0002fde0       ?process_op@?$cff2_cs_opset_t@Ucff2_cs_opset_path_t@@Ucff2_path_param_t@@Unumber_t@CFF@@Ucff2_path_procs_path_t@@@CFF@@SAXIAAU?$cff2_cs_interp_env_t@Unumber_t@CFF@@@2@AAUcff2_path_param_t@@@Z 10030de0 f i hb-ot-cff2-table.obj
 0001:0002ffd0       ?process_op@?$cs_opset_t@Unumber_t@CFF@@Ucff2_cs_opset_extents_t@@U?$cff2_cs_interp_env_t@Unumber_t@CFF@@@2@Ucff2_extents_param_t@@Ucff2_path_procs_extents_t@@@CFF@@SAXIAAU?$cff2_cs_interp_env_t@Unumber_t@CFF@@@2@AAUcff2_extents_param_t@@@Z 10030fd0 f i hb-ot-cff2-table.obj
 0001:000305c0       ?process_op@?$cs_opset_t@Unumber_t@CFF@@Ucff2_cs_opset_path_t@@U?$cff2_cs_interp_env_t@Unumber_t@CFF@@@2@Ucff2_path_param_t@@Ucff2_path_procs_path_t@@@CFF@@SAXIAAU?$cff2_cs_interp_env_t@Unumber_t@CFF@@@2@AAUcff2_path_param_t@@@Z 100315c0 f i hb-ot-cff2-table.obj
 0001:00030e80       ?process_post_move@?$cs_opset_t@Unumber_t@CFF@@Ucff2_cs_opset_extents_t@@U?$cff2_cs_interp_env_t@Unumber_t@CFF@@@2@Ucff2_extents_param_t@@Ucff2_path_procs_extents_t@@@CFF@@SAXIAAU?$cff2_cs_interp_env_t@Unumber_t@CFF@@@2@AAUcff2_extents_param_t@@@Z 10031e80 f i hb-ot-cff2-table.obj
 0001:00030e80       ?process_post_move@?$cs_opset_t@Unumber_t@CFF@@Ucff2_cs_opset_path_t@@U?$cff2_cs_interp_env_t@Unumber_t@CFF@@@2@Ucff2_path_param_t@@Ucff2_path_procs_path_t@@@CFF@@SAXIAAU?$cff2_cs_interp_env_t@Unumber_t@CFF@@@2@AAUcff2_path_param_t@@@Z 10031e80 f i hb-ot-cff2-table.obj
 0001:00030ee0       ?process_vsindex@?$cff2_cs_interp_env_t@Unumber_t@CFF@@@CFF@@QAEXXZ 10031ee0 f i hb-ot-cff2-table.obj
 0001:00030f50       ?rcurveline@?$path_procs_t@Ucff2_path_procs_extents_t@@U?$cff2_cs_interp_env_t@Unumber_t@CFF@@@CFF@@Ucff2_extents_param_t@@@CFF@@SAXAAU?$cff2_cs_interp_env_t@Unumber_t@CFF@@@2@AAUcff2_extents_param_t@@@Z 10031f50 f i hb-ot-cff2-table.obj
 0001:000314b0       ?rcurveline@?$path_procs_t@Ucff2_path_procs_path_t@@U?$cff2_cs_interp_env_t@Unumber_t@CFF@@@CFF@@Ucff2_path_param_t@@@CFF@@SAXAAU?$cff2_cs_interp_env_t@Unumber_t@CFF@@@2@AAUcff2_path_param_t@@@Z 100324b0 f i hb-ot-cff2-table.obj
 0001:00031810       ?rlinecurve@?$path_procs_t@Ucff2_path_procs_extents_t@@U?$cff2_cs_interp_env_t@Unumber_t@CFF@@@CFF@@Ucff2_extents_param_t@@@CFF@@SAXAAU?$cff2_cs_interp_env_t@Unumber_t@CFF@@@2@AAUcff2_extents_param_t@@@Z 10032810 f i hb-ot-cff2-table.obj
 0001:00031b90       ?rlinecurve@?$path_procs_t@Ucff2_path_procs_path_t@@U?$cff2_cs_interp_env_t@Unumber_t@CFF@@@CFF@@Ucff2_path_param_t@@@CFF@@SAXAAU?$cff2_cs_interp_env_t@Unumber_t@CFF@@@2@AAUcff2_path_param_t@@@Z 10032b90 f i hb-ot-cff2-table.obj
 0001:00031ef0       ?rlineto@?$path_procs_t@Ucff2_path_procs_extents_t@@U?$cff2_cs_interp_env_t@Unumber_t@CFF@@@CFF@@Ucff2_extents_param_t@@@CFF@@SAXAAU?$cff2_cs_interp_env_t@Unumber_t@CFF@@@2@AAUcff2_extents_param_t@@@Z 10032ef0 f i hb-ot-cff2-table.obj
 0001:000320f0       ?rrcurveto@?$path_procs_t@Ucff2_path_procs_extents_t@@U?$cff2_cs_interp_env_t@Unumber_t@CFF@@@CFF@@Ucff2_extents_param_t@@@CFF@@SAXAAU?$cff2_cs_interp_env_t@Unumber_t@CFF@@@2@AAUcff2_extents_param_t@@@Z 100330f0 f i hb-ot-cff2-table.obj
 0001:00032480       ?rrcurveto@?$path_procs_t@Ucff2_path_procs_path_t@@U?$cff2_cs_interp_env_t@Unumber_t@CFF@@@CFF@@Ucff2_path_param_t@@@CFF@@SAXAAU?$cff2_cs_interp_env_t@Unumber_t@CFF@@@2@AAUcff2_path_param_t@@@Z 10033480 f i hb-ot-cff2-table.obj
 0001:000326f0       ?vhcurveto@?$path_procs_t@Ucff2_path_procs_extents_t@@U?$cff2_cs_interp_env_t@Unumber_t@CFF@@@CFF@@Ucff2_extents_param_t@@@CFF@@SAXAAU?$cff2_cs_interp_env_t@Unumber_t@CFF@@@2@AAUcff2_extents_param_t@@@Z 100336f0 f i hb-ot-cff2-table.obj
 0001:000334a0       ?vhcurveto@?$path_procs_t@Ucff2_path_procs_path_t@@U?$cff2_cs_interp_env_t@Unumber_t@CFF@@@CFF@@Ucff2_path_param_t@@@CFF@@SAXAAU?$cff2_cs_interp_env_t@Unumber_t@CFF@@@2@AAUcff2_path_param_t@@@Z 100344a0 f i hb-ot-cff2-table.obj
 0001:00033e20       ?vlineto@?$path_procs_t@Ucff2_path_procs_extents_t@@U?$cff2_cs_interp_env_t@Unumber_t@CFF@@@CFF@@Ucff2_extents_param_t@@@CFF@@SAXAAU?$cff2_cs_interp_env_t@Unumber_t@CFF@@@2@AAUcff2_extents_param_t@@@Z 10034e20 f i hb-ot-cff2-table.obj
 0001:000342a0       ?vlineto@?$path_procs_t@Ucff2_path_procs_path_t@@U?$cff2_cs_interp_env_t@Unumber_t@CFF@@@CFF@@Ucff2_path_param_t@@@CFF@@SAXAAU?$cff2_cs_interp_env_t@Unumber_t@CFF@@@2@AAUcff2_path_param_t@@@Z 100352a0 f i hb-ot-cff2-table.obj
 0001:00034510       ?vvcurveto@?$path_procs_t@Ucff2_path_procs_extents_t@@U?$cff2_cs_interp_env_t@Unumber_t@CFF@@@CFF@@Ucff2_extents_param_t@@@CFF@@SAXAAU?$cff2_cs_interp_env_t@Unumber_t@CFF@@@2@AAUcff2_extents_param_t@@@Z 10035510 f i hb-ot-cff2-table.obj
 0001:00034880       ?vvcurveto@?$path_procs_t@Ucff2_path_procs_path_t@@U?$cff2_cs_interp_env_t@Unumber_t@CFF@@@CFF@@Ucff2_path_param_t@@@CFF@@SAXAAU?$cff2_cs_interp_env_t@Unumber_t@CFF@@@2@AAUcff2_path_param_t@@@Z 10035880 f i hb-ot-cff2-table.obj
 0001:00034ab0       ??$sanitize@$$V@?$OffsetTo@UDeltaSetIndexMap@OT@@U?$IntType@I$03@2@$00@OT@@QBE_NPAUhb_sanitize_context_t@@PBX@Z 10035ab0 f i hb-ot-color.obj
 0001:00034b80       ??$sanitize@$$V@?$OffsetTo@USBIXStrike@OT@@U?$IntType@I$03@2@$00@OT@@QBE_NPAUhb_sanitize_context_t@@PBX@Z 10035b80 f i hb-ot-color.obj
 0001:00034ce0       ??$sanitize_blob@UCBDT@OT@@@hb_sanitize_context_t@@QAEPAUhb_blob_t@@PAU1@@Z 10035ce0 f i hb-ot-color.obj
 0001:00034ed0       ??$sanitize_blob@UCBLC@OT@@@hb_sanitize_context_t@@QAEPAUhb_blob_t@@PAU1@@Z 10035ed0 f i hb-ot-color.obj
 0001:00035240       ??$sanitize_blob@Usbix@OT@@@hb_sanitize_context_t@@QAEPAUhb_blob_t@@PAU1@@Z 10036240 f i hb-ot-color.obj
 0001:000355b0       ?choose_strike@CBLC@OT@@IBEABUBitmapSizeTable@2@PAUhb_font_t@@@Z 100365b0 f i hb-ot-color.obj
 0001:00035710       ?choose_strike@accelerator_t@sbix@OT@@ABEABUSBIXStrike@3@PAUhb_font_t@@@Z 10036710 f i hb-ot-color.obj
 0001:000358c0       ?find_table@IndexSubtableArray@OT@@QBEPBUIndexSubtableRecord@2@II@Z 100368c0 f i hb-ot-color.obj
 0001:00035940       ?get_glyph_blob@SBIXStrike@OT@@QBEPAUhb_blob_t@@IPAU3@IPAH1IPAI@Z 10036940 f i hb-ot-color.obj
 0001:00035c40       ?get_image_data@IndexSubtable@OT@@QBE_NIPAI00@Z 10036c40 f i hb-ot-color.obj
 0001:00035e40       ?get_image_data@IndexSubtableRecord@OT@@QBE_NIPBXPAI11@Z 10036e40 f i hb-ot-color.obj
 0001:00035ec0       ?get_strike@sbix@OT@@QBEABUSBIXStrike@2@I@Z 10036ec0 f i hb-ot-color.obj
 0001:00035f60       ?sanitize@BitmapSizeTable@OT@@QBE_NPAUhb_sanitize_context_t@@PBX@Z 10036f60 f i hb-ot-color.obj
 0001:00036100       ?sanitize@CBDT@OT@@QBE_NPAUhb_sanitize_context_t@@@Z 10037100 f i hb-ot-color.obj
 0001:000361a0       ?sanitize@CBLC@OT@@QBE_NPAUhb_sanitize_context_t@@@Z 100371a0 f i hb-ot-color.obj
 0001:000362e0       ?sanitize@DeltaSetIndexMap@OT@@QBE_NPAUhb_sanitize_context_t@@@Z 100372e0 f i hb-ot-color.obj
 0001:00036450       ?sanitize@IndexSubtable@OT@@QBE_NPAUhb_sanitize_context_t@@I@Z 10037450 f i hb-ot-color.obj
 0001:000365e0       ?sanitize@IndexSubtableRecord@OT@@QBE_NPAUhb_sanitize_context_t@@PBX@Z 100375e0 f i hb-ot-color.obj
 0001:00036750       ?sanitize@sbix@OT@@QBE_NPAUhb_sanitize_context_t@@@Z 10037750 f i hb-ot-color.obj
 0001:00036880       ??$shrink_vector@U?$cff1_private_dict_values_base_t@Udict_val_t@CFF@@@CFF@@$0A@@?$hb_vector_t@U?$cff1_private_dict_values_base_t@Udict_val_t@CFF@@@CFF@@$0A@@@QAEXI@Z 10037880 f i hb-ot-face.obj
 0001:000368e0       ??$shrink_vector@Ucff2_font_dict_values_t@CFF@@$0A@@?$hb_vector_t@Ucff2_font_dict_values_t@CFF@@$0A@@@QAEXI@Z 100378e0 f i hb-ot-face.obj
 0001:000368e0       ??$shrink_vector@U?$cff2_private_dict_values_base_t@Udict_val_t@CFF@@@CFF@@$0A@@?$hb_vector_t@U?$cff2_private_dict_values_base_t@Udict_val_t@CFF@@@CFF@@$0A@@@QAEXI@Z 100378e0 f i hb-ot-face.obj
 0001:00036950       ??$shrink_vector@Ucff1_font_dict_values_t@CFF@@$0A@@?$hb_vector_t@Ucff1_font_dict_values_t@CFF@@$0A@@@QAEXI@Z 10037950 f i hb-ot-face.obj
 0001:000369b0       ??1?$accelerator_t@UGPOS@Layout@OT@@@GSUBGPOS@OT@@QAE@XZ 100379b0 f i hb-ot-face.obj
 0001:000369b0       ??1?$accelerator_t@UGSUB@1Layout@OT@@@GSUBGPOS@OT@@QAE@XZ 100379b0 f i hb-ot-face.obj
 0001:00036a30       ??1?$accelerator_templ_t@Ucff1_private_dict_opset_t@CFF@@U?$cff1_private_dict_values_base_t@Udict_val_t@CFF@@@2@@cff1@OT@@QAE@XZ 10037a30 f i hb-ot-face.obj
 0001:00036ad0       ??1?$accelerator_templ_t@Ucff2_private_dict_opset_t@CFF@@U?$cff2_private_dict_values_base_t@Udict_val_t@CFF@@@2@@cff2@OT@@QAE@XZ 10037ad0 f i hb-ot-face.obj
 0001:00036b60       ?_fini@?$accelerator_templ_t@Ucff2_private_dict_opset_t@CFF@@U?$cff2_private_dict_values_base_t@Udict_val_t@CFF@@@2@@cff2@OT@@QAEXXZ 10037b60 f i hb-ot-face.obj
 0001:00036c30       ?fini@?$accelerator_templ_t@Ucff1_private_dict_opset_t@CFF@@U?$cff1_private_dict_values_base_t@Udict_val_t@CFF@@@2@@cff1@OT@@QAEXXZ 10037c30 f i hb-ot-face.obj
 0001:00036d20       ?fini@hb_ot_face_t@@QAEXXZ 10037d20 f   hb-ot-face.obj
 0001:00037440       ?init0@hb_ot_face_t@@QAEXPAUhb_face_t@@@Z 10038440 f   hb-ot-face.obj
 0001:00037450       ??$check_array@U?$IntType@E$00@OT@@@hb_sanitize_context_t@@QBE_NPBU?$IntType@E$00@OT@@II@Z 10038450 f i hb-ot-font.obj
 0001:00037490       ??$get_extents@Uglyf_accelerator_t@OT@@@GlyphHeader@glyf_impl@OT@@QBE_NPAUhb_font_t@@ABUglyf_accelerator_t@2@IPAUhb_glyph_extents_t@@@Z 10038490 f i hb-ot-font.obj
 0001:00037680       ??$get_points@Uglyf_accelerator_t@OT@@@Glyph@glyf_impl@OT@@QBE_NPAUhb_font_t@@ABUglyf_accelerator_t@2@AAUcontour_point_vector_t@2@_NI@Z 10038680 f i hb-ot-font.obj
 0001:00038570       ??$get_points@Upoints_aggregator_t@glyf_accelerator_t@OT@@@glyf_accelerator_t@OT@@IBE_NPAUhb_font_t@@IUpoints_aggregator_t@01@@Z 10039570 f i hb-ot-font.obj
 0001:000388f0       ??$sanitize@Uhb_sanitize_context_t@@@?$hb_array_t@$$CBE@@QBE_NPAUhb_sanitize_context_t@@@Z 100398f0 f i hb-ot-font.obj
 0001:00038920       ??$sanitize_blob@UHVARVVAR@OT@@@hb_sanitize_context_t@@QAEPAUhb_blob_t@@PAU1@@Z 10039920 f i hb-ot-font.obj
 0001:00038c50       ??$sanitize_blob@UVORG@OT@@@hb_sanitize_context_t@@QAEPAUhb_blob_t@@PAU1@@Z 10039c50 f i hb-ot-font.obj
 0001:00038f40       ??$sanitize_blob@Ucff1@OT@@@hb_sanitize_context_t@@QAEPAUhb_blob_t@@PAU1@@Z 10039f40 f i hb-ot-font.obj
 0001:00039110       ??$sanitize_blob@Ucff2@OT@@@hb_sanitize_context_t@@QAEPAUhb_blob_t@@PAU1@@Z 1003a110 f i hb-ot-font.obj
 0001:000392e0       ??$sanitize_blob@Ugvar@OT@@@hb_sanitize_context_t@@QAEPAUhb_blob_t@@PAU1@@Z 1003a2e0 f i hb-ot-font.obj
 0001:00039460       ??$sanitize_blob@Uvhea@OT@@@hb_sanitize_context_t@@QAEPAUhb_blob_t@@PAU1@@Z 1003a460 f i hb-ot-font.obj
 0001:00039460       ??$sanitize_blob@Uhhea@OT@@@hb_sanitize_context_t@@QAEPAUhb_blob_t@@PAU1@@Z 1003a460 f i hb-ot-font.obj
 0001:00039650       ??$sanitize_blob@Upost@OT@@@hb_sanitize_context_t@@QAEPAUhb_blob_t@@PAU1@@Z 1003a650 f i hb-ot-font.obj
 0001:00039cd0       ??0?$accelerator_templ_t@Ucff2_private_dict_opset_t@CFF@@U?$cff2_private_dict_values_base_t@Udict_val_t@CFF@@@2@@cff2@OT@@QAE@PAUhb_face_t@@@Z 1003acd0 f i hb-ot-font.obj
 0001:0003a740       ??0Glyph@glyf_impl@OT@@QAE@U?$hb_array_t@$$CBD@@I@Z 1003b740 f i hb-ot-font.obj
 0001:0003a7a0       ??0accelerator_t@?$hmtxvmtx@Uhmtx@OT@@Uhhea@2@@OT@@QAE@PAUhb_face_t@@@Z 1003b7a0 f i hb-ot-font.obj
 0001:0003a9d0       ??0accelerator_t@?$hmtxvmtx@Uvmtx@OT@@Uvhea@2@@OT@@QAE@PAUhb_face_t@@@Z 1003b9d0 f i hb-ot-font.obj
 0001:0003ac00       ??0accelerator_t@post@OT@@QAE@PAUhb_face_t@@@Z 1003bc00 f i hb-ot-font.obj
 0001:0003ae00       ??0cff1_top_dict_interp_env_t@CFF@@QAE@ABU?$hb_array_t@$$CBE@@@Z 1003be00 f i hb-ot-font.obj
 0001:0003ae30       ??0glyf_accelerator_t@OT@@QAE@PAUhb_face_t@@@Z 1003be30 f i hb-ot-font.obj
 0001:0003b270       ??C?$hb_lazy_loader_t@Ucff1_accelerator_t@OT@@U?$hb_face_lazy_loader_t@Ucff1_accelerator_t@OT@@$0BA@@@Uhb_face_t@@$0BA@U12@@@QBEPBUcff1_accelerator_t@OT@@XZ 1003c270 f i hb-ot-font.obj
 0001:0003b440       ??C?$hb_lazy_loader_t@Ucff2_accelerator_t@OT@@U?$hb_face_lazy_loader_t@Ucff2_accelerator_t@OT@@$0BB@@@Uhb_face_t@@$0BB@U12@@@QBEPBUcff2_accelerator_t@OT@@XZ 1003c440 f i hb-ot-font.obj
 0001:0003b4c0       ??C?$hb_lazy_loader_t@Uglyf_accelerator_t@OT@@U?$hb_face_lazy_loader_t@Uglyf_accelerator_t@OT@@$0P@@@Uhb_face_t@@$0P@U12@@@QBEPBUglyf_accelerator_t@OT@@XZ 1003c4c0 f i hb-ot-font.obj
 0001:0003b540       ??C?$hb_lazy_loader_t@Uhhea@OT@@U?$hb_table_lazy_loader_t@Uhhea@OT@@$03$0A@@@Uhb_face_t@@$03Uhb_blob_t@@@@QBEPBUhhea@OT@@XZ 1003c540 f i hb-ot-font.obj
 0001:0003b610       ??C?$hb_lazy_loader_t@Upost_accelerator_t@OT@@U?$hb_face_lazy_loader_t@Upost_accelerator_t@OT@@$06@@Uhb_face_t@@$06U12@@@QBEPBUpost_accelerator_t@OT@@XZ 1003c610 f i hb-ot-font.obj
 0001:0003b6c0       ??C?$hb_lazy_loader_t@Uvhea@OT@@U?$hb_table_lazy_loader_t@Uvhea@OT@@$0L@$0A@@@Uhb_face_t@@$0L@Uhb_blob_t@@@@QBEPBUvhea@OT@@XZ 1003c6c0 f i hb-ot-font.obj
 0001:0003b790       ?_glyf_get_advance_var@@YAIPAUhb_font_t@@I_N@Z 1003c790 f   hb-ot-font.obj
 0001:0003b9e0       ?add_op@?$parsed_values_t@Udict_val_t@CFF@@@CFF@@QAEXIABUbyte_str_ref_t@2@ABUdict_val_t@2@@Z 1003c9e0 f i hb-ot-font.obj
 0001:0003bae0       ?add_op@?$parsed_values_t@Uop_str_t@CFF@@@CFF@@QAEXIABUbyte_str_ref_t@2@@Z 1003cae0 f i hb-ot-font.obj
 0001:0003bc10       ?apply_deltas_to_points@accelerator_t@gvar@OT@@QBE_NIPAUhb_font_t@@U?$hb_array_t@Ucontour_point_t@OT@@@@@Z 1003cc10 f i hb-ot-font.obj
 0001:0003c9c0       ?calculate_scalar@TupleVariationHeader@OT@@QBEMU?$hb_array_t@H@@IU?$hb_array_t@$$CBUF2DOT14@OT@@@@@Z 1003d9c0 f i hb-ot-font.obj
 0001:0003cce0       ?cmp@gname_t@accelerator_t@cff1@OT@@SAHPBX0@Z 1003dce0 f i hb-ot-font.obj
 0001:0003cd20       ?cmp_gids@accelerator_t@post@OT@@KAHPBX0PAX@Z 1003dd20 f i hb-ot-font.obj
 0001:0003cd80       ?consume_point@path_builder_t@glyf_impl@OT@@QAEXABUcontour_point_t@3@@Z 1003dd80 f i hb-ot-font.obj
 0001:0003d2c0       ?end@?$hb_iter_t@Ucomposite_iter_t@glyf_impl@OT@@ABUCompositeGlyphRecord@23@@@QBE?AUcomposite_iter_t@glyf_impl@OT@@XZ 1003e2c0 f i hb-ot-font.obj
 0001:0003d300       ?extend@contour_point_vector_t@OT@@QAEXABU?$hb_array_t@Ucontour_point_t@OT@@@@@Z 1003e300 f i hb-ot-font.obj
 0001:0003d360       ?find_glyph_name@accelerator_t@post@OT@@IBE?AU?$hb_array_t@$$CBD@@I@Z 1003e360 f i hb-ot-font.obj
 0001:0003d480       ?get@?$hb_lazy_loader_t@Uhmtx_accelerator_t@OT@@U?$hb_face_lazy_loader_t@Uhmtx_accelerator_t@OT@@$04@@Uhb_face_t@@$04U12@@@QBEPBUhmtx_accelerator_t@OT@@XZ 1003e480 f i hb-ot-font.obj
 0001:0003d510       ?get@?$hb_lazy_loader_t@Uvmtx_accelerator_t@OT@@U?$hb_face_lazy_loader_t@Uvmtx_accelerator_t@OT@@$0M@@@Uhb_face_t@@$0M@U12@@@QBEPBUvmtx_accelerator_t@OT@@XZ 1003e510 f i hb-ot-font.obj
 0001:0003d5a0       ?get_advance@accelerator_t@?$hmtxvmtx@Uvmtx@OT@@Uvhea@2@@OT@@QBEII@Z 1003e5a0 f i hb-ot-font.obj
 0001:0003d5a0       ?get_advance@accelerator_t@?$hmtxvmtx@Uhmtx@OT@@Uhhea@2@@OT@@QBEII@Z 1003e5a0 f i hb-ot-font.obj
 0001:0003d660       ?get_advance_var@HVARVVAR@OT@@QBEMIPAUhb_font_t@@PAM@Z 1003e660 f i hb-ot-font.obj
 0001:0003d6e0       ?get_composite_iterator@Glyph@glyf_impl@OT@@QBE?AUcomposite_iter_t@23@XZ 1003e6e0 f i hb-ot-font.obj
 0001:0003d750       ?get_contour_points@SimpleGlyph@glyf_impl@OT@@QBE_NAAUcontour_point_vector_t@3@_N@Z 1003e750 f i hb-ot-font.obj
 0001:0003d940       ?get_delta@VarData@OT@@QBEMIPBHIABUVarRegionList@2@PAM@Z 1003e940 f i hb-ot-font.obj
 0001:0003dfc0       ?get_delta@VariationStore@OT@@QBEMIPBHIPAM@Z 1003efc0 f i hb-ot-font.obj
 0001:0003e070       ?get_extents@SmallGlyphMetrics@OT@@QBEXPAUhb_font_t@@PAUhb_glyph_extents_t@@@Z 1003f070 f i hb-ot-font.obj
 0001:0003e110       ?get_extents@accelerator_t@CBDT@OT@@QBE_NPAUhb_font_t@@IPAUhb_glyph_extents_t@@@Z 1003f110 f i hb-ot-font.obj
 0001:0003e340       ?get_extents@glyf_accelerator_t@OT@@QBE_NPAUhb_font_t@@IPAUhb_glyph_extents_t@@@Z 1003f340 f i hb-ot-font.obj
 0001:0003e400       ?get_glyph@VariationSelectorRecord@OT@@QBE?AW4glyph_variant_t@2@IPAIPBX@Z 1003f400 f i hb-ot-font.obj
 0001:0003e590       ?get_glyph_from_name@accelerator_t@cff1@OT@@QBE_NPBDHPAI@Z 1003f590 f i hb-ot-font.obj
 0001:0003e950       ?get_glyph_from_name@accelerator_t@post@OT@@QBE_NPBDHPAI@Z 1003f950 f i hb-ot-font.obj
 0001:0003eaa0       ?get_offset@gvar@OT@@IBEII@Z 1003faa0 f i hb-ot-font.obj
 0001:0003eb10       ?get_png_extents@accelerator_t@sbix@OT@@ABE_NPAUhb_font_t@@IPAUhb_glyph_extents_t@@@Z 1003fb10 f i hb-ot-font.obj
 0001:0003eeb0       ?get_sid@Charset@CFF@@QBEIII@Z 1003feb0 f i hb-ot-font.obj
 0001:0003efd0       ?get_side_bearing@accelerator_t@?$hmtxvmtx@Uhmtx@OT@@Uhhea@2@@OT@@QBEHI@Z 1003ffd0 f i hb-ot-font.obj
 0001:0003efd0       ?get_side_bearing@accelerator_t@?$hmtxvmtx@Uvmtx@OT@@Uvhea@2@@OT@@QBEHI@Z 1003ffd0 f i hb-ot-font.obj
 0001:0003f060       ?get_side_bearing@accelerator_t@?$hmtxvmtx@Uvmtx@OT@@Uvhea@2@@OT@@QBEHPAUhb_font_t@@I@Z 10040060 f i hb-ot-font.obj
 0001:0003f300       ?get_size@?$CFFIndex@U?$IntType@G$01@OT@@@CFF@@QBEIXZ 10040300 f i hb-ot-font.obj
 0001:0003f360       ?get_transformation@CompositeGlyphRecord@glyf_impl@OT@@IBE_NAAY03MAAUcontour_point_t@3@@Z 10040360 f i hb-ot-font.obj
 0001:0003f590       ?glyph_for_gid@glyf_accelerator_t@OT@@QBE?BUGlyph@glyf_impl@2@I_N@Z 10040590 f i hb-ot-font.obj
 0001:0003f750       ?glyph_to_sid@?$accelerator_templ_t@Ucff1_private_dict_opset_t@CFF@@U?$cff1_private_dict_values_base_t@Udict_val_t@CFF@@@2@@cff1@OT@@QBEII@Z 10040750 f i hb-ot-font.obj
 0001:00040940       ?init@?$accelerator_templ_t@Ucff1_private_dict_opset_t@CFF@@U?$cff1_private_dict_values_base_t@Udict_val_t@CFF@@@2@@cff1@OT@@QAEXPAUhb_face_t@@@Z 10041940 f i hb-ot-font.obj
 0001:00041200       ?init@?$cff1_private_dict_values_base_t@Udict_val_t@CFF@@@CFF@@QAEXXZ 10042200 f i hb-ot-font.obj
 0001:00041230       ?init@cff1_top_dict_values_t@CFF@@QAEXXZ 10042230 f i hb-ot-font.obj
 0001:000412b0       ?interpret@?$dict_interpreter_t@Ucff1_font_dict_opset_t@CFF@@Ucff1_font_dict_values_t@2@U?$interp_env_t@Unumber_t@CFF@@@2@@CFF@@QAE_NAAUcff1_font_dict_values_t@2@@Z 100422b0 f i hb-ot-font.obj
 0001:00041520       ?interpret@?$dict_interpreter_t@Ucff1_private_dict_opset_t@CFF@@U?$cff1_private_dict_values_base_t@Udict_val_t@CFF@@@2@U?$interp_env_t@Unumber_t@CFF@@@2@@CFF@@QAE_NAAU?$cff1_private_dict_values_base_t@Udict_val_t@CFF@@@2@@Z 10042520 f i hb-ot-font.obj
 0001:00041770       ?interpret@?$dict_interpreter_t@Ucff2_font_dict_opset_t@CFF@@Ucff2_font_dict_values_t@2@U?$interp_env_t@Unumber_t@CFF@@@2@@CFF@@QAE_NAAUcff2_font_dict_values_t@2@@Z 10042770 f i hb-ot-font.obj
 0001:00041950       ?interpret@?$dict_interpreter_t@Ucff2_top_dict_opset_t@CFF@@Ucff2_top_dict_values_t@2@U?$interp_env_t@Unumber_t@CFF@@@2@@CFF@@QAE_NAAUcff2_top_dict_values_t@2@@Z 10042950 f i hb-ot-font.obj
 0001:00041c50       ?is_valid@tuple_iterator_t@GlyphVariationData@OT@@QBE_NXZ 10042c50 f i hb-ot-font.obj
 0001:00041ce0       ?iter@CompositeGlyph@glyf_impl@OT@@QBE?AUcomposite_iter_t@23@XZ 10042ce0 f i hb-ot-font.obj
 0001:00041d60       ?map@DeltaSetIndexMap@OT@@QBEII@Z 10042d60 f i hb-ot-font.obj
 0001:00041df0       ?parse_bcd@dict_opset_t@CFF@@SANAAUbyte_str_ref_t@2@@Z 10042df0 f i hb-ot-font.obj
 0001:00041f30       ?process_op@cff1_top_dict_opset_t@CFF@@SAXIAAUcff1_top_dict_interp_env_t@2@AAUcff1_top_dict_values_t@2@@Z 10042f30 f i hb-ot-font.obj
 0001:00042310       ?process_op@cff2_private_dict_opset_t@CFF@@SAXIAAUcff2_priv_dict_interp_env_t@2@AAU?$cff2_private_dict_values_base_t@Udict_val_t@CFF@@@2@@Z 10043310 f i hb-ot-font.obj
 0001:000424f0       ?process_op@dict_opset_t@CFF@@SAXIAAU?$interp_env_t@Unumber_t@CFF@@@2@@Z 100434f0 f i hb-ot-font.obj
 0001:00042640       ?quadratic_to@hb_draw_session_t@@QAEXMMMM@Z 10043640 f i hb-ot-font.obj
 0001:000426b0       ?read_points@SimpleGlyph@glyf_impl@OT@@SA_NAAPBU?$IntType@E$00@3@AAUcontour_point_vector_t@3@PBU43@PQcontour_point_t@3@MW4simple_glyph_flag_t@123@4@Z 100436b0 f i hb-ot-font.obj
 0001:000427b0       ?resize@?$hb_vector_t@H$0A@@@QAE_NH@Z 100437b0 f i hb-ot-font.obj
 0001:00042840       ?resize@?$hb_vector_t@U?$cff1_private_dict_values_base_t@Udict_val_t@CFF@@@CFF@@$0A@@@QAE_NH@Z 10043840 f i hb-ot-font.obj
 0001:000429f0       ?resize@?$hb_vector_t@U?$cff2_private_dict_values_base_t@Udict_val_t@CFF@@@CFF@@$0A@@@QAE_NH@Z 100439f0 f i hb-ot-font.obj
 0001:00042bc0       ?resize@?$hb_vector_t@Ucff1_font_dict_values_t@CFF@@$0A@@@QAE_NH@Z 10043bc0 f i hb-ot-font.obj
 0001:00042d90       ?resize@?$hb_vector_t@Ucff2_font_dict_values_t@CFF@@$0A@@@QAE_NH@Z 10043d90 f i hb-ot-font.obj
 0001:00042f60       ?resize@?$hb_vector_t@Ucontour_point_t@OT@@$0A@@@QAE_NH@Z 10043f60 f i hb-ot-font.obj
 0001:00042fd0       ?sanitize@?$CFFIndex@U?$IntType@G$01@OT@@@CFF@@QBE_NPAUhb_sanitize_context_t@@@Z 10043fd0 f i hb-ot-font.obj
 0001:000430e0       ?sanitize@?$CFFIndex@U?$IntType@I$03@OT@@@CFF@@QBE_NPAUhb_sanitize_context_t@@@Z 100440e0 f i hb-ot-font.obj
 0001:000431f0       ?sanitize@?$FDSelect3_4@U?$IntType@G$01@OT@@U?$IntType@E$00@2@@CFF@@QBE_NPAUhb_sanitize_context_t@@I@Z 100441f0 f i hb-ot-font.obj
 0001:00043450       ?sanitize@?$FDSelect3_4@U?$IntType@I$03@OT@@U?$IntType@G$01@2@@CFF@@QBE_NPAUhb_sanitize_context_t@@I@Z 10044450 f i hb-ot-font.obj
 0001:00043710       ?sanitize@?$_hea@Uvhea@OT@@@OT@@QBE_NPAUhb_sanitize_context_t@@@Z 10044710 f i hb-ot-font.obj
 0001:00043710       ?sanitize@?$_hea@Uhhea@OT@@@OT@@QBE_NPAUhb_sanitize_context_t@@@Z 10044710 f i hb-ot-font.obj
 0001:000437b0       ?sanitize@Charset@CFF@@QBE_NPAUhb_sanitize_context_t@@@Z 100447b0 f i hb-ot-font.obj
 0001:00043a20       ?sanitize@Encoding@CFF@@QBE_NPAUhb_sanitize_context_t@@@Z 10044a20 f i hb-ot-font.obj
 0001:00043b20       ?sanitize@FDSelect0@CFF@@QBE_NPAUhb_sanitize_context_t@@I@Z 10044b20 f i hb-ot-font.obj
 0001:00043b90       ?sanitize@HVARVVAR@OT@@QBE_NPAUhb_sanitize_context_t@@@Z 10044b90 f i hb-ot-font.obj
 0001:00043cc0       ?sanitize@VORG@OT@@QBE_NPAUhb_sanitize_context_t@@@Z 10044cc0 f i hb-ot-font.obj
 0001:00043d90       ?sanitize@cff1@OT@@QBE_NPAUhb_sanitize_context_t@@@Z 10044d90 f i hb-ot-font.obj
 0001:00043e10       ?sanitize@cff2@OT@@QBE_NPAUhb_sanitize_context_t@@@Z 10044e10 f i hb-ot-font.obj
 0001:00043e90       ?sanitize@post@OT@@QBE_NPAUhb_sanitize_context_t@@@Z 10044e90 f i hb-ot-font.obj
 0001:00043fb0       ?sanitize_shallow@gvar@OT@@QBE_NPAUhb_sanitize_context_t@@@Z 10044fb0 f i hb-ot-font.obj
 0001:00044160       ?sentinel@?$FDSelect3_4@U?$IntType@I$03@OT@@U?$IntType@G$01@2@@CFF@@QBEABU?$IntType@I$03@OT@@XZ 10045160 f i hb-ot-font.obj
 0001:000441b0       ?set_current@composite_iter_t@glyf_impl@OT@@QAEXPBUCompositeGlyphRecord@23@@Z 100451b0 f i hb-ot-font.obj
 0001:00044210       ?suppEncData@Encoding@CFF@@IBEABUCFF1SuppEncData@2@XZ 10045210 f i hb-ot-font.obj
 0001:00044260       ?translate@contour_point_vector_t@OT@@QAEXABUcontour_point_t@2@@Z 10045260 f i hb-ot-font.obj
 0001:00044370       ?trim_padding@SimpleGlyph@glyf_impl@OT@@QBE?BU?$hb_array_t@$$CBD@@XZ 10045370 f i hb-ot-font.obj
 0001:000444d0       ?unpack_deltas@GlyphVariationData@OT@@SA_NAAPBU?$IntType@E$00@2@AAU?$hb_vector_t@H$0A@@@PBU32@@Z 100454d0 f i hb-ot-font.obj
 0001:00044620       ?unpack_points@GlyphVariationData@OT@@SA_NAAPBU?$IntType@E$00@2@AAU?$hb_vector_t@I$0A@@@PBU32@@Z 10045620 f i hb-ot-font.obj
 0001:000447b0       _hb_ot_font_set_funcs      100457b0 f   hb-ot-font.obj
 0001:00044910       ??$?HPBUMarkMarkPosFormat1@GPOS_impl@Layout@OT@@$0A@@OT@@YAABUAnchorMatrix@GPOS_impl@Layout@0@ABQBUMarkMarkPosFormat1@230@ABU?$OffsetTo@UAnchorMatrix@GPOS_impl@Layout@OT@@U?$IntType@G$01@4@$00@0@@Z 10045910 f i hb-ot-layout.obj
 0001:00044910       ??$?HPBUMarkMarkPosFormat1@GPOS_impl@Layout@OT@@$0A@@OT@@YAABUCoverage@0@ABQBUMarkMarkPosFormat1@GPOS_impl@Layout@0@ABU?$OffsetTo@UCoverage@OT@@U?$IntType@G$01@2@$00@0@@Z 10045910 f i hb-ot-layout.obj
 0001:00044910       ??$?HPBUMarkLigPosFormat1@GPOS_impl@Layout@OT@@$0A@@OT@@YAABUMarkArray@GPOS_impl@Layout@0@ABQBUMarkLigPosFormat1@230@ABU?$OffsetTo@UMarkArray@GPOS_impl@Layout@OT@@U?$IntType@G$01@4@$00@0@@Z 10045910 f i hb-ot-layout.obj
 0001:00044910       ??$?HPBX$0A@@OT@@YAABUDevice@0@ABQBXABU?$OffsetTo@UDevice@OT@@U?$IntType@G$01@2@$00@0@@Z 10045910 f i hb-ot-layout.obj
 0001:00044910       ??$?HPBUMarkMarkPosFormat1@GPOS_impl@Layout@OT@@$0A@@OT@@YAABUMarkArray@GPOS_impl@Layout@0@ABQBUMarkMarkPosFormat1@230@ABU?$OffsetTo@UMarkArray@GPOS_impl@Layout@OT@@U?$IntType@G$01@4@$00@0@@Z 10045910 f i hb-ot-layout.obj
 0001:00044940       ??$_dispatch@U?$OffsetTo@ULigature@GSUB@Layout@OT@@U?$IntType@G$01@4@$00@OT@@PBULigatureSet@GSUB@Layout@2@@hb_sanitize_context_t@@AAE_NABU?$OffsetTo@ULigature@GSUB@Layout@OT@@U?$IntType@G$01@4@$00@OT@@U?$hb_priority@$00@@$$QAPBULigatureSet@GSUB@Layout@2@@Z 10045940 f i hb-ot-layout.obj
 0001:00044a60       ??$_dispatch@UContextFormat3@OT@@$$V@hb_sanitize_context_t@@AAE_NABUContextFormat3@OT@@U?$hb_priority@$00@@@Z 10045a60 f i hb-ot-layout.obj
 0001:00044b80       ??$_dispatch@UPairSet@GPOS_impl@Layout@OT@@PAUsanitize_closure_t@1234@@hb_sanitize_context_t@@AAE_NABUPairSet@GPOS_impl@Layout@OT@@U?$hb_priority@$00@@$$QAPAUsanitize_closure_t@1234@@Z 10045b80 f i hb-ot-layout.obj
 0001:00044c90       ??$apply@UGPOSProxy@@@hb_ot_map_t@@QBEXABUGPOSProxy@@PBUhb_ot_shape_plan_t@@PAUhb_font_t@@PAUhb_buffer_t@@@Z 10045c90 f i hb-ot-layout.obj
 0001:00044f20       ??$apply@UGSUBProxy@@@hb_ot_map_t@@QBEXABUGSUBProxy@@PBUhb_ot_shape_plan_t@@PAUhb_font_t@@PAUhb_buffer_t@@@Z 10045f20 f i hb-ot-layout.obj
 0001:00045220       ??$apply_cached_to@UAlternateSubstFormat1@GSUB@Layout@OT@@@hb_accelerate_subtables_context_t@OT@@SA_NPBXPAUhb_ot_apply_context_t@1@@Z 10046220 f i hb-ot-layout.obj
 0001:00045220       ??$apply_to@UAlternateSubstFormat1@GSUB@Layout@OT@@@hb_accelerate_subtables_context_t@OT@@SA_NPBXPAUhb_ot_apply_context_t@1@@Z 10046220 f i hb-ot-layout.obj
 0001:00045230       ??$apply_cached_to@UChainContextFormat1@OT@@@hb_accelerate_subtables_context_t@OT@@SA_NPBXPAUhb_ot_apply_context_t@1@@Z 10046230 f i hb-ot-layout.obj
 0001:00045230       ??$apply_to@UChainContextFormat1@OT@@@hb_accelerate_subtables_context_t@OT@@SA_NPBXPAUhb_ot_apply_context_t@1@@Z 10046230 f i hb-ot-layout.obj
 0001:00045240       ??$apply_cached_to@UChainContextFormat2@OT@@@hb_accelerate_subtables_context_t@OT@@SA_NPBXPAUhb_ot_apply_context_t@1@@Z 10046240 f i hb-ot-layout.obj
 0001:00045250       ??$apply_cached_to@UChainContextFormat3@OT@@@hb_accelerate_subtables_context_t@OT@@SA_NPBXPAUhb_ot_apply_context_t@1@@Z 10046250 f i hb-ot-layout.obj
 0001:00045250       ??$apply_to@UChainContextFormat3@OT@@@hb_accelerate_subtables_context_t@OT@@SA_NPBXPAUhb_ot_apply_context_t@1@@Z 10046250 f i hb-ot-layout.obj
 0001:00045260       ??$apply_cached_to@UContextFormat1@OT@@@hb_accelerate_subtables_context_t@OT@@SA_NPBXPAUhb_ot_apply_context_t@1@@Z 10046260 f i hb-ot-layout.obj
 0001:00045260       ??$apply_to@UContextFormat1@OT@@@hb_accelerate_subtables_context_t@OT@@SA_NPBXPAUhb_ot_apply_context_t@1@@Z 10046260 f i hb-ot-layout.obj
 0001:00045270       ??$apply_cached_to@UContextFormat2@OT@@@hb_accelerate_subtables_context_t@OT@@SA_NPBXPAUhb_ot_apply_context_t@1@@Z 10046270 f i hb-ot-layout.obj
 0001:00045280       ??$apply_to@UContextFormat3@OT@@@hb_accelerate_subtables_context_t@OT@@SA_NPBXPAUhb_ot_apply_context_t@1@@Z 10046280 f i hb-ot-layout.obj
 0001:00045280       ??$apply_cached_to@UContextFormat3@OT@@@hb_accelerate_subtables_context_t@OT@@SA_NPBXPAUhb_ot_apply_context_t@1@@Z 10046280 f i hb-ot-layout.obj
 0001:00045290       ??$apply_to@UCursivePosFormat1@GPOS_impl@Layout@OT@@@hb_accelerate_subtables_context_t@OT@@SA_NPBXPAUhb_ot_apply_context_t@1@@Z 10046290 f i hb-ot-layout.obj
 0001:00045290       ??$apply_cached_to@UCursivePosFormat1@GPOS_impl@Layout@OT@@@hb_accelerate_subtables_context_t@OT@@SA_NPBXPAUhb_ot_apply_context_t@1@@Z 10046290 f i hb-ot-layout.obj
 0001:000452a0       ??$apply_cached_to@ULigatureSubstFormat1@GSUB@Layout@OT@@@hb_accelerate_subtables_context_t@OT@@SA_NPBXPAUhb_ot_apply_context_t@1@@Z 100462a0 f i hb-ot-layout.obj
 0001:000452a0       ??$apply_to@ULigatureSubstFormat1@GSUB@Layout@OT@@@hb_accelerate_subtables_context_t@OT@@SA_NPBXPAUhb_ot_apply_context_t@1@@Z 100462a0 f i hb-ot-layout.obj
 0001:000452b0       ??$apply_to@UMarkBasePosFormat1@GPOS_impl@Layout@OT@@@hb_accelerate_subtables_context_t@OT@@SA_NPBXPAUhb_ot_apply_context_t@1@@Z 100462b0 f i hb-ot-layout.obj
 0001:000452b0       ??$apply_cached_to@UMarkBasePosFormat1@GPOS_impl@Layout@OT@@@hb_accelerate_subtables_context_t@OT@@SA_NPBXPAUhb_ot_apply_context_t@1@@Z 100462b0 f i hb-ot-layout.obj
 0001:000452c0       ??$apply_to@UMarkLigPosFormat1@GPOS_impl@Layout@OT@@@hb_accelerate_subtables_context_t@OT@@SA_NPBXPAUhb_ot_apply_context_t@1@@Z 100462c0 f i hb-ot-layout.obj
 0001:000452c0       ??$apply_cached_to@UMarkLigPosFormat1@GPOS_impl@Layout@OT@@@hb_accelerate_subtables_context_t@OT@@SA_NPBXPAUhb_ot_apply_context_t@1@@Z 100462c0 f i hb-ot-layout.obj
 0001:000452d0       ??$apply_cached_to@UMarkMarkPosFormat1@GPOS_impl@Layout@OT@@@hb_accelerate_subtables_context_t@OT@@SA_NPBXPAUhb_ot_apply_context_t@1@@Z 100462d0 f i hb-ot-layout.obj
 0001:000452d0       ??$apply_to@UMarkMarkPosFormat1@GPOS_impl@Layout@OT@@@hb_accelerate_subtables_context_t@OT@@SA_NPBXPAUhb_ot_apply_context_t@1@@Z 100462d0 f i hb-ot-layout.obj
 0001:000452e0       ??$apply_cached_to@UMultipleSubstFormat1@GSUB@Layout@OT@@@hb_accelerate_subtables_context_t@OT@@SA_NPBXPAUhb_ot_apply_context_t@1@@Z 100462e0 f i hb-ot-layout.obj
 0001:000452e0       ??$apply_to@UMultipleSubstFormat1@GSUB@Layout@OT@@@hb_accelerate_subtables_context_t@OT@@SA_NPBXPAUhb_ot_apply_context_t@1@@Z 100462e0 f i hb-ot-layout.obj
 0001:000452f0       ??$apply_to@UPairPosFormat1@GPOS_impl@Layout@OT@@@hb_accelerate_subtables_context_t@OT@@SA_NPBXPAUhb_ot_apply_context_t@1@@Z 100462f0 f i hb-ot-layout.obj
 0001:000452f0       ??$apply_cached_to@UPairPosFormat1@GPOS_impl@Layout@OT@@@hb_accelerate_subtables_context_t@OT@@SA_NPBXPAUhb_ot_apply_context_t@1@@Z 100462f0 f i hb-ot-layout.obj
 0001:00045300       ??$apply_to@UPairPosFormat2@GPOS_impl@Layout@OT@@@hb_accelerate_subtables_context_t@OT@@SA_NPBXPAUhb_ot_apply_context_t@1@@Z 10046300 f i hb-ot-layout.obj
 0001:00045300       ??$apply_cached_to@UPairPosFormat2@GPOS_impl@Layout@OT@@@hb_accelerate_subtables_context_t@OT@@SA_NPBXPAUhb_ot_apply_context_t@1@@Z 10046300 f i hb-ot-layout.obj
 0001:00045310       ??$apply_cached_to@UReverseChainSingleSubstFormat1@GSUB@Layout@OT@@@hb_accelerate_subtables_context_t@OT@@SA_NPBXPAUhb_ot_apply_context_t@1@@Z 10046310 f i hb-ot-layout.obj
 0001:00045310       ??$apply_to@UReverseChainSingleSubstFormat1@GSUB@Layout@OT@@@hb_accelerate_subtables_context_t@OT@@SA_NPBXPAUhb_ot_apply_context_t@1@@Z 10046310 f i hb-ot-layout.obj
 0001:00045320       ??$apply_cached_to@USinglePosFormat1@GPOS_impl@Layout@OT@@@hb_accelerate_subtables_context_t@OT@@SA_NPBXPAUhb_ot_apply_context_t@1@@Z 10046320 f i hb-ot-layout.obj
 0001:00045320       ??$apply_to@USinglePosFormat1@GPOS_impl@Layout@OT@@@hb_accelerate_subtables_context_t@OT@@SA_NPBXPAUhb_ot_apply_context_t@1@@Z 10046320 f i hb-ot-layout.obj
 0001:00045330       ??$apply_to@USinglePosFormat2@GPOS_impl@Layout@OT@@@hb_accelerate_subtables_context_t@OT@@SA_NPBXPAUhb_ot_apply_context_t@1@@Z 10046330 f i hb-ot-layout.obj
 0001:00045330       ??$apply_cached_to@USinglePosFormat2@GPOS_impl@Layout@OT@@@hb_accelerate_subtables_context_t@OT@@SA_NPBXPAUhb_ot_apply_context_t@1@@Z 10046330 f i hb-ot-layout.obj
 0001:00045340       ??$apply_cached_to@USingleSubstFormat1@GSUB@Layout@OT@@@hb_accelerate_subtables_context_t@OT@@SA_NPBXPAUhb_ot_apply_context_t@1@@Z 10046340 f i hb-ot-layout.obj
 0001:00045340       ??$apply_to@USingleSubstFormat1@GSUB@Layout@OT@@@hb_accelerate_subtables_context_t@OT@@SA_NPBXPAUhb_ot_apply_context_t@1@@Z 10046340 f i hb-ot-layout.obj
 0001:00045350       ??$apply_to@USingleSubstFormat2@GSUB@Layout@OT@@@hb_accelerate_subtables_context_t@OT@@SA_NPBXPAUhb_ot_apply_context_t@1@@Z 10046350 f i hb-ot-layout.obj
 0001:00045350       ??$apply_cached_to@USingleSubstFormat2@GSUB@Layout@OT@@@hb_accelerate_subtables_context_t@OT@@SA_NPBXPAUhb_ot_apply_context_t@1@@Z 10046350 f i hb-ot-layout.obj
 0001:00045420       ??$apply_to@UChainContextFormat2@OT@@@hb_accelerate_subtables_context_t@OT@@SA_NPBXPAUhb_ot_apply_context_t@1@@Z 10046420 f i hb-ot-layout.obj
 0001:00045430       ??$apply_to@UContextFormat2@OT@@@hb_accelerate_subtables_context_t@OT@@SA_NPBXPAUhb_ot_apply_context_t@1@@Z 10046430 f i hb-ot-layout.obj
 0001:00045440       ??$bsearch@Uhb_glyph_pair_t@AAT@@@?$SortedArrayOf@UKernPair@AAT@@U?$BinSearchHeader@U?$IntType@G$01@OT@@@OT@@@OT@@QBEABUKernPair@AAT@@ABUhb_glyph_pair_t@3@ABU23@@Z 10046440 f i hb-ot-layout.obj
 0001:000454f0       ??$cache_func_to@UMultipleSubstFormat1@GSUB@Layout@OT@@@hb_accelerate_subtables_context_t@OT@@SA_NPBXPAUhb_ot_apply_context_t@1@_N@Z 100464f0 f i hb-ot-layout.obj
 0001:000454f0       ??$cache_func_to@UPairPosFormat2@GPOS_impl@Layout@OT@@@hb_accelerate_subtables_context_t@OT@@SA_NPBXPAUhb_ot_apply_context_t@1@_N@Z 100464f0 f i hb-ot-layout.obj
 0001:000454f0       ??$cache_func_to@UChainContextFormat3@OT@@@hb_accelerate_subtables_context_t@OT@@SA_NPBXPAUhb_ot_apply_context_t@1@_N@Z 100464f0 f i hb-ot-layout.obj
 0001:000454f0       ??$cache_func_to@UMarkLigPosFormat1@GPOS_impl@Layout@OT@@@hb_accelerate_subtables_context_t@OT@@SA_NPBXPAUhb_ot_apply_context_t@1@_N@Z 100464f0 f i hb-ot-layout.obj
 0001:000454f0       ??$cache_func_to@USinglePosFormat2@GPOS_impl@Layout@OT@@@hb_accelerate_subtables_context_t@OT@@SA_NPBXPAUhb_ot_apply_context_t@1@_N@Z 100464f0 f i hb-ot-layout.obj
 0001:000454f0       ??$cache_func_to@ULigatureSubstFormat1@GSUB@Layout@OT@@@hb_accelerate_subtables_context_t@OT@@SA_NPBXPAUhb_ot_apply_context_t@1@_N@Z 100464f0 f i hb-ot-layout.obj
 0001:000454f0       ??$cache_func_to@UReverseChainSingleSubstFormat1@GSUB@Layout@OT@@@hb_accelerate_subtables_context_t@OT@@SA_NPBXPAUhb_ot_apply_context_t@1@_N@Z 100464f0 f i hb-ot-layout.obj
 0001:000454f0       ??$cache_func_to@UMarkMarkPosFormat1@GPOS_impl@Layout@OT@@@hb_accelerate_subtables_context_t@OT@@SA_NPBXPAUhb_ot_apply_context_t@1@_N@Z 100464f0 f i hb-ot-layout.obj
 0001:000454f0       ??$cache_func_to@UPairPosFormat1@GPOS_impl@Layout@OT@@@hb_accelerate_subtables_context_t@OT@@SA_NPBXPAUhb_ot_apply_context_t@1@_N@Z 100464f0 f i hb-ot-layout.obj
 0001:000454f0       ??$cache_func_to@UMarkBasePosFormat1@GPOS_impl@Layout@OT@@@hb_accelerate_subtables_context_t@OT@@SA_NPBXPAUhb_ot_apply_context_t@1@_N@Z 100464f0 f i hb-ot-layout.obj
 0001:000454f0       ??$cache_func_to@UContextFormat3@OT@@@hb_accelerate_subtables_context_t@OT@@SA_NPBXPAUhb_ot_apply_context_t@1@_N@Z 100464f0 f i hb-ot-layout.obj
 0001:000454f0       ??$cache_func_to@UCursivePosFormat1@GPOS_impl@Layout@OT@@@hb_accelerate_subtables_context_t@OT@@SA_NPBXPAUhb_ot_apply_context_t@1@_N@Z 100464f0 f i hb-ot-layout.obj
 0001:000454f0       ??$cache_func_to@UContextFormat1@OT@@@hb_accelerate_subtables_context_t@OT@@SA_NPBXPAUhb_ot_apply_context_t@1@_N@Z 100464f0 f i hb-ot-layout.obj
 0001:000454f0       ??$cache_func_to@USinglePosFormat1@GPOS_impl@Layout@OT@@@hb_accelerate_subtables_context_t@OT@@SA_NPBXPAUhb_ot_apply_context_t@1@_N@Z 100464f0 f i hb-ot-layout.obj
 0001:000454f0       ??$cache_func_to@UChainContextFormat1@OT@@@hb_accelerate_subtables_context_t@OT@@SA_NPBXPAUhb_ot_apply_context_t@1@_N@Z 100464f0 f i hb-ot-layout.obj
 0001:000454f0       ??$cache_func_to@USingleSubstFormat1@GSUB@Layout@OT@@@hb_accelerate_subtables_context_t@OT@@SA_NPBXPAUhb_ot_apply_context_t@1@_N@Z 100464f0 f i hb-ot-layout.obj
 0001:000454f0       ??$cache_func_to@UAlternateSubstFormat1@GSUB@Layout@OT@@@hb_accelerate_subtables_context_t@OT@@SA_NPBXPAUhb_ot_apply_context_t@1@_N@Z 100464f0 f i hb-ot-layout.obj
 0001:000454f0       ??$cache_func_to@USingleSubstFormat2@GSUB@Layout@OT@@@hb_accelerate_subtables_context_t@OT@@SA_NPBXPAUhb_ot_apply_context_t@1@_N@Z 100464f0 f i hb-ot-layout.obj
 0001:00045500       ??$cache_func_to@UContextFormat2@OT@@@hb_accelerate_subtables_context_t@OT@@SA_NPBXPAUhb_ot_apply_context_t@1@_N@Z 10046500 f i hb-ot-layout.obj
 0001:00045500       ??$cache_func_to@UChainContextFormat2@OT@@@hb_accelerate_subtables_context_t@OT@@SA_NPBXPAUhb_ot_apply_context_t@1@_N@Z 10046500 f i hb-ot-layout.obj
 0001:00045570       ??$check_struct@ULookup@OT@@@hb_sanitize_context_t@@QBE_NPBULookup@OT@@@Z 10046570 f i hb-ot-layout.obj
 0001:000455e0       ??$collect_coverage@U?$hb_set_digest_combiner_t@U?$hb_set_digest_bits_pattern_t@K$03@@U?$hb_set_digest_combiner_t@U?$hb_set_digest_bits_pattern_t@K$0A@@@U?$hb_set_digest_bits_pattern_t@K$08@@@@@@@Coverage@OT@@QBE_NPAU?$hb_set_digest_combiner_t@U?$hb_set_digest_bits_pattern_t@K$03@@U?$hb_set_digest_combiner_t@U?$hb_set_digest_bits_pattern_t@K$0A@@@U?$hb_set_digest_bits_pattern_t@K$08@@@@@@@Z 100465e0 f i hb-ot-layout.obj
 0001:000456a0       ??$collect_coverage@U?$hb_set_digest_combiner_t@U?$hb_set_digest_bits_pattern_t@K$03@@U?$hb_set_digest_combiner_t@U?$hb_set_digest_bits_pattern_t@K$0A@@@U?$hb_set_digest_bits_pattern_t@K$08@@@@@@@CoverageFormat2@OT@@ABE_NPAU?$hb_set_digest_combiner_t@U?$hb_set_digest_bits_pattern_t@K$03@@U?$hb_set_digest_combiner_t@U?$hb_set_digest_bits_pattern_t@K$0A@@@U?$hb_set_digest_bits_pattern_t@K$08@@@@@@@Z 100466a0 f i hb-ot-layout.obj
 0001:000457f0       ??$dispatch@U?$hb_collect_coverage_context_t@U?$hb_set_digest_combiner_t@U?$hb_set_digest_bits_pattern_t@K$03@@U?$hb_set_digest_combiner_t@U?$hb_set_digest_bits_pattern_t@K$0A@@@U?$hb_set_digest_bits_pattern_t@K$08@@@@@@@OT@@$$V@ChainContext@OT@@QBEABUCoverage@1@PAU?$hb_collect_coverage_context_t@U?$hb_set_digest_combiner_t@U?$hb_set_digest_bits_pattern_t@K$03@@U?$hb_set_digest_combiner_t@U?$hb_set_digest_bits_pattern_t@K$0A@@@U?$hb_set_digest_bits_pattern_t@K$08@@@@@@@1@@Z 100467f0 f i hb-ot-layout.obj
 0001:00045850       ??$dispatch@U?$hb_collect_coverage_context_t@U?$hb_set_digest_combiner_t@U?$hb_set_digest_bits_pattern_t@K$03@@U?$hb_set_digest_combiner_t@U?$hb_set_digest_bits_pattern_t@K$0A@@@U?$hb_set_digest_bits_pattern_t@K$08@@@@@@@OT@@$$V@Context@OT@@QBEABUCoverage@1@PAU?$hb_collect_coverage_context_t@U?$hb_set_digest_combiner_t@U?$hb_set_digest_bits_pattern_t@K$03@@U?$hb_set_digest_combiner_t@U?$hb_set_digest_bits_pattern_t@K$0A@@@U?$hb_set_digest_bits_pattern_t@K$08@@@@@@@1@@Z 10046850 f i hb-ot-layout.obj
 0001:000458b0       ??$dispatch@U?$hb_collect_coverage_context_t@U?$hb_set_digest_combiner_t@U?$hb_set_digest_bits_pattern_t@K$03@@U?$hb_set_digest_combiner_t@U?$hb_set_digest_bits_pattern_t@K$0A@@@U?$hb_set_digest_bits_pattern_t@K$08@@@@@@@OT@@$$V@PosLookupSubTable@GPOS_impl@Layout@OT@@QBEABUCoverage@3@PAU?$hb_collect_coverage_context_t@U?$hb_set_digest_combiner_t@U?$hb_set_digest_bits_pattern_t@K$03@@U?$hb_set_digest_combiner_t@U?$hb_set_digest_bits_pattern_t@K$0A@@@U?$hb_set_digest_bits_pattern_t@K$08@@@@@@@3@I@Z 100468b0 f i hb-ot-layout.obj
 0001:00045a20       ??$dispatch@U?$hb_collect_coverage_context_t@U?$hb_set_digest_combiner_t@U?$hb_set_digest_bits_pattern_t@K$03@@U?$hb_set_digest_combiner_t@U?$hb_set_digest_bits_pattern_t@K$0A@@@U?$hb_set_digest_bits_pattern_t@K$08@@@@@@@OT@@$$V@SubstLookupSubTable@GSUB@Layout@OT@@QBEABUCoverage@3@PAU?$hb_collect_coverage_context_t@U?$hb_set_digest_combiner_t@U?$hb_set_digest_bits_pattern_t@K$03@@U?$hb_set_digest_combiner_t@U?$hb_set_digest_bits_pattern_t@K$0A@@@U?$hb_set_digest_bits_pattern_t@K$08@@@@@@@3@I@Z 10046a20 f i hb-ot-layout.obj
 0001:00045b20       ??$dispatch@UPosLookupSubTable@GPOS_impl@Layout@OT@@U?$hb_collect_coverage_context_t@U?$hb_set_digest_combiner_t@U?$hb_set_digest_bits_pattern_t@K$03@@U?$hb_set_digest_combiner_t@U?$hb_set_digest_bits_pattern_t@K$0A@@@U?$hb_set_digest_bits_pattern_t@K$08@@@@@@@4@$$V@Lookup@OT@@QBEABUCoverage@1@PAU?$hb_collect_coverage_context_t@U?$hb_set_digest_combiner_t@U?$hb_set_digest_bits_pattern_t@K$03@@U?$hb_set_digest_combiner_t@U?$hb_set_digest_bits_pattern_t@K$0A@@@U?$hb_set_digest_bits_pattern_t@K$08@@@@@@@1@@Z 10046b20 f i hb-ot-layout.obj
 0001:00045d00       ??$dispatch@USubstLookupSubTable@GSUB@Layout@OT@@U?$hb_collect_coverage_context_t@U?$hb_set_digest_combiner_t@U?$hb_set_digest_bits_pattern_t@K$03@@U?$hb_set_digest_combiner_t@U?$hb_set_digest_bits_pattern_t@K$0A@@@U?$hb_set_digest_bits_pattern_t@K$08@@@@@@@4@$$V@Lookup@OT@@QBEABUCoverage@1@PAU?$hb_collect_coverage_context_t@U?$hb_set_digest_combiner_t@U?$hb_set_digest_bits_pattern_t@K$03@@U?$hb_set_digest_combiner_t@U?$hb_set_digest_bits_pattern_t@K$0A@@@U?$hb_set_digest_bits_pattern_t@K$08@@@@@@@1@@Z 10046d00 f i hb-ot-layout.obj
 0001:00045ee0       ??$dispatch@USubstLookupSubTable@GSUB@Layout@OT@@Uhb_ot_apply_context_t@4@$$V@Lookup@OT@@QBE_NPAUhb_ot_apply_context_t@1@@Z 10046ee0 f i hb-ot-layout.obj
 0001:00046170       ??$dispatch@Uhb_aat_apply_context_t@AAT@@$$V@?$KernSubTable@UKernAATSubTableHeader@OT@@@OT@@QBE_NPAUhb_aat_apply_context_t@AAT@@@Z 10047170 f i hb-ot-layout.obj
 0001:00046350       ??$dispatch@Uhb_accelerate_subtables_context_t@OT@@$$V@ChainContext@OT@@QBE?AUhb_empty_t@@PAUhb_accelerate_subtables_context_t@1@@Z 10047350 f i hb-ot-layout.obj
 0001:00046550       ??$dispatch@Uhb_accelerate_subtables_context_t@OT@@$$V@Context@OT@@QBE?AUhb_empty_t@@PAUhb_accelerate_subtables_context_t@1@@Z 10047550 f i hb-ot-layout.obj
 0001:00046740       ??$dispatch@Uhb_accelerate_subtables_context_t@OT@@$$V@PosLookupSubTable@GPOS_impl@Layout@OT@@QBE?AUhb_empty_t@@PAUhb_accelerate_subtables_context_t@3@I@Z 10047740 f i hb-ot-layout.obj
 0001:00046a90       ??$dispatch@Uhb_accelerate_subtables_context_t@OT@@$$V@SubstLookupSubTable@GSUB@Layout@OT@@QBE?AUhb_empty_t@@PAUhb_accelerate_subtables_context_t@3@I@Z 10047a90 f i hb-ot-layout.obj
 0001:00046d40       ??$dispatch@Uhb_ot_apply_context_t@OT@@$$V@ChainContext@OT@@QBE_NPAUhb_ot_apply_context_t@1@@Z 10047d40 f i hb-ot-layout.obj
 0001:00046d80       ??$dispatch@Uhb_ot_apply_context_t@OT@@$$V@Context@OT@@QBE_NPAUhb_ot_apply_context_t@1@@Z 10047d80 f i hb-ot-layout.obj
 0001:00046dc0       ??$dispatch@Uhb_ot_apply_context_t@OT@@$$V@PosLookupSubTable@GPOS_impl@Layout@OT@@QBE_NPAUhb_ot_apply_context_t@3@I@Z 10047dc0 f i hb-ot-layout.obj
 0001:00046f70       ??$dispatch@Uhb_ot_apply_context_t@OT@@$$V@SubstLookupSubTable@GSUB@Layout@OT@@QBE_NPAUhb_ot_apply_context_t@3@I@Z 10047f70 f i hb-ot-layout.obj
 0001:000470e0       ??$dispatch@Uhb_sanitize_context_t@@$$V@?$KernSubTable@UKernAATSubTableHeader@OT@@@OT@@QBE_NPAUhb_sanitize_context_t@@@Z 100480e0 f i hb-ot-layout.obj
 0001:00047300       ??$dispatch@Uhb_sanitize_context_t@@$$V@ChainContext@OT@@QBE_NPAUhb_sanitize_context_t@@@Z 10048300 f i hb-ot-layout.obj
 0001:00047520       ??$dispatch@Uhb_sanitize_context_t@@$$V@Context@OT@@QBE_NPAUhb_sanitize_context_t@@@Z 10048520 f i hb-ot-layout.obj
 0001:00047690       ??$dispatch@Uhb_sanitize_context_t@@$$V@PosLookupSubTable@GPOS_impl@Layout@OT@@QBE_NPAUhb_sanitize_context_t@@I@Z 10048690 f i hb-ot-layout.obj
 0001:00047b00       ??$dispatch@Uhb_sanitize_context_t@@$$V@SinglePos@GPOS_impl@Layout@OT@@QBE_NPAUhb_sanitize_context_t@@@Z 10048b00 f i hb-ot-layout.obj
 0001:00047cc0       ??$dispatch@Uhb_sanitize_context_t@@$$V@SubstLookupSubTable@GSUB@Layout@OT@@QBE_NPAUhb_sanitize_context_t@@I@Z 10048cc0 f i hb-ot-layout.obj
 0001:00048070       ??$dispatch@Uhb_sanitize_context_t@@$$V@kern@OT@@QBE_NPAUhb_sanitize_context_t@@@Z 10049070 f i hb-ot-layout.obj
 0001:000481a0       ??$dispatch@Uhb_would_apply_context_t@OT@@$$V@ChainContext@OT@@QBE_NPAUhb_would_apply_context_t@1@@Z 100491a0 f i hb-ot-layout.obj
 0001:00048420       ??$dispatch@Uhb_would_apply_context_t@OT@@$$V@Context@OT@@QBE_NPAUhb_would_apply_context_t@1@@Z 10049420 f i hb-ot-layout.obj
 0001:000485d0       ??$dispatch@Uhb_would_apply_context_t@OT@@$$V@SubstLookupSubTable@GSUB@Layout@OT@@QBE_NPAUhb_would_apply_context_t@3@I@Z 100495d0 f i hb-ot-layout.obj
 0001:00048770       ??$dispatch_recurse_func@Uhb_ot_apply_context_t@OT@@@PosLookup@GPOS_impl@Layout@OT@@SA_NPAUhb_ot_apply_context_t@3@I@Z 10049770 f i hb-ot-layout.obj
 0001:000488b0       ??$dispatch_recurse_func@Uhb_ot_apply_context_t@OT@@@SubstLookup@GSUB@Layout@OT@@SA_NPAUhb_ot_apply_context_t@3@I@Z 100498b0 f i hb-ot-layout.obj
 0001:00048970       ??$drive@Udriver_context_t@?$KerxSubTableFormat1@UKernAATSubTableHeader@OT@@@AAT@@@?$StateTableDriver@UObsoleteTypes@AAT@@X@AAT@@QAEXPAUdriver_context_t@?$KerxSubTableFormat1@UKernAATSubTableHeader@OT@@@1@@Z 10049970 f i hb-ot-layout.obj
 0001:00048c40       ??$get_subtable@UPosLookupSubTable@GPOS_impl@Layout@OT@@@Lookup@OT@@QBEABUPosLookupSubTable@GPOS_impl@Layout@1@I@Z 10049c40 f i hb-ot-layout.obj
 0001:00048c40       ??$get_subtable@USubstLookupSubTable@GSUB@Layout@OT@@@Lookup@OT@@QBEABUSubstLookupSubTable@GSUB@Layout@1@I@Z 10049c40 f i hb-ot-layout.obj
 0001:00048ca0       ??$init@UPosLookup@GPOS_impl@Layout@OT@@@hb_ot_layout_lookup_accelerator_t@OT@@QAEXABUPosLookup@GPOS_impl@Layout@1@@Z 10049ca0 f i hb-ot-layout.obj
 0001:00048e40       ??$init@USubstLookup@GSUB@Layout@OT@@@hb_ot_layout_lookup_accelerator_t@OT@@QAEXABUSubstLookup@GSUB@Layout@1@@Z 10049e40 f i hb-ot-layout.obj
 0001:00048fe0       ??$push@AAUhb_applicable_t@hb_accelerate_subtables_context_t@OT@@U123@$0A@@?$hb_vector_t@Uhb_applicable_t@hb_accelerate_subtables_context_t@OT@@$0A@@@QAEPAUhb_applicable_t@hb_accelerate_subtables_context_t@OT@@AAU123@@Z 10049fe0 f i hb-ot-layout.obj
 0001:000490b0       ??$sanitize@$$V@?$ArrayOf@UKernPair@AAT@@U?$BinSearchHeader@U?$IntType@G$01@OT@@@OT@@@OT@@QBE_NPAUhb_sanitize_context_t@@@Z 1004a0b0 f i hb-ot-layout.obj
 0001:00049150       ??$sanitize@$$V@?$ArrayOf@ULookupRecord@OT@@U?$IntType@G$01@2@@OT@@QBE_NPAUhb_sanitize_context_t@@@Z 1004a150 f i hb-ot-layout.obj
 0001:00049190       ??$sanitize@$$V@?$OffsetTo@U?$ClassTable@U?$IntType@G$01@OT@@@AAT@@U?$IntType@G$01@OT@@$0A@@OT@@QBE_NPAUhb_sanitize_context_t@@PBX@Z 1004a190 f i hb-ot-layout.obj
 0001:000492c0       ??$sanitize@$$V@?$OffsetTo@U?$List16OfOffset16To@UPosLookup@GPOS_impl@Layout@OT@@@OT@@U?$IntType@G$01@2@$00@OT@@QBE_NPAUhb_sanitize_context_t@@PBX@Z 1004a2c0 f i hb-ot-layout.obj
 0001:000493a0       ??$sanitize@$$V@?$OffsetTo@U?$RecordListOf@UFeature@OT@@@OT@@U?$IntType@G$01@2@$00@OT@@QBE_NPAUhb_sanitize_context_t@@PBX@Z 1004a3a0 f i hb-ot-layout.obj
 0001:000494f0       ??$sanitize@$$V@?$OffsetTo@UAnchor@GPOS_impl@Layout@OT@@U?$IntType@G$01@4@$00@OT@@QBE_NPAUhb_sanitize_context_t@@PBX@Z 1004a4f0 f i hb-ot-layout.obj
 0001:000495c0       ??$sanitize@$$V@?$OffsetTo@UChainRuleSet@OT@@U?$IntType@G$01@2@$00@OT@@QBE_NPAUhb_sanitize_context_t@@PBX@Z 1004a5c0 f i hb-ot-layout.obj
 0001:000496a0       ??$sanitize@$$V@?$OffsetTo@UCondition@OT@@U?$IntType@I$03@2@$00@OT@@QBE_NPAUhb_sanitize_context_t@@PBX@Z 1004a6a0 f i hb-ot-layout.obj
 0001:00049800       ??$sanitize@$$V@?$OffsetTo@UConditionSet@OT@@U?$IntType@I$03@2@$00@OT@@QBE_NPAUhb_sanitize_context_t@@PBX@Z 1004a800 f i hb-ot-layout.obj
 0001:00049950       ??$sanitize@$$V@?$OffsetTo@UFeatureTableSubstitution@OT@@U?$IntType@I$03@2@$00@OT@@QBE_NPAUhb_sanitize_context_t@@PBX@Z 1004a950 f i hb-ot-layout.obj
 0001:00049ad0       ??$sanitize@$$V@?$OffsetTo@UFeatureVariations@OT@@U?$IntType@I$03@2@$00@OT@@QBE_NPAUhb_sanitize_context_t@@PBX@Z 1004aad0 f i hb-ot-layout.obj
 0001:00049c90       ??$sanitize@$$V@?$OffsetTo@ULigatureSet@GSUB@Layout@OT@@U?$IntType@G$01@4@$00@OT@@QBE_NPAUhb_sanitize_context_t@@PBX@Z 1004ac90 f i hb-ot-layout.obj
 0001:00049de0       ??$sanitize@$$V@?$OffsetTo@UMarkArray@GPOS_impl@Layout@OT@@U?$IntType@G$01@4@$00@OT@@QBE_NPAUhb_sanitize_context_t@@PBX@Z 1004ade0 f i hb-ot-layout.obj
 0001:00049fc0       ??$sanitize@$$V@?$OffsetTo@URecordListOfScript@OT@@U?$IntType@G$01@2@$00@OT@@QBE_NPAUhb_sanitize_context_t@@PBX@Z 1004afc0 f i hb-ot-layout.obj
 0001:0004a090       ??$sanitize@$$V@?$OffsetTo@URule@OT@@U?$IntType@G$01@2@$00@OT@@QBE_NPAUhb_sanitize_context_t@@PBX@Z 1004b090 f i hb-ot-layout.obj
 0001:0004a1c0       ??$sanitize@$$V@?$OffsetTo@URuleSet@OT@@U?$IntType@G$01@2@$00@OT@@QBE_NPAUhb_sanitize_context_t@@PBX@Z 1004b1c0 f i hb-ot-layout.obj
 0001:0004a310       ??$sanitize@I@?$OffsetTo@UAnchorMatrix@GPOS_impl@Layout@OT@@U?$IntType@G$01@4@$00@OT@@QBE_NPAUhb_sanitize_context_t@@PBX$$QAI@Z 1004b310 f i hb-ot-layout.obj
 0001:0004a4f0       ??$sanitize@I@?$OffsetTo@UFeatureParams@OT@@U?$IntType@G$01@2@$00@OT@@QBE_NPAUhb_sanitize_context_t@@PBX$$QAI@Z 1004b4f0 f i hb-ot-layout.obj
 0001:0004a5d0       ??$sanitize@I@?$OffsetTo@ULigatureArray@GPOS_impl@Layout@OT@@U?$IntType@G$01@4@$00@OT@@QBE_NPAUhb_sanitize_context_t@@PBX$$QAI@Z 1004b5d0 f i hb-ot-layout.obj
 0001:0004a720       ??$sanitize@PBU?$List16OfOffset16To@UPosLookup@GPOS_impl@Layout@OT@@@OT@@@?$ArrayOf@U?$OffsetTo@UPosLookup@GPOS_impl@Layout@OT@@U?$IntType@G$01@4@$00@OT@@U?$IntType@G$01@2@@OT@@QBE_NPAUhb_sanitize_context_t@@$$QAPBU?$List16OfOffset16To@UPosLookup@GPOS_impl@Layout@OT@@@1@@Z 1004b720 f i hb-ot-layout.obj
 0001:0004a860       ??$sanitize@PBU?$List16OfOffset16To@USubstLookup@GSUB@Layout@OT@@@OT@@@?$ArrayOf@U?$OffsetTo@USubstLookup@GSUB@Layout@OT@@U?$IntType@G$01@4@$00@OT@@U?$IntType@G$01@2@@OT@@QBE_NPAUhb_sanitize_context_t@@$$QAPBU?$List16OfOffset16To@USubstLookup@GSUB@Layout@OT@@@1@@Z 1004b860 f i hb-ot-layout.obj
 0001:0004a9a0       ??$sanitize@PBUAlternateSubstFormat1@GSUB@Layout@OT@@@?$ArrayOf@U?$OffsetTo@UAlternateSet@GSUB@Layout@OT@@U?$IntType@G$01@4@$00@OT@@U?$IntType@G$01@2@@OT@@QBE_NPAUhb_sanitize_context_t@@$$QAPBUAlternateSubstFormat1@GSUB@Layout@1@@Z 1004b9a0 f i hb-ot-layout.obj
 0001:0004a9a0       ??$sanitize@PBUMultipleSubstFormat1@GSUB@Layout@OT@@@?$ArrayOf@U?$OffsetTo@USequence@GSUB@Layout@OT@@U?$IntType@G$01@4@$00@OT@@U?$IntType@G$01@2@@OT@@QBE_NPAUhb_sanitize_context_t@@$$QAPBUMultipleSubstFormat1@GSUB@Layout@1@@Z 1004b9a0 f i hb-ot-layout.obj
 0001:0004ab00       ??$sanitize@PBUReverseChainSingleSubstFormat1@GSUB@Layout@OT@@@?$ArrayOf@U?$OffsetTo@UCoverage@OT@@U?$IntType@G$01@2@$00@OT@@U?$IntType@G$01@2@@OT@@QBE_NPAUhb_sanitize_context_t@@$$QAPBUReverseChainSingleSubstFormat1@GSUB@Layout@1@@Z 1004bb00 f i hb-ot-layout.obj
 0001:0004ab00       ??$sanitize@PBUChainContextFormat3@OT@@@?$ArrayOf@U?$OffsetTo@UCoverage@OT@@U?$IntType@G$01@2@$00@OT@@U?$IntType@G$01@2@@OT@@QBE_NPAUhb_sanitize_context_t@@$$QAPBUChainContextFormat3@1@@Z 1004bb00 f i hb-ot-layout.obj
 0001:0004ab80       ??$sanitize@PBUChainRuleSet@OT@@@?$ArrayOf@U?$OffsetTo@UChainRule@OT@@U?$IntType@G$01@2@$00@OT@@U?$IntType@G$01@2@@OT@@QBE_NPAUhb_sanitize_context_t@@$$QAPBUChainRuleSet@1@@Z 1004bb80 f i hb-ot-layout.obj
 0001:0004acc0       ??$sanitize@PBULookup@OT@@I@?$ArrayOf@U?$OffsetTo@UPosLookupSubTable@GPOS_impl@Layout@OT@@U?$IntType@G$01@4@$00@OT@@U?$IntType@G$01@2@@OT@@QBE_NPAUhb_sanitize_context_t@@$$QAPBULookup@1@$$QAI@Z 1004bcc0 f i hb-ot-layout.obj
 0001:0004ae10       ??$sanitize@PBULookup@OT@@I@?$ArrayOf@U?$OffsetTo@USubstLookupSubTable@GSUB@Layout@OT@@U?$IntType@G$01@4@$00@OT@@U?$IntType@G$01@2@@OT@@QBE_NPAUhb_sanitize_context_t@@$$QAPBULookup@1@$$QAI@Z 1004be10 f i hb-ot-layout.obj
 0001:0004af60       ??$sanitize@PBUPairPosFormat1@GPOS_impl@Layout@OT@@PAUsanitize_closure_t@PairSet@234@@?$ArrayOf@U?$OffsetTo@UPairSet@GPOS_impl@Layout@OT@@U?$IntType@G$01@4@$00@OT@@U?$IntType@G$01@2@@OT@@QBE_NPAUhb_sanitize_context_t@@$$QAPBUPairPosFormat1@GPOS_impl@Layout@1@$$QAPAUsanitize_closure_t@PairSet@451@@Z 1004bf60 f i hb-ot-layout.obj
 0001:0004b0b0       ??$sanitize@PBURecord_sanitize_closure_t@OT@@@?$OffsetTo@UScript@OT@@U?$IntType@G$01@2@$00@OT@@QBE_NPAUhb_sanitize_context_t@@PBX$$QAPBURecord_sanitize_closure_t@1@@Z 1004c0b0 f i hb-ot-layout.obj
 0001:0004b1f0       ??$sanitize@PBUScript@OT@@@?$ArrayOf@U?$Record@ULangSys@OT@@@OT@@U?$IntType@G$01@2@@OT@@QBE_NPAUhb_sanitize_context_t@@$$QAPBUScript@1@@Z 1004c1f0 f i hb-ot-layout.obj
 0001:0004b350       ??$sanitize@UPosLookupSubTable@GPOS_impl@Layout@OT@@@Lookup@OT@@QBE_NPAUhb_sanitize_context_t@@@Z 1004c350 f i hb-ot-layout.obj
 0001:0004b4a0       ??$sanitize@USubstLookup@GSUB@Layout@OT@@@GSUBGPOS@OT@@QBE_NPAUhb_sanitize_context_t@@@Z 1004c4a0 f i hb-ot-layout.obj
 0001:0004b5f0       ??$sanitize@USubstLookupSubTable@GSUB@Layout@OT@@@Lookup@OT@@QBE_NPAUhb_sanitize_context_t@@@Z 1004c5f0 f i hb-ot-layout.obj
 0001:0004b740       ??$sanitize_blob@UGPOS@Layout@OT@@@hb_sanitize_context_t@@QAEPAUhb_blob_t@@PAU1@@Z 1004c740 f i hb-ot-layout.obj
 0001:0004b990       ??$sanitize_blob@UGSUB@1Layout@OT@@@hb_sanitize_context_t@@QAEPAUhb_blob_t@@PAU1@@Z 1004c990 f i hb-ot-layout.obj
 0001:0004bb10       ??$sanitize_blob@Ukern@OT@@@hb_sanitize_context_t@@QAEPAUhb_blob_t@@PAU1@@Z 1004cb10 f i hb-ot-layout.obj
 0001:0004bd80       ??A?$List16OfOffset16To@UAnchorMatrix@GPOS_impl@Layout@OT@@@OT@@QBEABUAnchorMatrix@GPOS_impl@Layout@1@H@Z 1004cd80 f i hb-ot-layout.obj
 0001:0004be20       ?_set_glyph_class@hb_ot_apply_context_t@OT@@QBEXII_N0@Z 1004ce20 f i hb-ot-layout.obj
 0001:0004bed0       ?apply@?$KerxTable@UKernAAT@OT@@@AAT@@QBE_NPAUhb_aat_apply_context_t@2@@Z 1004ced0 f i hb-ot-layout.obj
 0001:0004c0e0       ?apply@?$KerxTable@UKernOT@OT@@@AAT@@QBE_NPAUhb_aat_apply_context_t@2@@Z 1004d0e0 f i hb-ot-layout.obj
 0001:0004c340       ?apply@AlternateSubstFormat1@GSUB@Layout@OT@@QBE_NPAUhb_ot_apply_context_t@4@@Z 1004d340 f i hb-ot-layout.obj
 0001:0004c4a0       ?apply@ChainContextFormat1@OT@@QBE_NPAUhb_ot_apply_context_t@2@@Z 1004d4a0 f i hb-ot-layout.obj
 0001:0004c580       ?apply@ChainContextFormat2@OT@@QBE_NPAUhb_ot_apply_context_t@2@_N@Z 1004d580 f i hb-ot-layout.obj
 0001:0004c720       ?apply@ChainContextFormat3@OT@@QBE_NPAUhb_ot_apply_context_t@2@@Z 1004d720 f i hb-ot-layout.obj
 0001:0004c840       ?apply@ChainRuleSet@OT@@QBE_NPAUhb_ot_apply_context_t@2@AAUChainContextApplyLookupContext@2@@Z 1004d840 f i hb-ot-layout.obj
 0001:0004c9c0       ?apply@ContextFormat1@OT@@QBE_NPAUhb_ot_apply_context_t@2@@Z 1004d9c0 f i hb-ot-layout.obj
 0001:0004ca90       ?apply@ContextFormat2@OT@@QBE_NPAUhb_ot_apply_context_t@2@_N@Z 1004da90 f i hb-ot-layout.obj
 0001:0004cc00       ?apply@ContextFormat3@OT@@QBE_NPAUhb_ot_apply_context_t@2@@Z 1004dc00 f i hb-ot-layout.obj
 0001:0004ccb0       ?apply@CursivePosFormat1@GPOS_impl@Layout@OT@@QBE_NPAUhb_ot_apply_context_t@4@@Z 1004dcb0 f i hb-ot-layout.obj
 0001:0004d190       ?apply@LigatureSet@GSUB@Layout@OT@@QBE_NPAUhb_ot_apply_context_t@4@@Z 1004e190 f i hb-ot-layout.obj
 0001:0004d350       ?apply@LigatureSubstFormat1@GSUB@Layout@OT@@QBE_NPAUhb_ot_apply_context_t@4@@Z 1004e350 f i hb-ot-layout.obj
 0001:0004d410       ?apply@MarkArray@GPOS_impl@Layout@OT@@QBE_NPAUhb_ot_apply_context_t@4@IIABUAnchorMatrix@234@II@Z 1004e410 f i hb-ot-layout.obj
 0001:0004d650       ?apply@MarkBasePosFormat1@GPOS_impl@Layout@OT@@QBE_NPAUhb_ot_apply_context_t@4@@Z 1004e650 f i hb-ot-layout.obj
 0001:0004d960       ?apply@MarkLigPosFormat1@GPOS_impl@Layout@OT@@QBE_NPAUhb_ot_apply_context_t@4@@Z 1004e960 f i hb-ot-layout.obj
 0001:0004db80       ?apply@MarkMarkPosFormat1@GPOS_impl@Layout@OT@@QBE_NPAUhb_ot_apply_context_t@4@@Z 1004eb80 f i hb-ot-layout.obj
 0001:0004dda0       ?apply@MultipleSubstFormat1@GSUB@Layout@OT@@QBE_NPAUhb_ot_apply_context_t@4@@Z 1004eda0 f i hb-ot-layout.obj
 0001:0004de60       ?apply@PairPosFormat1@GPOS_impl@Layout@OT@@QBE_NPAUhb_ot_apply_context_t@4@@Z 1004ee60 f i hb-ot-layout.obj
 0001:0004df80       ?apply@PairPosFormat2@GPOS_impl@Layout@OT@@QBE_NPAUhb_ot_apply_context_t@4@@Z 1004ef80 f i hb-ot-layout.obj
 0001:0004e230       ?apply@PairSet@GPOS_impl@Layout@OT@@QBE_NPAUhb_ot_apply_context_t@4@PBUValueFormat@234@I@Z 1004f230 f i hb-ot-layout.obj
 0001:0004e440       ?apply@ReverseChainSingleSubstFormat1@GSUB@Layout@OT@@QBE_NPAUhb_ot_apply_context_t@4@@Z 1004f440 f i hb-ot-layout.obj
 0001:0004e610       ?apply@RuleSet@OT@@QBE_NPAUhb_ot_apply_context_t@2@AAUContextApplyLookupContext@2@@Z 1004f610 f i hb-ot-layout.obj
 0001:0004e740       ?apply@Sequence@GSUB@Layout@OT@@QBE_NPAUhb_ot_apply_context_t@4@@Z 1004f740 f i hb-ot-layout.obj
 0001:0004e8a0       ?apply@SinglePosFormat1@GPOS_impl@Layout@OT@@QBE_NPAUhb_ot_apply_context_t@4@@Z 1004f8a0 f i hb-ot-layout.obj
 0001:0004e920       ?apply@SinglePosFormat2@GPOS_impl@Layout@OT@@QBE_NPAUhb_ot_apply_context_t@4@@Z 1004f920 f i hb-ot-layout.obj
 0001:0004ea10       ?apply@SingleSubstFormat1@GSUB@Layout@OT@@QBE_NPAUhb_ot_apply_context_t@4@@Z 1004fa10 f i hb-ot-layout.obj
 0001:0004ea90       ?apply@SingleSubstFormat2@GSUB@Layout@OT@@QBE_NPAUhb_ot_apply_context_t@4@@Z 1004fa90 f i hb-ot-layout.obj
 0001:0004f4d0       ?apply_value@ValueFormat@GPOS_impl@Layout@OT@@QBE_NPAUhb_ot_apply_context_t@4@PBXPBU?$IntType@G$01@4@AAUhb_glyph_position_t@@@Z 100504d0 f i hb-ot-layout.obj
 0001:0004fad0       ?find_index@FeatureVariations@OT@@QBE_NPBHIPAI@Z 10050ad0 f i hb-ot-layout.obj
 0001:0004fc60       ?find_lang_sys_index@Script@OT@@QBE_NIPAI@Z 10050c60 f i hb-ot-layout.obj
 0001:0004fcf0       ?find_script_index@GSUBGPOS@OT@@QBE_NIPAI@Z 10050cf0 f i hb-ot-layout.obj
 0001:0004fda0       ?get_anchor@Anchor@GPOS_impl@Layout@OT@@QBEXPAUhb_ot_apply_context_t@4@IPAM1@Z 10050da0 f i hb-ot-layout.obj
 0001:00050050       ?get_coverage@ChainContextFormat3@OT@@QBEABUCoverage@2@XZ 10051050 f i hb-ot-layout.obj
 0001:000500c0       ?get_delta@HintingDevice@OT@@ABEHIH@Z 100510c0 f i hb-ot-layout.obj
 0001:000501c0       ?get_delta@VariationDevice@OT@@ABEMPAUhb_font_t@@ABUVariationStore@2@PAM@Z 100511c0 f i hb-ot-layout.obj
 0001:000502a0       ?get_feature@GSUBGPOS@OT@@QBEABUFeature@2@I@Z 100512a0 f i hb-ot-layout.obj
 0001:00050320       ?get_feature_tag@GSUBGPOS@OT@@QBEII@Z 10051320 f i hb-ot-layout.obj
 0001:000503a0       ?get_feature_variation@GSUBGPOS@OT@@QBEABUFeature@2@II@Z 100513a0 f i hb-ot-layout.obj
 0001:00050560       ?get_indexes@IndexArray@OT@@QBEIIPAI0@Z 10051560 f i hb-ot-layout.obj
 0001:00050680       ?get_lang_sys@Script@OT@@QBEABULangSys@2@I@Z 10051680 f i hb-ot-layout.obj
 0001:000506f0       ?get_len@ValueFormat@GPOS_impl@Layout@OT@@QBEIXZ 100516f0 f i hb-ot-layout.obj
 0001:00050730       ?get_lookup@GSUBGPOS@OT@@QBEABULookup@2@I@Z 10051730 f i hb-ot-layout.obj
 0001:000507a0       ?get_props@Lookup@OT@@QBEIXZ 100517a0 f i hb-ot-layout.obj
 0001:000507f0       ?get_script@GSUBGPOS@OT@@QBEABUScript@2@I@Z 100517f0 f i hb-ot-layout.obj
 0001:00050870       ?get_size@ValueFormat@GPOS_impl@Layout@OT@@QBEIXZ 10051870 f i hb-ot-layout.obj
 0001:000508b0       ?get_stored@?$hb_lazy_loader_t@UGPOS_accelerator_t@OT@@U?$hb_face_lazy_loader_t@UGPOS_accelerator_t@OT@@$0BJ@@@Uhb_face_t@@$0BJ@U12@@@QBEPAUGPOS_accelerator_t@OT@@XZ 100518b0 f i hb-ot-layout.obj
 0001:00050a60       ?get_stored@?$hb_lazy_loader_t@UGSUB_accelerator_t@OT@@U?$hb_face_lazy_loader_t@UGSUB_accelerator_t@OT@@$0BI@@@Uhb_face_t@@$0BI@U12@@@QBEPAUGSUB_accelerator_t@OT@@XZ 10051a60 f i hb-ot-layout.obj
 0001:00050c10       ?get_stored@?$hb_lazy_loader_t@Ukern@OT@@U?$hb_table_lazy_loader_t@Ukern@OT@@$0BG@$0A@@@Uhb_face_t@@$0BG@Uhb_blob_t@@@@QBEPAUhb_blob_t@@XZ 10051c10 f i hb-ot-layout.obj
 0001:00050ce0       ?get_type@?$Extension@UExtensionPos@GPOS_impl@Layout@OT@@@OT@@QBEIXZ 10051ce0 f i hb-ot-layout.obj
 0001:00050ce0       ?get_type@?$Extension@UExtensionSubst@GSUB@Layout@OT@@@OT@@QBEIXZ 10051ce0 f i hb-ot-layout.obj
 0001:00050d10       ?get_x_delta@Device@OT@@QBEHPAUhb_font_t@@ABUVariationStore@2@PAM@Z 10051d10 f i hb-ot-layout.obj
 0001:00050db0       ?get_y_delta@Device@OT@@QBEHPAUhb_font_t@@ABUVariationStore@2@PAM@Z 10051db0 f i hb-ot-layout.obj
 0001:00050e50       ?hb_ot_layout_delete_glyphs_inplace@@YAXPAUhb_buffer_t@@P6A_NPBUhb_glyph_info_t@@@Z@Z 10051e50 f   hb-ot-layout.obj
 0001:00050f70       ?hb_ot_layout_has_cross_kerning@@YA_NPAUhb_face_t@@@Z 10051f70 f   hb-ot-layout.obj
 0001:00051040       ?hb_ot_layout_has_kerning@@YA_NPAUhb_face_t@@@Z 10052040 f   hb-ot-layout.obj
 0001:00051080       ?hb_ot_layout_has_machine_kerning@@YA_NPAUhb_face_t@@@Z 10052080 f   hb-ot-layout.obj
 0001:00051150       ?hb_ot_layout_kern@@YAXPBUhb_ot_shape_plan_t@@PAUhb_font_t@@PAUhb_buffer_t@@@Z 10052150 f   hb-ot-layout.obj
 0001:000511f0       ?hb_ot_layout_position_finish_offsets@@YAXPAUhb_font_t@@PAUhb_buffer_t@@@Z 100521f0 f   hb-ot-layout.obj
 0001:000512d0       ?hb_ot_layout_position_start@@YAXPAUhb_font_t@@PAUhb_buffer_t@@@Z 100522d0 f   hb-ot-layout.obj
 0001:00051300       ?hb_ot_layout_substitute_lookup@@YAXPAUhb_ot_apply_context_t@OT@@ABUSubstLookup@GSUB@Layout@2@ABUhb_ot_layout_lookup_accelerator_t@2@@Z 10052300 f   hb-ot-layout.obj
 0001:00051310       ?hb_ot_layout_substitute_start@@YAXPAUhb_font_t@@PAUhb_buffer_t@@@Z 10052310 f   hb-ot-layout.obj
 0001:00051410       ?hb_ot_layout_table_find_feature@@YA_NPAUhb_face_t@@IIPAI@Z 10052410 f   hb-ot-layout.obj
 0001:00051520       ?is_blocklisted@GDEF@OT@@QBE_NPAUhb_blob_t@@PAUhb_face_t@@@Z 10052520 f   hb-ot-layout.obj
 0001:000518d0       ?kern@?$hb_kern_machine_t@U?$KernSubTableFormat3@UKernAATSubTableHeader@OT@@@OT@@@OT@@QBEXPAUhb_font_t@@PAUhb_buffer_t@@I_N@Z 100528d0 f i hb-ot-layout.obj
 0001:00051d80       ?kern@?$hb_kern_machine_t@Uaccelerator_t@?$KerxSubTableFormat0@UKernAATSubTableHeader@OT@@@AAT@@@OT@@QBEXPAUhb_font_t@@PAUhb_buffer_t@@I_N@Z 10052d80 f i hb-ot-layout.obj
 0001:000521a0       ?kern@?$hb_kern_machine_t@Uaccelerator_t@?$KerxSubTableFormat0@UKernOTSubTableHeader@OT@@@AAT@@@OT@@QBEXPAUhb_font_t@@PAUhb_buffer_t@@I_N@Z 100531a0 f i hb-ot-layout.obj
 0001:000525c0       ?kern@?$hb_kern_machine_t@Uaccelerator_t@?$KerxSubTableFormat2@UKernAATSubTableHeader@OT@@@AAT@@@OT@@QBEXPAUhb_font_t@@PAUhb_buffer_t@@I_N@Z 100535c0 f i hb-ot-layout.obj
 0001:00052ab0       ?kern@?$hb_kern_machine_t@Uaccelerator_t@?$KerxSubTableFormat2@UKernOTSubTableHeader@OT@@@AAT@@@OT@@QBEXPAUhb_font_t@@PAUhb_buffer_t@@I_N@Z 10053ab0 f i hb-ot-layout.obj
 0001:00053a30       ?position@hb_ot_map_t@@QBEXPBUhb_ot_shape_plan_t@@PAUhb_font_t@@PAUhb_buffer_t@@@Z 10054a30 f   hb-ot-layout.obj
 0001:00053ac0       ?prev@skipping_iterator_t@hb_ot_apply_context_t@OT@@QAE_NPAI@Z 10054ac0 f i hb-ot-layout.obj
 0001:00053cf0       ?replace_glyph@hb_ot_apply_context_t@OT@@QBEXI@Z 10054cf0 f i hb-ot-layout.obj
 0001:00053e00       ?sanitize@?$KernSubTable@UKernOTSubTableHeader@OT@@@OT@@QBE_NPAUhb_sanitize_context_t@@@Z 10054e00 f i hb-ot-layout.obj
 0001:00053f30       ?sanitize@?$KerxTable@UKernAAT@OT@@@AAT@@QBE_NPAUhb_sanitize_context_t@@@Z 10054f30 f i hb-ot-layout.obj
 0001:000540a0       ?sanitize@?$Record@UFeature@OT@@@OT@@QBE_NPAUhb_sanitize_context_t@@PBX@Z 100550a0 f i hb-ot-layout.obj
 0001:00054220       ?sanitize@?$RecordListOf@UScript@OT@@@OT@@QBE_NPAUhb_sanitize_context_t@@@Z 10055220 f i hb-ot-layout.obj
 0001:00054360       ?sanitize@Anchor@GPOS_impl@Layout@OT@@QBE_NPAUhb_sanitize_context_t@@@Z 10055360 f i hb-ot-layout.obj
 0001:000544e0       ?sanitize@ChainRule@OT@@QBE_NPAUhb_sanitize_context_t@@@Z 100554e0 f i hb-ot-layout.obj
 0001:000545f0       ?sanitize@Feature@OT@@QBE_NPAUhb_sanitize_context_t@@PBURecord_sanitize_closure_t@2@@Z 100555f0 f i hb-ot-layout.obj
 0001:00054780       ?sanitize@FeatureParams@OT@@QBE_NPAUhb_sanitize_context_t@@I@Z 10055780 f i hb-ot-layout.obj
 0001:000548d0       ?sanitize@FeatureParamsSize@OT@@QBE_NPAUhb_sanitize_context_t@@@Z 100558d0 f i hb-ot-layout.obj
 0001:00054a00       ?sanitize@FeatureTableSubstitutionRecord@OT@@QBE_NPAUhb_sanitize_context_t@@PBX@Z 10055a00 f i hb-ot-layout.obj
 0001:00054b40       ?sanitize@GPOS@Layout@OT@@QBE_NPAUhb_sanitize_context_t@@@Z 10055b40 f i hb-ot-layout.obj
 0001:00054bc0       ?sanitize@KernAATSubTableHeader@OT@@QBE_NPAUhb_sanitize_context_t@@@Z 10055bc0 f i hb-ot-layout.obj
 0001:00054c40       ?sanitize@KernOTSubTableHeader@OT@@QBE_NPAUhb_sanitize_context_t@@@Z 10055c40 f i hb-ot-layout.obj
 0001:00054cc0       ?sanitize@LangSys@OT@@QBE_NPAUhb_sanitize_context_t@@PBURecord_sanitize_closure_t@2@@Z 10055cc0 f i hb-ot-layout.obj
 0001:00054d70       ?sanitize@PairPosFormat1@GPOS_impl@Layout@OT@@QBE_NPAUhb_sanitize_context_t@@@Z 10055d70 f i hb-ot-layout.obj
 0001:00054ec0       ?sanitize@PairPosFormat2@GPOS_impl@Layout@OT@@QBE_NPAUhb_sanitize_context_t@@@Z 10055ec0 f i hb-ot-layout.obj
 0001:00055050       ?sanitize_shallow@?$OffsetTo@ULangSys@OT@@U?$IntType@G$01@2@$00@OT@@QBE_NPAUhb_sanitize_context_t@@PBX@Z 10056050 f i hb-ot-layout.obj
 0001:00055100       ?sanitize_value_devices@ValueFormat@GPOS_impl@Layout@OT@@ABE_NPAUhb_sanitize_context_t@@PBXPBU?$IntType@G$01@4@@Z 10056100 f i hb-ot-layout.obj
 0001:000551a0       ?sanitize_values@ValueFormat@GPOS_impl@Layout@OT@@QBE_NPAUhb_sanitize_context_t@@PBXPBU?$IntType@G$01@4@I@Z 100561a0 f i hb-ot-layout.obj
 0001:00055300       ?sanitize_values_stride_unsafe@ValueFormat@GPOS_impl@Layout@OT@@QBE_NPAUhb_sanitize_context_t@@PBXPBU?$IntType@G$01@4@II@Z 10056300 f i hb-ot-layout.obj
 0001:000553f0       ?substitute@hb_ot_map_t@@QBEXPBUhb_ot_shape_plan_t@@PAUhb_font_t@@PAUhb_buffer_t@@@Z 100563f0 f   hb-ot-layout.obj
 0001:00055480       ?transition@driver_context_t@?$KerxSubTableFormat1@UKernAATSubTableHeader@OT@@@AAT@@QAEXPAU?$StateTableDriver@UObsoleteTypes@AAT@@X@3@ABU?$Entry@X@3@@Z 10056480 f i hb-ot-layout.obj
 0001:000557c0       ?unsafe_to_concat_from_outbuffer@hb_buffer_t@@QAEXII@Z 100567c0 f i hb-ot-layout.obj
 0001:00055860       ?would_apply@ChainRuleSet@OT@@QBE_NPAUhb_would_apply_context_t@2@AAUChainContextApplyLookupContext@2@@Z 10056860 f i hb-ot-layout.obj
 0001:000559d0       ?would_apply@LigatureSubstFormat1@GSUB@Layout@OT@@QBE_NPAUhb_would_apply_context_t@4@@Z 100569d0 f i hb-ot-layout.obj
 0001:00055bb0       ?would_apply@RuleSet@OT@@QBE_NPAUhb_would_apply_context_t@2@AAUContextApplyLookupContext@2@@Z 10056bb0 f i hb-ot-layout.obj
 0001:00055d70       _hb_ot_layout_feature_with_variations_get_lookups 10056d70 f   hb-ot-layout.obj
 0001:00055db0       _hb_ot_layout_has_glyph_classes 10056db0 f   hb-ot-layout.obj
 0001:00055e00       _hb_ot_layout_has_positioning 10056e00 f   hb-ot-layout.obj
 0001:00055e50       _hb_ot_layout_has_substitution 10056e50 f   hb-ot-layout.obj
 0001:00055ea0       _hb_ot_layout_language_find_feature 10056ea0 f   hb-ot-layout.obj
 0001:00055fc0       _hb_ot_layout_language_get_required_feature 10056fc0 f   hb-ot-layout.obj
 0001:00056050       _hb_ot_layout_lookup_would_substitute 10057050 f   hb-ot-layout.obj
 0001:000561d0       _hb_ot_layout_script_select_language 100571d0 f   hb-ot-layout.obj
 0001:000562e0       _hb_ot_layout_table_find_feature_variations 100572e0 f   hb-ot-layout.obj
 0001:00056360       _hb_ot_layout_table_get_lookup_count 10057360 f   hb-ot-layout.obj
 0001:000563b0       _hb_ot_layout_table_select_script 100573b0 f   hb-ot-layout.obj
 0001:00056560       ??0hb_ot_map_builder_t@@QAE@PAUhb_face_t@@PBUhb_segment_properties_t@@@Z 10057560 f   hb-ot-map.obj
 0001:00056690       ??1hb_ot_map_builder_t@@QAE@XZ 10057690 f   hb-ot-map.obj
 0001:00056750       ?add_feature@hb_ot_map_builder_t@@QAEXIW4hb_ot_map_feature_flags_t@@I@Z 10057750 f   hb-ot-map.obj
 0001:00056870       ?add_lookups@hb_ot_map_builder_t@@AAEXAAUhb_ot_map_t@@IIII_N111@Z 10057870 f   hb-ot-map.obj
 0001:00056a70       ?add_pause@hb_ot_map_builder_t@@AAEXIP6AXPBUhb_ot_shape_plan_t@@PAUhb_font_t@@PAUhb_buffer_t@@@Z@Z 10057a70 f   hb-ot-map.obj
 0001:00056b50       ?cmp@feature_info_t@hb_ot_map_builder_t@@SAHPBX0@Z 10057b50 f i hb-ot-map.obj
 0001:00056b80       ?cmp@lookup_map_t@hb_ot_map_t@@SAHPBX0@Z 10057b80 f i hb-ot-map.obj
 0001:00056ba0       ?compile@hb_ot_map_builder_t@@QAEXAAUhb_ot_map_t@@ABUhb_ot_shape_plan_key_t@@@Z 10057ba0 f   hb-ot-map.obj
 0001:00057c90       ??$sanitize_blob@UMVAR@OT@@@hb_sanitize_context_t@@QAEPAUhb_blob_t@@PAU1@@Z 10058c90 f i hb-ot-metrics.obj
 0001:000580b0       ??C?$hb_lazy_loader_t@UMVAR@OT@@U?$hb_table_lazy_loader_t@UMVAR@OT@@$0BF@$0A@@@Uhb_face_t@@$0BF@Uhb_blob_t@@@@QBEPBUMVAR@OT@@XZ 100590b0 f i hb-ot-metrics.obj
 0001:00058200       ?_hb_ot_metrics_get_position_common@@YA_NPAUhb_font_t@@W4hb_ot_metrics_tag_t@@PAH@Z 10059200 f   hb-ot-metrics.obj
 0001:00058810       ?get_var@MVAR@OT@@QBEMIPBHI@Z 10059810 f i hb-ot-metrics.obj
 0001:00058930       ?has_data@OS2@OT@@QBE_NXZ  10059930 f i hb-ot-metrics.obj
 0001:00058990       ?sanitize@MVAR@OT@@QBE_NPAUhb_sanitize_context_t@@@Z 10059990 f i hb-ot-metrics.obj
 0001:00058b50       ?_hb_ot_shape_fallback_kern@@YAXPBUhb_ot_shape_plan_t@@PAUhb_font_t@@PAUhb_buffer_t@@@Z 10059b50 f   hb-ot-shape-fallback.obj
 0001:00058c10       ?_hb_ot_shape_fallback_mark_position@@YAXPBUhb_ot_shape_plan_t@@PAUhb_font_t@@PAUhb_buffer_t@@_N@Z 10059c10 f   hb-ot-shape-fallback.obj
 0001:00058d20       ?_hb_ot_shape_fallback_mark_position_recategorize_marks@@YAXPBUhb_ot_shape_plan_t@@PAUhb_font_t@@PAUhb_buffer_t@@@Z 10059d20 f   hb-ot-shape-fallback.obj
 0001:00058f70       ?_hb_ot_shape_fallback_spaces@@YAXPBUhb_ot_shape_plan_t@@PAUhb_font_t@@PAUhb_buffer_t@@@Z 10059f70 f   hb-ot-shape-fallback.obj
 0001:000591e0       ?kern@?$hb_kern_machine_t@Uhb_ot_shape_fallback_kern_driver_t@@@OT@@QBEXPAUhb_font_t@@PAUhb_buffer_t@@I_N@Z 1005a1e0 f i hb-ot-shape-fallback.obj
 0001:00059f40       ?_hb_ot_shape_normalize@@YAXPBUhb_ot_shape_plan_t@@PAUhb_buffer_t@@PAUhb_font_t@@@Z 1005af40 f   hb-ot-shape-normalize.obj
 0001:0005b0d0       ??$bsearch@I$00$0A@@?$hb_vector_t@Ufeature_map_t@hb_ot_map_t@@$00@@QBEPBUfeature_map_t@hb_ot_map_t@@ABIPBU12@@Z 1005c0d0 f i hb-ot-shape.obj
 0001:0005b150       ?compile@hb_ot_shape_planner_t@@QAEXAAUhb_ot_shape_plan_t@@ABUhb_ot_shape_plan_key_t@@@Z 1005c150 f   hb-ot-shape.obj
 0001:0005b560       ?fini@hb_ot_map_t@@QAEXXZ  1005c560 f i hb-ot-shape.obj
 0001:0005b5f0       ?fini@hb_ot_shape_plan_t@@QAEXXZ 1005c5f0 f   hb-ot-shape.obj
 0001:0005b640       ?get_1_mask@hb_ot_map_t@@QBEII@Z 1005c640 f i hb-ot-shape.obj
 0001:0005b660       ?has_glyph@hb_font_t@@QAE_NI@Z 1005c660 f i hb-ot-shape.obj
 0001:0005d090       ?init0@hb_ot_shape_plan_t@@QAE_NPAUhb_face_t@@PBUhb_shape_plan_key_t@@@Z 1005e090 f   hb-ot-shape.obj
 0001:0005d3a0       __hb_ot_shape              1005e3a0 f   hb-ot-shape.obj
 0001:0005d690       ?data_create_arabic@@YAPAXPBUhb_ot_shape_plan_t@@@Z 1005e690 f   hb-ot-shaper-arabic.obj
 0001:0005d7a0       ?data_destroy_arabic@@YAXPAX@Z 1005e7a0 f   hb-ot-shaper-arabic.obj
 0001:0005d8e0       ??$add_link@U?$OffsetTo@ULigatureSet@GSUB@Layout@OT@@U?$IntType@G$01@4@$00@OT@@@hb_serialize_context_t@@QAEXAAU?$OffsetTo@ULigatureSet@GSUB@Layout@OT@@U?$IntType@G$01@4@$00@OT@@IW4whence_t@0@I@Z 1005e8e0 f i hb-ot-shaper-arabic.obj
 0001:0005d8e0       ??$add_link@U?$OffsetTo@USubstLookupSubTable@GSUB@Layout@OT@@U?$IntType@G$01@4@$00@OT@@@hb_serialize_context_t@@QAEXAAU?$OffsetTo@USubstLookupSubTable@GSUB@Layout@OT@@U?$IntType@G$01@4@$00@OT@@IW4whence_t@0@I@Z 1005e8e0 f i hb-ot-shaper-arabic.obj
 0001:0005d8e0       ??$add_link@U?$OffsetTo@UCoverage@OT@@U?$IntType@G$01@2@$00@OT@@@hb_serialize_context_t@@QAEXAAU?$OffsetTo@UCoverage@OT@@U?$IntType@G$01@2@$00@OT@@IW4whence_t@0@I@Z 1005e8e0 f i hb-ot-shaper-arabic.obj
 0001:0005d8e0       ??$add_link@U?$OffsetTo@ULigature@GSUB@Layout@OT@@U?$IntType@G$01@4@$00@OT@@@hb_serialize_context_t@@QAEXAAU?$OffsetTo@ULigature@GSUB@Layout@OT@@U?$IntType@G$01@4@$00@OT@@IW4whence_t@0@I@Z 1005e8e0 f i hb-ot-shaper-arabic.obj
 0001:0005d950       ??$allocate_size@U?$IntType@G$01@OT@@@hb_serialize_context_t@@QAEPAU?$IntType@G$01@OT@@I@Z 1005e950 f i hb-ot-shaper-arabic.obj
 0001:0005e400       ??$copy@USubstLookup@GSUB@Layout@OT@@@hb_serialize_context_t@@QBEPAUSubstLookup@GSUB@Layout@OT@@XZ 1005f400 f i hb-ot-shaper-arabic.obj
 0001:0005e460       ??$extend@ULookup@OT@@$$V@hb_serialize_context_t@@QAEPAULookup@OT@@PAU12@@Z 1005f460 f i hb-ot-shaper-arabic.obj
 0001:0005e4a0       ??$extend_min@ULigatureSet@GSUB@Layout@OT@@@hb_serialize_context_t@@QAEPAULigatureSet@GSUB@Layout@OT@@PAU1234@@Z 1005f4a0 f i hb-ot-shaper-arabic.obj
 0001:0005e4a0       ??$extend_min@UCoverage@OT@@@hb_serialize_context_t@@QAEPAUCoverage@OT@@PAU12@@Z 1005f4a0 f i hb-ot-shaper-arabic.obj
 0001:0005e510       ??$extend_min@UCoverageFormat2@OT@@@hb_serialize_context_t@@QAEPAUCoverageFormat2@OT@@PAU12@@Z 1005f510 f i hb-ot-shaper-arabic.obj
 0001:0005e510       ??$extend_min@ULigature@GSUB@Layout@OT@@@hb_serialize_context_t@@QAEPAULigature@GSUB@Layout@OT@@PAU1234@@Z 1005f510 f i hb-ot-shaper-arabic.obj
 0001:0005e580       ??$extend_min@ULigatureSubstFormat1@GSUB@Layout@OT@@@hb_serialize_context_t@@QAEPAULigatureSubstFormat1@GSUB@Layout@OT@@PAU1234@@Z 1005f580 f i hb-ot-shaper-arabic.obj
 0001:0005e580       ??$extend_min@USingleSubstFormat1@GSUB@Layout@OT@@@hb_serialize_context_t@@QAEPAUSingleSubstFormat1@GSUB@Layout@OT@@PAU1234@@Z 1005f580 f i hb-ot-shaper-arabic.obj
 0001:0005e580       ??$extend_min@USingleSubstFormat2@GSUB@Layout@OT@@@hb_serialize_context_t@@QAEPAUSingleSubstFormat2@GSUB@Layout@OT@@PAU1234@@Z 1005f580 f i hb-ot-shaper-arabic.obj
 0001:0005e5f0       ??$extend_size@ULookup@OT@@@hb_serialize_context_t@@QAEPAULookup@OT@@PAU12@I@Z 1005f5f0 f i hb-ot-shaper-arabic.obj
 0001:0005e5f0       ??$extend_size@U?$ArrayOf@U?$Offset@U?$IntType@G$01@OT@@$00@OT@@U?$IntType@G$01@2@@OT@@@hb_serialize_context_t@@QAEPAU?$ArrayOf@U?$Offset@U?$IntType@G$01@OT@@$00@OT@@U?$IntType@G$01@2@@OT@@PAU12@I@Z 1005f5f0 f i hb-ot-shaper-arabic.obj
 0001:0005e5f0       ??$extend_size@U?$ArrayOf@U?$OffsetTo@ULigatureSet@GSUB@Layout@OT@@U?$IntType@G$01@4@$00@OT@@U?$IntType@G$01@2@@OT@@@hb_serialize_context_t@@QAEPAU?$ArrayOf@U?$OffsetTo@ULigatureSet@GSUB@Layout@OT@@U?$IntType@G$01@4@$00@OT@@U?$IntType@G$01@2@@OT@@PAU12@I@Z 1005f5f0 f i hb-ot-shaper-arabic.obj
 0001:0005e5f0       ??$extend_size@U?$ArrayOf@U?$OffsetTo@ULigature@GSUB@Layout@OT@@U?$IntType@G$01@4@$00@OT@@U?$IntType@G$01@2@@OT@@@hb_serialize_context_t@@QAEPAU?$ArrayOf@U?$OffsetTo@ULigature@GSUB@Layout@OT@@U?$IntType@G$01@4@$00@OT@@U?$IntType@G$01@2@@OT@@PAU12@I@Z 1005f5f0 f i hb-ot-shaper-arabic.obj
 0001:0005e5f0       ??$extend_size@U?$ArrayOf@UHBGlyphID16@OT@@U?$IntType@G$01@2@@OT@@@hb_serialize_context_t@@QAEPAU?$ArrayOf@UHBGlyphID16@OT@@U?$IntType@G$01@2@@OT@@PAU12@I@Z 1005f5f0 f i hb-ot-shaper-arabic.obj
 0001:0005e5f0       ??$extend_size@U?$ArrayOf@URangeRecord@OT@@U?$IntType@G$01@2@@OT@@@hb_serialize_context_t@@QAEPAU?$ArrayOf@URangeRecord@OT@@U?$IntType@G$01@2@@OT@@PAU12@I@Z 1005f5f0 f i hb-ot-shaper-arabic.obj
 0001:0005e5f0       ??$extend_size@U?$HeadlessArrayOf@UHBGlyphID16@OT@@U?$IntType@G$01@2@@OT@@@hb_serialize_context_t@@QAEPAU?$HeadlessArrayOf@UHBGlyphID16@OT@@U?$IntType@G$01@2@@OT@@PAU12@I@Z 1005f5f0 f i hb-ot-shaper-arabic.obj
 0001:0005e710       ??$serialize@U?$hb_map_iter_t@U?$hb_zip_iter_t@U?$hb_sorted_array_t@$$CBUHBGlyphID16@OT@@@@U?$hb_array_t@$$CBUHBGlyphID16@OT@@@@@@ABU<unnamed-type-hb_first>@@$00$0A@@@$0A@@CoverageFormat2@OT@@AAE_NPAUhb_serialize_context_t@@U?$hb_map_iter_t@U?$hb_zip_iter_t@U?$hb_sorted_array_t@$$CBUHBGlyphID16@OT@@@@U?$hb_array_t@$$CBUHBGlyphID16@OT@@@@@@ABU<unnamed-type-hb_first>@@$00$0A@@@@Z 1005f710 f i hb-ot-shaper-arabic.obj
 0001:0005e9b0       ??$serialize@U?$hb_sorted_array_t@$$CBUHBGlyphID16@OT@@@@$0A@@Coverage@OT@@QAE_NPAUhb_serialize_context_t@@U?$hb_sorted_array_t@$$CBUHBGlyphID16@OT@@@@@Z 1005f9b0 f i hb-ot-shaper-arabic.obj
 0001:0005eb60       ??$serialize@U?$hb_sorted_array_t@$$CBUHBGlyphID16@OT@@@@$0A@@CoverageFormat2@OT@@AAE_NPAUhb_serialize_context_t@@U?$hb_sorted_array_t@$$CBUHBGlyphID16@OT@@@@@Z 1005fb60 f i hb-ot-shaper-arabic.obj
 0001:0005edf0       ??$serialize@U?$hb_zip_iter_t@U?$hb_sorted_array_t@$$CBUHBGlyphID16@OT@@@@U?$hb_array_t@$$CBUHBGlyphID16@OT@@@@@@$0A@@SingleSubst@GSUB@Layout@OT@@QAE_NPAUhb_serialize_context_t@@U?$hb_zip_iter_t@U?$hb_sorted_array_t@$$CBUHBGlyphID16@OT@@@@U?$hb_array_t@$$CBUHBGlyphID16@OT@@@@@@@Z 1005fdf0 f i hb-ot-shaper-arabic.obj
 0001:0005f130       ??$serialize_serialize@AAU?$hb_map_iter_t@U?$hb_zip_iter_t@U?$hb_sorted_array_t@$$CBUHBGlyphID16@OT@@@@U?$hb_array_t@$$CBUHBGlyphID16@OT@@@@@@ABU<unnamed-type-hb_first>@@$00$0A@@@@?$OffsetTo@UCoverage@OT@@U?$IntType@G$01@2@$00@OT@@QAE_NPAUhb_serialize_context_t@@AAU?$hb_map_iter_t@U?$hb_zip_iter_t@U?$hb_sorted_array_t@$$CBUHBGlyphID16@OT@@@@U?$hb_array_t@$$CBUHBGlyphID16@OT@@@@@@ABU<unnamed-type-hb_first>@@$00$0A@@@@Z 10060130 f i hb-ot-shaper-arabic.obj
 0001:0005f420       ??$serialize_serialize@AAU?$hb_sorted_array_t@$$CBUHBGlyphID16@OT@@@@@?$OffsetTo@UCoverage@OT@@U?$IntType@G$01@2@$00@OT@@QAE_NPAUhb_serialize_context_t@@AAU?$hb_sorted_array_t@$$CBUHBGlyphID16@OT@@@@@Z 10060420 f i hb-ot-shaper-arabic.obj
 0001:0005f4f0       ??$start_serialize@USubstLookup@GSUB@Layout@OT@@@hb_serialize_context_t@@QAEPAUSubstLookup@GSUB@Layout@OT@@XZ 100604f0 f i hb-ot-shaper-arabic.obj
 0001:0005f560       ?__item__@?$hb_zip_iter_t@U?$hb_sorted_array_t@$$CBUHBGlyphID16@OT@@@@U?$hb_array_t@$$CBUHBGlyphID16@OT@@@@@@QBE?AU?$hb_pair_t@ABUHBGlyphID16@OT@@ABU12@@@XZ 10060560 f i hb-ot-shaper-arabic.obj
 0001:0005f5d0       ?__next__@?$hb_zip_iter_t@U?$hb_sorted_array_t@$$CBUHBGlyphID16@OT@@@@U?$hb_array_t@$$CBUHBGlyphID16@OT@@@@@@QAEXXZ 100605d0 f i hb-ot-shaper-arabic.obj
 0001:000607a0       ?cmp@?$IntType@G$01@OT@@SAHPBU12@0@Z 100617a0 f i hb-ot-shaper-arabic.obj
 0001:00060800       ?discard_stale_objects@hb_serialize_context_t@@QAEXXZ 10061800 f i hb-ot-shaper-arabic.obj
 0001:000609b0       ?end@?$hb_iter_t@U?$hb_map_iter_t@U?$hb_zip_iter_t@U?$hb_sorted_array_t@$$CBUHBGlyphID16@OT@@@@U?$hb_array_t@$$CBUHBGlyphID16@OT@@@@@@ABU<unnamed-type-hb_first>@@$00$0A@@@ABUHBGlyphID16@OT@@@@QBE?AU?$hb_map_iter_t@U?$hb_zip_iter_t@U?$hb_sorted_array_t@$$CBUHBGlyphID16@OT@@@@U?$hb_array_t@$$CBUHBGlyphID16@OT@@@@@@ABU<unnamed-type-hb_first>@@$00$0A@@@XZ 100619b0 f i hb-ot-shaper-arabic.obj
 0001:00060c00       ?push@?$hb_vector_t@Ulink_t@object_t@hb_serialize_context_t@@$0A@@@QAEPAUlink_t@object_t@hb_serialize_context_t@@XZ 10061c00 f i hb-ot-shaper-arabic.obj
 0001:00060ce0       ?serialize@?$ArrayOf@UHBGlyphID16@OT@@U?$IntType@G$01@2@@OT@@QAE_NPAUhb_serialize_context_t@@I@Z 10061ce0 f i hb-ot-shaper-arabic.obj
 0001:00060d60       ?serialize@?$HeadlessArrayOf@UHBGlyphID16@OT@@U?$IntType@G$01@2@@OT@@QAE_NPAUhb_serialize_context_t@@I@Z 10061d60 f i hb-ot-shaper-arabic.obj
 0001:00060df0       ?serialize@?$SortedArrayOf@URangeRecord@OT@@U?$IntType@G$01@2@@OT@@QAE_NPAUhb_serialize_context_t@@I@Z 10061df0 f i hb-ot-shaper-arabic.obj
 0001:00060e70       ?serialize@LigatureSet@GSUB@Layout@OT@@QAE_NPAUhb_serialize_context_t@@U?$hb_array_t@$$CBUHBGlyphID16@OT@@@@U?$hb_array_t@$$CBI@@AAU6@@Z 10061e70 f i hb-ot-shaper-arabic.obj
 0001:00061140       ?serialize@LigatureSubstFormat1@GSUB@Layout@OT@@QAE_NPAUhb_serialize_context_t@@U?$hb_sorted_array_t@$$CBUHBGlyphID16@OT@@@@U?$hb_array_t@$$CBI@@U?$hb_array_t@$$CBUHBGlyphID16@OT@@@@23@Z 10062140 f i hb-ot-shaper-arabic.obj
 0001:00061390       ?serialize@Lookup@OT@@QAE_NPAUhb_serialize_context_t@@III@Z 10062390 f i hb-ot-shaper-arabic.obj
 0001:000614b0       ?serialize_ligature@SubstLookup@GSUB@Layout@OT@@QAE_NPAUhb_serialize_context_t@@IU?$hb_sorted_array_t@$$CBUHBGlyphID16@OT@@@@U?$hb_array_t@$$CBI@@U?$hb_array_t@$$CBUHBGlyphID16@OT@@@@23@Z 100624b0 f i hb-ot-shaper-arabic.obj
 0001:00061640       ?setup_masks_arabic_plan@@YAXPBUarabic_shape_plan_t@@PAUhb_buffer_t@@W4hb_script_t@@@Z 10062640 f   hb-ot-shaper-arabic.obj
 0001:00062390       ?hb_indic_get_categories@@YAGI@Z 10063390 f   hb-ot-shaper-indic-table.obj
 0001:00063470       ?find_syllables_indic@@YAXPAUhb_buffer_t@@@Z 10064470 f i hb-ot-shaper-indic.obj
 0001:00063a40       ?init@hb_indic_would_substitute_feature_t@@QAEXPBUhb_ot_map_t@@I_N@Z 10064a40 f i hb-ot-shaper-indic.obj
 0001:00064970       ?would_substitute@hb_indic_would_substitute_feature_t@@QBE_NPBIIPAUhb_face_t@@@Z 10065970 f i hb-ot-shaper-indic.obj
 0001:00064d00       ?find_syllables_khmer@@YAXPAUhb_buffer_t@@@Z 10065d00 f i hb-ot-shaper-khmer.obj
 0001:00065570       ?find_syllables_myanmar@@YAXPAUhb_buffer_t@@@Z 10066570 f i hb-ot-shaper-myanmar.obj
 0001:00065b80       ?hb_syllabic_clear_var@@YAXPBUhb_ot_shape_plan_t@@PAUhb_font_t@@PAUhb_buffer_t@@@Z 10066b80 f   hb-ot-shaper-syllabic.obj
 0001:00065b90       ?hb_syllabic_insert_dotted_circles@@YAXPAUhb_font_t@@PAUhb_buffer_t@@IIHH@Z 10066b90 f   hb-ot-shaper-syllabic.obj
 0001:00066640       ??4?$machine_index_t@U?$hb_zip_iter_t@U?$hb_iota_iter_t@II@@U?$hb_filter_iter_t@U?$hb_filter_iter_t@U?$hb_zip_iter_t@U?$hb_iota_iter_t@II@@U?$hb_array_t@Uhb_glyph_info_t@@@@@@V<lambda_ce8f76acbbe9af6df8f1b6105ce8238a>@@ABU<unnamed-type-hb_second>@@$0A@@@V<lambda_daa85cc6b6d559953d3cb9980857ae51>@@ABU<unnamed-type-hb_identity>@@$0A@@@@@@@QAEXABU0@@Z 10067640 f i hb-ot-shaper-use.obj
 0001:000666b0       ??E?$hb_iter_t@U?$hb_filter_iter_t@U?$hb_filter_iter_t@U?$hb_zip_iter_t@U?$hb_iota_iter_t@II@@U?$hb_array_t@Uhb_glyph_info_t@@@@@@V<lambda_ce8f76acbbe9af6df8f1b6105ce8238a>@@ABU<unnamed-type-hb_second>@@$0A@@@V<lambda_daa85cc6b6d559953d3cb9980857ae51>@@ABU<unnamed-type-hb_identity>@@$0A@@@U?$hb_pair_t@IAAUhb_glyph_info_t@@@@@@QGAEAAU?$hb_filter_iter_t@U?$hb_filter_iter_t@U?$hb_zip_iter_t@U?$hb_iota_iter_t@II@@U?$hb_array_t@Uhb_glyph_info_t@@@@@@V<lambda_ce8f76acbbe9af6df8f1b6105ce8238a>@@ABU<unnamed-type-hb_second>@@$0A@@@V<lambda_daa85cc6b6d559953d3cb9980857ae51>@@ABU<unnamed-type-hb_identity>@@$0A@@@XZ 100676b0 f i hb-ot-shaper-use.obj
 0001:000667c0       ??F?$hb_iter_t@U?$hb_filter_iter_t@U?$hb_filter_iter_t@U?$hb_zip_iter_t@U?$hb_iota_iter_t@II@@U?$hb_array_t@Uhb_glyph_info_t@@@@@@V<lambda_ce8f76acbbe9af6df8f1b6105ce8238a>@@ABU<unnamed-type-hb_second>@@$0A@@@V<lambda_daa85cc6b6d559953d3cb9980857ae51>@@ABU<unnamed-type-hb_identity>@@$0A@@@U?$hb_pair_t@IAAUhb_glyph_info_t@@@@@@QGAEAAU?$hb_filter_iter_t@U?$hb_filter_iter_t@U?$hb_zip_iter_t@U?$hb_iota_iter_t@II@@U?$hb_array_t@Uhb_glyph_info_t@@@@@@V<lambda_ce8f76acbbe9af6df8f1b6105ce8238a>@@ABU<unnamed-type-hb_second>@@$0A@@@V<lambda_daa85cc6b6d559953d3cb9980857ae51>@@ABU<unnamed-type-hb_identity>@@$0A@@@XZ 100677c0 f i hb-ot-shaper-use.obj
 0001:000668e0       ??F?$hb_iter_t@U?$machine_index_t@U?$hb_zip_iter_t@U?$hb_iota_iter_t@II@@U?$hb_filter_iter_t@U?$hb_filter_iter_t@U?$hb_zip_iter_t@U?$hb_iota_iter_t@II@@U?$hb_array_t@Uhb_glyph_info_t@@@@@@V<lambda_ce8f76acbbe9af6df8f1b6105ce8238a>@@ABU<unnamed-type-hb_second>@@$0A@@@V<lambda_daa85cc6b6d559953d3cb9980857ae51>@@ABU<unnamed-type-hb_identity>@@$0A@@@@@@@U?$hb_pair_t@IU?$hb_pair_t@IAAUhb_glyph_info_t@@@@@@@@QAE?AU?$machine_index_t@U?$hb_zip_iter_t@U?$hb_iota_iter_t@II@@U?$hb_filter_iter_t@U?$hb_filter_iter_t@U?$hb_zip_iter_t@U?$hb_iota_iter_t@II@@U?$hb_array_t@Uhb_glyph_info_t@@@@@@V<lambda_ce8f76acbbe9af6df8f1b6105ce8238a>@@ABU<unnamed-type-hb_second>@@$0A@@@V<lambda_daa85cc6b6d559953d3cb9980857ae51>@@ABU<unnamed-type-hb_identity>@@$0A@@@@@@@H@Z 100678e0 f i hb-ot-shaper-use.obj
 0001:00066930       ??G?$hb_iter_t@U?$machine_index_t@U?$hb_zip_iter_t@U?$hb_iota_iter_t@II@@U?$hb_filter_iter_t@U?$hb_filter_iter_t@U?$hb_zip_iter_t@U?$hb_iota_iter_t@II@@U?$hb_array_t@Uhb_glyph_info_t@@@@@@V<lambda_ce8f76acbbe9af6df8f1b6105ce8238a>@@ABU<unnamed-type-hb_second>@@$0A@@@V<lambda_daa85cc6b6d559953d3cb9980857ae51>@@ABU<unnamed-type-hb_identity>@@$0A@@@@@@@U?$hb_pair_t@IU?$hb_pair_t@IAAUhb_glyph_info_t@@@@@@@@QBE?AU?$machine_index_t@U?$hb_zip_iter_t@U?$hb_iota_iter_t@II@@U?$hb_filter_iter_t@U?$hb_filter_iter_t@U?$hb_zip_iter_t@U?$hb_iota_iter_t@II@@U?$hb_array_t@Uhb_glyph_info_t@@@@@@V<lambda_ce8f76acbbe9af6df8f1b6105ce8238a>@@ABU<unnamed-type-hb_second>@@$0A@@@V<lambda_daa85cc6b6d559953d3cb9980857ae51>@@ABU<unnamed-type-hb_identity>@@$0A@@@@@@@I@Z 10067930 f i hb-ot-shaper-use.obj
 0001:000669a0       ??H?$hb_iter_t@U?$machine_index_t@U?$hb_zip_iter_t@U?$hb_iota_iter_t@II@@U?$hb_filter_iter_t@U?$hb_filter_iter_t@U?$hb_zip_iter_t@U?$hb_iota_iter_t@II@@U?$hb_array_t@Uhb_glyph_info_t@@@@@@V<lambda_ce8f76acbbe9af6df8f1b6105ce8238a>@@ABU<unnamed-type-hb_second>@@$0A@@@V<lambda_daa85cc6b6d559953d3cb9980857ae51>@@ABU<unnamed-type-hb_identity>@@$0A@@@@@@@U?$hb_pair_t@IU?$hb_pair_t@IAAUhb_glyph_info_t@@@@@@@@QBE?AU?$machine_index_t@U?$hb_zip_iter_t@U?$hb_iota_iter_t@II@@U?$hb_filter_iter_t@U?$hb_filter_iter_t@U?$hb_zip_iter_t@U?$hb_iota_iter_t@II@@U?$hb_array_t@Uhb_glyph_info_t@@@@@@V<lambda_ce8f76acbbe9af6df8f1b6105ce8238a>@@ABU<unnamed-type-hb_second>@@$0A@@@V<lambda_daa85cc6b6d559953d3cb9980857ae51>@@ABU<unnamed-type-hb_identity>@@$0A@@@@@@@I@Z 100679a0 f i hb-ot-shaper-use.obj
 0001:00066a10       ??Y?$hb_iter_t@U?$hb_zip_iter_t@U?$hb_iota_iter_t@II@@U?$hb_filter_iter_t@U?$hb_filter_iter_t@U?$hb_zip_iter_t@U?$hb_iota_iter_t@II@@U?$hb_array_t@Uhb_glyph_info_t@@@@@@V<lambda_ce8f76acbbe9af6df8f1b6105ce8238a>@@ABU<unnamed-type-hb_second>@@$0A@@@V<lambda_daa85cc6b6d559953d3cb9980857ae51>@@ABU<unnamed-type-hb_identity>@@$0A@@@@@U?$hb_pair_t@IU?$hb_pair_t@IAAUhb_glyph_info_t@@@@@@@@QGAEAAU?$hb_zip_iter_t@U?$hb_iota_iter_t@II@@U?$hb_filter_iter_t@U?$hb_filter_iter_t@U?$hb_zip_iter_t@U?$hb_iota_iter_t@II@@U?$hb_array_t@Uhb_glyph_info_t@@@@@@V<lambda_ce8f76acbbe9af6df8f1b6105ce8238a>@@ABU<unnamed-type-hb_second>@@$0A@@@V<lambda_daa85cc6b6d559953d3cb9980857ae51>@@ABU<unnamed-type-hb_identity>@@$0A@@@@@I@Z 10067a10 f i hb-ot-shaper-use.obj
 0001:00066a50       ??Z?$hb_iter_t@U?$hb_zip_iter_t@U?$hb_iota_iter_t@II@@U?$hb_filter_iter_t@U?$hb_filter_iter_t@U?$hb_zip_iter_t@U?$hb_iota_iter_t@II@@U?$hb_array_t@Uhb_glyph_info_t@@@@@@V<lambda_ce8f76acbbe9af6df8f1b6105ce8238a>@@ABU<unnamed-type-hb_second>@@$0A@@@V<lambda_daa85cc6b6d559953d3cb9980857ae51>@@ABU<unnamed-type-hb_identity>@@$0A@@@@@U?$hb_pair_t@IU?$hb_pair_t@IAAUhb_glyph_info_t@@@@@@@@QGAEAAU?$hb_zip_iter_t@U?$hb_iota_iter_t@II@@U?$hb_filter_iter_t@U?$hb_filter_iter_t@U?$hb_zip_iter_t@U?$hb_iota_iter_t@II@@U?$hb_array_t@Uhb_glyph_info_t@@@@@@V<lambda_ce8f76acbbe9af6df8f1b6105ce8238a>@@ABU<unnamed-type-hb_second>@@$0A@@@V<lambda_daa85cc6b6d559953d3cb9980857ae51>@@ABU<unnamed-type-hb_identity>@@$0A@@@@@I@Z 10067a50 f i hb-ot-shaper-use.obj
 0001:00066a90       ?__forward__@?$hb_iter_fallback_mixin_t@U?$hb_filter_iter_t@U?$hb_filter_iter_t@U?$hb_zip_iter_t@U?$hb_iota_iter_t@II@@U?$hb_array_t@Uhb_glyph_info_t@@@@@@V<lambda_ce8f76acbbe9af6df8f1b6105ce8238a>@@ABU<unnamed-type-hb_second>@@$0A@@@V<lambda_daa85cc6b6d559953d3cb9980857ae51>@@ABU<unnamed-type-hb_identity>@@$0A@@@U?$hb_pair_t@IAAUhb_glyph_info_t@@@@@@QAEXI@Z 10067a90 f i hb-ot-shaper-use.obj
 0001:00066cc0       ?__item__@?$hb_zip_iter_t@U?$hb_iota_iter_t@II@@U?$hb_array_t@Uhb_glyph_info_t@@@@@@QBE?AU?$hb_pair_t@IAAUhb_glyph_info_t@@@@XZ 10067cc0 f i hb-ot-shaper-use.obj
 0001:00066d30       ?__rewind__@?$hb_iter_fallback_mixin_t@U?$hb_filter_iter_t@U?$hb_filter_iter_t@U?$hb_zip_iter_t@U?$hb_iota_iter_t@II@@U?$hb_array_t@Uhb_glyph_info_t@@@@@@V<lambda_ce8f76acbbe9af6df8f1b6105ce8238a>@@ABU<unnamed-type-hb_second>@@$0A@@@V<lambda_daa85cc6b6d559953d3cb9980857ae51>@@ABU<unnamed-type-hb_identity>@@$0A@@@U?$hb_pair_t@IAAUhb_glyph_info_t@@@@@@QAEXI@Z 10067d30 f i hb-ot-shaper-use.obj
 0001:00068e80       ?_hb_preprocess_text_vowel_constraints@@YAXPBUhb_ot_shape_plan_t@@PAUhb_buffer_t@@PAUhb_font_t@@@Z 10069e80 f   hb-ot-shaper-vowel-constraints.obj
 0001:0006c0b0       _hb_ot_tag_to_language     1006d0b0 f   hb-ot-tag.obj
 0001:0006c220       _hb_ot_tags_from_script_and_language 1006d220 f   hb-ot-tag.obj
 0001:0006c5f0       _hb_ot_var_named_instance_get_design_coords 1006d5f0 f   hb-ot-var.obj
 0001:0006c6b0       _hb_ot_var_normalize_coords 1006d6b0 f   hb-ot-var.obj
 0001:0006c950       ?init@hb_shape_plan_key_t@@QAE_N_NPAUhb_face_t@@PBUhb_segment_properties_t@@PBUhb_feature_t@@IPBHIPBQBD@Z 1006d950 f   hb-shape-plan.obj
 0001:0006cc50       _hb_shape_plan_create2     1006dc50 f   hb-shape-plan.obj
 0001:0006cd30       _hb_shape_plan_create_cached2 1006dd30 f   hb-shape-plan.obj
 0001:0006d000       _hb_shape_plan_destroy     1006e000 f   hb-shape-plan.obj
 0001:0006d060       _hb_shape_plan_execute     1006e060 f   hb-shape-plan.obj
 0001:0006d0a0       _hb_shape_full             1006e0a0 f   hb-shape.obj
 0001:0006d180       ?_hb_shapers_get@@YAPBUhb_shaper_entry_t@@XZ 1006e180 f   hb-shaper.obj
 0001:0006d790       _hb_ucd_get_unicode_funcs  1006e790 f   hb-ucd.obj
 0001:0006d890       ?_hb_unicode_is_emoji_Extended_Pictographic@@YA_NI@Z 1006e890 f   hb-unicode.obj
 0001:0006d8f0       _hb_unicode_funcs_create   1006e8f0 f   hb-unicode.obj
 0001:0006d980       _hb_unicode_funcs_destroy  1006e980 f   hb-unicode.obj
 0001:0006da60       _hb_unicode_funcs_get_default 1006ea60 f   hb-unicode.obj
 0001:0006da70       _hb_unicode_funcs_get_empty 1006ea70 f   hb-unicode.obj
 0001:0006da80       _hb_unicode_funcs_set_combining_class_func 1006ea80 f   hb-unicode.obj
 0001:0006dad0       _hb_unicode_funcs_set_compose_func 1006ead0 f   hb-unicode.obj
 0001:0006db20       _hb_unicode_funcs_set_decompose_func 1006eb20 f   hb-unicode.obj
 0001:0006db70       _hb_unicode_funcs_set_general_category_func 1006eb70 f   hb-unicode.obj
 0001:0006dbc0       _hb_unicode_funcs_set_mirroring_func 1006ebc0 f   hb-unicode.obj
 0001:0006dc10       _hb_unicode_funcs_set_script_func 1006ec10 f   hb-unicode.obj
 0001:0006dc60       _Java_sun_font_FileFontStrike__1getGlyphImageFromWindows@32 1006ec60 f   lcdglyph.obj
 0001:0006e5c0       _Java_sun_font_FileFontStrike_initNative@8 1006f5c0 f   lcdglyph.obj
 0001:0006e5e0       _getHBScriptCode           1006f5e0 f   scriptMapping.obj
 0001:0006e600       _Java_sun_font_NullFontScaler_getGlyphImage@20 1006f600 f   sunFont.obj
 0001:0006e620       _Java_sun_font_NullFontScaler_getNullScalerContext@8 1006f620 f   sunFont.obj
 0001:0006e640       _Java_sun_font_StrikeCache_freeIntMemory@20 1006f640 f   sunFont.obj
 0001:0006e6f0       _Java_sun_font_StrikeCache_freeIntPointer@12 1006f6f0 f   sunFont.obj
 0001:0006e710       _Java_sun_font_StrikeCache_freeLongMemory@20 1006f710 f   sunFont.obj
 0001:0006e7c0       _Java_sun_font_StrikeCache_freeLongPointer@16 1006f7c0 f   sunFont.obj
 0001:0006e7e0       _Java_sun_font_StrikeCache_getGlyphCacheDescription@12 1006f7e0 f   sunFont.obj
 0001:0006e900       _Java_sun_font_SunFontManager_initIDs@8 1006f900 f   sunFont.obj
 0001:0006e910       _getSunFontIDs             1006f910 f   sunFont.obj
 0001:0006ef30       _isNullScalerContext       1006ff30 f   sunFont.obj
 0001:0006ef40       _FT_Init_FreeType          1006ff40 f   freetype:freetype.dll
 0001:0006ef46       _FT_Done_FreeType          1006ff46 f   freetype:freetype.dll
 0001:0006ef4c       _FT_New_Memory_Face        1006ff4c f   freetype:freetype.dll
 0001:0006ef52       _FT_Open_Face              1006ff52 f   freetype:freetype.dll
 0001:0006ef58       _FT_Done_Face              1006ff58 f   freetype:freetype.dll
 0001:0006ef5e       _FT_Set_Char_Size          1006ff5e f   freetype:freetype.dll
 0001:0006ef64       _FT_Load_Glyph             1006ff64 f   freetype:freetype.dll
 0001:0006ef6a       _FT_Set_Transform          1006ff6a f   freetype:freetype.dll
 0001:0006ef70       _FT_Render_Glyph           1006ff70 f   freetype:freetype.dll
 0001:0006ef76       _FT_Get_Char_Index         1006ff76 f   freetype:freetype.dll
 0001:0006ef7c       _FT_MulFix                 1006ff7c f   freetype:freetype.dll
 0001:0006ef82       _FT_Matrix_Multiply        1006ff82 f   freetype:freetype.dll
 0001:0006ef88       _FT_Outline_Get_BBox       1006ff88 f   freetype:freetype.dll
 0001:0006ef8e       _FT_Activate_Size          1006ff8e f   freetype:freetype.dll
 0001:0006ef94       _FT_Outline_Decompose      1006ff94 f   freetype:freetype.dll
 0001:0006ef9a       _FT_Outline_Get_CBox       1006ff9a f   freetype:freetype.dll
 0001:0006efa0       _FT_Outline_Translate      1006ffa0 f   freetype:freetype.dll
 0001:0006efa6       _FT_Outline_Embolden       1006ffa6 f   freetype:freetype.dll
 0001:0006efac       _FT_Library_SetLcdFilter   1006ffac f   freetype:freetype.dll
 0001:0006efb2       _FT_Property_Set           1006ffb2 f   freetype:freetype.dll
 0001:0006efb8       _JNU_ThrowOutOfMemoryError@8 1006ffb8 f   java:java.dll
 0001:0006efbe       _JNU_ThrowInternalError@8  1006ffbe f   java:java.dll
 0001:0006efc4       _JNU_ThrowArrayIndexOutOfBoundsException@8 1006ffc4 f   java:java.dll
 0001:0006efca       _JNU_NewStringPlatform@8   1006ffca f   java:java.dll
 0001:0006efd0       _SurfaceData_GetOps@8      1006ffd0 f   awt:awt.dll
 0001:0006efd6       _SurfaceData_IntersectBounds@8 1006ffd6 f   awt:awt.dll
 0001:0006efdc       _SurfaceData_InitOps@12    1006ffdc f   awt:awt.dll
 0001:0006efe2       _GetNativePrim@8           1006ffe2 f   awt:awt.dll
 0001:0006efe8       _GrPrim_Sg2dGetCompInfo@16 1006ffe8 f   awt:awt.dll
 0001:0006efee       _GrPrim_Sg2dGetClip@12     1006ffee f   awt:awt.dll
 0001:0006eff4       _GrPrim_Sg2dGetPixel@8     1006fff4 f   awt:awt.dll
 0001:0006effa       _GrPrim_Sg2dGetEaRGB@8     1006fffa f   awt:awt.dll
 0001:0006f000       _GrPrim_Sg2dGetLCDTextContrast@8 10070000 f   awt:awt.dll
 0001:0006f006       _AccelGlyphCache_RemoveAllCellInfos 10070006 f   awt:awt.dll
 0001:0006f00c       @__security_check_cookie@4 1007000c f   MSVCRT:secchk.obj
 0001:0006f020       __ftoui3                   10070020 f   MSVCRT:ftol3.obj
 0001:0006f066       __ftoul3                   10070066 f   MSVCRT:ftol3.obj
 0001:0006f0d8       __ftol3                    100700d8 f   MSVCRT:ftol3.obj
 0001:0006f145       __dtoui3                   10070145 f   MSVCRT:ftol3.obj
 0001:0006f1b9       __dtoul3                   100701b9 f   MSVCRT:ftol3.obj
 0001:0006f25b       __dtol3                    1007025b f   MSVCRT:ftol3.obj
 0001:0006f310       __ultod3                   10070310 f   MSVCRT:ftol3.obj
 0001:0006f370       __ltod3                    10070370 f   MSVCRT:ftol3.obj
 0001:0006f3c0       __allmul                   100703c0 f   MSVCRT:llmul.obj
 0001:0006f3f4       ___raise_securityfailure   100703f4 f   MSVCRT:gs_report.obj
 0001:0006f41c       ___report_gsfailure        1007041c f   MSVCRT:gs_report.obj
 0001:0006f515       ___report_rangecheckfailure 10070515 f   MSVCRT:gs_report.obj
 0001:0006f521       ___report_securityfailure  10070521 f   MSVCRT:gs_report.obj
 0001:0006f5f0       __alldiv                   100705f0 f   MSVCRT:lldiv.obj
 0001:0006f6a0       __alloca_probe             100706a0 f   MSVCRT:chkstk.obj
 0001:0006f6a0       __chkstk                   100706a0 f   MSVCRT:chkstk.obj
 0001:0006f6d0       __ftoi2                    100706d0 f   MSVCRT:ftol2.obj
 0001:0006f6d0       __ftol2_sse_excpt          100706d0     MSVCRT:ftol2.obj
 0001:0006f6d0       __ftol2_sse                100706d0     MSVCRT:ftol2.obj
 0001:0006f750       __ftoui2                   10070750 f   MSVCRT:ftol2.obj
 0001:0006f800       __ftol2                    10070800 f   MSVCRT:ftol2.obj
 0001:0006f8b0       __ftoul2                   100708b0 f   MSVCRT:ftol2.obj
 0001:0006f970       __alloca_probe_16          10070970 f   MSVCRT:alloca16.obj
 0001:0006f986       __alloca_probe_8           10070986     MSVCRT:alloca16.obj
 0001:0006fcdc       __DllMainCRTStartup@12     10070cdc f   MSVCRT:dll_dllmain.obj
 0001:0006fcff       ___isa_available_init      10070cff f   MSVCRT:cpu_disp.obj
 0001:0006ff1c       ___security_init_cookie    10070f1c f   MSVCRT:gs_support.obj
 0001:0006ff67       _DllMain@12                10070f67 f   MSVCRT:dll_dllmain_stub.obj
 0001:0006ff89       ?__scrt_initialize_type_info@@YAXXZ 10070f89 f   MSVCRT:tncleanup.obj
 0001:0006ff95       ?__scrt_uninitialize_type_info@@YAXXZ 10070f95 f   MSVCRT:tncleanup.obj
 0001:0006ffa1       ___local_stdio_scanf_options 10070fa1 f i MSVCRT:default_local_stdio_options.obj
 0001:0006ffa7       ___scrt_initialize_default_local_stdio_options 10070fa7 f   MSVCRT:default_local_stdio_options.obj
 0001:00070008       ___scrt_acquire_startup_lock 10071008 f   MSVCRT:utility.obj
 0001:0007003a       ___scrt_dllmain_after_initialize_c 1007103a f   MSVCRT:utility.obj
 0001:00070065       ___scrt_dllmain_before_initialize_c 10071065 f   MSVCRT:utility.obj
 0001:00070073       ___scrt_dllmain_crt_thread_attach 10071073 f   MSVCRT:utility.obj
 0001:00070092       ___scrt_dllmain_crt_thread_detach 10071092 f   MSVCRT:utility.obj
 0001:0007009f       ___scrt_dllmain_exception_filter 1007109f f   MSVCRT:utility.obj
 0001:000700d3       ___scrt_dllmain_uninitialize_c 100710d3 f   MSVCRT:utility.obj
 0001:000700f6       ___scrt_dllmain_uninitialize_critical 100710f6 f   MSVCRT:utility.obj
 0001:00070103       ___scrt_initialize_crt     10071103 f   MSVCRT:utility.obj
 0001:0007013c       ___scrt_initialize_onexit_tables 1007113c f   MSVCRT:utility.obj
 0001:000701c3       ___scrt_is_nonwritable_in_current_image 100711c3 f   MSVCRT:utility.obj
 0001:00070257       ___scrt_release_startup_lock 10071257 f   MSVCRT:utility.obj
 0001:00070274       ___scrt_uninitialize_crt   10071274 f   MSVCRT:utility.obj
 0001:0007029c       ___scrt_get_dyn_tls_init_callback 1007129c f   MSVCRT:dyn_tls_init.obj
 0001:000702a2       ___scrt_fastfail           100712a2 f   MSVCRT:utility_desktop.obj
 0001:000703bc       __crt_debugger_hook        100713bc f   MSVCRT:utility_desktop.obj
 0001:000703c4       __RTC_Initialize           100713c4 f   MSVCRT:initsect.obj
 0001:000703f0       __RTC_Terminate            100713f0 f   MSVCRT:initsect.obj
 0001:00070420       __SEH_prolog4              10071420 f   MSVCRT:sehprolg4.obj
 0001:00070464       __SEH_epilog4              10071464 f   MSVCRT:sehprolg4.obj
 0001:00070478       __except_handler4          10071478 f   MSVCRT:chandler4gs.obj
 0001:000704a7       __get_startup_argv_mode    100714a7 f   MSVCRT:argv_mode.obj
 0001:000704ab       ___scrt_is_ucrt_dll_in_use 100714ab f   MSVCRT:ucrt_detection.obj
 0001:000704b7       _IsProcessorFeaturePresent@4 100714b7 f   kernel32:KERNEL32.dll
 0001:000704bd       _memset                    100714bd f   vcruntime:VCRUNTIME140.dll
 0001:000704c3       _strrchr                   100714c3 f   vcruntime:VCRUNTIME140.dll
 0001:000704c9       _wcsrchr                   100714c9 f   vcruntime:VCRUNTIME140.dll
 0001:000704cf       _wcsstr                    100714cf f   vcruntime:VCRUNTIME140.dll
 0001:000704d5       _strstr                    100714d5 f   vcruntime:VCRUNTIME140.dll
 0001:000704db       _memcpy                    100714db f   vcruntime:VCRUNTIME140.dll
 0001:000704e1       _memmove                   100714e1 f   vcruntime:VCRUNTIME140.dll
 0001:000704e7       _strchr                    100714e7 f   vcruntime:VCRUNTIME140.dll
 0001:000704ed       ___std_type_info_destroy_list 100714ed f   vcruntime:VCRUNTIME140.dll
 0001:000704f3       __except_handler4_common   100714f3 f   vcruntime:VCRUNTIME140.dll
 0001:000704f9       __libm_sse2_pow_precise    100714f9 f   ucrt:api-ms-win-crt-math-l1-1-0.dll
 0001:000704ff       _floor                     100714ff f   ucrt:api-ms-win-crt-math-l1-1-0.dll
 0001:00070505       __libm_sse2_sqrt_precise   10071505 f   ucrt:api-ms-win-crt-math-l1-1-0.dll
 0001:0007050b       _ceil                      1007150b f   ucrt:api-ms-win-crt-math-l1-1-0.dll
 0001:00070511       __initterm                 10071511 f   ucrt:api-ms-win-crt-runtime-l1-1-0.dll
 0001:00070517       __initterm_e               10071517 f   ucrt:api-ms-win-crt-runtime-l1-1-0.dll
 0001:0007051d       __seh_filter_dll           1007151d f   ucrt:api-ms-win-crt-runtime-l1-1-0.dll
 0001:00070523       __configure_narrow_argv    10071523 f   ucrt:api-ms-win-crt-runtime-l1-1-0.dll
 0001:00070529       __initialize_narrow_environment 10071529 f   ucrt:api-ms-win-crt-runtime-l1-1-0.dll
 0001:0007052f       __initialize_onexit_table  1007152f f   ucrt:api-ms-win-crt-runtime-l1-1-0.dll
 0001:00070535       __execute_onexit_table     10071535 f   ucrt:api-ms-win-crt-runtime-l1-1-0.dll
 0001:0007053b       __cexit                    1007153b f   ucrt:api-ms-win-crt-runtime-l1-1-0.dll
 0001:00070541       ___vcrt_initialize         10071541 f   MSVCRT:ucrt_stubs.obj
 0001:00070541       ___acrt_initialize         10071541 f   MSVCRT:ucrt_stubs.obj
 0001:00070541       ___scrt_stub_for_acrt_thread_attach 10071541 f   MSVCRT:ucrt_stubs.obj
 0001:00070541       ___vcrt_uninitialize       10071541 f   MSVCRT:ucrt_stubs.obj
 0001:00070541       ___acrt_thread_attach      10071541 f   MSVCRT:ucrt_stubs.obj
 0001:00070541       ___vcrt_thread_detach      10071541 f   MSVCRT:ucrt_stubs.obj
 0001:00070541       ___vcrt_thread_attach      10071541 f   MSVCRT:ucrt_stubs.obj
 0001:00070541       ___acrt_thread_detach      10071541 f   MSVCRT:ucrt_stubs.obj
 0001:00070541       ___acrt_uninitialize       10071541 f   MSVCRT:ucrt_stubs.obj
 0001:00070541       ___scrt_stub_for_acrt_initialize 10071541 f   MSVCRT:ucrt_stubs.obj
 0001:00070541       ___scrt_stub_for_acrt_uninitialize_critical 10071541 f   MSVCRT:ucrt_stubs.obj
 0001:00070541       ___acrt_uninitialize_critical 10071541 f   MSVCRT:ucrt_stubs.obj
 0001:00070541       ___scrt_stub_for_acrt_uninitialize 10071541 f   MSVCRT:ucrt_stubs.obj
 0001:00070541       ___vcrt_uninitialize_critical 10071541 f   MSVCRT:ucrt_stubs.obj
 0001:00070541       ___scrt_stub_for_acrt_thread_detach 10071541 f   MSVCRT:ucrt_stubs.obj
 0001:00070544       __filter_x86_sse2_floating_point_exception 10071544 f   MSVCRT:x86_exception_filter.obj
 0001:00070544       __filter_x86_sse2_floating_point_exception_default 10071544 f   MSVCRT:x86_exception_filter.obj
 0002:00000000       __imp__RegCloseKey@4       10072000     advapi32:ADVAPI32.dll
 0002:00000004       __imp__RegOpenKeyExA@20    10072004     advapi32:ADVAPI32.dll
 0002:00000008       __imp__RegQueryInfoKeyW@48 10072008     advapi32:ADVAPI32.dll
 0002:0000000c       __imp__RegEnumValueW@32    1007200c     advapi32:ADVAPI32.dll
 0002:00000010       \177ADVAPI32_NULL_THUNK_DATA 10072010     advapi32:ADVAPI32.dll
 0002:00000014       __imp__DeleteObject@4      10072014     gdi32:GDI32.dll
 0002:00000018       __imp__CreateFontIndirectW@4 10072018     gdi32:GDI32.dll
 0002:0000001c       __imp__CreateCompatibleDC@4 1007201c     gdi32:GDI32.dll
 0002:00000020       __imp__CreateCompatibleBitmap@12 10072020     gdi32:GDI32.dll
 0002:00000024       __imp__GetDIBits@28        10072024     gdi32:GDI32.dll
 0002:00000028       __imp__SelectObject@8      10072028     gdi32:GDI32.dll
 0002:0000002c       __imp__SetBkColor@8        1007202c     gdi32:GDI32.dll
 0002:00000030       __imp__SetMapMode@8        10072030     gdi32:GDI32.dll
 0002:00000034       __imp__GetTextMetricsA@8   10072034     gdi32:GDI32.dll
 0002:00000038       __imp__ExtTextOutW@32      10072038     gdi32:GDI32.dll
 0002:0000003c       __imp__GetDeviceCaps@8     1007203c     gdi32:GDI32.dll
 0002:00000040       __imp__GetFontData@20      10072040     gdi32:GDI32.dll
 0002:00000044       __imp__GetGlyphOutlineA@28 10072044     gdi32:GDI32.dll
 0002:00000048       __imp__EnumFontFamiliesExW@20 10072048     gdi32:GDI32.dll
 0002:0000004c       __imp__SetTextColor@8      1007204c     gdi32:GDI32.dll
 0002:00000050       __imp__GetStockObject@4    10072050     gdi32:GDI32.dll
 0002:00000054       \177GDI32_NULL_THUNK_DATA  10072054     gdi32:GDI32.dll
 0002:00000058       __imp__GetSystemDirectoryA@8 10072058     kernel32:KERNEL32.dll
 0002:0000005c       __imp__EnterCriticalSection@4 1007205c     kernel32:KERNEL32.dll
 0002:00000060       __imp__LeaveCriticalSection@4 10072060     kernel32:KERNEL32.dll
 0002:00000064       __imp__DeleteCriticalSection@4 10072064     kernel32:KERNEL32.dll
 0002:00000068       __imp__UnhandledExceptionFilter@4 10072068     kernel32:KERNEL32.dll
 0002:0000006c       __imp__SetUnhandledExceptionFilter@4 1007206c     kernel32:KERNEL32.dll
 0002:00000070       __imp__GetCurrentProcess@0 10072070     kernel32:KERNEL32.dll
 0002:00000074       __imp__TerminateProcess@8  10072074     kernel32:KERNEL32.dll
 0002:00000078       __imp__IsProcessorFeaturePresent@4 10072078     kernel32:KERNEL32.dll
 0002:0000007c       __imp__QueryPerformanceCounter@4 1007207c     kernel32:KERNEL32.dll
 0002:00000080       __imp__GetCurrentProcessId@0 10072080     kernel32:KERNEL32.dll
 0002:00000084       __imp__GetCurrentThreadId@0 10072084     kernel32:KERNEL32.dll
 0002:00000088       __imp__GetSystemTimeAsFileTime@4 10072088     kernel32:KERNEL32.dll
 0002:0000008c       __imp__DisableThreadLibraryCalls@4 1007208c     kernel32:KERNEL32.dll
 0002:00000090       __imp__InitializeSListHead@4 10072090     kernel32:KERNEL32.dll
 0002:00000094       __imp__IsDebuggerPresent@0 10072094     kernel32:KERNEL32.dll
 0002:00000098       __imp__GetWindowsDirectoryA@8 10072098     kernel32:KERNEL32.dll
 0002:0000009c       \177KERNEL32_NULL_THUNK_DATA 1007209c     kernel32:KERNEL32.dll
 0002:000000a0       __imp__GetDesktopWindow@0  100720a0     user32:USER32.dll
 0002:000000a4       __imp__FillRect@12         100720a4     user32:USER32.dll
 0002:000000a8       __imp__GetWindowDC@4       100720a8     user32:USER32.dll
 0002:000000ac       __imp__ReleaseDC@8         100720ac     user32:USER32.dll
 0002:000000b0       __imp__GetDC@4             100720b0     user32:USER32.dll
 0002:000000b4       __imp__SystemParametersInfoA@16 100720b4     user32:USER32.dll
 0002:000000b8       \177USER32_NULL_THUNK_DATA 100720b8     user32:USER32.dll
 0002:000000bc       __imp__memmove             100720bc     vcruntime:VCRUNTIME140.dll
 0002:000000c0       __imp__strchr              100720c0     vcruntime:VCRUNTIME140.dll
 0002:000000c4       __imp__strstr              100720c4     vcruntime:VCRUNTIME140.dll
 0002:000000c8       __imp__wcsstr              100720c8     vcruntime:VCRUNTIME140.dll
 0002:000000cc       __imp__wcsrchr             100720cc     vcruntime:VCRUNTIME140.dll
 0002:000000d0       __imp__strrchr             100720d0     vcruntime:VCRUNTIME140.dll
 0002:000000d4       __imp__memset              100720d4     vcruntime:VCRUNTIME140.dll
 0002:000000d8       __imp___except_handler4_common 100720d8     vcruntime:VCRUNTIME140.dll
 0002:000000dc       __imp__memcpy              100720dc     vcruntime:VCRUNTIME140.dll
 0002:000000e0       __imp____std_type_info_destroy_list 100720e0     vcruntime:VCRUNTIME140.dll
 0002:000000e4       \177VCRUNTIME140_NULL_THUNK_DATA 100720e4     vcruntime:VCRUNTIME140.dll
 0002:000000e8       __imp__strtol              100720e8     ucrt:api-ms-win-crt-convert-l1-1-0.dll
 0002:000000ec       \177api-ms-win-crt-convert-l1-1-0_NULL_THUNK_DATA 100720ec     ucrt:api-ms-win-crt-convert-l1-1-0.dll
 0002:000000f0       __imp__getenv              100720f0     ucrt:api-ms-win-crt-environment-l1-1-0.dll
 0002:000000f4       \177api-ms-win-crt-environment-l1-1-0_NULL_THUNK_DATA 100720f4     ucrt:api-ms-win-crt-environment-l1-1-0.dll
 0002:000000f8       __imp__realloc             100720f8     ucrt:api-ms-win-crt-heap-l1-1-0.dll
 0002:000000fc       __imp__malloc              100720fc     ucrt:api-ms-win-crt-heap-l1-1-0.dll
 0002:00000100       __imp__free                10072100     ucrt:api-ms-win-crt-heap-l1-1-0.dll
 0002:00000104       __imp__calloc              10072104     ucrt:api-ms-win-crt-heap-l1-1-0.dll
 0002:00000108       \177api-ms-win-crt-heap-l1-1-0_NULL_THUNK_DATA 10072108     ucrt:api-ms-win-crt-heap-l1-1-0.dll
 0002:0000010c       __imp___libm_sse2_pow_precise 1007210c     ucrt:api-ms-win-crt-math-l1-1-0.dll
 0002:00000110       __imp__ceil                10072110     ucrt:api-ms-win-crt-math-l1-1-0.dll
 0002:00000114       __imp___libm_sse2_sqrt_precise 10072114     ucrt:api-ms-win-crt-math-l1-1-0.dll
 0002:00000118       __imp__floor               10072118     ucrt:api-ms-win-crt-math-l1-1-0.dll
 0002:0000011c       \177api-ms-win-crt-math-l1-1-0_NULL_THUNK_DATA 1007211c     ucrt:api-ms-win-crt-math-l1-1-0.dll
 0002:00000120       __imp___cexit              10072120     ucrt:api-ms-win-crt-runtime-l1-1-0.dll
 0002:00000124       __imp___configure_narrow_argv 10072124     ucrt:api-ms-win-crt-runtime-l1-1-0.dll
 0002:00000128       __imp___initterm_e         10072128     ucrt:api-ms-win-crt-runtime-l1-1-0.dll
 0002:0000012c       __imp___seh_filter_dll     1007212c     ucrt:api-ms-win-crt-runtime-l1-1-0.dll
 0002:00000130       __imp___initialize_onexit_table 10072130     ucrt:api-ms-win-crt-runtime-l1-1-0.dll
 0002:00000134       __imp___initialize_narrow_environment 10072134     ucrt:api-ms-win-crt-runtime-l1-1-0.dll
 0002:00000138       __imp___execute_onexit_table 10072138     ucrt:api-ms-win-crt-runtime-l1-1-0.dll
 0002:0000013c       __imp___errno              1007213c     ucrt:api-ms-win-crt-runtime-l1-1-0.dll
 0002:00000140       __imp___initterm           10072140     ucrt:api-ms-win-crt-runtime-l1-1-0.dll
 0002:00000144       \177api-ms-win-crt-runtime-l1-1-0_NULL_THUNK_DATA 10072144     ucrt:api-ms-win-crt-runtime-l1-1-0.dll
 0002:00000148       __imp____stdio_common_vsprintf 10072148     ucrt:api-ms-win-crt-stdio-l1-1-0.dll
 0002:0000014c       __imp____stdio_common_vfprintf 1007214c     ucrt:api-ms-win-crt-stdio-l1-1-0.dll
 0002:00000150       __imp____acrt_iob_func     10072150     ucrt:api-ms-win-crt-stdio-l1-1-0.dll
 0002:00000154       \177api-ms-win-crt-stdio-l1-1-0_NULL_THUNK_DATA 10072154     ucrt:api-ms-win-crt-stdio-l1-1-0.dll
 0002:00000158       __imp___stricmp            10072158     ucrt:api-ms-win-crt-string-l1-1-0.dll
 0002:00000158       __imp__stricmp             10072158     ucrt:api-ms-win-crt-string-l1-1-0.dll
 0002:0000015c       __imp__strncmp             1007215c     ucrt:api-ms-win-crt-string-l1-1-0.dll
 0002:00000160       __imp__strncpy             10072160     ucrt:api-ms-win-crt-string-l1-1-0.dll
 0002:00000164       __imp__wcsicmp             10072164     ucrt:api-ms-win-crt-string-l1-1-0.dll
 0002:00000164       __imp___wcsicmp            10072164     ucrt:api-ms-win-crt-string-l1-1-0.dll
 0002:00000168       \177api-ms-win-crt-string-l1-1-0_NULL_THUNK_DATA 10072168     ucrt:api-ms-win-crt-string-l1-1-0.dll
 0002:0000016c       __imp__SurfaceData_IntersectBounds@8 1007216c     awt:awt.dll
 0002:00000170       __imp__SurfaceData_InitOps@12 10072170     awt:awt.dll
 0002:00000174       __imp__GetNativePrim@8     10072174     awt:awt.dll
 0002:00000178       __imp__GrPrim_Sg2dGetCompInfo@16 10072178     awt:awt.dll
 0002:0000017c       __imp__SurfaceData_GetOps@8 1007217c     awt:awt.dll
 0002:00000180       __imp__GrPrim_Sg2dGetPixel@8 10072180     awt:awt.dll
 0002:00000184       __imp__GrPrim_Sg2dGetEaRGB@8 10072184     awt:awt.dll
 0002:00000188       __imp__GrPrim_Sg2dGetLCDTextContrast@8 10072188     awt:awt.dll
 0002:0000018c       __imp__AccelGlyphCache_RemoveAllCellInfos 1007218c     awt:awt.dll
 0002:00000190       __imp__GrPrim_Sg2dGetClip@12 10072190     awt:awt.dll
 0002:00000194       \177awt_NULL_THUNK_DATA    10072194     awt:awt.dll
 0002:00000198       __imp__FT_Render_Glyph     10072198     freetype:freetype.dll
 0002:0000019c       __imp__FT_Done_FreeType    1007219c     freetype:freetype.dll
 0002:000001a0       __imp__FT_Property_Set     100721a0     freetype:freetype.dll
 0002:000001a4       __imp__FT_Library_SetLcdFilter 100721a4     freetype:freetype.dll
 0002:000001a8       __imp__FT_Outline_Embolden 100721a8     freetype:freetype.dll
 0002:000001ac       __imp__FT_Outline_Translate 100721ac     freetype:freetype.dll
 0002:000001b0       __imp__FT_Outline_Get_CBox 100721b0     freetype:freetype.dll
 0002:000001b4       __imp__FT_Outline_Decompose 100721b4     freetype:freetype.dll
 0002:000001b8       __imp__FT_Activate_Size    100721b8     freetype:freetype.dll
 0002:000001bc       __imp__FT_Outline_Get_BBox 100721bc     freetype:freetype.dll
 0002:000001c0       __imp__FT_Matrix_Multiply  100721c0     freetype:freetype.dll
 0002:000001c4       __imp__FT_MulFix           100721c4     freetype:freetype.dll
 0002:000001c8       __imp__FT_Get_Char_Index   100721c8     freetype:freetype.dll
 0002:000001cc       __imp__FT_Init_FreeType    100721cc     freetype:freetype.dll
 0002:000001d0       __imp__FT_Set_Transform    100721d0     freetype:freetype.dll
 0002:000001d4       __imp__FT_Load_Glyph       100721d4     freetype:freetype.dll
 0002:000001d8       __imp__FT_Set_Char_Size    100721d8     freetype:freetype.dll
 0002:000001dc       __imp__FT_New_Memory_Face  100721dc     freetype:freetype.dll
 0002:000001e0       __imp__FT_Open_Face        100721e0     freetype:freetype.dll
 0002:000001e4       __imp__FT_Done_Face        100721e4     freetype:freetype.dll
 0002:000001e8       \177freetype_NULL_THUNK_DATA 100721e8     freetype:freetype.dll
 0002:000001ec       __imp__JNU_ThrowInternalError@8 100721ec     java:java.dll
 0002:000001f0       __imp__JNU_NewStringPlatform@8 100721f0     java:java.dll
 0002:000001f4       __imp__JNU_ThrowOutOfMemoryError@8 100721f4     java:java.dll
 0002:000001f8       __imp__JNU_ThrowArrayIndexOutOfBoundsException@8 100721f8     java:java.dll
 0002:000001fc       \177java_NULL_THUNK_DATA   100721fc     java:java.dll
 0002:00000200       ___guard_check_icall_fptr  10072200     MSVCRT:guard_support.obj
 0002:00000204       ___xc_a                    10072204     MSVCRT:initializers.obj
 0002:00000208       ___xc_z                    10072208     MSVCRT:initializers.obj
 0002:0000020c       ___xi_a                    1007220c     MSVCRT:initializers.obj
 0002:00000210       ___xi_z                    10072210     MSVCRT:initializers.obj
 0002:00000214       ___xp_a                    10072214     MSVCRT:initializers.obj
 0002:00000218       ___xp_z                    10072218     MSVCRT:initializers.obj
 0002:0000021c       ___xt_a                    1007221c     MSVCRT:initializers.obj
 0002:00000220       ___xt_z                    10072220     MSVCRT:initializers.obj
 0002:00000230       ??_C@_0CJ@PGKOGMIO@Unsupported?5mode?5for?5glyph?5imag@ 10072230     ColorGlyphSurfaceData.obj
 0002:0000025c       ??_C@_0CP@FKLHLEEM@Initialization?5of?5ColorGlyphSur@ 1007225c     ColorGlyphSurfaceData.obj
 0002:0000028c       __real@3eaaaaaa            1007228c     DrawGlyphList.obj
 0002:00000290       __real@3ff0000000000000    10072290     DrawGlyphList.obj
 0002:00000298       __real@40400000            10072298     DrawGlyphList.obj
 0002:000002a0       __real@4059000000000000    100722a0     DrawGlyphList.obj
 0002:000002a8       __real@406fe00000000000    100722a8     DrawGlyphList.obj
 0002:000002b0       ??_C@_0BM@DODCGPJL@sun?1font?1GlyphLayout$GVData@ 100722b0     HBShaper.obj
 0002:000002cc       ??_C@_01JPJNBJEM@I@        100722cc     HBShaper.obj
 0002:000002d0       ??_C@_06HHPHCOMB@_count@   100722d0     HBShaper.obj
 0002:000002d8       ??_C@_06PPHBKICC@_flags@   100722d8     HBShaper.obj
 0002:000002e0       ??_C@_02EBOMBDPA@?$FLI@    100722e0     HBShaper.obj
 0002:000002e4       ??_C@_07PKNHOODJ@_glyphs@  100722e4     HBShaper.obj
 0002:000002ec       ??_C@_02MGHEAPDP@?$FLF@    100722ec     HBShaper.obj
 0002:000002f0       ??_C@_0L@BHNDECPI@_positions@ 100722f0     HBShaper.obj
 0002:000002fc       ??_C@_08MEOKMKLN@_indices@ 100722fc     HBShaper.obj
 0002:00000308       ??_C@_03GAEACAIP@?$CI?$CJV@ 10072308     HBShaper.obj
 0002:0000030c       ??_C@_04PAAMKIIE@grow@     1007230c     HBShaper.obj
 0002:00000311       ??_C@_00CNPNBAHC@@         10072311     HBShaper.obj
 0002:00000314       ??_C@_0L@LCGIKEMB@HB_NODEVTX@ 10072314     HBShaper.obj
 0002:00000320       ??_C@_04HHMMLDJI@kern@     10072320     HBShaper.obj
 0002:00000328       ??_C@_05LLBOPDMO@?9kern@   10072328     HBShaper.obj
 0002:00000330       ??_C@_04BCEPKNGE@liga@     10072330     HBShaper.obj
 0002:00000338       ??_C@_05NOJNONDC@?9liga@   10072338     HBShaper.obj
 0002:00000340       __real@37800000            10072340     HBShaper.obj
 0002:00000344       __real@3f000000            10072344     HBShaper.obj
 0002:00000348       __real@3f800000            10072348     HBShaper.obj
 0002:00000350       __xmm@80000000800000008000000080000000 10072350     HBShaper.obj
 0002:000003c4       ??_C@_07GCCENIMJ@?2System@ 100723c4     fontpath.obj
 0002:000003cc       ??_C@_09FJGNFLHN@?2System32@ 100723cc     fontpath.obj
 0002:000003d8       ??_C@_06MIJGMACG@?2Fonts@  100723d8     fontpath.obj
 0002:000003e0       ??_C@_01ICJEACDI@?$DL@     100723e0     fontpath.obj
 0002:000003e4       ??_C@_17BCGMALNF@?$AA?5?$AA?$CG?$AA?5@ 100723e4     fontpath.obj
 0002:000003ec       ??_C@_19OLAFNMII@?$AA?4?$AAt?$AAt?$AAf@ 100723ec     fontpath.obj
 0002:000003f8       ??_C@_19MKNEPBPF@?$AA?4?$AAo?$AAt?$AAf@ 100723f8     fontpath.obj
 0002:00000404       ??_C@_0BC@LEKPNIDO@java?1util?1HashMap@ 10072404     fontpath.obj
 0002:00000418       ??_C@_0DJ@FLFJBGBN@?$CILjava?1lang?1Object?$DLLjava?1lang?1O@ 10072418     fontpath.obj
 0002:00000454       ??_C@_03KMONJGDG@put@      10072454     fontpath.obj
 0002:00000458       ??_C@_0BG@DHOOFEJE@?$CILjava?1lang?1Object?$DL?$CJZ@ 10072458     fontpath.obj
 0002:00000470       ??_C@_0M@ILMAKOC@containsKey@ 10072470     fontpath.obj
 0002:0000047c       ??_C@_0BE@GPOIDJOH@java?1util?1ArrayList@ 1007247c     fontpath.obj
 0002:00000490       ??_C@_04PFANPMCN@?$CII?$CJV@ 10072490     fontpath.obj
 0002:00000498       ??_C@_06FALKBLGB@?$DMinit?$DO@ 10072498     fontpath.obj
 0002:000004a0       ??_C@_03BDGOHNNK@add@      100724a0     fontpath.obj
 0002:000004a4       ??_C@_0BB@FLFAIHG@java?1lang?1String@ 100724a4     fontpath.obj
 0002:000004b8       ??_C@_0CH@BHMNPKMP@?$CILjava?1util?1Locale?$DL?$CJLjava?1lang?1@ 100724b8     fontpath.obj
 0002:000004e0       ??_C@_0M@IMBDOEKL@toLowerCase@ 100724e0     fontpath.obj
 0002:00000504       ??_C@_0BB@NIMAMPFF@invalidateScaler@ 10072504     freetypeScaler.obj
 0002:00000518       ??_C@_0BE@LLDKDDBI@FREETYPE_PROPERTIES@ 10072518     freetypeScaler.obj
 0002:0000052c       ??_C@_08OKLLNAKL@truetype@ 1007252c     freetypeScaler.obj
 0002:00000538       ??_C@_0BE@OJJAFABD@interpreter?9version@ 10072538     freetypeScaler.obj
 0002:0000054c       __real@00000000            1007254c     freetypeScaler.obj
 0002:00000550       __real@3c800000            10072550     freetypeScaler.obj
 0002:00000558       __real@3ef0000000000000    10072558     freetypeScaler.obj
 0002:00000560       __real@3f90000000000000    10072560     freetypeScaler.obj
 0002:00000568       __real@4050000000000000    10072568     freetypeScaler.obj
 0002:00000570       __real@40f0000000000000    10072570     freetypeScaler.obj
 0002:00000578       __real@42800000            10072578     freetypeScaler.obj
 0002:00000580       __real@c0f0000000000000    10072580     freetypeScaler.obj
 0002:00000590       __xmm@00010000000000000000366a00010000 10072590     freetypeScaler.obj
 0002:000005a0       __xmm@80000000000000008000000000000000 100725a0     freetypeScaler.obj
 0002:00000a88       ??_C@_08EMNHGPIL@SANITIZE@ 10072a88     hb-aat-layout.obj
 0002:00000a94       ??_C@_0BL@LJCAAAA@start?5?$FL?$CFp?4?4?$CFp?$FN?5?$CI?$CFlu?5bytes?$CJ@ 10072a94     hb-aat-layout.obj
 0002:00000ab0       ??_C@_0BO@NFKLCDNJ@end?5?$FL?$CFp?4?4?$CFp?$FN?5?$CFu?5edit?5requests@ 10072ab0     hb-aat-layout.obj
 0002:00000ad0       ??_C@_02GIPFHKNO@OK@       10072ad0     hb-aat-layout.obj
 0002:00000ad4       ??_C@_0N@FLBMHONH@OUT?9OF?9RANGE@ 10072ad4     hb-aat-layout.obj
 0002:00000ae4       ??_C@_0DC@HBKIOHH@check_range?5?$FL?$CFp?4?4?$CFp?$FN?5?$CI?$CFd?5bytes?$CJ@ 10072ae4     hb-aat-layout.obj
 0002:00000b18       ??_C@_07IICDHBMC@GRANTED@  10072b18     hb-aat-layout.obj
 0002:00000b20       ??_C@_06GONJNOIB@DENIED@   10072b20     hb-aat-layout.obj
 0002:00000b28       ??_C@_0DD@HNPKOALM@may_edit?$CI?$CFu?$CJ?5?$FL?$CFp?4?4?$CFp?$FN?5?$CI?$CFd?5bytes@ 10072b28     hb-aat-layout.obj
 0002:00000b5c       ??_C@_0BB@HBIIGPNG@start?5table?5morx@ 10072b5c     hb-aat-layout.obj
 0002:00000b70       ??_C@_0P@CBPBJJBN@end?5table?5morx@ 10072b70     hb-aat-layout.obj
 0002:00000b80       ??_C@_0BB@NNDNCANK@start?5table?5mort@ 10072b80     hb-aat-layout.obj
 0002:00000b94       ??_C@_0P@INEENGBB@end?5table?5mort@ 10072b94     hb-aat-layout.obj
 0002:00000ba4       ??_C@_0BB@JBHFHKBC@start?5table?5kerx@ 10072ba4     hb-aat-layout.obj
 0002:00000bb8       ??_C@_0P@MBAMIMNJ@end?5table?5kerx@ 10072bb8     hb-aat-layout.obj
 0002:00000bc8       ??_C@_0BC@MAKNDEOG@start?5subtable?5?$CFd@ 10072bc8     hb-aat-layout.obj
 0002:00000bdc       ??_C@_0BA@MMELFGCI@end?5subtable?5?$CFd@ 10072bdc     hb-aat-layout.obj
 0002:00000bec       ??_C@_0BH@CNFMEJEM@start?5chainsubtable?5?$CFd@ 10072bec     hb-aat-layout.obj
 0002:00000c04       ??_C@_0BF@OLIMMDGA@end?5chainsubtable?5?$CFd@ 10072c04     hb-aat-layout.obj
 0002:00000c1c       ??_C@_0L@PIONBGHN@start?5kern@ 10072c1c     hb-aat-layout.obj
 0002:00000c28       ??_C@_08PMCHELIJ@end?5kern@ 10072c28     hb-aat-layout.obj
 0002:00000c38       __real@3fe999999999999a    10072c38     hb-aat-layout.obj
 0002:00000c48       ??_C@_04HDKFADDE@BLOB@     10072c48     hb-blob.obj
 0002:00000c50       ??_C@_0BH@NNGJHJOL@current?5data?5is?5?9?$DO?5?$CFp?6@ 10072c50     hb-blob.obj
 0002:00000c68       ??_C@_0DD@LDEEFHJD@bool?5__thiscall?5hb_blob_t?3?3try_@ 10072c68     hb-blob.obj
 0002:00000c9c       ??_C@_0BL@NAAIMIGO@dupped?5successfully?5?9?$DO?5?$CFp?6@ 10072c9c     hb-blob.obj
 0002:00000cb8       ??_C@_04CIMGMMMG@text@     10072cb8     hb-buffer-serialize.obj
 0002:00000cc0       ??_C@_04CLCAKCEI@json@     10072cc0     hb-buffer-serialize.obj
 0002:00002548       ??_C@_02GMHACPFF@?$CFu@    10074548     hb-buffer-serialize.obj
 0002:0000254c       ??_C@_08ELFBALIN@?0?$CCcl?$CC?3?$CFu@ 1007454c     hb-buffer-serialize.obj
 0002:00002558       ??_C@_04MAFNGINP@?$CCu?$CC?3@ 10074558     hb-buffer-serialize.obj
 0002:00002560       ??_C@_03LADEAJCH@?$DN?$CFu@ 10074560     hb-buffer-serialize.obj
 0002:00002564       ??_C@_06NGBPNBKB@U?$CL?$CF04X@ 10074564     hb-buffer-serialize.obj
 0002:0000256c       ??_C@_09CPCAOBOK@harfbuzz?5@ 1007456c     hb-buffer-verify.obj
 0002:00002578       ??_C@_01EEMJAFIK@?6@       10074578     hb-buffer-verify.obj
 0002:0000257c       ??_C@_0DA@OHKIDNHD@buffer?5verify?5error?3?5clusters?5a@ 1007457c     hb-buffer-verify.obj
 0002:000025ac       ??_C@_0DM@MPDBGHGJ@buffer?5verify?5error?3?5shaping?5fa@ 100745ac     hb-buffer-verify.obj
 0002:000025e8       ??_C@_0DC@KJMJOHEC@buffer?5verify?5error?3?5unsafe?9to?9@ 100745e8     hb-buffer-verify.obj
 0002:0000261c       ??_C@_0DD@CKNGEJOG@buffer?5verify?5error?3?5unsafe?9to?9@ 1007461c     hb-buffer-verify.obj
 0002:00002650       ??_C@_0CD@DIKIFAKO@buffer?5verify?5error?3?5text?5was?3?5@ 10074650     hb-buffer-verify.obj
 0002:00002790       ?_hb_Null_OT_Index@@3QBEB  10074790     hb-common.obj
 0002:00002794       ?_hb_Null_OT_VarIdx@@3QBEB 10074794     hb-common.obj
 0002:00002798       ?_hb_Null_OT_RangeRecord@@3QBEB 10074798     hb-common.obj
 0002:000027a8       ?minus_1@@3IB              100747a8     hb-common.obj
 0002:000027ac       ?_hb_Null_AAT_Lookup@@3QBEB 100747ac     hb-common.obj
 0002:000032d8       ?_hb_Null_OT_LangSys@@3QBEB 100752d8     hb-common.obj
 0002:000032e0       ?_hb_Null_AAT_SettingName@@3QBEB 100752e0     hb-common.obj
 0002:000032e4       ?_hb_Null_OT_CmapSubtableLongGroup@@3QBEB 100752e4     hb-common.obj
 0002:00004250       ?_hb_NullPool@@3QB_KB      10076250     hb-common.obj
 0002:00004410       ??_C@_0L@PGCGEAJK@HB_OPTIONS@ 10076410     hb-common.obj
 0002:0000441c       ??_C@_0BJ@EELCEACD@uniscribe?9bug?9compatible@ 1007641c     hb-common.obj
 0002:00004438       __real@3eaaaaab            10076438     hb-draw.obj
 0002:000053ac       ??_C@_0L@LHCHIOPJ@successful@ 100773ac     hb-face.obj
 0002:000053b8       ??_C@_0N@KIEOCLDL@UNSUCCESSFUL@ 100773b8     hb-face.obj
 0002:000053c8       ??_C@_0CF@PIDDOBFK@end?5?$FL?$CFp?4?4?$CFp?$FN?5serialized?5?$CFu?5byte@ 100773c8     hb-face.obj
 0002:000053f0       ??_C@_09EPPNEDIL@SERIALIZE@ 100773f0     hb-face.obj
 0002:0000540c       __real@38800000            1007740c     hb-font.obj
 0002:00005410       __real@46800000            10077410     hb-font.obj
 0002:00005420       __xmm@41f00000000000000000000000000000 10077420     hb-font.obj
 0002:00005430       __real@47800000            10077430     hb-jdk-font.obj
 0002:00005588       __real@0010000000000000    10077588     hb-number.obj
 0002:00005590       __real@4024000000000000    10077590     hb-number.obj
 0002:00005598       __real@42f9999999999990    10077598     hb-number.obj
 0002:000055a0       __real@7fefffffffffffff    100775a0     hb-number.obj
 0002:000055a8       __real@8010000000000000    100775a8     hb-number.obj
 0002:000055b0       __real@bff0000000000000    100775b0     hb-number.obj
 0002:000055b8       __real@ffefffffffffffff    100775b8     hb-number.obj
 0002:00007270       __xmm@41dfffffffc0000041dfffffffc00000 10079270     hb-ot-cff1-table.obj
 0002:00007280       __xmm@7fffffffffffffff7fffffffffffffff 10079280     hb-ot-cff1-table.obj
 0002:00007290       __xmm@c1e0000000000000c1e0000000000000 10079290     hb-ot-cff1-table.obj
 0002:000072a8       __real@40000000            100792a8     hb-ot-cff2-table.obj
 0002:0000cf58       ??_C@_0BB@HNNCONOI@0123456789?4EE?$DP?9?$DP@ 1007ef58     hb-ot-font.obj
 0002:0000cf6c       __real@4f000000            1007ef6c     hb-ot-font.obj
 0002:0000cf70       __real@7f7fffff            1007ef70     hb-ot-font.obj
 0002:0000cf74       __real@ff7fffff            1007ef74     hb-ot-font.obj
 0002:0000cf80       __xmm@ff7fffffff7fffff7f7fffff7f7fffff 1007ef80     hb-ot-font.obj
 0002:0000cf90       __xmm@ffffffffffffffffffffffffffffffff 1007ef90     hb-ot-font.obj
 0002:0000d7a0       ??_C@_0BB@INONMPMF@start?5table?5kern@ 1007f7a0     hb-ot-layout.obj
 0002:0000d7b4       ??_C@_0P@NNJEDJAO@end?5table?5kern@ 1007f7b4     hb-ot-layout.obj
 0002:0000d7c4       ??_C@_0BB@FIKPJBHG@start?5table?5GSUB@ 1007f7c4     hb-ot-layout.obj
 0002:0000d7d8       ??_C@_0P@INGGHLN@end?5table?5GSUB@ 1007f7d8     hb-ot-layout.obj
 0002:0000d7e8       ??_C@_0BB@IHCDLCO@start?5table?5GPOS@ 1007f7e8     hb-ot-layout.obj
 0002:0000d7fc       ??_C@_0P@FIALMNOF@end?5table?5GPOS@ 1007f7fc     hb-ot-layout.obj
 0002:0000d80c       ??_C@_0BA@PGADGHOK@start?5lookup?5?$CFd@ 1007f80c     hb-ot-layout.obj
 0002:0000d81c       ??_C@_0O@IKIEJAJK@end?5lookup?5?$CFd@ 1007f81c     hb-ot-layout.obj
 0002:0000eb90       __xmm@7fffffff7fffffff7fffffff7fffffff 10080b90     hb-ot-metrics.obj
 0002:0000ebb0       ??_C@_0BE@JHLPALHA@start?5fallback?5mark@ 10080bb0     hb-ot-shape-fallback.obj
 0002:0000ebc4       ??_C@_0BC@GBHKPNCC@end?5fallback?5mark@ 10080bc4     hb-ot-shape-fallback.obj
 0002:0000ebd8       ??_C@_0BE@OKOKJNMC@start?5fallback?5kern@ 10080bd8     hb-ot-shape-fallback.obj
 0002:0000ebec       ??_C@_0BC@BMCPGLJA@end?5fallback?5kern@ 10080bec     hb-ot-shape-fallback.obj
 0002:0000ec08       ??_C@_0O@PHODME@start?5reorder@ 10080c08     hb-ot-shape-normalize.obj
 0002:0000ec18       ??_C@_0M@MGJODAHL@end?5reorder@ 10080c18     hb-ot-shape-normalize.obj
 0002:0000ec9c       ??_C@_0BJ@JCPBKLAK@start?5postprocess?9glyphs@ 10080c9c     hb-ot-shape.obj
 0002:0000ecb8       ??_C@_0BH@KGKNGMEK@end?5postprocess?9glyphs@ 10080cb8     hb-ot-shape.obj
 0002:0000ecd0       ??_C@_0BG@KEPPLGKM@start?5preprocess?9text@ 10080cd0     hb-ot-shape.obj
 0002:0000ece8       ??_C@_0BE@HIKMCIJG@end?5preprocess?9text@ 10080ce8     hb-ot-shape.obj
 0002:0000ecfc       ??_C@_02IGGBGAC@ot@        10080cfc     hb-ot-shape.obj
 0002:0000ed00       __xmm@00000003000000030000000300000003 10080d00     hb-ot-shape.obj
 0002:0000ed18       ?_hb_ot_shaper_arabic@@3Uhb_ot_shaper_t@@B 10080d18     hb-ot-shaper-arabic.obj
 0002:0000ff40       ??_C@_09BJHPDKCP@measuring@ 10081f40     hb-ot-shaper-arabic.obj
 0002:0000ff4c       ??_C@_07MINDNCFJ@cutting@  10081f4c     hb-ot-shaper-arabic.obj
 0002:0000ff54       ??_C@_0BJ@ECIMFCKL@?$CFs?5stretch?5at?5?$CI?$CFd?0?$CFd?0?$CFd?$CJ@ 10081f54     hb-ot-shaper-arabic.obj
 0002:0000ff70       ??_C@_06DBDILMHG@ARABIC@   10081f70     hb-ot-shaper-arabic.obj
 0002:0000ff80       ?_hb_ot_shaper_default@@3Uhb_ot_shaper_t@@B 10081f80     hb-ot-shaper-default.obj
 0002:0000ffb8       ?_hb_ot_shaper_dumber@@3Uhb_ot_shaper_t@@B 10081fb8     hb-ot-shaper-default.obj
 0002:0000fff8       ?_hb_ot_shaper_hangul@@3Uhb_ot_shaper_t@@B 10081ff8     hb-ot-shaper-hangul.obj
 0002:00010048       ?_hb_ot_shaper_hebrew@@3Uhb_ot_shaper_t@@B 10082048     hb-ot-shaper-hebrew.obj
 0002:00012968       ?_hb_ot_shaper_indic@@3Uhb_ot_shaper_t@@B 10084968     hb-ot-shaper-indic.obj
 0002:000135a0       ??_C@_0BP@PFJNIBAL@start?5reordering?5indic?5initial@ 100855a0     hb-ot-shaper-indic.obj
 0002:000135c0       ??_C@_0BN@DEJECPK@end?5reordering?5indic?5initial@ 100855c0     hb-ot-shaper-indic.obj
 0002:000135e0       ??_C@_0BN@BEFMFOMM@start?5reordering?5indic?5final@ 100855e0     hb-ot-shaper-indic.obj
 0002:00013600       ??_C@_0BL@CMBCGANJ@end?5reordering?5indic?5final@ 10085600     hb-ot-shaper-indic.obj
 0002:00013628       ?_hb_ot_shaper_khmer@@3Uhb_ot_shaper_t@@B 10085628     hb-ot-shaper-khmer.obj
 0002:00013c60       ??_C@_0BH@LEEFGPFH@start?5reordering?5khmer@ 10085c60     hb-ot-shaper-khmer.obj
 0002:00013c78       ??_C@_0BF@HCJFOFHL@end?5reordering?5khmer@ 10085c78     hb-ot-shaper-khmer.obj
 0002:00013c98       ?_hb_ot_shaper_myanmar@@3Uhb_ot_shaper_t@@B 10085c98     hb-ot-shaper-myanmar.obj
 0002:00013cd0       ?_hb_ot_shaper_myanmar_zawgyi@@3Uhb_ot_shaper_t@@B 10085cd0     hb-ot-shaper-myanmar.obj
 0002:00014770       ??_C@_0BJ@HDEFJBCC@start?5reordering?5myanmar@ 10086770     hb-ot-shaper-myanmar.obj
 0002:0001478c       ??_C@_0BH@EHBJFGGC@end?5reordering?5myanmar@ 1008678c     hb-ot-shaper-myanmar.obj
 0002:000147b8       ?_hb_ot_shaper_thai@@3Uhb_ot_shaper_t@@B 100867b8     hb-ot-shaper-thai.obj
 0002:00014a18       ?_hb_ot_shaper_use@@3Uhb_ot_shaper_t@@B 10086a18     hb-ot-shaper-use.obj
 0002:00019144       ??_C@_0BF@INKMBGAO@start?5reordering?5USE@ 1008b144     hb-ot-shaper-use.obj
 0002:0001915c       ??_C@_0BD@IDPODCA@end?5reordering?5USE@ 1008b15c     hb-ot-shaper-use.obj
 0002:0001bd98       ??_C@_08LOEDBOED@?9fonnapa@ 1008dd98     hb-ot-tag.obj
 0002:0001bda4       ??_C@_08GMLKJDFJ@?9polyton@ 1008dda4     hb-ot-tag.obj
 0002:0001bdb0       ??_C@_08NJCBHCMA@?9arevmda@ 1008ddb0     hb-ot-tag.obj
 0002:0001bdbc       ??_C@_08DCLOKPKI@?9provenc@ 1008ddbc     hb-ot-tag.obj
 0002:0001bdc8       ??_C@_07KBFBNAFC@?9fonipa@ 1008ddc8     hb-ot-tag.obj
 0002:0001bdd0       ??_C@_05BHGHNKKJ@?9geok@   1008ddd0     hb-ot-tag.obj
 0002:0001bdd8       ??_C@_05BCLFBOGB@?9syre@   1008ddd8     hb-ot-tag.obj
 0002:0001bde0       ??_C@_05JFCNACKO@?9syrj@   1008dde0     hb-ot-tag.obj
 0002:0001bde8       ??_C@_05PBEBMHKK@?9syrn@   1008dde8     hb-ot-tag.obj
 0002:0001bdf0       ??_C@_09GEIHALDG@rt?9lojban@ 1008ddf0     hb-ot-tag.obj
 0002:0001bdfc       ??_C@_0L@KFNBBKMN@do?9hant?9hk@ 1008ddfc     hb-ot-tag.obj
 0002:0001be08       ??_C@_0L@MHHGBNCC@do?9hant?9mo@ 1008de08     hb-ot-tag.obj
 0002:0001be14       ??_C@_0L@NNBHMAGE@jy?9hant?9hk@ 1008de14     hb-ot-tag.obj
 0002:0001be20       ??_C@_0L@LPLAMHIL@jy?9hant?9mo@ 1008de20     hb-ot-tag.obj
 0002:0001be2c       ??_C@_0L@DBFOEPHG@mn?9hant?9hk@ 1008de2c     hb-ot-tag.obj
 0002:0001be38       ??_C@_0L@FDPJEIJJ@mn?9hant?9mo@ 1008de38     hb-ot-tag.obj
 0002:0001be44       ??_C@_0L@JBNLJICM@np?9hant?9hk@ 1008de44     hb-ot-tag.obj
 0002:0001be50       ??_C@_0L@PDHMJPMD@np?9hant?9mo@ 1008de50     hb-ot-tag.obj
 0002:0001be5c       ??_C@_0L@HOIMDHBF@px?9hant?9hk@ 1008de5c     hb-ot-tag.obj
 0002:0001be68       ??_C@_0L@BMCLDAPK@px?9hant?9mo@ 1008de68     hb-ot-tag.obj
 0002:0001be74       ??_C@_0L@PELJBBOA@sp?9hant?9hk@ 1008de74     hb-ot-tag.obj
 0002:0001be80       ??_C@_0L@JGBOBGAP@sp?9hant?9mo@ 1008de80     hb-ot-tag.obj
 0002:0001be8c       ??_C@_0L@LLINOOHJ@zh?9hant?9hk@ 1008de8c     hb-ot-tag.obj
 0002:0001be98       ??_C@_0L@NJCKOJJG@zh?9hant?9mo@ 1008de98     hb-ot-tag.obj
 0002:0001bea4       ??_C@_0L@FJFBPFAA@zo?9hant?9hk@ 1008dea4     hb-ot-tag.obj
 0002:0001beb0       ??_C@_0L@DLPGPCOP@zo?9hant?9mo@ 1008deb0     hb-ot-tag.obj
 0002:0001bebc       ??_C@_07GEDDMEMG@do?9hans@ 1008debc     hb-ot-tag.obj
 0002:0001bec4       ??_C@_07CLHCFCAB@do?9hant@ 1008dec4     hb-ot-tag.obj
 0002:0001becc       ??_C@_07HFLHHPAA@jy?9hans@ 1008decc     hb-ot-tag.obj
 0002:0001bed4       ??_C@_07DKPGOJMH@jy?9hant@ 1008ded4     hb-ot-tag.obj
 0002:0001bedc       ??_C@_07NNALNEFJ@mn?9hans@ 1008dedc     hb-ot-tag.obj
 0002:0001bee4       ??_C@_07JCEKECJO@mn?9hant@ 1008dee4     hb-ot-tag.obj
 0002:0001beec       ??_C@_07GEGFDECJ@np?9hans@ 1008deec     hb-ot-tag.obj
 0002:0001bef4       ??_C@_07CLCEKCOO@np?9hant@ 1008def4     hb-ot-tag.obj
 0002:0001befc       ??_C@_07DOLLFJFH@px?9hans@ 1008defc     hb-ot-tag.obj
 0002:0001bf04       ??_C@_07HBPKMPJA@px?9hant@ 1008df04     hb-ot-tag.obj
 0002:0001bf0c       ??_C@_07IDNLBAND@sp?9hans@ 1008df0c     hb-ot-tag.obj
 0002:0001bf14       ??_C@_07MMJKIGBE@sp?9hant@ 1008df14     hb-ot-tag.obj
 0002:0001bf1c       ??_C@_07MIKFNJFB@zh?9hans@ 1008df1c     hb-ot-tag.obj
 0002:0001bf24       ??_C@_07IHOEEPJG@zh?9hant@ 1008df24     hb-ot-tag.obj
 0002:0001bf2c       ??_C@_07NACOHNP@zo?9hans@  1008df2c     hb-ot-tag.obj
 0002:0001bf34       ??_C@_07ECEDHBBI@zo?9hant@ 1008df34     hb-ot-tag.obj
 0002:0001bf3c       ??_C@_03JFOJGEF@do?9@      1008df3c     hb-ot-tag.obj
 0002:0001bf40       ??_C@_03EMCOHPPE@?9hk@     1008df40     hb-ot-tag.obj
 0002:0001bf44       ??_C@_03COIJHIBL@?9mo@     1008df44     hb-ot-tag.obj
 0002:0001bf48       ??_C@_03LPGFHILN@?9tw@     1008df48     hb-ot-tag.obj
 0002:0001bf4c       ??_C@_03PBCKDOLE@jy?9@     1008df4c     hb-ot-tag.obj
 0002:0001bf50       ??_C@_03HFJELDPI@mn?9@     1008df50     hb-ot-tag.obj
 0002:0001bf54       ??_C@_03HBJJJCGM@np?9@     1008df54     hb-ot-tag.obj
 0002:0001bf58       ??_C@_03MPEMODHI@px?9@     1008df58     hb-ot-tag.obj
 0002:0001bf5c       ??_C@_03NDOKBNCO@sp?9@     1008df5c     hb-ot-tag.obj
 0002:0001bf60       ??_C@_03LMNHKAGM@zh?9@     1008df60     hb-ot-tag.obj
 0002:0001bf64       ??_C@_03LJJILGOJ@zo?9@     1008df64     hb-ot-tag.obj
 0002:0001bf68       ??_C@_0L@DLEENNLB@an?9hant?9hk@ 1008df68     hb-ot-tag.obj
 0002:0001bf74       ??_C@_0L@FJODNKFO@an?9hant?9mo@ 1008df74     hb-ot-tag.obj
 0002:0001bf80       ??_C@_07IKKEMBBG@an?9hans@ 1008df80     hb-ot-tag.obj
 0002:0001bf88       ??_C@_07MFOFFHNB@an?9hant@ 1008df88     hb-ot-tag.obj
 0002:0001bf90       ??_C@_06FCHMEGPO@a?9latg@  1008df90     hb-ot-tag.obj
 0002:0001bf98       ??_C@_03DPECAMEA@an?9@     1008df98     hb-ot-tag.obj
 0002:0001bf9c       ??_C@_0L@NNGNBGPF@ak?9hant?9hk@ 1008df9c     hb-ot-tag.obj
 0002:0001bfa8       ??_C@_0L@LPMKBBBK@ak?9hant?9mo@ 1008dfa8     hb-ot-tag.obj
 0002:0001bfb4       ??_C@_0L@MNNOKALL@sn?9hant?9hk@ 1008dfb4     hb-ot-tag.obj
 0002:0001bfc0       ??_C@_0L@KPHJKHFE@sn?9hant?9mo@ 1008dfc0     hb-ot-tag.obj
 0002:0001bfcc       ??_C@_07NIJMOOLB@ak?9hans@ 1008dfcc     hb-ot-tag.obj
 0002:0001bfd4       ??_C@_07JHNNHIHG@ak?9hant@ 1008dfd4     hb-ot-tag.obj
 0002:0001bfdc       ??_C@_07LEDKPHEA@sn?9hans@ 1008dfdc     hb-ot-tag.obj
 0002:0001bfe4       ??_C@_07PLHLGBIH@sn?9hant@ 1008dfe4     hb-ot-tag.obj
 0002:0001bfec       ??_C@_03DJIJMOKL@ak?9@     1008dfec     hb-ot-tag.obj
 0002:0001bff0       ??_C@_03MFFCJDFE@sn?9@     1008dff0     hb-ot-tag.obj
 0002:0001bff4       ??_C@_07LCKCAAMB@?9navajo@ 1008dff4     hb-ot-tag.obj
 0002:0001bffc       ??_C@_04DBACCPMA@?9hak@    1008dffc     hb-ot-tag.obj
 0002:0001c004       ??_C@_04MEKAPCKJ@?9lux@    1008e004     hb-ot-tag.obj
 0002:0001c00c       ??_C@_03HENGIEOJ@nw?9@     1008e00c     hb-ot-tag.obj
 0002:0001c010       ??_C@_03HCDPHGCD@?9th@     1008e010     hb-ot-tag.obj
 0002:0001c014       ??_C@_05NKGDAJJP@o?9bok@   1008e014     hb-ot-tag.obj
 0002:0001c01c       ??_C@_05PFGJJNKA@o?9nyn@   1008e01c     hb-ot-tag.obj
 0002:0001c024       ??_C@_02GDBPPABP@o?9@      1008e024     hb-ot-tag.obj
 0002:0001c028       ??_C@_03MNHNKBNA@?9md@     1008e028     hb-ot-tag.obj
 0002:0001c02c       ??_C@_0L@PKCFBAOH@uu?9hant?9hk@ 1008e02c     hb-ot-tag.obj
 0002:0001c038       ??_C@_0L@JIICBHAI@uu?9hant?9mo@ 1008e038     hb-ot-tag.obj
 0002:0001c044       ??_C@_07BHIMDGPD@uu?9hans@ 1008e044     hb-ot-tag.obj
 0002:0001c04c       ??_C@_07FIMNKADE@uu?9hant@ 1008e04c     hb-ot-tag.obj
 0002:0001c054       ??_C@_03PAEKIABJ@uu?9@     1008e054     hb-ot-tag.obj
 0002:0001c058       ??_C@_07HAFCKKDN@ue?9hans@ 1008e058     hb-ot-tag.obj
 0002:0001c060       ??_C@_09CPANDNJE@h?9hant?9hk@ 1008e060     hb-ot-tag.obj
 0002:0001c06c       ??_C@_09ENKKDKHL@h?9hant?9mo@ 1008e06c     hb-ot-tag.obj
 0002:0001c078       ??_C@_09JKAGOIDE@h?9min?9nan@ 1008e078     hb-ot-tag.obj
 0002:0001c084       ??_C@_06NHLFEBO@h?9hans@   1008e084     hb-ot-tag.obj
 0002:0001c08c       ??_C@_06ECDKMCNJ@h?9hant@  1008e08c     hb-ot-tag.obj
 0002:0001c094       ??_C@_05OGPPKBIG@h?9min@   1008e094     hb-ot-tag.obj
 0002:0001c09c       ??_C@_02GGFAOGJK@h?9@      1008e09c     hb-ot-tag.obj
 0002:0001c0a0       ??_C@_03FHLPDODD@alt@      1008e0a0     hb-ot-tag.obj
 0002:0001c0a4       ??_C@_0M@EFNICDFC@und?9fonnapa@ 1008e0a4     hb-ot-tag.obj
 0002:0001c0b0       ??_C@_02FEKCJMIO@ar@       1008e0b0     hb-ot-tag.obj
 0002:0001c0b4       ??_C@_03OPDALMNL@rki@      1008e0b4     hb-ot-tag.obj
 0002:0001c0b8       ??_C@_03KDPNJBKG@ath@      1008e0b8     hb-ot-tag.obj
 0002:0001c0bc       ??_C@_03BMIBANNE@ber@      1008e0bc     hb-ot-tag.obj
 0002:0001c0c0       ??_C@_03IOJLFNKI@bik@      1008e0c0     hb-ot-tag.obj
 0002:0001c0c4       ??_C@_03JKGFGNIL@btk@      1008e0c4     hb-ot-tag.obj
 0002:0001c0c8       ??_C@_03IPGCLNMG@crp@      1008e0c8     hb-ot-tag.obj
 0002:0001c0cc       ??_C@_03EHLLDHMO@crx@      1008e0cc     hb-ot-tag.obj
 0002:0001c0d0       ??_C@_03JNELBMEE@doi@      1008e0d0     hb-ot-tag.obj
 0002:0001c0d4       ??_C@_03NGIHPGDB@din@      1008e0d4     hb-ot-tag.obj
 0002:0001c0d8       ??_C@_03OGODBGHE@prs@      1008e0d8     hb-ot-tag.obj
 0002:0001c0dc       ??_C@_02JKLANEGN@dz@       1008e0dc     hb-ot-tag.obj
 0002:0001c0e0       ??_C@_02FPBJDNE@et@        1008e0e0     hb-ot-tag.obj
 0002:0001c0e4       ??_C@_02DAACMLJJ@fa@       1008e0e4     hb-ot-tag.obj
 0002:0001c0e8       ??_C@_03MALPCFGN@gon@      1008e0e8     hb-ot-tag.obj
 0002:0001c0ec       ??_C@_03NPJADACO@mrj@      1008e0ec     hb-ot-tag.obj
 0002:0001c0f0       ??_C@_03JLFIOBFF@hmn@      1008e0f0     hb-ot-tag.obj
 0002:0001c0f4       ??_C@_03GDPBLHIG@hnd@      1008e0f4     hb-ot-tag.obj
 0002:0001c0f8       ??_C@_03BLHHEDOB@hyw@      1008e0f8     hb-ot-tag.obj
 0002:0001c0fc       ??_C@_03KPCANNMC@iba@      1008e0fc     hb-ot-tag.obj
 0002:0001c100       ??_C@_03DPLAKBPE@ijo@      1008e100     hb-ot-tag.obj
 0002:0001c104       ??_C@_02BFPAFLPB@iu@       1008e104     hb-ot-tag.obj
 0002:0001c108       ??_C@_02MBLBGECO@ik@       1008e108     hb-ot-tag.obj
 0002:0001c10c       ??_C@_0L@OOCAKEAN@und?9fonipa@ 1008e10c     hb-ot-tag.obj
 0002:0001c118       ??_C@_07LBNNMAEP@ga?9Latg@ 1008e118     hb-ot-tag.obj
 0002:0001c120       ??_C@_02OPKBKFNM@yi@       1008e120     hb-ot-tag.obj
 0002:0001c124       ??_C@_03IICPCEIM@kln@      1008e124     hb-ot-tag.obj
 0002:0001c128       ??_C@_08IBMBBMEF@und?9Geok@ 1008e128     hb-ot-tag.obj
 0002:0001c134       ??_C@_02FJDFBJFI@kr@       1008e134     hb-ot-tag.obj
 0002:0001c138       ??_C@_03CJCPPGJN@okm@      1008e138     hb-ot-tag.obj
 0002:0001c13c       ??_C@_03PHBOGOJA@kok@      1008e13c     hb-ot-tag.obj
 0002:0001c140       ??_C@_02DNFJNMFM@kv@       1008e140     hb-ot-tag.obj
 0002:0001c144       ??_C@_03HOOHKHFD@kpe@      1008e144     hb-ot-tag.obj
 0002:0001c148       ??_C@_03GGIAOKIC@kar@      1008e148     hb-ot-tag.obj
 0002:0001c14c       ??_C@_03HCOHIEGC@uki@      1008e14c     hb-ot-tag.obj
 0002:0001c150       ??_C@_02BGHEIPJP@ku@       1008e150     hb-ot-tag.obj
 0002:0001c154       ??_C@_03EMDKIONB@mhr@      1008e154     hb-ot-tag.obj
 0002:0001c158       ??_C@_03DIMAAFM@luy@       1008e158     hb-ot-tag.obj
 0002:0001c15c       ??_C@_02DIBGMKNJ@lv@       1008e15c     hb-ot-tag.obj
 0002:0001c160       ??_C@_03FLEAGKJM@mwr@      1008e160     hb-ot-tag.obj
 0002:0001c164       ??_C@_02GKANIDPO@mg@       1008e164     hb-ot-tag.obj
 0002:0001c168       ??_C@_02EEKDFEKL@ms@       1008e168     hb-ot-tag.obj
 0002:0001c16c       ??_C@_02LLMPDILH@mn@       1008e16c     hb-ot-tag.obj
 0002:0001c170       ??_C@_03KFJMOIAD@man@      1008e170     hb-ot-tag.obj
 0002:0001c174       ??_C@_05KNLKPBHL@ro?9MD@   1008e174     hb-ot-tag.obj
 0002:0001c17c       ??_C@_06PALDGLND@mnw?9TH@  1008e17c     hb-ot-tag.obj
 0002:0001c184       ??_C@_03LHKJBKML@myn@      1008e184     hb-ot-tag.obj
 0002:0001c188       ??_C@_03OBHDOAGL@nah@      1008e188     hb-ot-tag.obj
 0002:0001c18c       ??_C@_02FKHNFPCF@ne@       1008e18c     hb-ot-tag.obj
 0002:0001c190       ??_C@_03JFNCHPFJ@njz@      1008e190     hb-ot-tag.obj
 0002:0001c194       ??_C@_02KAJCLHKP@no@       1008e194     hb-ot-tag.obj
 0002:0001c198       ??_C@_02NMCHCJNN@oj@       1008e198     hb-ot-tag.obj
 0002:0001c19c       ??_C@_02JDGGLPBK@om@       1008e19c     hb-ot-tag.obj
 0002:0001c1a0       ??_C@_02FAFNGEII@ps@       1008e1a0     hb-ot-tag.obj
 0002:0001c1a4       ??_C@_0L@LGMOIJP@el?9polyton@ 1008e1a4     hb-ot-tag.obj
 0002:0001c1b0       ??_C@_03JEELCJ@pro@        1008e1b0     hb-ot-tag.obj
 0002:0001c1b4       ??_C@_03PCCGKMAO@quh@      1008e1b4     hb-ot-tag.obj
 0002:0001c1b8       ??_C@_02HMFKJDJ@qu@        1008e1b8     hb-ot-tag.obj
 0002:0001c1bc       ??_C@_03OJHLCDBG@qvi@      1008e1bc     hb-ot-tag.obj
 0002:0001c1c0       ??_C@_03PBKCHIGA@qwh@      1008e1c0     hb-ot-tag.obj
 0002:0001c1c4       ??_C@_03MJIKGKMO@raj@      1008e1c4     hb-ot-tag.obj
 0002:0001c1c8       ??_C@_02LFKOONLL@ro@       1008e1c8     hb-ot-tag.obj
 0002:0001c1cc       ??_C@_03IMFFNBAD@rom@      1008e1cc     hb-ot-tag.obj
 0002:0001c1d0       ??_C@_02GACNLIFD@sq@       1008e1d0     hb-ot-tag.obj
 0002:0001c1d4       ??_C@_02ELAAOLJA@sr@       1008e1d4     hb-ot-tag.obj
 0002:0001c1d8       ??_C@_03KNGLMNJH@xnj@      1008e1d8     hb-ot-tag.obj
 0002:0001c1dc       ??_C@_03OBBIGHDK@syr@      1008e1dc     hb-ot-tag.obj
 0002:0001c1e0       ??_C@_08IEBDNIIN@und?9Syre@ 1008e1e0     hb-ot-tag.obj
 0002:0001c1ec       ??_C@_08DILMEEC@und?9Syrj@ 1008e1ec     hb-ot-tag.obj
 0002:0001c1f8       ??_C@_08GHOHABEG@und?9Syrn@ 1008e1f8     hb-ot-tag.obj
 0002:0001c204       ??_C@_03NHMNKOPE@tmh@      1008e204     hb-ot-tag.obj
 0002:0001c208       ??_C@_03MDOLKBCN@xwo@      1008e208     hb-ot-tag.obj
 0002:0001c20c       ??_C@_05HCJKHBCC@zh?9HK@   1008e20c     hb-ot-tag.obj
 0002:0001c214       ??_C@_07JGEPGFF@zh?9Hans@  1008e214     hb-ot-tag.obj
 0002:0001c21c       ??_C@_07EGCFGAJC@zh?9Hant@ 1008e21c     hb-ot-tag.obj
 0002:0001c224       ??_C@_05BADNHGMN@zh?9MO@   1008e224     hb-ot-tag.obj
 0002:0001c22c       ??_C@_03PPLJNHHL@zza@      1008e22c     hb-ot-tag.obj
 0002:0001c230       ??_C@_05NFAFKFNN@?9hbsc@   1008e230     hb-ot-tag.obj
 0002:0001c238       ??_C@_05MFLKHLFP@?9hbot@   1008e238     hb-ot-tag.obj
 0002:0001c240       ??_C@_0M@MFILKOCI@x?9hbot?9?$CF08x@ 1008e240     hb-ot-tag.obj
 0002:0001c264       ??_C@_08LFBOCJLE@fallback@ 1008e264     hb-shape-plan.obj
 0002:0001c270       ??_C@_0DF@LPDLEJCD@face?$DN?$CFp?5num_features?$DN?$CFd?5num_coo@ 1008e270     hb-shape-plan.obj
 0002:0001c2a8       ??_C@_0MH@MMALGGGN@struct?5hb_shape_plan_t?5?$CK__cdecl@ 1008e2a8     hb-shape-plan.obj
 0002:0001c370       ??_C@_0L@HJBOBLCO@SHAPE_PLAN@ 1008e370     hb-shape-plan.obj
 0002:0001c37c       ??_C@_0CP@IPGKIIHP@num_features?$DN?$CFd?5shaper_func?$DN?$CFp?0@ 1008e37c     hb-shape-plan.obj
 0002:0001c3b0       ??_C@_0JI@JOJJJOPA@bool?5__cdecl?5_hb_shape_plan_exe@ 1008e3b0     hb-shape-plan.obj
 0002:0001c448       ??_C@_0CH@NAFHBKKC@face?$DN?$CFp?5num_features?$DN?$CFd?5shaper_@ 1008e448     hb-shape-plan.obj
 0002:0001c470       ??_C@_0MO@MGHFPDJG@struct?5hb_shape_plan_t?5?$CK__cdecl@ 1008e470     hb-shape-plan.obj
 0002:0001c574       ??_C@_0P@GEOKODDH@HB_SHAPER_LIST@ 1008e574     hb-shaper.obj
 0002:00034ad0       ?_hb_modified_combining_class@@3QBEB 100a6ad0     hb-unicode.obj
 0002:00034df0       ??_C@_0BG@NKHBBPH@sun?1font?1TrueTypeFont@ 100a6df0     sunFont.obj
 0002:00034e08       ??_C@_0BL@GAAGJDLL@?$CILjava?1nio?1ByteBuffer?$DLII?$CJI@ 100a6e08     sunFont.obj
 0002:00034e24       ??_C@_09CKAKNPHP@readBlock@ 100a6e24     sunFont.obj
 0002:00034e30       ??_C@_06JMOJDKIE@?$CIII?$CJ?$FLB@ 100a6e30     sunFont.obj
 0002:00034e38       ??_C@_09IDIEPDPI@readBytes@ 100a6e38     sunFont.obj
 0002:00034e44       ??_C@_0BD@OPLCIPMH@sun?1font?1Type1Font@ 100a6e44     sunFont.obj
 0002:00034e58       ??_C@_0BJ@LMHMPPKE@?$CILjava?1nio?1ByteBuffer?$DL?$CJV@ 100a6e58     sunFont.obj
 0002:00034e74       ??_C@_08CJNGBMAG@readFile@ 100a6e74     sunFont.obj
 0002:00034e80       ??_C@_0BM@DGICEJAA@java?1awt?1geom?1Point2D$Float@ 100a6e80     sunFont.obj
 0002:00034e9c       ??_C@_05BHHDPELC@?$CIFF?$CJV@ 100a6e9c     sunFont.obj
 0002:00034ea4       ??_C@_01BIAFAFID@F@        100a6ea4     sunFont.obj
 0002:00034ea8       ??_C@_01FJMABOPO@x@        100a6ea8     sunFont.obj
 0002:00034eac       ??_C@_01EANLCPLP@y@        100a6eac     sunFont.obj
 0002:00034eb0       ??_C@_0BH@ENELCGL@sun?1font?1StrikeMetrics@ 100a6eb0     sunFont.obj
 0002:00034ec8       ??_C@_0O@LBAHCNJL@?$CIFFFFFFFFFF?$CJV@ 100a6ec8     sunFont.obj
 0002:00034ed8       ??_C@_0CA@PDMBNICK@java?1awt?1geom?1Rectangle2D$Float@ 100a6ed8     sunFont.obj
 0002:00034ef8       ??_C@_07PMCFNNPC@?$CIFFFF?$CJV@ 100a6ef8     sunFont.obj
 0002:00034f00       ??_C@_05IGKADHGO@width@    100a6f00     sunFont.obj
 0002:00034f08       ??_C@_06LNLHEAAG@height@   100a6f08     sunFont.obj
 0002:00034f10       ??_C@_0BK@COJNCHEM@java?1awt?1geom?1GeneralPath@ 100a6f10     sunFont.obj
 0002:00034f2c       ??_C@_0L@MDPODKN@?$CII?$FLBI?$FLFI?$CJV@ 100a6f2c     sunFont.obj
 0002:00034f38       ??_C@_0BA@OKNBFGCN@sun?1font?1Font2D@ 100a6f38     sunFont.obj
 0002:00034f48       ??_C@_04DIFHPCLD@?$CII?$CJI@ 100a6f48     sunFont.obj
 0002:00034f50       ??_C@_0M@NMGOHDEJ@charToGlyph@ 100a6f50     sunFont.obj
 0002:00034f5c       ??_C@_05BKHNKL@?$CIII?$CJI@ 100a6f5c     sunFont.obj
 0002:00034f64       ??_C@_0BF@NFJAPLLH@charToVariationGlyph@ 100a6f64     sunFont.obj
 0002:00034f7c       ??_C@_0BP@CBNLOFNN@?$CI?$CJLsun?1font?1CharToGlyphMapper?$DL@ 100a6f7c     sunFont.obj
 0002:00034f9c       ??_C@_09DGCMEJKL@getMapper@ 100a6f9c     sunFont.obj
 0002:00034fa8       ??_C@_05IPLNOPFN@?$CII?$CJ?$FLB@ 100a6fa8     sunFont.obj
 0002:00034fb0       ??_C@_0O@DBNIPDIH@getTableBytes@ 100a6fb0     sunFont.obj
 0002:00034fc0       ??_C@_04DGAFFDEF@?$CIC?$CJZ@ 100a6fc0     sunFont.obj
 0002:00034fc8       ??_C@_0L@PGEPPKMA@canDisplay@ 100a6fc8     sunFont.obj
 0002:00034fd4       ??_C@_0BL@GAPGNAAC@sun?1font?1CharToGlyphMapper@ 100a6fd4     sunFont.obj
 0002:00034ff0       ??_C@_0BI@GDBHNKM@sun?1font?1PhysicalStrike@ 100a6ff0     sunFont.obj
 0002:00035008       ??_C@_0CB@IBGFEOCM@?$CII?$CJLjava?1awt?1geom?1Point2D$Float@ 100a7008     sunFont.obj
 0002:0003502c       ??_C@_0BA@FMKHNFIF@getGlyphMetrics@ 100a702c     sunFont.obj
 0002:0003503c       ??_C@_0CC@IBLMDHKA@?$CIII?$CJLjava?1awt?1geom?1Point2D$Floa@ 100a703c     sunFont.obj
 0002:00035060       ??_C@_0O@NHLNHECD@getGlyphPoint@ 100a7060     sunFont.obj
 0002:00035070       ??_C@_0CB@CONGGNHA@?$CILjava?1awt?1geom?1Point2D$Float?$DL?$CJ@ 100a7070     sunFont.obj
 0002:00035094       ??_C@_0M@MJABIGBP@adjustPoint@ 100a7094     sunFont.obj
 0002:000350a0       ??_C@_01LELAEKIP@J@        100a70a0     sunFont.obj
 0002:000350a4       ??_C@_0P@DPIICNJB@pScalerContext@ 100a70a4     sunFont.obj
 0002:000350b4       ??_C@_0BD@LPHBDEDB@sun?1font?1GlyphList@ 100a70b4     sunFont.obj
 0002:000350c8       ??_C@_05HAAKEDND@gposx@    100a70c8     sunFont.obj
 0002:000350d0       ??_C@_05GJBBHCJC@gposy@    100a70d0     sunFont.obj
 0002:000350d8       ??_C@_03BKCJCHLK@len@      100a70d8     sunFont.obj
 0002:000350dc       ??_C@_02GKMBEADD@?$FLJ@    100a70dc     sunFont.obj
 0002:000350e0       ??_C@_06IAHKIHIK@images@   100a70e0     sunFont.obj
 0002:000350e8       ??_C@_01POHCFINO@Z@        100a70e8     sunFont.obj
 0002:000350ec       ??_C@_0N@CLHDJEN@usePositions@ 100a70ec     sunFont.obj
 0002:000350fc       ??_C@_09HEJILCIA@positions@ 100a70fc     sunFont.obj
 0002:00035108       ??_C@_0M@IOGNPDID@lcdRGBOrder@ 100a7108     sunFont.obj
 0002:00035114       ??_C@_0N@OIMCCICM@lcdSubPixPos@ 100a7114     sunFont.obj
 0002:0003515c       __pRawDllMain              100a715c     MSVCRT:dll_dllmain.obj
 0002:0003515c       __pDefaultRawDllMain       100a715c     MSVCRT:dll_dllmain.obj
 0002:000351d0       __load_config_used         100a71d0     MSVCRT:loadcfg.obj
 0002:00035288       ___safe_se_handler_table   100a7288     <linker-defined>
 0002:00035514       ___rtc_iaa                 100a7514     MSVCRT:initsect.obj
 0002:00035518       ___rtc_izz                 100a7518     MSVCRT:initsect.obj
 0002:0003551c       ___rtc_taa                 100a751c     MSVCRT:initsect.obj
 0002:00035520       ___rtc_tzz                 100a7520     MSVCRT:initsect.obj
 0002:00035f08       __IMPORT_DESCRIPTOR_freetype 100a7f08     freetype:freetype.dll
 0002:00035f1c       __IMPORT_DESCRIPTOR_java   100a7f1c     java:java.dll
 0002:00035f30       __IMPORT_DESCRIPTOR_ADVAPI32 100a7f30     advapi32:ADVAPI32.dll
 0002:00035f44       __IMPORT_DESCRIPTOR_USER32 100a7f44     user32:USER32.dll
 0002:00035f58       __IMPORT_DESCRIPTOR_GDI32  100a7f58     gdi32:GDI32.dll
 0002:00035f6c       __IMPORT_DESCRIPTOR_awt    100a7f6c     awt:awt.dll
 0002:00035f80       __IMPORT_DESCRIPTOR_KERNEL32 100a7f80     kernel32:KERNEL32.dll
 0002:00035f94       __IMPORT_DESCRIPTOR_VCRUNTIME140 100a7f94     vcruntime:VCRUNTIME140.dll
 0002:00035fa8       __IMPORT_DESCRIPTOR_api-ms-win-crt-heap-l1-1-0 100a7fa8     ucrt:api-ms-win-crt-heap-l1-1-0.dll
 0002:00035fbc       __IMPORT_DESCRIPTOR_api-ms-win-crt-math-l1-1-0 100a7fbc     ucrt:api-ms-win-crt-math-l1-1-0.dll
 0002:00035fd0       __IMPORT_DESCRIPTOR_api-ms-win-crt-environment-l1-1-0 100a7fd0     ucrt:api-ms-win-crt-environment-l1-1-0.dll
 0002:00035fe4       __IMPORT_DESCRIPTOR_api-ms-win-crt-convert-l1-1-0 100a7fe4     ucrt:api-ms-win-crt-convert-l1-1-0.dll
 0002:00035ff8       __IMPORT_DESCRIPTOR_api-ms-win-crt-stdio-l1-1-0 100a7ff8     ucrt:api-ms-win-crt-stdio-l1-1-0.dll
 0002:0003600c       __IMPORT_DESCRIPTOR_api-ms-win-crt-string-l1-1-0 100a800c     ucrt:api-ms-win-crt-string-l1-1-0.dll
 0002:00036020       __IMPORT_DESCRIPTOR_api-ms-win-crt-runtime-l1-1-0 100a8020     ucrt:api-ms-win-crt-runtime-l1-1-0.dll
 0002:00036034       __NULL_IMPORT_DESCRIPTOR   100a8034     freetype:freetype.dll
 0003:00000000       _defaultGammaLUT           100a9000     DrawGlyphList.obj
 0003:00000100       _defaultInvGammaLUT        100a9100     DrawGlyphList.obj
 0003:00000218       ?_hb_Null_hb_buffer_t@@3Uhb_buffer_t@@B 100a9218     hb-buffer.obj
 0003:000002c4       ?_hb_Null_hb_draw_funcs_t@@3Uhb_draw_funcs_t@@B 100a92c4     hb-draw.obj
 0003:000002f0       ?_hb_Null_hb_face_t@@3Uhb_face_t@@B 100a92f0     hb-face.obj
 0003:000003c8       ?_hb_Null_hb_font_funcs_t@@3Uhb_font_funcs_t@@B 100a93c8     hb-font.obj
 0003:00000428       ?_hb_Null_hb_font_t@@3Uhb_font_t@@B 100a9428     hb-font.obj
 0003:00000650       ?_hb_Null_hb_unicode_funcs_t@@3Uhb_unicode_funcs_t@@B 100a9650     hb-unicode.obj
 0003:000006c0       _MAX_ICU_SCRIPTCODE        100a96c0     scriptMapping.obj
 0003:000006c8       _ICU_to_Harfbuzz_ScriptCode 100a96c8     scriptMapping.obj
 0003:00000780       ___security_cookie_complement 100a9780     MSVCRT:gs_cookie.obj
 0003:00000784       ___security_cookie         100a9784     MSVCRT:gs_cookie.obj
 0003:00000788       __fltused                  100a9788     MSVCRT:fltused.obj
 0003:00000790       ___isa_enabled             100a9790     MSVCRT:cpu_disp.obj
 0003:00000794       ___scrt_native_dllmain_reason 100a9794     MSVCRT:utility.obj
 0003:000007a0       ___scrt_ucrt_dll_is_in_use 100a97a0     MSVCRT:ucrt_stubs.obj
 0003:000007e8       ?_OptionsStorage@?1??__local_stdio_printf_options@@9@4_KA 100a97e8     hb-buffer-serialize.obj
 0003:000007f0       ?_hb_options@@3Uhb_atomic_int_t@@A 100a97f0     hb-common.obj
 0003:000007f8       ?_hb_CrapPool@@3PA_KA      100a97f8     hb-common.obj
 0003:00000ee8       ___isa_available           100a9ee8     MSVCRT:cpu_disp.obj
 0003:00000eec       ___favor                   100a9eec     MSVCRT:cpu_disp.obj
 0003:00000ef0       ?__type_info_root_node@@3U__type_info_node@@A 100a9ef0     MSVCRT:tncleanup.obj
 0003:00000ef8       ?_OptionsStorage@?1??__local_stdio_scanf_options@@9@4_KA 100a9ef8     MSVCRT:default_local_stdio_options.obj
 0003:00000f00       ___scrt_current_native_startup_state 100a9f00     MSVCRT:utility.obj
 0003:00000f04       ___scrt_native_startup_lock 100a9f04     MSVCRT:utility.obj
 0003:00000f24       ___scrt_debugger_hook_flag 100a9f24     MSVCRT:utility_desktop.obj
 0003:00000f40       _sunFontIDs                100a9f40     <common>
 0003:00000fe0       _lcdInvGammaLUT            100a9fe0     <common>
 0003:00001240       _lcdGammaLUT               100aa240     <common>
 0003:0000149c       ___dyn_tls_init_callback   100aa49c     <common>

 entry point at        0001:0006fcdc

 Static symbols

 0000:fff4f000       .debug$S                   10000000     fontmanager.exp
 0000:fff4f000       .debug$S                   10000000     vcruntime:VCRUNTIME140.dll
 0000:fff4f000       .debug$S                   10000000     vcruntime:VCRUNTIME140.dll
 0000:fff4f000       .debug$S                   10000000     vcruntime:VCRUNTIME140.dll
 0000:fff4f000       .debug$S                   10000000     vcruntime:VCRUNTIME140.dll
 0000:fff4f000       .debug$S                   10000000     vcruntime:VCRUNTIME140.dll
 0000:fff4f000       .debug$S                   10000000     vcruntime:VCRUNTIME140.dll
 0000:fff4f000       .debug$S                   10000000     vcruntime:VCRUNTIME140.dll
 0000:fff4f000       .debug$S                   10000000     vcruntime:VCRUNTIME140.dll
 0000:fff4f000       .debug$S                   10000000     vcruntime:VCRUNTIME140.dll
 0000:fff4f000       .debug$S                   10000000     vcruntime:VCRUNTIME140.dll
 0000:fff4f000       .debug$S                   10000000     vcruntime:VCRUNTIME140.dll
 0000:fff4f000       .debug$S                   10000000     vcruntime:VCRUNTIME140.dll
 0000:fff4f000       .debug$S                   10000000     ucrt:api-ms-win-crt-convert-l1-1-0.dll
 0000:fff4f000       .debug$S                   10000000     ucrt:api-ms-win-crt-convert-l1-1-0.dll
 0000:fff4f000       .debug$S                   10000000     ucrt:api-ms-win-crt-convert-l1-1-0.dll
 0000:fff4f000       .debug$S                   10000000     ucrt:api-ms-win-crt-environment-l1-1-0.dll
 0000:fff4f000       .debug$S                   10000000     ucrt:api-ms-win-crt-heap-l1-1-0.dll
 0000:fff4f000       .debug$S                   10000000     ucrt:api-ms-win-crt-heap-l1-1-0.dll
 0000:fff4f000       .debug$S                   10000000     ucrt:api-ms-win-crt-heap-l1-1-0.dll
 0000:fff4f000       .debug$S                   10000000     ucrt:api-ms-win-crt-heap-l1-1-0.dll
 0000:fff4f000       .debug$S                   10000000     ucrt:api-ms-win-crt-math-l1-1-0.dll
 0000:fff4f000       .debug$S                   10000000     ucrt:api-ms-win-crt-math-l1-1-0.dll
 0000:fff4f000       .debug$S                   10000000     ucrt:api-ms-win-crt-math-l1-1-0.dll
 0000:fff4f000       .debug$S                   10000000     ucrt:api-ms-win-crt-math-l1-1-0.dll
 0000:fff4f000       .debug$S                   10000000     ucrt:api-ms-win-crt-math-l1-1-0.dll
 0000:fff4f000       .debug$S                   10000000     ucrt:api-ms-win-crt-math-l1-1-0.dll
 0000:fff4f000       .debug$S                   10000000     ucrt:api-ms-win-crt-math-l1-1-0.dll
 0000:fff4f000       .debug$S                   10000000     ucrt:api-ms-win-crt-runtime-l1-1-0.dll
 0000:fff4f000       .debug$S                   10000000     ucrt:api-ms-win-crt-runtime-l1-1-0.dll
 0000:fff4f000       .debug$S                   10000000     ucrt:api-ms-win-crt-runtime-l1-1-0.dll
 0000:fff4f000       .debug$S                   10000000     ucrt:api-ms-win-crt-runtime-l1-1-0.dll
 0000:fff4f000       .debug$S                   10000000     ucrt:api-ms-win-crt-runtime-l1-1-0.dll
 0000:fff4f000       .debug$S                   10000000     ucrt:api-ms-win-crt-runtime-l1-1-0.dll
 0000:fff4f000       .debug$S                   10000000     ucrt:api-ms-win-crt-runtime-l1-1-0.dll
 0000:fff4f000       .debug$S                   10000000     ucrt:api-ms-win-crt-runtime-l1-1-0.dll
 0000:fff4f000       .debug$S                   10000000     ucrt:api-ms-win-crt-runtime-l1-1-0.dll
 0000:fff4f000       .debug$S                   10000000     ucrt:api-ms-win-crt-runtime-l1-1-0.dll
 0000:fff4f000       .debug$S                   10000000     ucrt:api-ms-win-crt-runtime-l1-1-0.dll
 0000:fff4f000       .debug$S                   10000000     ucrt:api-ms-win-crt-runtime-l1-1-0.dll
 0000:fff4f000       .debug$S                   10000000     ucrt:api-ms-win-crt-runtime-l1-1-0.dll
 0000:fff4f000       .debug$S                   10000000     ucrt:api-ms-win-crt-stdio-l1-1-0.dll
 0000:fff4f000       .debug$S                   10000000     ucrt:api-ms-win-crt-stdio-l1-1-0.dll
 0000:fff4f000       .debug$S                   10000000     ucrt:api-ms-win-crt-stdio-l1-1-0.dll
 0000:fff4f000       .debug$S                   10000000     ucrt:api-ms-win-crt-stdio-l1-1-0.dll
 0000:fff4f000       .debug$S                   10000000     ucrt:api-ms-win-crt-stdio-l1-1-0.dll
 0000:fff4f000       .debug$S                   10000000     ucrt:api-ms-win-crt-stdio-l1-1-0.dll
 0000:fff4f000       .debug$S                   10000000     ucrt:api-ms-win-crt-stdio-l1-1-0.dll
 0000:fff4f000       .debug$S                   10000000     ucrt:api-ms-win-crt-stdio-l1-1-0.dll
 0000:fff4f000       .debug$S                   10000000     ucrt:api-ms-win-crt-string-l1-1-0.dll
 0000:fff4f000       .debug$S                   10000000     ucrt:api-ms-win-crt-string-l1-1-0.dll
 0000:fff4f000       .debug$S                   10000000     ucrt:api-ms-win-crt-string-l1-1-0.dll
 0000:fff4f000       .debug$S                   10000000     ucrt:api-ms-win-crt-string-l1-1-0.dll
 0000:fff4f000       .debug$S                   10000000     advapi32:ADVAPI32.dll
 0000:fff4f000       .debug$S                   10000000     advapi32:ADVAPI32.dll
 0000:fff4f000       .debug$S                   10000000     advapi32:ADVAPI32.dll
 0000:fff4f000       .debug$S                   10000000     advapi32:ADVAPI32.dll
 0000:fff4f000       .debug$S                   10000000     gdi32:GDI32.dll
 0000:fff4f000       .debug$S                   10000000     gdi32:GDI32.dll
 0000:fff4f000       .debug$S                   10000000     gdi32:GDI32.dll
 0000:fff4f000       .debug$S                   10000000     gdi32:GDI32.dll
 0000:fff4f000       .debug$S                   10000000     gdi32:GDI32.dll
 0000:fff4f000       .debug$S                   10000000     gdi32:GDI32.dll
 0000:fff4f000       .debug$S                   10000000     gdi32:GDI32.dll
 0000:fff4f000       .debug$S                   10000000     gdi32:GDI32.dll
 0000:fff4f000       .debug$S                   10000000     gdi32:GDI32.dll
 0000:fff4f000       .debug$S                   10000000     gdi32:GDI32.dll
 0000:fff4f000       .debug$S                   10000000     gdi32:GDI32.dll
 0000:fff4f000       .debug$S                   10000000     gdi32:GDI32.dll
 0000:fff4f000       .debug$S                   10000000     gdi32:GDI32.dll
 0000:fff4f000       .debug$S                   10000000     gdi32:GDI32.dll
 0000:fff4f000       .debug$S                   10000000     gdi32:GDI32.dll
 0000:fff4f000       .debug$S                   10000000     gdi32:GDI32.dll
 0000:fff4f000       .debug$S                   10000000     kernel32:KERNEL32.dll
 0000:fff4f000       .debug$S                   10000000     kernel32:KERNEL32.dll
 0000:fff4f000       .debug$S                   10000000     kernel32:KERNEL32.dll
 0000:fff4f000       .debug$S                   10000000     kernel32:KERNEL32.dll
 0000:fff4f000       .debug$S                   10000000     kernel32:KERNEL32.dll
 0000:fff4f000       .debug$S                   10000000     kernel32:KERNEL32.dll
 0000:fff4f000       .debug$S                   10000000     kernel32:KERNEL32.dll
 0000:fff4f000       .debug$S                   10000000     kernel32:KERNEL32.dll
 0000:fff4f000       .debug$S                   10000000     kernel32:KERNEL32.dll
 0000:fff4f000       .debug$S                   10000000     kernel32:KERNEL32.dll
 0000:fff4f000       .debug$S                   10000000     kernel32:KERNEL32.dll
 0000:fff4f000       .debug$S                   10000000     kernel32:KERNEL32.dll
 0000:fff4f000       .debug$S                   10000000     kernel32:KERNEL32.dll
 0000:fff4f000       .debug$S                   10000000     kernel32:KERNEL32.dll
 0000:fff4f000       .debug$S                   10000000     kernel32:KERNEL32.dll
 0000:fff4f000       .debug$S                   10000000     kernel32:KERNEL32.dll
 0000:fff4f000       .debug$S                   10000000     kernel32:KERNEL32.dll
 0000:fff4f000       .debug$S                   10000000     kernel32:KERNEL32.dll
 0000:fff4f000       .debug$S                   10000000     kernel32:KERNEL32.dll
 0000:fff4f000       .debug$S                   10000000     kernel32:KERNEL32.dll
 0000:fff4f000       .debug$S                   10000000     kernel32:KERNEL32.dll
 0000:fff4f000       .debug$S                   10000000     kernel32:KERNEL32.dll
 0000:fff4f000       .debug$S                   10000000     kernel32:KERNEL32.dll
 0000:fff4f000       .debug$S                   10000000     kernel32:KERNEL32.dll
 0000:fff4f000       .debug$S                   10000000     kernel32:KERNEL32.dll
 0000:fff4f000       .debug$S                   10000000     kernel32:KERNEL32.dll
 0000:fff4f000       .debug$S                   10000000     user32:USER32.dll
 0000:fff4f000       .debug$S                   10000000     user32:USER32.dll
 0000:fff4f000       .debug$S                   10000000     user32:USER32.dll
 0000:fff4f000       .debug$S                   10000000     user32:USER32.dll
 0000:fff4f000       .debug$S                   10000000     user32:USER32.dll
 0000:fff4f000       .debug$S                   10000000     user32:USER32.dll
 0000:fff4f000       .debug$S                   10000000     java:java.dll
 0000:fff4f000       .debug$S                   10000000     java:java.dll
 0000:fff4f000       .debug$S                   10000000     java:java.dll
 0000:fff4f000       .debug$S                   10000000     java:java.dll
 0000:fff4f000       .debug$S                   10000000     awt:awt.dll
 0000:fff4f000       .debug$S                   10000000     awt:awt.dll
 0000:fff4f000       .debug$S                   10000000     awt:awt.dll
 0000:fff4f000       .debug$S                   10000000     awt:awt.dll
 0000:fff4f000       .debug$S                   10000000     awt:awt.dll
 0000:fff4f000       .debug$S                   10000000     awt:awt.dll
 0000:fff4f000       .debug$S                   10000000     awt:awt.dll
 0000:fff4f000       .debug$S                   10000000     awt:awt.dll
 0000:fff4f000       .debug$S                   10000000     awt:awt.dll
 0000:fff4f000       .debug$S                   10000000     awt:awt.dll
 0000:fff4f000       .debug$S                   10000000     freetype:freetype.dll
 0000:fff4f000       .debug$S                   10000000     freetype:freetype.dll
 0000:fff4f000       .debug$S                   10000000     freetype:freetype.dll
 0000:fff4f000       .debug$S                   10000000     freetype:freetype.dll
 0000:fff4f000       .debug$S                   10000000     freetype:freetype.dll
 0000:fff4f000       .debug$S                   10000000     freetype:freetype.dll
 0000:fff4f000       .debug$S                   10000000     freetype:freetype.dll
 0000:fff4f000       .debug$S                   10000000     freetype:freetype.dll
 0000:fff4f000       .debug$S                   10000000     freetype:freetype.dll
 0000:fff4f000       .debug$S                   10000000     freetype:freetype.dll
 0000:fff4f000       .debug$S                   10000000     freetype:freetype.dll
 0000:fff4f000       .debug$S                   10000000     freetype:freetype.dll
 0000:fff4f000       .debug$S                   10000000     freetype:freetype.dll
 0000:fff4f000       .debug$S                   10000000     freetype:freetype.dll
 0000:fff4f000       .debug$S                   10000000     freetype:freetype.dll
 0000:fff4f000       .debug$S                   10000000     freetype:freetype.dll
 0000:fff4f000       .debug$S                   10000000     freetype:freetype.dll
 0000:fff4f000       .debug$S                   10000000     freetype:freetype.dll
 0000:fff4f000       .debug$S                   10000000     freetype:freetype.dll
 0000:fff4f000       .debug$S                   10000000     freetype:freetype.dll
 0001:00000000       _Glyph_GetRasInfo          10001000 f   ColorGlyphSurfaceData.obj
 0001:00000030       _Glyph_Lock                10001030 f   ColorGlyphSurfaceData.obj
 0001:00000350       _drawGlyphList             10001350 f   DrawGlyphList.obj
 0001:000004c0       _drawGlyphListLCD          100014c0 f   DrawGlyphList.obj
 0001:00001680       _euclidianDistance         10002680 f   HBShaper.obj
 0001:00001c60       _CheckFontFamilyProcW@16   10002c60 f   fontpath.obj
 0001:00001cb0       _EnumFamilyNamesW@16       10002cb0 f   fontpath.obj
 0001:00001f60       _EnumFontFacesInFamilyProcW@16 10002f60 f   fontpath.obj
 0001:000024c0       _populateFontFileNameFromRegistryKey 100034c0 f   fontpath.obj
 0001:00002710       _registerFontW             10003710 f   fontpath.obj
 0001:00002950       _moveTo                    10003950 f   freetypeScaler.obj
 0001:000029c0       _lineTo                    100039c0 f   freetypeScaler.obj
 0001:00002a20       _conicTo                   10003a20 f   freetypeScaler.obj
 0001:00002ac0       _cubicTo                   10003ac0 f   freetypeScaler.obj
 0001:00002ba0       _GlyphSlot_Embolden        10003ba0 f   freetypeScaler.obj
 0001:00003cb0       _ReadTTFontFileFunc        10004cb0 f   freetypeScaler.obj
 0001:00003e10       _addToGP                   10004e10 f   freetypeScaler.obj
 0001:00003e50       _allocateSpaceForGP        10004e50 f   freetypeScaler.obj
 0001:00003f30       _getFTOutline              10004f30 f   freetypeScaler.obj
 0001:00004000       _getGlyphImageNativeInternal 10005000 f   freetypeScaler.obj
 0001:000046e0       _invalidateJavaScaler      100056e0 f   freetypeScaler.obj
 0001:00004760       _setupFTContext            10005760 f   freetypeScaler.obj
 0001:00004930       ??$_hb_cmp_method@I$$CBURangeRecord@OT@@$$V@@YAHPBX0@Z 10005930 f   hb-aat-layout.obj
 0001:00004970       ??$_hb_cmp_method@IU?$LookupSegmentArray@U?$IntType@G$01@OT@@@AAT@@$$V@@YAHPBX0@Z 10005970 f   hb-aat-layout.obj
 0001:00004970       ??$_hb_cmp_method@IU?$LookupSegmentArray@U?$IntType@I$03@OT@@@AAT@@$$V@@YAHPBX0@Z 10005970 f   hb-aat-layout.obj
 0001:00004970       ??$_hb_cmp_method@IU?$LookupSegmentArray@U?$OffsetTo@U?$ArrayOf@UAnchor@AAT@@U?$IntType@I$03@OT@@@OT@@U?$IntType@G$01@2@$0A@@OT@@@AAT@@$$V@@YAHPBX0@Z 10005970 f   hb-aat-layout.obj
 0001:00004970       ??$_hb_cmp_method@IU?$LookupSegmentArray@UHBGlyphID16@OT@@@AAT@@$$V@@YAHPBX0@Z 10005970 f   hb-aat-layout.obj
 0001:00004970       ??$_hb_cmp_method@IU?$LookupSegmentSingle@U?$IntType@G$01@OT@@@AAT@@$$V@@YAHPBX0@Z 10005970 f   hb-aat-layout.obj
 0001:00004970       ??$_hb_cmp_method@IU?$LookupSegmentSingle@U?$IntType@I$03@OT@@@AAT@@$$V@@YAHPBX0@Z 10005970 f   hb-aat-layout.obj
 0001:00004970       ??$_hb_cmp_method@IU?$LookupSegmentSingle@U?$OffsetTo@U?$ArrayOf@UAnchor@AAT@@U?$IntType@I$03@OT@@@OT@@U?$IntType@G$01@2@$0A@@OT@@@AAT@@$$V@@YAHPBX0@Z 10005970 f   hb-aat-layout.obj
 0001:00004970       ??$_hb_cmp_method@IU?$LookupSegmentSingle@UHBGlyphID16@OT@@@AAT@@$$V@@YAHPBX0@Z 10005970 f   hb-aat-layout.obj
 0001:000049b0       ??$_hb_cmp_method@IU?$LookupSingle@U?$IntType@G$01@OT@@@AAT@@$$V@@YAHPBX0@Z 100059b0 f   hb-aat-layout.obj
 0001:000049b0       ??$_hb_cmp_method@IU?$LookupSingle@U?$IntType@I$03@OT@@@AAT@@$$V@@YAHPBX0@Z 100059b0 f   hb-aat-layout.obj
 0001:000049b0       ??$_hb_cmp_method@IU?$LookupSingle@U?$OffsetTo@U?$ArrayOf@UAnchor@AAT@@U?$IntType@I$03@OT@@@OT@@U?$IntType@G$01@2@$0A@@OT@@@AAT@@$$V@@YAHPBX0@Z 100059b0 f   hb-aat-layout.obj
 0001:000049b0       ??$_hb_cmp_method@IU?$LookupSingle@UHBGlyphID16@OT@@@AAT@@$$V@@YAHPBX0@Z 100059b0 f   hb-aat-layout.obj
 0001:000049e0       ??$_hb_debug_msg@$0A@@@YAXPBDPBX0_NIH0ZZ 100059e0 f   hb-aat-layout.obj
 0001:000049e0       ??$_hb_debug_msg@$0A@@@YAXPBDPBX0_NIH0ZZ 100059e0 f   hb-blob.obj
 0001:000049e0       ??$_hb_debug_msg@$0A@@@YAXPBDPBX0_NIH0ZZ 100059e0 f   hb-common.obj
 0001:000049e0       ?hb_draw_close_path_nil@@YAXPAUhb_draw_funcs_t@@PAXPAUhb_draw_state_t@@1@Z 100059e0 f   hb-draw.obj
 0001:000049e0       ?hb_draw_cubic_to_nil@@YAXPAUhb_draw_funcs_t@@PAXPAUhb_draw_state_t@@MMMMMM1@Z 100059e0 f   hb-draw.obj
 0001:000049e0       ?hb_draw_line_to_nil@@YAXPAUhb_draw_funcs_t@@PAXPAUhb_draw_state_t@@MM1@Z 100059e0 f   hb-draw.obj
 0001:000049e0       ?hb_draw_move_to_nil@@YAXPAUhb_draw_funcs_t@@PAXPAUhb_draw_state_t@@MM1@Z 100059e0 f   hb-draw.obj
 0001:000049e0       ??$_hb_debug_msg@$0A@@@YAXPBDPBX0_NIH0ZZ 100059e0 f   hb-face.obj
 0001:000049e0       ??$_hb_debug_msg@$0A@@@YAXPBDPBX0_NIH0ZZ 100059e0 f   hb-font.obj
 0001:000049e0       ?hb_font_get_glyph_shape_nil@@YAXPAUhb_font_t@@PAXIPAUhb_draw_funcs_t@@11@Z 100059e0 f   hb-font.obj
 0001:000049e0       ?_do_nothing@@YAXXZ        100059e0 f   hb-jdk-font.obj
 0001:000049e0       ??$_hb_debug_msg@$0A@@@YAXPBDPBX0_NIH0ZZ 100059e0 f   hb-ot-color.obj
 0001:000049e0       ??$_hb_debug_msg@$0A@@@YAXPBDPBX0_NIH0ZZ 100059e0 f   hb-ot-face.obj
 0001:000049e0       ??$_hb_debug_msg@$0A@@@YAXPBDPBX0_NIH0ZZ 100059e0 f   hb-ot-font.obj
 0001:000049e0       ??$_hb_debug_msg@$0A@@@YAXPBDPBX0_NIH0ZZ 100059e0 f   hb-ot-layout.obj
 0001:000049e0       ??$_hb_debug_msg@$0A@@@YAXPBDPBX0_NIH0ZZ 100059e0 f   hb-ot-metrics.obj
 0001:000049e0       ??$_hb_debug_msg@$0A@@@YAXPBDPBX0_NIH0ZZ 100059e0 f   hb-ot-shaper-arabic.obj
 0001:000049e0       ??$_hb_debug_msg@$0A@@@YAXPBDPBX0_NIH0ZZ 100059e0 f   hb-shape-plan.obj
 0001:00004fbc       $LN259                     10005fbc     hb-aat-layout.obj
 0001:00005324       $LN259                     10006324     hb-aat-layout.obj
 0001:00005620       $LN144                     10006620     hb-aat-layout.obj
 0001:0000590c       $LN159                     1000690c     hb-aat-layout.obj
 0001:00005b20       $LN155                     10006b20     hb-aat-layout.obj
 0001:00005dd4       $LN133                     10006dd4     hb-aat-layout.obj
 0001:000080f0       ??$hb_bsearch_impl@$$CBURangeRecord@OT@@I$$V@@YA_NPAIABIPBURangeRecord@OT@@IIP6AHPBX3@Z@Z 100090f0 f   hb-aat-layout.obj
 0001:000080f0       ??$hb_bsearch_impl@$$CBXI$$V@@YA_NPAIABIPBXIIP6AH22@Z@Z 100090f0 f   hb-aat-layout.obj
 0001:0000dac8       $LN122                     1000eac8     hb-aat-layout.obj
 0001:0000dac8       $LN122                     1000eac8     hb-aat-layout.obj
 0001:0000dac8       $LN122                     1000eac8     hb-aat-layout.obj
 0001:0000dd18       $LN122                     1000ed18     hb-aat-layout.obj
 0001:0000e8f0       ?is_deleted_glyph@@YA_NPBUhb_glyph_info_t@@@Z 1000f8f0 f   hb-aat-layout.obj
 0001:0000f4d0       ?kerxTupleKern@AAT@@YAHHIPBXPAUhb_aat_apply_context_t@1@@Z 100104d0 f   hb-aat-layout.obj
 0001:000101b4       $LN256                     100111b4     hb-aat-layout.obj
 0001:000101b4       $LN256                     100111b4     hb-aat-layout.obj
 0001:00010428       $LN256                     10011428     hb-aat-layout.obj
 0001:000105bc       $LN40                      100115bc     hb-aat-layout.obj
 0001:000146d0       ??$sort_r_simple@$$V@@YAXPAXIIP6AHPBX1@Z@Z 100156d0 f   hb-aat-map.obj
 0001:000146d0       ??$sort_r_simple@$$V@@YAXPAXIIP6AHPBX1@Z@Z 100156d0 f   hb-ot-font.obj
 0001:000146d0       ??$sort_r_simple@$$V@@YAXPAXIIP6AHPBX1@Z@Z 100156d0 f   hb-ot-map.obj
 0001:00014de0       ?_hb_blob_destroy@@YAXPAX@Z 10015de0 f   hb-blob.obj
 0001:000155e0       ?buffer_verify_error@@YAXPAUhb_buffer_t@@PAUhb_font_t@@PBDZZ 100165e0 f   hb-buffer-verify.obj
 0001:00015660       ?buffer_verify_unsafe_to_break@@YA_NPAUhb_buffer_t@@0PAUhb_font_t@@PBUhb_feature_t@@IPBQBD@Z 10016660 f   hb-buffer-verify.obj
 0001:00015910       ?buffer_verify_unsafe_to_concat@@YA_NPAUhb_buffer_t@@0PAUhb_font_t@@PBUhb_feature_t@@IPBQBD@Z 10016910 f   hb-buffer-verify.obj
 0001:00015df0       ??$hb_buffer_add_utf@U?$hb_utf16_xe_t@G@@@@YAXPAUhb_buffer_t@@PBGHIH@Z 10016df0 f   hb-buffer.obj
 0001:00017d60       ?lang_find_or_insert@@YAPAUhb_language_item_t@@PBD@Z 10018d60 f   hb-common.obj
 0001:00017f30       ?parse_feature_value_postfix@@YA_NPAPBDPBDPAUhb_feature_t@@@Z 10018f30 f   hb-common.obj
 0001:00018090       ?parse_one_feature@@YA_NPAPBDPBDPAUhb_feature_t@@@Z 10019090 f   hb-common.obj
 0001:000181f0       ?parse_space@@YA_NPAPBDPBD@Z 100191f0 f   hb-common.obj
 0001:00018230       ?parse_tag@@YA_NPAPBDPBDPAI@Z 10019230 f   hb-common.obj
 0001:00018810       ?hb_draw_quadratic_to_nil@@YAXPAUhb_draw_funcs_t@@PAXPAUhb_draw_state_t@@MMMM1@Z 10019810 f   hb-draw.obj
 0001:00018da0       ??$get_glyph_from_symbol@UCmapSubtable@OT@@$1?_hb_arabic_pua_simp_map@@YAII@Z@accelerator_t@cmap@OT@@KA_NPBXIPAI@Z 10019da0 f   hb-face.obj
 0001:00018de0       ??$get_glyph_from_symbol@UCmapSubtable@OT@@$1?_hb_arabic_pua_trad_map@@YAII@Z@accelerator_t@cmap@OT@@KA_NPBXIPAI@Z 10019de0 f   hb-face.obj
 0001:00018e20       ??$get_glyph_from_symbol@UCmapSubtable@OT@@$1?_hb_symbol_pua_map@2@YAII@Z@accelerator_t@cmap@OT@@KA_NPBXIPAI@Z 10019e20 f   hb-face.obj
 0001:00019d30       ?_hb_arabic_pua_simp_map@@YAII@Z 1001ad30 f   hb-face.obj
 0001:00019db0       ?_hb_arabic_pua_trad_map@@YAII@Z 1001adb0 f   hb-face.obj
 0001:0001a78c       $LN86                      1001b78c     hb-face.obj
 0001:0001a7a8       $LN85                      1001b7a8     hb-face.obj
 0001:0001a9a0       ?hb_memcmp@@YAHPBX0I@Z     1001b9a0 f   hb-face.obj
 0001:0001a9a0       ?hb_memcmp@@YAHPBX0I@Z     1001b9a0 f   hb-ot-font.obj
 0001:0001b89c       $LN236                     1001c89c     hb-face.obj
 0001:0001b8b8       $LN235                     1001c8b8     hb-face.obj
 0001:0001c500       $LN119                     1001d500     hb-fallback-shape.obj
 0001:0001c514       $LN118                     1001d514     hb-fallback-shape.obj
 0001:0001c530       ?hb_jdk_get_glyph_h_origin@@YAHPAUhb_font_t@@PAXIPAH21@Z 1001d530 f   hb-jdk-font.obj
 0001:0001c530       ?hb_unicode_eastasian_width_nil@@YAIPAUhb_unicode_funcs_t@@IPAX@Z 1001d530 f   hb-unicode.obj
 0001:0001c540       ?hb_font_get_font_h_extents_nil@@YAHPAUhb_font_t@@PAXPAUhb_font_extents_t@@1@Z 1001d540 f   hb-font.obj
 0001:0001c540       ?hb_font_get_font_v_extents_nil@@YAHPAUhb_font_t@@PAXPAUhb_font_extents_t@@1@Z 1001d540 f   hb-font.obj
 0001:0001c560       ?hb_font_get_font_h_extents_default@@YAHPAUhb_font_t@@PAXPAUhb_font_extents_t@@1@Z 1001d560 f   hb-font.obj
 0001:0001c640       ?hb_font_get_font_v_extents_default@@YAHPAUhb_font_t@@PAXPAUhb_font_extents_t@@1@Z 1001d640 f   hb-font.obj
 0001:0001c720       ?hb_font_get_nominal_glyph_nil@@YAHPAUhb_font_t@@PAXIPAI1@Z 1001d720 f   hb-font.obj
 0001:0001c730       ?hb_font_get_nominal_glyph_default@@YAHPAUhb_font_t@@PAXIPAI1@Z 1001d730 f   hb-font.obj
 0001:0001c7b0       ?hb_font_get_nominal_glyphs_default@@YAIPAUhb_font_t@@PAXIPBIIPAII1@Z 1001d7b0 f   hb-font.obj
 0001:0001c860       ?hb_font_get_glyph_from_name_nil@@YAHPAUhb_font_t@@PAXPBDHPAI1@Z 1001d860 f   hb-font.obj
 0001:0001c860       ?hb_font_get_variation_glyph_nil@@YAHPAUhb_font_t@@PAXIIPAI1@Z 1001d860 f   hb-font.obj
 0001:0001c870       ?hb_font_get_variation_glyph_default@@YAHPAUhb_font_t@@PAXIIPAI1@Z 1001d870 f   hb-font.obj
 0001:0001c8b0       ?hb_font_get_glyph_h_advance_nil@@YAHPAUhb_font_t@@PAXI1@Z 1001d8b0 f   hb-font.obj
 0001:0001c8c0       ?hb_font_get_glyph_h_advance_default@@YAHPAUhb_font_t@@PAXI1@Z 1001d8c0 f   hb-font.obj
 0001:0001c950       ?hb_font_get_glyph_v_advance_nil@@YAHPAUhb_font_t@@PAXI1@Z 1001d950 f   hb-font.obj
 0001:0001c960       ?hb_font_get_glyph_v_advance_default@@YAHPAUhb_font_t@@PAXI1@Z 1001d960 f   hb-font.obj
 0001:0001c9f0       ?hb_font_get_glyph_h_advances_default@@YAXPAUhb_font_t@@PAXIPBIIPAHI1@Z 1001d9f0 f   hb-font.obj
 0001:0001cad0       ?hb_font_get_glyph_v_advances_default@@YAXPAUhb_font_t@@PAXIPBIIPAHI1@Z 1001dad0 f   hb-font.obj
 0001:0001cbb0       ?hb_font_get_glyph_h_origin_nil@@YAHPAUhb_font_t@@PAXIPAH21@Z 1001dbb0 f   hb-font.obj
 0001:0001cbd0       ?hb_font_get_glyph_h_origin_default@@YAHPAUhb_font_t@@PAXIPAH21@Z 1001dbd0 f   hb-font.obj
 0001:0001cc30       ?hb_font_get_glyph_v_origin_nil@@YAHPAUhb_font_t@@PAXIPAH21@Z 1001dc30 f   hb-font.obj
 0001:0001cc50       ?hb_font_get_glyph_v_origin_default@@YAHPAUhb_font_t@@PAXIPAH21@Z 1001dc50 f   hb-font.obj
 0001:0001ccb0       ?hb_font_get_glyph_h_kerning_nil@@YAHPAUhb_font_t@@PAXII1@Z 1001dcb0 f   hb-font.obj
 0001:0001ccb0       ?hb_font_get_glyph_v_kerning_nil@@YAHPAUhb_font_t@@PAXII1@Z 1001dcb0 f   hb-font.obj
 0001:0001ccb0       ?hb_jdk_get_glyph_extents@@YAHPAUhb_font_t@@PAXIPAUhb_glyph_extents_t@@1@Z 1001dcb0 f   hb-jdk-font.obj
 0001:0001ccb0       ?hb_jdk_get_glyph_from_name@@YAHPAUhb_font_t@@PAXPBDHPAI1@Z 1001dcb0 f   hb-jdk-font.obj
 0001:0001ccb0       ?hb_jdk_get_glyph_h_kerning@@YAHPAUhb_font_t@@PAXII1@Z 1001dcb0 f   hb-jdk-font.obj
 0001:0001ccb0       ?hb_jdk_get_glyph_name@@YAHPAUhb_font_t@@PAXIPADI1@Z 1001dcb0 f   hb-jdk-font.obj
 0001:0001ccb0       ?hb_jdk_get_glyph_v_kerning@@YAHPAUhb_font_t@@PAXII1@Z 1001dcb0 f   hb-jdk-font.obj
 0001:0001ccb0       ?hb_jdk_get_glyph_v_origin@@YAHPAUhb_font_t@@PAXIPAH21@Z 1001dcb0 f   hb-jdk-font.obj
 0001:0001ccb0       ?hb_unicode_combining_class_nil@@YA?AW4hb_unicode_combining_class_t@@PAUhb_unicode_funcs_t@@IPAX@Z 1001dcb0 f   hb-unicode.obj
 0001:0001ccb0       ?hb_unicode_compose_nil@@YAHPAUhb_unicode_funcs_t@@IIPAIPAX@Z 1001dcb0 f   hb-unicode.obj
 0001:0001ccb0       ?hb_unicode_decompose_compatibility_nil@@YAIPAUhb_unicode_funcs_t@@IPAIPAX@Z 1001dcb0 f   hb-unicode.obj
 0001:0001ccb0       ?hb_unicode_decompose_nil@@YAHPAUhb_unicode_funcs_t@@IPAI1PAX@Z 1001dcb0 f   hb-unicode.obj
 0001:0001ccc0       ?hb_font_get_glyph_h_kerning_default@@YAHPAUhb_font_t@@PAXII1@Z 1001dcc0 f   hb-font.obj
 0001:0001cd20       ?hb_font_get_glyph_v_kerning_default@@YAHPAUhb_font_t@@PAXII1@Z 1001dd20 f   hb-font.obj
 0001:0001cd80       ?hb_font_get_glyph_extents_nil@@YAHPAUhb_font_t@@PAXIPAUhb_glyph_extents_t@@1@Z 1001dd80 f   hb-font.obj
 0001:0001cd90       ?hb_font_get_glyph_extents_default@@YAHPAUhb_font_t@@PAXIPAUhb_glyph_extents_t@@1@Z 1001dd90 f   hb-font.obj
 0001:0001ce50       ?hb_font_get_glyph_contour_point_nil@@YAHPAUhb_font_t@@PAXIIPAH21@Z 1001de50 f   hb-font.obj
 0001:0001ce70       ?hb_font_get_glyph_contour_point_default@@YAHPAUhb_font_t@@PAXIIPAH21@Z 1001de70 f   hb-font.obj
 0001:0001ced0       ?hb_font_get_glyph_name_nil@@YAHPAUhb_font_t@@PAXIPADI1@Z 1001ded0 f   hb-font.obj
 0001:0001cef0       ?hb_font_get_glyph_name_default@@YAHPAUhb_font_t@@PAXIPADI1@Z 1001def0 f   hb-font.obj
 0001:0001cf30       ?hb_font_get_glyph_from_name_default@@YAHPAUhb_font_t@@PAXPBDHPAI1@Z 1001df30 f   hb-font.obj
 0001:0001cf80       ?hb_draw_move_to_default@@YAXPAUhb_draw_funcs_t@@PAXPAUhb_draw_state_t@@MM1@Z 1001df80 f   hb-font.obj
 0001:0001cfd0       ?hb_draw_line_to_default@@YAXPAUhb_draw_funcs_t@@PAXPAUhb_draw_state_t@@MM1@Z 1001dfd0 f   hb-font.obj
 0001:0001d040       ?hb_draw_quadratic_to_default@@YAXPAUhb_draw_funcs_t@@PAXPAUhb_draw_state_t@@MMMM1@Z 1001e040 f   hb-font.obj
 0001:0001d0d0       ?hb_draw_cubic_to_default@@YAXPAUhb_draw_funcs_t@@PAXPAUhb_draw_state_t@@MMMMMM1@Z 1001e0d0 f   hb-font.obj
 0001:0001d180       ?hb_draw_close_path_default@@YAXPAUhb_draw_funcs_t@@PAXPAUhb_draw_state_t@@1@Z 1001e180 f   hb-font.obj
 0001:0001d1b0       ?hb_font_get_glyph_shape_default@@YAXPAUhb_font_t@@PAXIPAUhb_draw_funcs_t@@11@Z 1001e1b0 f   hb-font.obj
 0001:0001da80       ?_hb_font_create@@YAPAUhb_font_t@@PAUhb_face_t@@@Z 1001ea80 f   hb-font.obj
 0001:0001fdc0       ?cleanupFontInfo@@YAXPAX@Z 10020dc0 f   hb-jdk-font.obj
 0001:0001fe00       ?hb_jdk_get_glyph_contour_point@@YAHPAUhb_font_t@@PAXIIPAH21@Z 10020e00 f   hb-jdk-font.obj
 0001:0001fed0       ?hb_jdk_get_glyph_h_advance@@YAHPAUhb_font_t@@PAXI1@Z 10020ed0 f   hb-jdk-font.obj
 0001:0001ff50       ?hb_jdk_get_glyph_v_advance@@YAHPAUhb_font_t@@PAXI1@Z 10020f50 f   hb-jdk-font.obj
 0001:0001ffc0       ?hb_jdk_get_nominal_glyph@@YAHPAUhb_font_t@@PAXIPAI1@Z 10020fc0 f   hb-jdk-font.obj
 0001:00020010       ?hb_jdk_get_variation_glyph@@YAHPAUhb_font_t@@PAXIIPAI1@Z 10021010 f   hb-jdk-font.obj
 0001:00020070       ?reference_table@@YAPAUhb_blob_t@@PAUhb_face_t@@IPAX@Z 10021070 f   hb-jdk-font.obj
 0001:000202d0       ?_pow10@@YANI@Z            100212d0 f   hb-number.obj
 0001:00020430       ?strtod_rl@@YANPBDPAPBD@Z  10021430 f   hb-number.obj
 0001:00020718       $LN63                      10021718     hb-number.obj
 0001:00020b70       ?_get_bounds@@YA_NPBUaccelerator_t@cff1@OT@@IAAUbounds_t@@_N@Z 10021b70 f   hb-ot-cff1-table.obj
 0001:00020c90       ?_get_path@@YA_NPBUaccelerator_t@cff1@OT@@PAUhb_font_t@@IAAUhb_draw_session_t@@_NPAUpoint_t@CFF@@@Z 10021c90 f   hb-ot-cff1-table.obj
 0001:00020f90       $LN11                      10021f90     hb-ot-cff1-table.obj
 0001:00020f90       $LN11                      10021f90     hb-ot-cff1-table.obj
 0001:00020fa0       $LN10                      10021fa0     hb-ot-cff1-table.obj
 0001:00020fa0       $LN10                      10021fa0     hb-ot-cff1-table.obj
 0001:00025e30       $LN247                     10026e30     hb-ot-cff1-table.obj
 0001:00025e88       $LN246                     10026e88     hb-ot-cff1-table.obj
 0001:00026674       $LN330                     10027674     hb-ot-cff1-table.obj
 0001:000266cc       $LN329                     100276cc     hb-ot-cff1-table.obj
 0001:000269c8       $LN112                     100279c8     hb-ot-cff1-table.obj
 0001:000269d8       $LN111                     100279d8     hb-ot-cff1-table.obj
 0001:0002fdb0       $LN83                      10030db0     hb-ot-cff2-table.obj
 0001:0002fdc0       $LN82                      10030dc0     hb-ot-cff2-table.obj
 0001:0002ffa0       $LN83                      10030fa0     hb-ot-cff2-table.obj
 0001:0002ffb0       $LN82                      10030fb0     hb-ot-cff2-table.obj
 0001:0003045c       $LN236                     1003145c     hb-ot-cff2-table.obj
 0001:000304b4       $LN235                     100314b4     hb-ot-cff2-table.obj
 0001:00030d28       $LN379                     10031d28     hb-ot-cff2-table.obj
 0001:00030d80       $LN378                     10031d80     hb-ot-cff2-table.obj
 0001:00039980       ??$sort_r_simple@PAX@@YAXPAXIIP6AHPBX10@Z0@Z 1003a980 f   hb-ot-font.obj
 0001:0003b970       ?_hb_ot_font_destroy@@YAXPAX@Z 1003c970 f   hb-ot-font.obj
 0001:0003b9a0       ?_hb_roundf@@YAMM@Z        1003c9a0 f   hb-ot-font.obj
 0001:0003b9a0       ?_hb_roundf@@YAMM@Z        1003c9a0 f   hb-ot-layout.obj
 0001:0003d450       ?format1_names@@YA?AU?$hb_array_t@$$CBD@@I@Z 1003e450 f   hb-ot-font.obj
 0001:0003f7c0       ?hb_ot_get_font_h_extents@@YAHPAUhb_font_t@@PAXPAUhb_font_extents_t@@1@Z 100407c0 f   hb-ot-font.obj
 0001:0003f820       ?hb_ot_get_font_v_extents@@YAHPAUhb_font_t@@PAXPAUhb_font_extents_t@@1@Z 10040820 f   hb-ot-font.obj
 0001:0003f880       ?hb_ot_get_glyph_extents@@YAHPAUhb_font_t@@PAXIPAUhb_glyph_extents_t@@1@Z 10040880 f   hb-ot-font.obj
 0001:0003fb80       ?hb_ot_get_glyph_from_name@@YAHPAUhb_font_t@@PAXPBDHPAI1@Z 10040b80 f   hb-ot-font.obj
 0001:0003fbd0       ?hb_ot_get_glyph_h_advances@@YAXPAUhb_font_t@@PAXIPBIIPAHI1@Z 10040bd0 f   hb-ot-font.obj
 0001:0003ff90       ?hb_ot_get_glyph_name@@YAHPAUhb_font_t@@PAXIPADI1@Z 10040f90 f   hb-ot-font.obj
 0001:00040070       ?hb_ot_get_glyph_shape@@YAXPAUhb_font_t@@PAXIPAUhb_draw_funcs_t@@11@Z 10041070 f   hb-ot-font.obj
 0001:00040300       ?hb_ot_get_glyph_v_advances@@YAXPAUhb_font_t@@PAXIPBIIPAHI1@Z 10041300 f   hb-ot-font.obj
 0001:00040550       ?hb_ot_get_glyph_v_origin@@YAHPAUhb_font_t@@PAXIPAH21@Z 10041550 f   hb-ot-font.obj
 0001:00040820       ?hb_ot_get_nominal_glyph@@YAHPAUhb_font_t@@PAXIPAI1@Z 10041820 f   hb-ot-font.obj
 0001:00040850       ?hb_ot_get_nominal_glyphs@@YAIPAUhb_font_t@@PAXIPBIIPAII1@Z 10041850 f   hb-ot-font.obj
 0001:000408c0       ?hb_ot_get_variation_glyph@@YAHPAUhb_font_t@@PAXIIPAI1@Z 100418c0 f   hb-ot-font.obj
 0001:00041730       $LN135                     10042730     hb-ot-font.obj
 0001:00041740       $LN134                     10042740     hb-ot-font.obj
 0001:00041750       $LN137                     10042750     hb-ot-font.obj
 0001:0004175c       $LN136                     1004275c     hb-ot-font.obj
 0001:00042294       $LN171                     10043294     hb-ot-font.obj
 0001:000422ac       $LN170                     100432ac     hb-ot-font.obj
 0001:000422c0       $LN173                     100432c0     hb-ot-font.obj
 0001:000422d8       $LN172                     100432d8     hb-ot-font.obj
 0001:00042300       $LN174                     10043300     hb-ot-font.obj
 0001:000424a8       $LN79                      100434a8     hb-ot-font.obj
 0001:000424bc       $LN78                      100434bc     hb-ot-font.obj
 0001:000424d0       $LN81                      100434d0     hb-ot-font.obj
 0001:000424dc       $LN80                      100434dc     hb-ot-font.obj
 0001:00045360       ??$apply_string@UGSUBProxy@@@@YAXPAUhb_ot_apply_context_t@OT@@ABUSubstLookup@GSUB@Layout@1@ABUhb_ot_layout_lookup_accelerator_t@1@@Z 10046360 f   hb-ot-layout.obj
 0001:000459f8       $LN308                     100469f8     hb-ot-layout.obj
 0001:00045afc       $LN249                     10046afc     hb-ot-layout.obj
 0001:00045cd4       $LN361                     10046cd4     hb-ot-layout.obj
 0001:00045eb4       $LN302                     10046eb4     hb-ot-layout.obj
 0001:0004614c       $LN214                     1004714c     hb-ot-layout.obj
 0001:00046334       $LN98                      10047334     hb-ot-layout.obj
 0001:00046a60       $LN428                     10047a60     hb-ot-layout.obj
 0001:00046d20       $LN345                     10047d20     hb-ot-layout.obj
 0001:00046f40       $LN140                     10047f40     hb-ot-layout.obj
 0001:000470b8       $LN123                     100480b8     hb-ot-layout.obj
 0001:000472ec       $LN83                      100482ec     hb-ot-layout.obj
 0001:00047ad4       $LN265                     10048ad4     hb-ot-layout.obj
 0001:00048048       $LN291                     10049048     hb-ot-layout.obj
 0001:00048748       $LN238                     10049748     hb-ot-layout.obj
 0001:0004bdd0       ?_hb_allocate_lig_id@@YAEPAUhb_buffer_t@@@Z 1004cdd0 f   hb-ot-layout.obj
 0001:0004be00       ?_hb_glyph_info_get_lig_comp@@YAIPBUhb_glyph_info_t@@@Z 1004ce00 f   hb-ot-layout.obj
 0001:0004c330       $LN173                     1004d330     hb-ot-layout.obj
 0001:0004d180       $LN131                     1004e180     hb-ot-layout.obj
 0001:0004eb20       ?apply_backward@@YA_NPAUhb_ot_apply_context_t@OT@@ABUhb_ot_layout_lookup_accelerator_t@2@@Z 1004fb20 f   hb-ot-layout.obj
 0001:0004eda0       ?apply_forward@@YA_NPAUhb_ot_apply_context_t@OT@@ABUhb_ot_layout_lookup_accelerator_t@2@@Z 1004fda0 f   hb-ot-layout.obj
 0001:0004f190       ?apply_lookup@OT@@YAXPAUhb_ot_apply_context_t@1@IQAIIQBULookupRecord@1@I@Z 10050190 f   hb-ot-layout.obj
 0001:0004f820       ?chain_context_apply_lookup@OT@@YA_NPAUhb_ot_apply_context_t@1@IQBU?$IntType@G$01@1@I1I1IQBULookupRecord@1@AAUChainContextApplyLookupContext@1@@Z 10050820 f   hb-ot-layout.obj
 0001:0004f990       ?context_apply_lookup@OT@@YA_NPAUhb_ot_apply_context_t@1@IQBU?$IntType@G$01@1@IQBULookupRecord@1@AAUContextApplyLookupContext@1@@Z 10050990 f   hb-ot-layout.obj
 0001:000504f0       ?get_gsubgpos_table@@YAABUGSUBGPOS@OT@@PAUhb_face_t@@I@Z 100514f0 f   hb-ot-layout.obj
 0001:00052fa0       ?ligate_input@OT@@YA_NPAUhb_ot_apply_context_t@1@IQBIIII@Z 10053fa0 f   hb-ot-layout.obj
 0001:000532c0       ?match_backtrack@OT@@YA_NPAUhb_ot_apply_context_t@1@IQBU?$IntType@G$01@1@P6A_NAAUhb_glyph_info_t@@ABU31@PBX@Z4PAI@Z 100542c0 f   hb-ot-layout.obj
 0001:00053460       ?match_class@OT@@YA_NAAUhb_glyph_info_t@@ABU?$IntType@G$01@1@PBX@Z 10054460 f   hb-ot-layout.obj
 0001:00053490       ?match_class_cached@OT@@YA_NAAUhb_glyph_info_t@@ABU?$IntType@G$01@1@PBX@Z 10054490 f   hb-ot-layout.obj
 0001:000534f0       ?match_coverage@OT@@YA_NAAUhb_glyph_info_t@@ABU?$IntType@G$01@1@PBX@Z 100544f0 f   hb-ot-layout.obj
 0001:00053540       ?match_glyph@OT@@YA_NAAUhb_glyph_info_t@@ABU?$IntType@G$01@1@PBX@Z 10054540 f   hb-ot-layout.obj
 0001:00053560       ?match_input@OT@@YA_NPAUhb_ot_apply_context_t@1@IQBU?$IntType@G$01@1@P6A_NAAUhb_glyph_info_t@@ABU31@PBX@Z4PAIQAI6@Z 10054560 f   hb-ot-layout.obj
 0001:000538a0       ?match_lookahead@OT@@YA_NPAUhb_ot_apply_context_t@1@IQBU?$IntType@G$01@1@P6A_NAAUhb_glyph_info_t@@ABU31@PBX@Z4IPAI@Z 100548a0 f   hb-ot-layout.obj
 0001:00053be0       ?propagate_attachment_offsets@Layout@OT@@YAXPAUhb_glyph_position_t@@IIW4hb_direction_t@@I@Z 10054be0 f   hb-ot-layout.obj
 0001:00053d60       ?reverse_cursive_minor_offset@GPOS_impl@Layout@OT@@YAXPAUhb_glyph_position_t@@IW4hb_direction_t@@I@Z 10054d60 f   hb-ot-layout.obj
 0001:00053f14       $LN95                      10054f14     hb-ot-layout.obj
 0001:00055cd0       ?would_match_input@OT@@YA_NPAUhb_would_apply_context_t@1@IQBU?$IntType@G$01@1@P6A_NAAUhb_glyph_info_t@@ABU31@PBX@Z4@Z 10056cd0 f   hb-ot-layout.obj
 0001:00058180       ?_fix_ascender_descender@@YAMMW4hb_ot_metrics_tag_t@@@Z 10059180 f   hb-ot-metrics.obj
 0001:00058e10       $LN58                      10059e10     hb-ot-shape-fallback.obj
 0001:00058e20       $LN57                      10059e20     hb-ot-shape-fallback.obj
 0001:00058ec0       $LN60                      10059ec0     hb-ot-shape-fallback.obj
 0001:00058edc       $LN59                      10059edc     hb-ot-shape-fallback.obj
 0001:000591ac       $LN86                      1005a1ac     hb-ot-shape-fallback.obj
 0001:000591c4       $LN85                      1005a1c4     hb-ot-shape-fallback.obj
 0001:00059630       ?position_around_base@@YAXPBUhb_ot_shape_plan_t@@PAUhb_font_t@@PAUhb_buffer_t@@II_N@Z 1005a630 f   hb-ot-shape-fallback.obj
 0001:00059a10       ?position_cluster@@YAXPBUhb_ot_shape_plan_t@@PAUhb_font_t@@PAUhb_buffer_t@@II_N@Z 1005aa10 f   hb-ot-shape-fallback.obj
 0001:00059a90       ?position_mark@@YAXPBUhb_ot_shape_plan_t@@PAUhb_font_t@@PAUhb_buffer_t@@AAUhb_glyph_extents_t@@II@Z 1005aa90 f   hb-ot-shape-fallback.obj
 0001:00059c40       $LN36                      1005ac40     hb-ot-shape-fallback.obj
 0001:00059c50       $LN35                      1005ac50     hb-ot-shape-fallback.obj
 0001:00059c74       $LN38                      1005ac74     hb-ot-shape-fallback.obj
 0001:00059c88       $LN37                      1005ac88     hb-ot-shape-fallback.obj
 0001:00059cb0       ?_hb_glyph_info_set_unicode_props@@YAXPAUhb_glyph_info_t@@PAUhb_buffer_t@@@Z 1005acb0 f   hb-ot-shape-normalize.obj
 0001:00059cb0       ?_hb_glyph_info_set_unicode_props@@YAXPAUhb_glyph_info_t@@PAUhb_buffer_t@@@Z 1005acb0 f   hb-ot-shape.obj
 0001:00059f0c       $LN96                      1005af0c     hb-ot-shape-normalize.obj
 0001:00059f0c       $LN96                      1005af0c     hb-ot-shape.obj
 0001:00059f20       $LN95                      1005af20     hb-ot-shape-normalize.obj
 0001:00059f20       $LN95                      1005af20     hb-ot-shape.obj
 0001:0005a7b8       $LN371                     1005b7b8     hb-ot-shape-normalize.obj
 0001:0005a7e8       $LN370                     1005b7e8     hb-ot-shape-normalize.obj
 0001:0005a850       ?compare_combining_class@@YAHPBUhb_glyph_info_t@@0@Z 1005b850 f   hb-ot-shape-normalize.obj
 0001:0005a8a0       ?compose_unicode@@YA_NPBUhb_ot_shape_normalize_context_t@@IIPAI@Z 1005b8a0 f   hb-ot-shape-normalize.obj
 0001:0005a8e0       ?decompose@@YAIPBUhb_ot_shape_normalize_context_t@@_NI@Z 1005b8e0 f   hb-ot-shape-normalize.obj
 0001:0005aa30       ?decompose_current_character@@YAXPBUhb_ot_shape_normalize_context_t@@_N@Z 1005ba30 f   hb-ot-shape-normalize.obj
 0001:0005acb0       $LN97                      1005bcb0     hb-ot-shape-normalize.obj
 0001:0005ace0       $LN96                      1005bce0     hb-ot-shape-normalize.obj
 0001:0005ad40       ?decompose_unicode@@YA_NPBUhb_ot_shape_normalize_context_t@@IPAI1@Z 1005bd40 f   hb-ot-shape-normalize.obj
 0001:0005ad80       ?handle_variation_selector_cluster@@YAXPBUhb_ot_shape_normalize_context_t@@I_N@Z 1005bd80 f   hb-ot-shape-normalize.obj
 0001:0005b040       ?output_char@@YAXPAUhb_buffer_t@@II@Z 1005c040 f   hb-ot-shape-normalize.obj
 0001:0005b120       ?_hb_glyph_info_is_default_ignorable@@YA_NPBUhb_glyph_info_t@@@Z 1005c120 f   hb-ot-shape.obj
 0001:0005b140       ?_hb_grapheme_group_func@@YA_NABUhb_glyph_info_t@@0@Z 1005c140 f   hb-ot-shape.obj
 0001:0005b6a0       ?hb_form_clusters@@YAXPAUhb_buffer_t@@@Z 1005c6a0 f   hb-ot-shape.obj
 0001:0005b7e0       ?hb_ot_position@@YAXPBUhb_ot_shape_context_t@@@Z 1005c7e0 f   hb-ot-shape.obj
 0001:0005b930       ?hb_ot_position_plan@@YAXPBUhb_ot_shape_context_t@@@Z 1005c930 f   hb-ot-shape.obj
 0001:0005bb90       ?hb_ot_rotate_chars@@YAXPBUhb_ot_shape_context_t@@@Z 1005cb90 f   hb-ot-shape.obj
 0001:0005be54       $LN87                      1005ce54     hb-ot-shape.obj
 0001:0005be68       $LN86                      1005ce68     hb-ot-shape.obj
 0001:0005bf48       $LN89                      1005cf48     hb-ot-shape.obj
 0001:0005bf5c       $LN88                      1005cf5c     hb-ot-shape.obj
 0001:0005bf70       $LN90                      1005cf70     hb-ot-shape.obj
 0001:0005bfcc       $LN92                      1005cfcc     hb-ot-shape.obj
 0001:0005c000       $LN91                      1005d000     hb-ot-shape.obj
 0001:0005c060       ?hb_ot_shape_collect_features@@YAXPAUhb_ot_shape_planner_t@@PBUhb_feature_t@@I@Z 1005d060 f   hb-ot-shape.obj
 0001:0005c250       ?hb_ot_shape_internal@@YAXPAUhb_ot_shape_context_t@@@Z 1005d250 f   hb-ot-shape.obj
 0001:0005c6b0       ?hb_ot_shape_setup_masks_fraction@@YAXPBUhb_ot_shape_context_t@@@Z 1005d6b0 f   hb-ot-shape.obj
 0001:0005c870       ?hb_ot_shaper_categorize@@YAPBUhb_ot_shaper_t@@PBUhb_ot_shape_planner_t@@@Z 1005d870 f   hb-ot-shape.obj
 0001:0005cd40       ?hb_ot_substitute_pre@@YAXPBUhb_ot_shape_context_t@@@Z 1005dd40 f   hb-ot-shape.obj
 0001:0005cef0       ?hb_propagate_flags@@YAXPAUhb_buffer_t@@@Z 1005def0 f   hb-ot-shape.obj
 0001:0005d340       ?zero_mark_widths_by_gdef@@YAXPAUhb_buffer_t@@_N@Z 1005e340 f   hb-ot-shape.obj
 0001:0005d3f0       ?setup_masks_arabic@@YAXPBUhb_ot_shape_plan_t@@PAUhb_buffer_t@@PAUhb_font_t@@@Z 1005e3f0 f   hb-ot-shaper-arabic.obj
 0001:0005d480       ?postprocess_glyphs_arabic@@YAXPBUhb_ot_shape_plan_t@@PAUhb_buffer_t@@PAUhb_font_t@@@Z 1005e480 f   hb-ot-shaper-arabic.obj
 0001:0005d490       ?reorder_marks_arabic@@YAXPBUhb_ot_shape_plan_t@@PAUhb_buffer_t@@II@Z 1005e490 f   hb-ot-shaper-arabic.obj
 0001:0005d7c0       ?collect_features_arabic@@YAXPAUhb_ot_shape_planner_t@@@Z 1005e7c0 f   hb-ot-shaper-arabic.obj
 0001:0005d9b0       ??$arabic_fallback_synthesize_lookup_ligature@$$BY00Uligature_3_set_t@@@@YAPAUSubstLookup@GSUB@Layout@OT@@PBUhb_ot_shape_plan_t@@PAUhb_font_t@@AAY00$$CBUligature_3_set_t@@I@Z 1005e9b0 f   hb-ot-shaper-arabic.obj
 0001:0005dd40       ??$arabic_fallback_synthesize_lookup_ligature@$$BY00Uligature_mark_set_t@@@@YAPAUSubstLookup@GSUB@Layout@OT@@PBUhb_ot_shape_plan_t@@PAUhb_font_t@@AAY00$$CBUligature_mark_set_t@@I@Z 1005ed40 f   hb-ot-shaper-arabic.obj
 0001:0005e090       ??$arabic_fallback_synthesize_lookup_ligature@$$BY0BC@Uligature_set_t@@@@YAPAUSubstLookup@GSUB@Layout@OT@@PBUhb_ot_shape_plan_t@@PAUhb_font_t@@AAY0BC@$$CBUligature_set_t@@I@Z 1005f090 f   hb-ot-shaper-arabic.obj
 0001:0005e660       ??$hb_stable_sort@UHBGlyphID16@OT@@U?$IntType@G$01@2@I@@YAXPAUHBGlyphID16@OT@@IP6AHPBU?$IntType@G$01@1@1@ZPAI@Z 1005f660 f   hb-ot-shaper-arabic.obj
 0001:0005f660       ?apply_stch@@YAXPBUhb_ot_shape_plan_t@@PAUhb_buffer_t@@PAUhb_font_t@@@Z 10060660 f   hb-ot-shaper-arabic.obj
 0001:0005fa90       ?arabic_fallback_plan_destroy@@YAXPAUarabic_fallback_plan_t@@@Z 10060a90 f   hb-ot-shaper-arabic.obj
 0001:0005fb10       ?arabic_fallback_plan_init_win1256@@YA_NPAUarabic_fallback_plan_t@@PBUhb_ot_shape_plan_t@@PAUhb_font_t@@@Z 10060b10 f   hb-ot-shaper-arabic.obj
 0001:0005fd00       ?arabic_fallback_shape@@YAXPBUhb_ot_shape_plan_t@@PAUhb_font_t@@PAUhb_buffer_t@@@Z 10060d00 f   hb-ot-shaper-arabic.obj
 0001:0005ff20       ?arabic_fallback_synthesize_lookup_single@@YAPAUSubstLookup@GSUB@Layout@OT@@PBUhb_ot_shape_plan_t@@PAUhb_font_t@@I@Z 10060f20 f   hb-ot-shaper-arabic.obj
 0001:000602e0       ?arabic_joining@@YAXPAUhb_buffer_t@@@Z 100612e0 f   hb-ot-shaper-arabic.obj
 0001:000607f0       ?deallocate_buffer_var@@YAXPBUhb_ot_shape_plan_t@@PAUhb_font_t@@PAUhb_buffer_t@@@Z 100617f0 f   hb-ot-shaper-arabic.obj
 0001:00060a90       ?get_joining_type@@YAIIW4hb_unicode_general_category_t@@@Z 10061a90 f   hb-ot-shaper-arabic.obj
 0001:00060bb4       $LN49                      10061bb4     hb-ot-shaper-arabic.obj
 0001:00060bd4       $LN48                      10061bd4     hb-ot-shaper-arabic.obj
 0001:00060c80       ?record_stch@@YAXPBUhb_ot_shape_plan_t@@PAUhb_font_t@@PAUhb_buffer_t@@@Z 10061c80 f   hb-ot-shaper-arabic.obj
 0001:000616c0       ?collect_features_hangul@@YAXPAUhb_ot_shape_planner_t@@@Z 100626c0 f   hb-ot-shaper-hangul.obj
 0001:000616f0       ?override_features_hangul@@YAXPAUhb_ot_shape_planner_t@@@Z 100626f0 f   hb-ot-shaper-hangul.obj
 0001:00061710       ?data_create_hangul@@YAPAXPBUhb_ot_shape_plan_t@@@Z 10062710 f   hb-ot-shaper-hangul.obj
 0001:000617c0       ?data_destroy_hangul@@YAXPAX@Z 100627c0 f   hb-ot-shaper-hangul.obj
 0001:000617c0       ?data_destroy_indic@@YAXPAX@Z 100627c0 f   hb-ot-shaper-indic.obj
 0001:000617c0       ?data_destroy_khmer@@YAXPAX@Z 100627c0 f   hb-ot-shaper-khmer.obj
 0001:000617d0       ?preprocess_text_hangul@@YAXPBUhb_ot_shape_plan_t@@PAUhb_buffer_t@@PAUhb_font_t@@@Z 100627d0 f   hb-ot-shaper-hangul.obj
 0001:00062140       ?setup_masks_hangul@@YAXPBUhb_ot_shape_plan_t@@PAUhb_buffer_t@@PAUhb_font_t@@@Z 10063140 f   hb-ot-shaper-hangul.obj
 0001:00062190       ?compose_hebrew@@YA_NPBUhb_ot_shape_normalize_context_t@@IIPAI@Z 10063190 f   hb-ot-shaper-hebrew.obj
 0001:00062358       $LN42                      10063358     hb-ot-shaper-hebrew.obj
 0001:0006237c       $LN41                      1006337c     hb-ot-shaper-hebrew.obj
 0001:000624f4       $LN57                      100634f4     hb-ot-shaper-indic-table.obj
 0001:00062510       $LN56                      10063510     hb-ot-shaper-indic-table.obj
 0001:00062530       ?collect_features_indic@@YAXPAUhb_ot_shape_planner_t@@@Z 10063530 f   hb-ot-shaper-indic.obj
 0001:000625e0       ?override_features_indic@@YAXPAUhb_ot_shape_planner_t@@@Z 100635e0 f   hb-ot-shaper-indic.obj
 0001:00062610       ?data_create_indic@@YAPAXPBUhb_ot_shape_plan_t@@@Z 10063610 f   hb-ot-shaper-indic.obj
 0001:00062770       ?setup_masks_indic@@YAXPBUhb_ot_shape_plan_t@@PAUhb_buffer_t@@PAUhb_font_t@@@Z 10063770 f   hb-ot-shaper-indic.obj
 0001:000627c0       ?preprocess_text_indic@@YAXPBUhb_ot_shape_plan_t@@PAUhb_buffer_t@@PAUhb_font_t@@@Z 100637c0 f   hb-ot-shaper-indic.obj
 0001:000627e0       ?decompose_indic@@YA_NPBUhb_ot_shape_normalize_context_t@@IPAI1@Z 100637e0 f   hb-ot-shaper-indic.obj
 0001:00062840       ?compose_indic@@YA_NPBUhb_ot_shape_normalize_context_t@@IIPAI@Z 10063840 f   hb-ot-shaper-indic.obj
 0001:000628e0       ?_hb_next_syllable@@YAIPAUhb_buffer_t@@I@Z 100638e0 f   hb-ot-shaper-indic.obj
 0001:00062910       ?final_reordering_indic@@YAXPBUhb_ot_shape_plan_t@@PAUhb_font_t@@PAUhb_buffer_t@@@Z 10063910 f   hb-ot-shaper-indic.obj
 0001:000629b0       ?final_reordering_syllable_indic@@YAXPBUhb_ot_shape_plan_t@@PAUhb_buffer_t@@II@Z 100639b0 f   hb-ot-shaper-indic.obj
 0001:000639ec       $LN241                     100649ec     hb-ot-shaper-indic.obj
 0001:00063b00       ?initial_reordering_consonant_syllable@@YAXPBUhb_ot_shape_plan_t@@PAUhb_face_t@@PAUhb_buffer_t@@II@Z 10064b00 f   hb-ot-shaper-indic.obj
 0001:00064540       ?initial_reordering_indic@@YAXPBUhb_ot_shape_plan_t@@PAUhb_font_t@@PAUhb_buffer_t@@@Z 10065540 f   hb-ot-shaper-indic.obj
 0001:00064634       $LN38                      10065634     hb-ot-shaper-indic.obj
 0001:00064650       ?is_joiner@@YA_NABUhb_glyph_info_t@@@Z 10065650 f   hb-ot-shaper-indic.obj
 0001:00064680       ?is_one_of@@YA_NABUhb_glyph_info_t@@I@Z 10065680 f   hb-ot-shaper-indic.obj
 0001:000646c0       ?setup_syllables_indic@@YAXPBUhb_ot_shape_plan_t@@PAUhb_font_t@@PAUhb_buffer_t@@@Z 100656c0 f   hb-ot-shaper-indic.obj
 0001:000647d0       ?update_consonant_positions_indic@@YAXPBUhb_ot_shape_plan_t@@PAUhb_font_t@@PAUhb_buffer_t@@@Z 100657d0 f   hb-ot-shaper-indic.obj
 0001:000649c0       ?collect_features_khmer@@YAXPAUhb_ot_shape_planner_t@@@Z 100659c0 f   hb-ot-shaper-khmer.obj
 0001:00064a60       ?override_features_khmer@@YAXPAUhb_ot_shape_planner_t@@@Z 10065a60 f   hb-ot-shaper-khmer.obj
 0001:00064ac0       ?data_create_khmer@@YAPAXPBUhb_ot_shape_plan_t@@@Z 10065ac0 f   hb-ot-shaper-khmer.obj
 0001:00064b70       ?setup_masks_khmer@@YAXPBUhb_ot_shape_plan_t@@PAUhb_buffer_t@@PAUhb_font_t@@@Z 10065b70 f   hb-ot-shaper-khmer.obj
 0001:00064ba0       ?decompose_khmer@@YA_NPBUhb_ot_shape_normalize_context_t@@IPAI1@Z 10065ba0 f   hb-ot-shaper-khmer.obj
 0001:00064c5c       $LN12                      10065c5c     hb-ot-shaper-khmer.obj
 0001:00064c80       ?compose_khmer@@YA_NPBUhb_ot_shape_normalize_context_t@@IIPAI@Z 10065c80 f   hb-ot-shaper-khmer.obj
 0001:00064c80       ?compose_use@@YA_NPBUhb_ot_shape_normalize_context_t@@IIPAI@Z 10065c80 f   hb-ot-shaper-use.obj
 0001:00065060       $LN149                     10066060     hb-ot-shaper-khmer.obj
 0001:00065090       ?reorder_consonant_syllable@@YAXPBUhb_ot_shape_plan_t@@PAUhb_face_t@@PAUhb_buffer_t@@II@Z 10066090 f   hb-ot-shaper-khmer.obj
 0001:00065290       ?reorder_khmer@@YAXPBUhb_ot_shape_plan_t@@PAUhb_font_t@@PAUhb_buffer_t@@@Z 10066290 f   hb-ot-shaper-khmer.obj
 0001:00065370       ?setup_syllables_khmer@@YAXPBUhb_ot_shape_plan_t@@PAUhb_font_t@@PAUhb_buffer_t@@@Z 10066370 f   hb-ot-shaper-khmer.obj
 0001:00065480       ?collect_features_myanmar@@YAXPAUhb_ot_shape_planner_t@@@Z 10066480 f   hb-ot-shaper-myanmar.obj
 0001:00065520       ?setup_masks_myanmar@@YAXPBUhb_ot_shape_plan_t@@PAUhb_buffer_t@@PAUhb_font_t@@@Z 10066520 f   hb-ot-shaper-myanmar.obj
 0001:00065550       ?compare_myanmar_order@@YAHPBUhb_glyph_info_t@@0@Z 10066550 f   hb-ot-shaper-myanmar.obj
 0001:00065808       $LN125                     10066808     hb-ot-shaper-myanmar.obj
 0001:00065830       ?initial_reordering_consonant_syllable@@YAXPAUhb_buffer_t@@II@Z 10066830 f   hb-ot-shaper-myanmar.obj
 0001:000659a0       ?reorder_myanmar@@YAXPBUhb_ot_shape_plan_t@@PAUhb_font_t@@PAUhb_buffer_t@@@Z 100669a0 f   hb-ot-shaper-myanmar.obj
 0001:00065a70       ?setup_syllables_myanmar@@YAXPBUhb_ot_shape_plan_t@@PAUhb_font_t@@PAUhb_buffer_t@@@Z 10066a70 f   hb-ot-shaper-myanmar.obj
 0001:00065d90       ?preprocess_text_thai@@YAXPBUhb_ot_shape_plan_t@@PAUhb_buffer_t@@PAUhb_font_t@@@Z 10066d90 f   hb-ot-shaper-thai.obj
 0001:00066040       ?do_thai_pua_shaping@@YAXPBUhb_ot_shape_plan_t@@PAUhb_buffer_t@@PAUhb_font_t@@@Z 10067040 f   hb-ot-shaper-thai.obj
 0001:000662e0       ?thai_pua_shape@@YAIIW4thai_action_t@@PAUhb_font_t@@@Z 100672e0 f   hb-ot-shaper-thai.obj
 0001:00066384       $LN22                      10067384     hb-ot-shaper-thai.obj
 0001:000663a0       ?collect_features_use@@YAXPAUhb_ot_shape_planner_t@@@Z 100673a0 f   hb-ot-shaper-use.obj
 0001:000664e0       ?data_create_use@@YAPAXPBUhb_ot_shape_plan_t@@@Z 100674e0 f   hb-ot-shaper-use.obj
 0001:000665a0       ?data_destroy_use@@YAXPAX@Z 100675a0 f   hb-ot-shaper-use.obj
 0001:000665d0       ?setup_masks_use@@YAXPBUhb_ot_shape_plan_t@@PAUhb_buffer_t@@PAUhb_font_t@@@Z 100675d0 f   hb-ot-shaper-use.obj
 0001:00066630       ?preprocess_text_use@@YAXPBUhb_ot_shape_plan_t@@PAUhb_buffer_t@@PAUhb_font_t@@@Z 10067630 f   hb-ot-shaper-use.obj
 0001:00066f60       ?_hb_clear_substitution_flags@@YAXPBUhb_ot_shape_plan_t@@PAUhb_font_t@@PAUhb_buffer_t@@@Z 10067f60 f   hb-ot-shaper-use.obj
 0001:00066f90       ?find_syllables_use@@YAXPAUhb_buffer_t@@@Z 10067f90 f   hb-ot-shaper-use.obj
 0001:00068078       $LN2101                    10069078     hb-ot-shaper-use.obj
 0001:000680c0       ?hb_use_get_category@@YAEUhb_glyph_info_t@@@Z 100690c0 f   hb-ot-shaper-use.obj
 0001:00068538       $LN190                     10069538     hb-ot-shaper-use.obj
 0001:00068574       $LN189                     10069574     hb-ot-shaper-use.obj
 0001:00068660       ?record_pref_use@@YAXPBUhb_ot_shape_plan_t@@PAUhb_font_t@@PAUhb_buffer_t@@@Z 10069660 f   hb-ot-shaper-use.obj
 0001:000686f0       ?record_rphf_use@@YAXPBUhb_ot_shape_plan_t@@PAUhb_font_t@@PAUhb_buffer_t@@@Z 100696f0 f   hb-ot-shaper-use.obj
 0001:000687a0       ?reorder_syllable_use@@YAXPAUhb_buffer_t@@II@Z 100697a0 f   hb-ot-shaper-use.obj
 0001:000689d0       ?reorder_use@@YAXPBUhb_ot_shape_plan_t@@PAUhb_font_t@@PAUhb_buffer_t@@@Z 100699d0 f   hb-ot-shaper-use.obj
 0001:00068a80       ?setup_syllables_use@@YAXPBUhb_ot_shape_plan_t@@PAUhb_font_t@@PAUhb_buffer_t@@@Z 10069a80 f   hb-ot-shaper-use.obj
 0001:00068c40       ?setup_topographical_masks@@YAXPBUhb_ot_shape_plan_t@@PAUhb_buffer_t@@@Z 10069c40 f   hb-ot-shaper-use.obj
 0001:00068e60       $LN111                     10069e60     hb-ot-shaper-use.obj
 0001:00068e68       $LN110                     10069e68     hb-ot-shaper-use.obj
 0001:00069798       $LN360                     1006a798     hb-ot-shaper-vowel-constraints.obj
 0001:000697b0       $LN359                     1006a7b0     hb-ot-shaper-vowel-constraints.obj
 0001:000697dc       $LN362                     1006a7dc     hb-ot-shaper-vowel-constraints.obj
 0001:000697e4       $LN361                     1006a7e4     hb-ot-shaper-vowel-constraints.obj
 0001:00069804       $LN364                     1006a804     hb-ot-shaper-vowel-constraints.obj
 0001:0006980c       $LN363                     1006a80c     hb-ot-shaper-vowel-constraints.obj
 0001:0006981c       $LN366                     1006a81c     hb-ot-shaper-vowel-constraints.obj
 0001:0006982c       $LN365                     1006a82c     hb-ot-shaper-vowel-constraints.obj
 0001:00069838       $LN368                     1006a838     hb-ot-shaper-vowel-constraints.obj
 0001:0006984c       $LN367                     1006a84c     hb-ot-shaper-vowel-constraints.obj
 0001:0006985c       $LN370                     1006a85c     hb-ot-shaper-vowel-constraints.obj
 0001:00069864       $LN369                     1006a864     hb-ot-shaper-vowel-constraints.obj
 0001:0006987c       $LN372                     1006a87c     hb-ot-shaper-vowel-constraints.obj
 0001:0006988c       $LN371                     1006a88c     hb-ot-shaper-vowel-constraints.obj
 0001:000698b8       $LN374                     1006a8b8     hb-ot-shaper-vowel-constraints.obj
 0001:000698c4       $LN373                     1006a8c4     hb-ot-shaper-vowel-constraints.obj
 0001:00069900       ?_output_with_dotted_circle@@YAXPAUhb_buffer_t@@@Z 1006a900 f   hb-ot-shaper-vowel-constraints.obj
 0001:00069990       ?TOLOWER@@YAEE@Z           1006a990 f   hb-ot-tag.obj
 0001:000699b0       ?hb_ot_ambiguous_tag_to_language@@YAPBUhb_language_impl_t@@I@Z 1006a9b0 f   hb-ot-tag.obj
 0001:0006a1c0       ?hb_ot_tags_from_complex_language@@YA_NPBD0PAI1@Z 1006b1c0 f   hb-ot-tag.obj
 0001:0006bc5c       $LN376                     1006cc5c     hb-ot-tag.obj
 0001:0006bc90       $LN375                     1006cc90     hb-ot-tag.obj
 0001:0006bcb0       ?hb_ot_tags_from_language@@YAXPBD0PAI1@Z 1006ccb0 f   hb-ot-tag.obj
 0001:0006be90       ?lang_matches@@YA_NPBD00I@Z 1006ce90 f   hb-ot-tag.obj
 0001:0006bed0       ?parse_private_use_subtag@@YA_NPBDPAI10P6AEE@Z@Z 1006ced0 f   hb-ot-tag.obj
 0001:0006c040       ?subtag_matches@@YA_NPBD00I@Z 1006d040 f   hb-ot-tag.obj
 0001:0006c820       ?_hb_shape_plan_execute_internal@@YA_NPAUhb_shape_plan_t@@PAUhb_font_t@@PAUhb_buffer_t@@PBUhb_feature_t@@I@Z 1006d820 f   hb-shape-plan.obj
 0001:0006d330       ?hb_ucd_combining_class@@YA?AW4hb_unicode_combining_class_t@@PAUhb_unicode_funcs_t@@IPAX@Z 1006e330 f   hb-ucd.obj
 0001:0006d370       ?hb_ucd_compose@@YAHPAUhb_unicode_funcs_t@@IIPAIPAX@Z 1006e370 f   hb-ucd.obj
 0001:0006d500       ?hb_ucd_decompose@@YAHPAUhb_unicode_funcs_t@@IPAI1PAX@Z 1006e500 f   hb-ucd.obj
 0001:0006d680       ?hb_ucd_general_category@@YA?AW4hb_unicode_general_category_t@@PAUhb_unicode_funcs_t@@IPAX@Z 1006e680 f   hb-ucd.obj
 0001:0006d6d0       ?hb_ucd_mirroring@@YAIPAUhb_unicode_funcs_t@@IPAX@Z 1006e6d0 f   hb-ucd.obj
 0001:0006d730       ?hb_ucd_script@@YA?AW4hb_script_t@@PAUhb_unicode_funcs_t@@IPAX@Z 1006e730 f   hb-ucd.obj
 0001:0006d860       ?hb_unicode_general_category_nil@@YA?AW4hb_unicode_general_category_t@@PAUhb_unicode_funcs_t@@IPAX@Z 1006e860 f   hb-unicode.obj
 0001:0006d870       ?hb_unicode_mirroring_nil@@YAIPAUhb_unicode_funcs_t@@IPAX@Z 1006e870 f   hb-unicode.obj
 0001:0006d880       ?hb_unicode_script_nil@@YA?AW4hb_script_t@@PAUhb_unicode_funcs_t@@IPAX@Z 1006e880 f   hb-unicode.obj
 0001:0006e940       _initFontIDs               1006f940 f   sunFont.obj
 0001:0006f020       $$000000                   10070020     MSVCRT:ftol3.obj
 0001:0006f3c0       $$000000                   100703c0     MSVCRT:llmul.obj
 0001:0006f5f0       $$000000                   100705f0     MSVCRT:lldiv.obj
 0001:0006f6a0       $$000000                   100706a0     MSVCRT:chkstk.obj
 0001:0006f6d0       $$000000                   100706d0     MSVCRT:ftol2.obj
 0001:0006f970       $$000000                   10070970     MSVCRT:alloca16.obj
 0001:0006f99c       ?dllmain_crt_dispatch@@YGHQAUHINSTANCE__@@KQAX@Z 1007099c f   MSVCRT:dll_dllmain.obj
 0001:0006f9ef       ?dllmain_crt_process_attach@@YAHQAUHINSTANCE__@@QAX@Z 100709ef f   MSVCRT:dll_dllmain.obj
 0001:0006faf6       ?dllmain_crt_process_detach@@YAH_N@Z 10070af6 f   MSVCRT:dll_dllmain.obj
 0001:0006fba6       ?dllmain_dispatch@@YAHQAUHINSTANCE__@@KQAX@Z 10070ba6 f   MSVCRT:dll_dllmain.obj
 0001:0006fcb1       ?dllmain_raw@@YGHQAUHINSTANCE__@@KQAX@Z 10070cb1 f   MSVCRT:dll_dllmain.obj
 0001:0006fecf       ___get_entropy             10070ecf f   MSVCRT:gs_support.obj
 0001:0006ffc4       ?find_pe_section@@YAPAU_IMAGE_SECTION_HEADER@@QAEI@Z 10070fc4 f   MSVCRT:utility.obj
 0001:00070420       $$000000                   10071420     MSVCRT:sehprolg4.obj
 0002:00000360       _FONTKEY_NT                10072360     fontpath.obj
 0002:00000394       ?TTSUFFIX@?1??RegistryToBaseTTNameW@@9@9 10072394     fontpath.obj
 0002:000003ac       ?OTSUFFIX@?1??RegistryToBaseTTNameW@@9@9 100723ac     fontpath.obj
 0002:000004ec       ?outline_funcs@?1??addToGP@@9@9 100724ec     freetypeScaler.obj
 0002:000005b0       ?feature_mappings@@3QBUhb_aat_feature_mapping_t@@B 100725b0     hb-aat-layout.obj
 0002:00000a80       ?table_tags@@3QBIB         10072a80     hb-aat-layout.obj
 0002:00000c40       ?table_tags@@3QBIB         10072c40     hb-aat-map.obj
 0002:00000cc8       ?_deserialize_json_trans_keys@@3QBEB 10072cc8     hb-buffer-serialize.obj
 0002:00000d34       ?_deserialize_json_key_spans@@3QBDB 10072d34     hb-buffer-serialize.obj
 0002:00000d68       ?_deserialize_json_index_offsets@@3QBFB 10072d68     hb-buffer-serialize.obj
 0002:00000dd0       ?_deserialize_json_indicies@@3QBDB 10072dd0     hb-buffer-serialize.obj
 0002:000019a8       ?_deserialize_json_trans_targs@@3QBDB 100739a8     hb-buffer-serialize.obj
 0002:00001a00       ?_deserialize_json_trans_actions@@3QBDB 10073a00     hb-buffer-serialize.obj
 0002:00001a58       ?_deserialize_text_trans_keys@@3QBEB 10073a58     hb-buffer-serialize.obj
 0002:00001aa4       ?_deserialize_text_key_spans@@3QBDB 10073aa4     hb-buffer-serialize.obj
 0002:00001ad0       ?_deserialize_text_index_offsets@@3QBFB 10073ad0     hb-buffer-serialize.obj
 0002:00001b20       ?_deserialize_text_indicies@@3QBDB 10073b20     hb-buffer-serialize.obj
 0002:00002480       ?_deserialize_text_trans_targs@@3QBDB 10074480     hb-buffer-serialize.obj
 0002:000024d0       ?_deserialize_text_trans_actions@@3QBDB 100744d0     hb-buffer-serialize.obj
 0002:00002520       ?_deserialize_text_eof_actions@@3QBDB 10074520     hb-buffer-serialize.obj
 0002:00002674       ?table_tags@@3QBIB         10074674     hb-buffer.obj
 0002:00002680       ?direction_strings@@3QAY03$$CBDA 10074680     hb-common.obj
 0002:00002690       ?canon_map@@3QBDB          10074690     hb-common.obj
 0002:000027a0       ?table_tags@@3QBIB         100747a0     hb-common.obj
 0002:000027b0       ?_hb_ms_language_map@@3QBUhb_ot_language_map_t@@B 100747b0     hb-common.obj
 0002:00002f30       ?_hb_mac_language_map@@3QBUhb_ot_language_map_t@@B 10074f30     hb-common.obj
 0002:000032f0       ?_hb_os2_unicode_ranges@OT@@3QBUOS2Range@1@B 100752f0     hb-common.obj
 0002:00003ae0       ?_hb_arabic_u8@@3QBEB      10075ae0     hb-common.obj
 0002:00003cb0       ?_hb_arabic_u16@@3QBGB     10075cb0     hb-common.obj
 0002:00004440       ?table_tags@@3QBIB         10076440     hb-face.obj
 0002:00004448       ?_hb_os2_unicode_ranges@OT@@3QBUOS2Range@1@B 10076448     hb-face.obj
 0002:00004c38       ?_hb_arabic_u8@@3QBEB      10076c38     hb-face.obj
 0002:00004e08       ?_hb_arabic_u16@@3QBGB     10076e08     hb-face.obj
 0002:000053a8       ?hb_identity@@3U<unnamed-type-hb_identity>@@B 100773a8     hb-face.obj
 0002:000053a9       ?hb_ridentity@@3U<unnamed-type-hb_ridentity>@@B 100773a9     hb-face.obj
 0002:000053aa       ?hb_hash@@3U<unnamed-type-hb_hash>@@B 100773aa     hb-face.obj
 0002:000053fc       ?table_tags@@3QBIB         100773fc     hb-fallback-shape.obj
 0002:00005404       ?table_tags@@3QBIB         10077404     hb-font.obj
 0002:00005434       ?hb_identity@@3U<unnamed-type-hb_identity>@@B 10077434     hb-map.obj
 0002:00005438       ?_double_parser_trans_keys@@3QBEB 10077438     hb-number.obj
 0002:0000544c       ?_double_parser_key_spans@@3QBDB 1007744c     hb-number.obj
 0002:00005458       ?_double_parser_index_offsets@@3QBEB 10077458     hb-number.obj
 0002:00005468       ?_double_parser_indicies@@3QBDB 10077468     hb-number.obj
 0002:00005528       ?_double_parser_trans_targs@@3QBDB 10077528     hb-number.obj
 0002:00005534       ?_double_parser_trans_actions@@3QBDB 10077534     hb-number.obj
 0002:00005540       ?_powers_of_10@?1??_pow10@@YANI@Z@4QBNB 10077540     hb-number.obj
 0002:000055c0       ?standard_encoding_to_code@@3QBEB 100775c0     hb-ot-cff1-table.obj
 0002:00005658       ?expert_encoding_to_code@@3QBEB 10077658     hb-ot-cff1-table.obj
 0002:000057d8       ?expert_charset_to_sid@@3QBGB 100777d8     hb-ot-cff1-table.obj
 0002:00005928       ?expert_subset_charset_to_sid@@3QBGB 10077928     hb-ot-cff1-table.obj
 0002:000059d8       ?expert_charset_sid_to_gid@@3QBUsid_to_gid_t@@B 100779d8     hb-ot-cff1-table.obj
 0002:00005c70       ?expert_subset_charset_sid_to_gid@@3QBUsid_to_gid_t@@B 10077c70     hb-ot-cff1-table.obj
 0002:00005dc8       ?standard_encoding_to_sid@@3QBEB 10077dc8     hb-ot-cff1-table.obj
 0002:00005ec8       ?table_tags@@3QBIB         10077ec8     hb-ot-cff1-table.obj
 0002:00005ed0       ?cff1_std_strings_msgstr@@3Tcff1_std_strings_msgstr_t@@B 10077ed0     hb-ot-cff1-table.obj
 0002:00006c48       ?cff1_std_strings_msgidx@@3QBIB 10078c48     hb-ot-cff1-table.obj
 0002:000072a0       ?table_tags@@3QBIB         100792a0     hb-ot-cff2-table.obj
 0002:000072ac       ?table_tags@@3QBIB         100792ac     hb-ot-color.obj
 0002:000072b8       ?_hb_os2_unicode_ranges@OT@@3QBUOS2Range@1@B 100792b8     hb-ot-face.obj
 0002:00007aa8       ?_hb_arabic_u8@@3QBEB      10079aa8     hb-ot-face.obj
 0002:00007c78       ?_hb_arabic_u16@@3QBGB     10079c78     hb-ot-face.obj
 0002:00008218       ?format1_names_msgstr@@3Tformat1_names_msgstr_t@@B 1007a218     hb-ot-face.obj
 0002:00008958       ?format1_names_msgidx@@3QBIB 1007a958     hb-ot-face.obj
 0002:00008d64       ?table_tags@@3QBIB         1007ad64     hb-ot-face.obj
 0002:00008d70       ?cff1_std_strings_msgstr@@3Tcff1_std_strings_msgstr_t@@B 1007ad70     hb-ot-face.obj
 0002:00009ae8       ?cff1_std_strings_msgidx@@3QBIB 1007bae8     hb-ot-face.obj
 0002:0000a108       ?format1_names_msgstr@@3Tformat1_names_msgstr_t@@B 1007c108     hb-ot-font.obj
 0002:0000a848       ?format1_names_msgidx@@3QBIB 1007c848     hb-ot-font.obj
 0002:0000ac54       ?table_tags@@3QBIB         1007cc54     hb-ot-font.obj
 0002:0000ac60       ?_hb_os2_unicode_ranges@OT@@3QBUOS2Range@1@B 1007cc60     hb-ot-font.obj
 0002:0000b450       ?_hb_arabic_u8@@3QBEB      1007d450     hb-ot-font.obj
 0002:0000b620       ?_hb_arabic_u16@@3QBGB     1007d620     hb-ot-font.obj
 0002:0000bbc0       ?cff1_std_strings_msgstr@@3Tcff1_std_strings_msgstr_t@@B 1007dbc0     hb-ot-font.obj
 0002:0000c938       ?cff1_std_strings_msgidx@@3QBIB 1007e938     hb-ot-font.obj
 0002:0000cfa0       ?table_tags@@3QBIB         1007efa0     hb-ot-layout.obj
 0002:0000cfa8       ?_hb_os2_unicode_ranges@OT@@3QBUOS2Range@1@B 1007efa8     hb-ot-layout.obj
 0002:0000d794       ?hb_identity@@3U<unnamed-type-hb_identity>@@B 1007f794     hb-ot-layout.obj
 0002:0000d795       ?hb_first@@3U<unnamed-type-hb_first>@@B 1007f795     hb-ot-layout.obj
 0002:0000d796       ?hb_second@@3U<unnamed-type-hb_second>@@B 1007f796     hb-ot-layout.obj
 0002:0000d797       ?hb_bitwise_and@@3U<unnamed-type-hb_bitwise_and>@@B 1007f797     hb-ot-layout.obj
 0002:0000d798       ?hb_bitwise_or@@3U<unnamed-type-hb_bitwise_or>@@B 1007f798     hb-ot-layout.obj
 0002:0000d799       ?hb_bitwise_lt@@3U<unnamed-type-hb_bitwise_lt>@@B 1007f799     hb-ot-layout.obj
 0002:0000d79a       ?hb_bitwise_gt@@3U<unnamed-type-hb_bitwise_gt>@@B 1007f79a     hb-ot-layout.obj
 0002:0000d79b       ?hb_add@@3U<unnamed-type-hb_add>@@B 1007f79b     hb-ot-layout.obj
 0002:0000d79c       ?hb_zip@@3U<unnamed-type-hb_zip>@@B 1007f79c     hb-ot-layout.obj
 0002:0000d82c       ?table_tags@@3QBIB         1007f82c     hb-ot-map.obj
 0002:0000d834       ?table_tags@@3QBIB         1007f834     hb-ot-math.obj
 0002:0000d83c       ?table_tags@@3QBIB         1007f83c     hb-ot-meta.obj
 0002:0000d848       ?_hb_os2_unicode_ranges@OT@@3QBUOS2Range@1@B 1007f848     hb-ot-metrics.obj
 0002:0000e034       ?table_tags@@3QBIB         10080034     hb-ot-metrics.obj
 0002:0000e040       ?format1_names_msgstr@@3Tformat1_names_msgstr_t@@B 10080040     hb-ot-metrics.obj
 0002:0000e780       ?format1_names_msgidx@@3QBIB 10080780     hb-ot-metrics.obj
 0002:0000eba0       ?table_tags@@3QBIB         10080ba0     hb-ot-name.obj
 0002:0000eba8       ?table_tags@@3QBIB         10080ba8     hb-ot-shape-fallback.obj
 0002:0000ec00       ?table_tags@@3QBIB         10080c00     hb-ot-shape-normalize.obj
 0002:0000ec24       ?table_tags@@3QBIB         10080c24     hb-ot-shape.obj
 0002:0000ec2c       ?common_features@@3QBUhb_ot_map_feature_t@@B 10080c2c     hb-ot-shape.obj
 0002:0000ec64       ?horizontal_features@@3QBUhb_ot_map_feature_t@@B 10080c64     hb-ot-shape.obj
 0002:0000ed10       ?table_tags@@3QBIB         10080d10     hb-ot-shaper-arabic.obj
 0002:0000ed50       ?joining_table@@3QBEB      10080d50     hb-ot-shaper-arabic.obj
 0002:0000f2e8       ?shaping_table@@3QAY03$$CBGA 100812e8     hb-ot-shaper-arabic.obj
 0002:0000f880       ?ligature_table@@3QBUligature_set_t@@B 10081880     hb-ot-shaper-arabic.obj
 0002:0000fc94       ?ligature_mark_table@@3QBUligature_mark_set_t@@B 10081c94     hb-ot-shaper-arabic.obj
 0002:0000fcac       ?ligature_3_table@@3QBUligature_3_set_t@@B 10081cac     hb-ot-shaper-arabic.obj
 0002:0000fcc0       ?arabic_features@@3QBIB    10081cc0     hb-ot-shaper-arabic.obj
 0002:0000fce0       ?arabic_state_table@@3QAY05$$CBUarabic_state_table_entry@@A 10081ce0     hb-ot-shaper-arabic.obj
 0002:0000fd88       ?arabic_fallback_features@@3QBIB 10081d88     hb-ot-shaper-arabic.obj
 0002:0000fda8       ?arabic_win1256_gsub_lookups@@3U0@B 10081da8     hb-ot-shaper-arabic.obj
 0002:0000ff3a       ?hb_hash@@3U<unnamed-type-hb_hash>@@B 10081f3a     hb-ot-shaper-arabic.obj
 0002:0000ff3b       ?hb_first@@3U<unnamed-type-hb_first>@@B 10081f3b     hb-ot-shaper-arabic.obj
 0002:0000ff3c       ?hb_second@@3U<unnamed-type-hb_second>@@B 10081f3c     hb-ot-shaper-arabic.obj
 0002:0000ff3d       ?hb_add@@3U<unnamed-type-hb_add>@@B 10081f3d     hb-ot-shaper-arabic.obj
 0002:0000ff78       ?table_tags@@3QBIB         10081f78     hb-ot-shaper-default.obj
 0002:0000fff0       ?table_tags@@3QBIB         10081ff0     hb-ot-shaper-hangul.obj
 0002:00010030       ?hangul_features@@3QBIB    10082030     hb-ot-shaper-hangul.obj
 0002:00010040       ?table_tags@@3QBIB         10082040     hb-ot-shaper-hebrew.obj
 0002:00010080       ?sDageshForms@?1??compose_hebrew@@YA_NPBUhb_ot_shape_normalize_context_t@@IIPAI@Z@4QBIB 10082080     hb-ot-shaper-hebrew.obj
 0002:000100f0       ?table_tags@@3QBIB         100820f0     hb-ot-shaper-indic-table.obj
 0002:000100f8       ?_indic_syllable_machine_trans_keys@@3QBEB 100820f8     hb-ot-shaper-indic-table.obj
 0002:00010200       ?_indic_syllable_machine_key_spans@@3QBDB 10082200     hb-ot-shaper-indic-table.obj
 0002:00010288       ?_indic_syllable_machine_index_offsets@@3QBFB 10082288     hb-ot-shaper-indic-table.obj
 0002:00010390       ?_indic_syllable_machine_indicies@@3QBEB 10082390     hb-ot-shaper-indic-table.obj
 0002:00010848       ?_indic_syllable_machine_trans_targs@@3QBEB 10082848     hb-ot-shaper-indic-table.obj
 0002:000108d8       ?_indic_syllable_machine_trans_actions@@3QBDB 100828d8     hb-ot-shaper-indic-table.obj
 0002:00010968       ?_indic_syllable_machine_to_state_actions@@3QBDB 10082968     hb-ot-shaper-indic-table.obj
 0002:000109f0       ?_indic_syllable_machine_from_state_actions@@3QBDB 100829f0     hb-ot-shaper-indic-table.obj
 0002:00010a78       ?_indic_syllable_machine_eof_trans@@3QBFB 10082a78     hb-ot-shaper-indic-table.obj
 0002:00010b80       ?_khmer_syllable_machine_trans_keys@@3QBEB 10082b80     hb-ot-shaper-indic-table.obj
 0002:00010bd8       ?_khmer_syllable_machine_key_spans@@3QBDB 10082bd8     hb-ot-shaper-indic-table.obj
 0002:00010c08       ?_khmer_syllable_machine_index_offsets@@3QBFB 10082c08     hb-ot-shaper-indic-table.obj
 0002:00010c60       ?_khmer_syllable_machine_indicies@@3QBDB 10082c60     hb-ot-shaper-indic-table.obj
 0002:00011020       ?_khmer_syllable_machine_trans_targs@@3QBDB 10083020     hb-ot-shaper-indic-table.obj
 0002:00011054       ?_khmer_syllable_machine_trans_actions@@3QBDB 10083054     hb-ot-shaper-indic-table.obj
 0002:00011088       ?_khmer_syllable_machine_to_state_actions@@3QBDB 10083088     hb-ot-shaper-indic-table.obj
 0002:000110b4       ?_khmer_syllable_machine_from_state_actions@@3QBDB 100830b4     hb-ot-shaper-indic-table.obj
 0002:000110e0       ?_khmer_syllable_machine_eof_trans@@3QBFB 100830e0     hb-ot-shaper-indic-table.obj
 0002:00011138       ?_myanmar_syllable_machine_trans_keys@@3QBEB 10083138     hb-ot-shaper-indic-table.obj
 0002:000111a8       ?_myanmar_syllable_machine_key_spans@@3QBDB 100831a8     hb-ot-shaper-indic-table.obj
 0002:000111e0       ?_myanmar_syllable_machine_index_offsets@@3QBFB 100831e0     hb-ot-shaper-indic-table.obj
 0002:00011250       ?_myanmar_syllable_machine_indicies@@3QBDB 10083250     hb-ot-shaper-indic-table.obj
 0002:00011a20       ?_myanmar_syllable_machine_trans_targs@@3QBDB 10083a20     hb-ot-shaper-indic-table.obj
 0002:00011a60       ?_myanmar_syllable_machine_trans_actions@@3QBDB 10083a60     hb-ot-shaper-indic-table.obj
 0002:00011aa0       ?_myanmar_syllable_machine_to_state_actions@@3QBDB 10083aa0     hb-ot-shaper-indic-table.obj
 0002:00011ad8       ?_myanmar_syllable_machine_from_state_actions@@3QBDB 10083ad8     hb-ot-shaper-indic-table.obj
 0002:00011b10       ?_myanmar_syllable_machine_eof_trans@@3QBFB 10083b10     hb-ot-shaper-indic-table.obj
 0002:00011b80       ?indic_table@@3QBGB        10083b80     hb-ot-shaper-indic-table.obj
 0002:00012960       ?table_tags@@3QBIB         10084960     hb-ot-shaper-indic.obj
 0002:000129a0       ?_indic_syllable_machine_trans_keys@@3QBEB 100849a0     hb-ot-shaper-indic.obj
 0002:00012aa8       ?_indic_syllable_machine_key_spans@@3QBDB 10084aa8     hb-ot-shaper-indic.obj
 0002:00012b30       ?_indic_syllable_machine_index_offsets@@3QBFB 10084b30     hb-ot-shaper-indic.obj
 0002:00012c38       ?_indic_syllable_machine_indicies@@3QBEB 10084c38     hb-ot-shaper-indic.obj
 0002:000130f0       ?_indic_syllable_machine_trans_targs@@3QBEB 100850f0     hb-ot-shaper-indic.obj
 0002:00013180       ?_indic_syllable_machine_trans_actions@@3QBDB 10085180     hb-ot-shaper-indic.obj
 0002:00013210       ?_indic_syllable_machine_to_state_actions@@3QBDB 10085210     hb-ot-shaper-indic.obj
 0002:00013298       ?_indic_syllable_machine_from_state_actions@@3QBDB 10085298     hb-ot-shaper-indic.obj
 0002:00013320       ?_indic_syllable_machine_eof_trans@@3QBFB 10085320     hb-ot-shaper-indic.obj
 0002:00013428       ?indic_configs@@3QBUindic_config_t@@B 10085428     hb-ot-shaper-indic.obj
 0002:00013518       ?indic_features@@3QBUhb_ot_map_feature_t@@B 10085518     hb-ot-shaper-indic.obj
 0002:00013620       ?table_tags@@3QBIB         10085620     hb-ot-shaper-khmer.obj
 0002:00013660       ?_khmer_syllable_machine_trans_keys@@3QBEB 10085660     hb-ot-shaper-khmer.obj
 0002:000136b8       ?_khmer_syllable_machine_key_spans@@3QBDB 100856b8     hb-ot-shaper-khmer.obj
 0002:000136e8       ?_khmer_syllable_machine_index_offsets@@3QBFB 100856e8     hb-ot-shaper-khmer.obj
 0002:00013740       ?_khmer_syllable_machine_indicies@@3QBDB 10085740     hb-ot-shaper-khmer.obj
 0002:00013b00       ?_khmer_syllable_machine_trans_targs@@3QBDB 10085b00     hb-ot-shaper-khmer.obj
 0002:00013b34       ?_khmer_syllable_machine_trans_actions@@3QBDB 10085b34     hb-ot-shaper-khmer.obj
 0002:00013b68       ?_khmer_syllable_machine_to_state_actions@@3QBDB 10085b68     hb-ot-shaper-khmer.obj
 0002:00013b94       ?_khmer_syllable_machine_from_state_actions@@3QBDB 10085b94     hb-ot-shaper-khmer.obj
 0002:00013bc0       ?_khmer_syllable_machine_eof_trans@@3QBFB 10085bc0     hb-ot-shaper-khmer.obj
 0002:00013c18       ?khmer_features@@3QBUhb_ot_map_feature_t@@B 10085c18     hb-ot-shaper-khmer.obj
 0002:00013c90       ?table_tags@@3QBIB         10085c90     hb-ot-shaper-myanmar.obj
 0002:00013d08       ?_myanmar_syllable_machine_trans_keys@@3QBEB 10085d08     hb-ot-shaper-myanmar.obj
 0002:00013d78       ?_myanmar_syllable_machine_key_spans@@3QBDB 10085d78     hb-ot-shaper-myanmar.obj
 0002:00013db0       ?_myanmar_syllable_machine_index_offsets@@3QBFB 10085db0     hb-ot-shaper-myanmar.obj
 0002:00013e20       ?_myanmar_syllable_machine_indicies@@3QBDB 10085e20     hb-ot-shaper-myanmar.obj
 0002:000145f0       ?_myanmar_syllable_machine_trans_targs@@3QBDB 100865f0     hb-ot-shaper-myanmar.obj
 0002:00014630       ?_myanmar_syllable_machine_trans_actions@@3QBDB 10086630     hb-ot-shaper-myanmar.obj
 0002:00014670       ?_myanmar_syllable_machine_to_state_actions@@3QBDB 10086670     hb-ot-shaper-myanmar.obj
 0002:000146a8       ?_myanmar_syllable_machine_from_state_actions@@3QBDB 100866a8     hb-ot-shaper-myanmar.obj
 0002:000146e0       ?_myanmar_syllable_machine_eof_trans@@3QBFB 100866e0     hb-ot-shaper-myanmar.obj
 0002:00014750       ?myanmar_basic_features@@3QBIB 10086750     hb-ot-shaper-myanmar.obj
 0002:00014760       ?myanmar_other_features@@3QBIB 10086760     hb-ot-shaper-myanmar.obj
 0002:000147a4       ?table_tags@@3QBIB         100867a4     hb-ot-shaper-syllabic.obj
 0002:000147b0       ?table_tags@@3QBIB         100867b0     hb-ot-shaper-thai.obj
 0002:000147f0       ?thai_above_state_machine@@3QAY02$$CBUthai_above_state_machine_edge_t@@A 100867f0     hb-ot-shaper-thai.obj
 0002:00014850       ?thai_below_state_machine@@3QAY02$$CBUthai_below_state_machine_edge_t@@A 10086850     hb-ot-shaper-thai.obj
 0002:00014898       ?SD_mappings@?1??thai_pua_shape@@YAIIW4thai_action_t@@PAUhb_font_t@@@Z@4QBUthai_pua_mapping_t@?1??1@YAII01@Z@B 10086898     hb-ot-shaper-thai.obj
 0002:00014908       ?SDL_mappings@?1??thai_pua_shape@@YAIIW4thai_action_t@@PAUhb_font_t@@@Z@4QBUthai_pua_mapping_t@?1??1@YAII01@Z@B 10086908     hb-ot-shaper-thai.obj
 0002:00014950       ?SL_mappings@?1??thai_pua_shape@@YAIIW4thai_action_t@@PAUhb_font_t@@@Z@4QBUthai_pua_mapping_t@?1??1@YAII01@Z@B 10086950     hb-ot-shaper-thai.obj
 0002:000149ec       ?RD_mappings@?1??thai_pua_shape@@YAIIW4thai_action_t@@PAUhb_font_t@@@Z@4QBUthai_pua_mapping_t@?1??1@YAII01@Z@B 100869ec     hb-ot-shaper-thai.obj
 0002:00014a10       ?table_tags@@3QBIB         10086a10     hb-ot-shaper-use.obj
 0002:00014a50       ?_use_syllable_machine_trans_keys@@3QBEB 10086a50     hb-ot-shaper-use.obj
 0002:00014b48       ?_use_syllable_machine_key_spans@@3QBDB 10086b48     hb-ot-shaper-use.obj
 0002:00014bc0       ?_use_syllable_machine_index_offsets@@3QBFB 10086bc0     hb-ot-shaper-use.obj
 0002:00014cb0       ?_use_syllable_machine_indicies@@3QBEB 10086cb0     hb-ot-shaper-use.obj
 0002:000159d0       ?_use_syllable_machine_trans_targs@@3QBDB 100879d0     hb-ot-shaper-use.obj
 0002:00015a58       ?_use_syllable_machine_trans_actions@@3QBDB 10087a58     hb-ot-shaper-use.obj
 0002:00015ae0       ?_use_syllable_machine_to_state_actions@@3QBDB 10087ae0     hb-ot-shaper-use.obj
 0002:00015b58       ?_use_syllable_machine_from_state_actions@@3QBDB 10087b58     hb-ot-shaper-use.obj
 0002:00015bd0       ?_use_syllable_machine_eof_trans@@3QBFB 10087bd0     hb-ot-shaper-use.obj
 0002:00015cc0       ?use_table@@3QBEB          10087cc0     hb-ot-shaper-use.obj
 0002:00019100       ?use_basic_features@@3QBIB 1008b100     hb-ot-shaper-use.obj
 0002:0001911c       ?use_topographical_features@@3QBIB 1008b11c     hb-ot-shaper-use.obj
 0002:0001912c       ?use_other_features@@3QBIB 1008b12c     hb-ot-shaper-use.obj
 0002:00019140       ?hb_identity@@3U<unnamed-type-hb_identity>@@B 1008b140     hb-ot-shaper-use.obj
 0002:00019141       ?hb_second@@3U<unnamed-type-hb_second>@@B 1008b141     hb-ot-shaper-use.obj
 0002:00019170       ?table_tags@@3QBIB         1008b170     hb-ot-shaper-vowel-constraints.obj
 0002:00019178       ?ot_languages2@@3QBULangTag@@B 1008b178     hb-ot-tag.obj
 0002:000197d0       ?ot_languages3@@3QBULangTag@@B 1008b7d0     hb-ot-tag.obj
 0002:0001c24c       ?table_tags@@3QBIB         1008e24c     hb-ot-var.obj
 0002:0001c254       ?hb_bitwise_and@@3U<unnamed-type-hb_bitwise_and>@@B 1008e254     hb-set.obj
 0002:0001c255       ?hb_bitwise_or@@3U<unnamed-type-hb_bitwise_or>@@B 1008e255     hb-set.obj
 0002:0001c256       ?hb_bitwise_xor@@3U<unnamed-type-hb_bitwise_xor>@@B 1008e256     hb-set.obj
 0002:0001c257       ?hb_bitwise_lt@@3U<unnamed-type-hb_bitwise_lt>@@B 1008e257     hb-set.obj
 0002:0001c258       ?hb_bitwise_gt@@3U<unnamed-type-hb_bitwise_gt>@@B 1008e258     hb-set.obj
 0002:0001c25c       ?table_tags@@3QBIB         1008e25c     hb-shape-plan.obj
 0002:0001c540       ?table_tags@@3QBIB         1008e540     hb-shape.obj
 0002:0001c548       ?nil_shaper_list@@3QBQBDB  1008e548     hb-shape.obj
 0002:0001c54c       ?_hb_all_shapers@@3QBUhb_shaper_entry_t@@B 1008e54c     hb-shaper.obj
 0002:0001c588       ?table_tags@@3QBIB         1008e588     hb-static.obj
 0002:0001c590       ?_hb_os2_unicode_ranges@OT@@3QBUOS2Range@1@B 1008e590     hb-static.obj
 0002:0001cd80       ?_hb_arabic_u8@@3QBEB      1008ed80     hb-static.obj
 0002:0001cf50       ?_hb_arabic_u16@@3QBGB     1008ef50     hb-static.obj
 0002:0001d4f0       ?table_tags@@3QBIB         1008f4f0     hb-style.obj
 0002:0001d4f8       ?_hb_os2_unicode_ranges@OT@@3QBUOS2Range@1@B 1008f4f8     hb-style.obj
 0002:0001dce8       ?format1_names_msgstr@@3Tformat1_names_msgstr_t@@B 1008fce8     hb-style.obj
 0002:0001e428       ?format1_names_msgidx@@3QBIB 10090428     hb-style.obj
 0002:0001e834       ?table_tags@@3QBIB         10090834     hb-subset-cff-common.obj
 0002:0001e840       ?table_tags@@3QBIB         10090840     hb-subset-cff1.obj
 0002:0001e848       ?cff1_std_strings_msgstr@@3Tcff1_std_strings_msgstr_t@@B 10090848     hb-subset-cff1.obj
 0002:0001f5c0       ?cff1_std_strings_msgidx@@3QBIB 100915c0     hb-subset-cff1.obj
 0002:0001fbe0       ?hb_identity@@3U<unnamed-type-hb_identity>@@B 10091be0     hb-subset-cff1.obj
 0002:0001fbe1       ?hb_hash@@3U<unnamed-type-hb_hash>@@B 10091be1     hb-subset-cff1.obj
 0002:0001fbe4       ?table_tags@@3QBIB         10091be4     hb-subset-cff2.obj
 0002:0001fbec       ?hb_identity@@3U<unnamed-type-hb_identity>@@B 10091bec     hb-subset-cff2.obj
 0002:0001fbed       ?hb_hash@@3U<unnamed-type-hb_hash>@@B 10091bed     hb-subset-cff2.obj
 0002:0001fbf0       ?table_tags@@3QBIB         10091bf0     hb-subset-input.obj
 0002:0001fbf8       ?_hb_os2_unicode_ranges@OT@@3QBUOS2Range@1@B 10091bf8     hb-subset-plan.obj
 0002:000203e8       ?_hb_arabic_u8@@3QBEB      100923e8     hb-subset-plan.obj
 0002:000205b8       ?_hb_arabic_u16@@3QBGB     100925b8     hb-subset-plan.obj
 0002:00020b58       ?cff1_std_strings_msgstr@@3Tcff1_std_strings_msgstr_t@@B 10092b58     hb-subset-plan.obj
 0002:000218d0       ?cff1_std_strings_msgidx@@3QBIB 100938d0     hb-subset-plan.obj
 0002:00021ef0       ?table_tags@@3QBIB         10093ef0     hb-subset-plan.obj
 0002:00021ef8       ?hb_identity@@3U<unnamed-type-hb_identity>@@B 10093ef8     hb-subset-plan.obj
 0002:00021ef9       ?hb_bool@@3U<unnamed-type-hb_bool>@@B 10093ef9     hb-subset-plan.obj
 0002:00021efa       ?hb_has@@3U<unnamed-type-hb_has>@@B 10093efa     hb-subset-plan.obj
 0002:00021efb       ?hb_first@@3U<unnamed-type-hb_first>@@B 10093efb     hb-subset-plan.obj
 0002:00021efc       ?hb_second@@3U<unnamed-type-hb_second>@@B 10093efc     hb-subset-plan.obj
 0002:00021efd       ?hb_bitwise_and@@3U<unnamed-type-hb_bitwise_and>@@B 10093efd     hb-subset-plan.obj
 0002:00021efe       ?hb_bitwise_or@@3U<unnamed-type-hb_bitwise_or>@@B 10093efe     hb-subset-plan.obj
 0002:00021eff       ?hb_bitwise_lt@@3U<unnamed-type-hb_bitwise_lt>@@B 10093eff     hb-subset-plan.obj
 0002:00021f00       ?hb_bitwise_gt@@3U<unnamed-type-hb_bitwise_gt>@@B 10093f00     hb-subset-plan.obj
 0002:00021f01       ?hb_add@@3U<unnamed-type-hb_add>@@B 10093f01     hb-subset-plan.obj
 0002:00021f02       ?hb_zip@@3U<unnamed-type-hb_zip>@@B 10093f02     hb-subset-plan.obj
 0002:00021f08       ?format1_names_msgstr@@3Tformat1_names_msgstr_t@@B 10093f08     hb-subset.obj
 0002:00022648       ?format1_names_msgidx@@3QBIB 10094648     hb-subset.obj
 0002:00022a54       ?table_tags@@3QBIB         10094a54     hb-subset.obj
 0002:00022a60       ?cff1_std_strings_msgstr@@3Tcff1_std_strings_msgstr_t@@B 10094a60     hb-subset.obj
 0002:000237d8       ?cff1_std_strings_msgidx@@3QBIB 100957d8     hb-subset.obj
 0002:00023df8       ?_hb_os2_unicode_ranges@OT@@3QBUOS2Range@1@B 10095df8     hb-subset.obj
 0002:000245e8       ?_hb_arabic_u8@@3QBEB      100965e8     hb-subset.obj
 0002:000247b8       ?_hb_arabic_u16@@3QBGB     100967b8     hb-subset.obj
 0002:00024d58       ?hb_identity@@3U<unnamed-type-hb_identity>@@B 10096d58     hb-subset.obj
 0002:00024d59       ?hb_ridentity@@3U<unnamed-type-hb_ridentity>@@B 10096d59     hb-subset.obj
 0002:00024d5a       ?hb_hash@@3U<unnamed-type-hb_hash>@@B 10096d5a     hb-subset.obj
 0002:00024d5b       ?hb_first@@3U<unnamed-type-hb_first>@@B 10096d5b     hb-subset.obj
 0002:00024d5c       ?hb_second@@3U<unnamed-type-hb_second>@@B 10096d5c     hb-subset.obj
 0002:00024d5d       ?hb_add@@3U<unnamed-type-hb_add>@@B 10096d5d     hb-subset.obj
 0002:00024d5e       ?hb_iter@@3U<unnamed-type-hb_iter>@@B 10096d5e     hb-subset.obj
 0002:00024d5f       ?hb_zip@@3U<unnamed-type-hb_zip>@@B 10096d5f     hb-subset.obj
 0002:00024d60       ?hb_all@@3U<unnamed-type-hb_all>@@B 10096d60     hb-subset.obj
 0002:00024d68       ?_hb_ucd_sc_map@@3QBW4hb_script_t@@B 10096d68     hb-ucd.obj
 0002:00024ff8       ?_hb_ucd_dm1_p0_map@@3QBGB 10096ff8     hb-ucd.obj
 0002:00025670       ?_hb_ucd_dm1_p2_map@@3QBGB 10097670     hb-ucd.obj
 0002:00025750       ?_hb_ucd_dm2_u32_map@@3QBIB 10097750     hb-ucd.obj
 0002:00026148       ?_hb_ucd_dm2_u64_map@@3QB_KB 10098148     hb-ucd.obj
 0002:00026d68       ?_hb_ucd_u8@@3QBEB         10098d68     hb-ucd.obj
 0002:0002eec8       ?_hb_ucd_u16@@3QBGB        100a0ec8     hb-ucd.obj
 0002:00034948       ?_hb_ucd_i16@@3QBFB        100a6948     hb-ucd.obj
 0002:00034bd0       ?_hb_emoji_u8@@3QBEB       100a6bd0     hb-unicode.obj
 0002:00035130       _NaN                       100a7130     MSVCRT:ftol3.obj
 0002:00035134       _onept5                    100a7134     MSVCRT:ftol3.obj
 0002:00035138       _Int32ToUInt32             100a7138     MSVCRT:ftol3.obj
 0002:00035148       _GS_ExceptionPointers      100a7148     MSVCRT:gs_report.obj
 0002:00035150       two32                      100a7150     MSVCRT:ftol2.obj
 0002:00035154       two63                      100a7154     MSVCRT:ftol2.obj
 0002:00035158       _NaN                       100a7158     MSVCRT:ftol2.obj
 0002:00035528       __sehtable$?dllmain_crt_process_attach@@YAHQAUHINSTANCE__@@QAX@Z 100a7528     MSVCRT:dll_dllmain.obj
 0002:00035548       __sehtable$?dllmain_crt_process_detach@@YAH_N@Z 100a7548     MSVCRT:dll_dllmain.obj
 0002:00035570       __sehtable$?dllmain_dispatch@@YAHQAUHINSTANCE__@@KQAX@Z 100a7570     MSVCRT:dll_dllmain.obj
 0002:00035590       __sehtable$___scrt_is_nonwritable_in_current_image 100a7590     MSVCRT:utility.obj
 0002:000355b0       .edata                     100a75b0     fontmanager.exp
 0002:000355d8       rgpv                       100a75d8     fontmanager.exp
 0002:00035670       rgszName                   100a7670     fontmanager.exp
 0002:00035708       rgwOrd                     100a7708     fontmanager.exp
 0002:00035754       szName                     100a7754     fontmanager.exp
 0002:00035764       $N00001                    100a7764     fontmanager.exp
 0002:00035792       $N00002                    100a7792     fontmanager.exp
 0002:000357cd       $N00003                    100a77cd     fontmanager.exp
 0002:000357fc       $N00004                    100a77fc     fontmanager.exp
 0002:00035834       $N00005                    100a7834     fontmanager.exp
 0002:00035870       $N00006                    100a7870     fontmanager.exp
 0002:0003589b       $N00007                    100a789b     fontmanager.exp
 0002:000358da       $N00008                    100a78da     fontmanager.exp
 0002:00035913       $N00009                    100a7913     fontmanager.exp
 0002:0003594d       $N00010                    100a794d     fontmanager.exp
 0002:00035988       $N00011                    100a7988     fontmanager.exp
 0002:000359c0       $N00012                    100a79c0     fontmanager.exp
 0002:000359f9       $N00013                    100a79f9     fontmanager.exp
 0002:00035a34       $N00014                    100a7a34     fontmanager.exp
 0002:00035a75       $N00015                    100a7a75     fontmanager.exp
 0002:00035ab0       $N00016                    100a7ab0     fontmanager.exp
 0002:00035ae9       $N00017                    100a7ae9     fontmanager.exp
 0002:00035b2a       $N00018                    100a7b2a     fontmanager.exp
 0002:00035b69       $N00019                    100a7b69     fontmanager.exp
 0002:00035ba1       $N00020                    100a7ba1     fontmanager.exp
 0002:00035bda       $N00021                    100a7bda     fontmanager.exp
 0002:00035c07       $N00022                    100a7c07     fontmanager.exp
 0002:00035c3d       $N00023                    100a7c3d     fontmanager.exp
 0002:00035c6c       $N00024                    100a7c6c     fontmanager.exp
 0002:00035ca1       $N00025                    100a7ca1     fontmanager.exp
 0002:00035ccd       $N00026                    100a7ccd     fontmanager.exp
 0002:00035cfa       $N00027                    100a7cfa     fontmanager.exp
 0002:00035d27       $N00028                    100a7d27     fontmanager.exp
 0002:00035d55       $N00029                    100a7d55     fontmanager.exp
 0002:00035d8c       $N00030                    100a7d8c     fontmanager.exp
 0002:00035db4       $N00031                    100a7db4     fontmanager.exp
 0002:00035de1       $N00032                    100a7de1     fontmanager.exp
 0002:00035e0f       $N00033                    100a7e0f     fontmanager.exp
 0002:00035e37       $N00034                    100a7e37     fontmanager.exp
 0002:00035e71       $N00035                    100a7e71     fontmanager.exp
 0002:00035ead       $N00036                    100a7ead     fontmanager.exp
 0002:00035ee3       $N00037                    100a7ee3     fontmanager.exp
 0002:00035ef1       $N00038                    100a7ef1     fontmanager.exp
 0002:000363d8       .idata$6                   100a83d8     freetype:freetype.dll
 0002:0003646c       .idata$6                   100a846c     java:java.dll
 0002:000364b8       .idata$6                   100a84b8     advapi32:ADVAPI32.dll
 0002:00036520       .idata$6                   100a8520     user32:USER32.dll
 0002:00036644       .idata$6                   100a8644     gdi32:GDI32.dll
 0002:0003676c       .idata$6                   100a876c     awt:awt.dll
 0002:0003690e       .idata$6                   100a890e     kernel32:KERNEL32.dll
 0002:000369a6       .idata$6                   100a89a6     vcruntime:VCRUNTIME140.dll
 0002:00036b58       .idata$6                   100a8b58     ucrt:api-ms-win-crt-heap-l1-1-0.dll
 0002:00036b78       .idata$6                   100a8b78     ucrt:api-ms-win-crt-math-l1-1-0.dll
 0002:00036b98       .idata$6                   100a8b98     ucrt:api-ms-win-crt-environment-l1-1-0.dll
 0002:00036bbe       .idata$6                   100a8bbe     ucrt:api-ms-win-crt-convert-l1-1-0.dll
 0002:00036be0       .idata$6                   100a8be0     ucrt:api-ms-win-crt-stdio-l1-1-0.dll
 0002:00036c00       .idata$6                   100a8c00     ucrt:api-ms-win-crt-string-l1-1-0.dll
 0002:00036c22       .idata$6                   100a8c22     ucrt:api-ms-win-crt-runtime-l1-1-0.dll
 0003:00000200       _gvdClassName              100a9200     HBShaper.obj
 0003:00000204       ?PADBYTES@?1??getGlyphImageNativeInternal@@9@9 100a9204     freetypeScaler.obj
 0003:00000208       ?_hb_buffer_serialize_formats@@3PAPBDA 100a9208     hb-buffer-serialize.obj
 0003:000004a0       ?_hb_draw_funcs_default@@3Uhb_draw_funcs_t@@B 100a94a0     hb-font.obj
 0003:000004c8       ?_hb_font_funcs_default@@3Uhb_font_funcs_t@@B 100a94c8     hb-font.obj
 0003:00000524       ?modifier_combining_marks@@3PAIA 100a9524     hb-ot-shaper-arabic.obj
 0003:0000055c       ?thai_above_start_state@@3PAW4thai_above_state_t@@A 100a955c     hb-ot-shaper-thai.obj
 0003:00000570       ?thai_below_start_state@@3PAW4thai_below_state_t@@A 100a9570     hb-ot-shaper-thai.obj
 0003:00000588       ?known_tables@@3PAIA       100a9588     hb-subset.obj
 0003:000007c0       _gvdClass                  100a97c0     HBShaper.obj
 0003:000007c4       _gvdCountFID               100a97c4     HBShaper.obj
 0003:000007c8       _gvdFlagsFID               100a97c8     HBShaper.obj
 0003:000007cc       _gvdGlyphsFID              100a97cc     HBShaper.obj
 0003:000007d0       _gvdPositionsFID           100a97d0     HBShaper.obj
 0003:000007d4       _gvdIndicesFID             100a97d4     HBShaper.obj
 0003:000007d8       _gvdGrowMID                100a97d8     HBShaper.obj
 0003:000007dc       _jniInited                 100a97dc     HBShaper.obj
 0003:000007e0       _screenDC                  100a97e0     fontpath.obj
 0003:000007e4       _invalidateScalerMID       100a97e4     freetypeScaler.obj
 0003:000009b8       ?langs@@3U?$hb_atomic_ptr_t@Uhb_language_item_t@@@@A 100a99b8     hb-common.obj
 0003:000009bc       ?jdk_ffuncs@?1??_hb_jdk_get_font_funcs@@YAPAUhb_font_funcs_t@@XZ@4PAU2@A 100a99bc     hb-jdk-font.obj
 0003:000009c0       ?static_ot_funcs@@3Uhb_ot_font_funcs_lazy_loader_t@@A 100a99c0     hb-ot-font.obj
 0003:000009c4       ?last_tag_idx@?4??hb_ot_tags_from_language@@YAXPBD0PAI1@Z@4Uhb_atomic_int_t@@A 100a99c4     hb-ot-tag.obj
 0003:000009c8       ?static_shaper_list@@3Uhb_shaper_list_lazy_loader_t@@A 100a99c8     hb-shape.obj
 0003:000009cc       ?static_shapers@@3Uhb_shapers_lazy_loader_t@@A 100a99cc     hb-shaper.obj
 0003:000009d0       ?static_ucd_funcs@@3Uhb_ucd_unicode_funcs_lazy_loader_t@@A 100a99d0     hb-ucd.obj
 0003:000009d8       _igLUTable                 100a99d8     lcdglyph.obj
 0003:00000bbc       _theNullScalerContext      100a9bbc     sunFont.obj
 0003:00000bc0       _initialisedFontIDs        100a9bc0     sunFont.obj
 0003:00000bc8       _GS_ExceptionRecord        100a9bc8     MSVCRT:gs_report.obj
 0003:00000c18       _GS_ContextRecord          100a9c18     MSVCRT:gs_report.obj
 0003:00000ee4       ?__proc_attached@@3HA      100a9ee4     MSVCRT:dll_dllmain.obj
 0003:00000f08       ?is_initialized_as_dll@@3_NA 100a9f08     MSVCRT:utility.obj
 0003:00000f09       ?module_local_atexit_table_initialized@@3_NA 100a9f09     MSVCRT:utility.obj
 0003:00000f0c       ?module_local_atexit_table@@3U_onexit_table_t@@A 100a9f0c     MSVCRT:utility.obj
 0003:00000f18       ?module_local_at_quick_exit_table@@3U_onexit_table_t@@A 100a9f18     MSVCRT:utility.obj
 0004:00000060       $R000000                   100ab060     fontmanager.dll.res
